 javaaccessbridge

 Timestamp is ffffffff (Sun Feb  7 06:28:15 2106)

 Preferred load address is 10000000

 Start         Length     Name                   Class
 0001:00000000 00020973H .text$mn                CODE
 0001:00020973 00000000H .text$x                 CODE
 0002:00000000 0000016cH .idata$5                DATA
 0002:0000016c 00000004H .00cfg                  DATA
 0002:00000170 00000004H .CRT$XCA                DATA
 0002:00000174 00000004H .CRT$XCZ                DATA
 0002:00000178 00000004H .CRT$XIA                DATA
 0002:0000017c 0000000cH .CRT$XIC                DATA
 0002:00000188 00000004H .CRT$XIZ                DATA
 0002:0000018c 00000004H .CRT$XPA                DATA
 0002:00000190 00000008H .CRT$XPX                DATA
 0002:00000198 00000004H .CRT$XPXA               DATA
 0002:0000019c 00000004H .CRT$XPZ                DATA
 0002:000001a0 00000004H .CRT$XTA                DATA
 0002:000001a4 0000000cH .CRT$XTZ                DATA
 0002:000001a8 00000000H .gfids$y                DATA
 0002:000001b0 00014bb8H .rdata                  DATA
 0002:00014d68 0000012cH .rdata$r                DATA
 0002:00014e94 0000000cH .rdata$sxdata           DATA
 0002:00014ea0 000002f0H .rdata$zzzdbg           DATA
 0002:00015190 00000004H .rtc$IAA                DATA
 0002:00015194 00000004H .rtc$IZZ                DATA
 0002:00015198 00000004H .rtc$TAA                DATA
 0002:0001519c 00000004H .rtc$TZZ                DATA
 0002:000151a0 00000580H .xdata$x                DATA
 0002:00015720 00000a78H .edata                  DATA
 0002:00016198 0000003cH .idata$2                DATA
 0002:000161d4 00000014H .idata$3                DATA
 0002:000161e8 0000016cH .idata$4                DATA
 0002:00016354 00000680H .idata$6                DATA
 0003:00000000 00000890H .data                   DATA
 0003:00000890 00000078H .data$r                 DATA
 0003:00000908 00000a74H .bss                    DATA
 0004:00000000 00000120H .rsrc$01                DATA
 0004:00000120 00000630H .rsrc$02                DATA

  Address         Publics by Value              Rva+Base       Lib:Object

 0000:00000000       ___hybrid_code_map_count   00000000     <absolute>
 0000:00000000       ___guard_fids_count        00000000     <absolute>
 0000:00000000       ___x64_code_ranges_to_entry_points 00000000     <absolute>
 0000:00000000       ___guard_eh_cont_count     00000000     <absolute>
 0000:00000000       ___arm64x_redirection_metadata 00000000     <absolute>
 0000:00000000       ___arm64x_extra_rfe_table_size 00000000     <absolute>
 0000:00000000       ___arm64x_native_entrypoint 00000000     <absolute>
 0000:00000000       ___arm64x_extra_rfe_table  00000000     <absolute>
 0000:00000000       ___guard_iat_count         00000000     <absolute>
 0000:00000000       ___dynamic_value_reloc_table 00000000     <absolute>
 0000:00000000       ___guard_longjmp_count     00000000     <absolute>
 0000:00000000       ___guard_fids_table        00000000     <absolute>
 0000:00000000       __except_list              00000000     <absolute>
 0000:00000000       ___guard_longjmp_table     00000000     <absolute>
 0000:00000000       ___guard_iat_table         00000000     <absolute>
 0000:00000000       ___hybrid_auxiliary_iat    00000000     <absolute>
 0000:00000000       ___arm64x_redirection_metadata_count 00000000     <absolute>
 0000:00000000       ___enclave_config          00000000     <absolute>
 0000:00000000       ___volatile_metadata       00000000     <absolute>
 0000:00000000       ___guard_eh_cont_table     00000000     <absolute>
 0000:00000000       ___AbsoluteZero            00000000     <absolute>
 0000:00000000       ___x64_code_ranges_to_entry_points_count 00000000     <absolute>
 0000:00000000       ___hybrid_code_map         00000000     <absolute>
 0000:00000003       ___safe_se_handler_count   00000003     <absolute>
 0000:00000100       ___guard_flags             00000100     <absolute>
 0000:00000000       ___ImageBase               10000000     <linker-defined>
 0001:00000000       ??0AccessBridgeATInstance@@QAE@PAUHWND__@@0PADPAV0@@Z 10001000 f   AccessBridgeATInstance.obj
 0001:0000003a       ??1AccessBridgeATInstance@@QAE@XZ 1000103a f   AccessBridgeATInstance.obj
 0001:00000196       ?findABATInstanceFromATHWND@AccessBridgeATInstance@@QAEPAV1@PAUHWND__@@@Z 10001196 f   AccessBridgeATInstance.obj
 0001:000001b5       ?initiateIPC@AccessBridgeATInstance@@QAEJXZ 100011b5 f   AccessBridgeATInstance.obj
 0001:00000279       ?sendAccessibilityEventPackage@AccessBridgeATInstance@@QAEJPADHJ@Z 10001279 f   AccessBridgeATInstance.obj
 0001:000002b5       ?sendJavaEventPackage@AccessBridgeATInstance@@QAEJPADHJ@Z 100012b5 f   AccessBridgeATInstance.obj
 0001:000002fd       _PrintDebugString          100012fd f   AccessBridgeDebug.obj
 0001:00000347       ___local_stdio_printf_options 10001347 f i AccessBridgeDebug.obj
 0001:0000034d       __vfprintf_l               1000134d f i AccessBridgeDebug.obj
 0001:00000370       __vfwprintf_l              10001370 f i AccessBridgeDebug.obj
 0001:00000393       _finalizeFileLogger        10001393 f   AccessBridgeDebug.obj
 0001:000003ab       _fprintf                   100013ab f i AccessBridgeDebug.obj
 0001:000003c3       _getTimeStamp              100013c3 f   AccessBridgeDebug.obj
 0001:000003f1       _initializeFileLogger      100013f1 f   AccessBridgeDebug.obj
 0001:000004b1       _printf                    100014b1 f i AccessBridgeDebug.obj
 0001:000004ce       _wPrintDebugString         100014ce f   AccessBridgeDebug.obj
 0001:000004ce       _wPrintJavaDebugString     100014ce f   AccessBridgeDebug.obj
 0001:00000518       ??0AccessBridgeJavaEntryPoints@@QAE@PAUJNIEnv_@@PAV_jobject@@@Z 10001518 f   AccessBridgeJavaEntryPoints.obj
 0001:0000053d       ?BuildJavaEntryPoints@AccessBridgeJavaEntryPoints@@QAEHXZ 1000153d f   AccessBridgeJavaEntryPoints.obj
 0001:00001ade       ?CallBooleanMethod@JNIEnv_@@QAAEPAV_jobject@@PAU_jmethodID@@ZZ 10002ade f i AccessBridgeJavaEntryPoints.obj
 0001:00001af9       ?CallCharMethod@JNIEnv_@@QAAGPAV_jobject@@PAU_jmethodID@@ZZ 10002af9 f i AccessBridgeJavaEntryPoints.obj
 0001:00001b14       ?CallFloatMethod@JNIEnv_@@QAAMPAV_jobject@@PAU_jmethodID@@ZZ 10002b14 f i AccessBridgeJavaEntryPoints.obj
 0001:00001b2f       ?CallIntMethod@JNIEnv_@@QAAJPAV_jobject@@PAU_jmethodID@@ZZ 10002b2f f i AccessBridgeJavaEntryPoints.obj
 0001:00001b4a       ?CallObjectMethod@JNIEnv_@@QAAPAV_jobject@@PAV2@PAU_jmethodID@@ZZ 10002b4a f i AccessBridgeJavaEntryPoints.obj
 0001:00001b65       ?CallVoidMethod@JNIEnv_@@QAAXPAV_jobject@@PAU_jmethodID@@ZZ 10002b65 f i AccessBridgeJavaEntryPoints.obj
 0001:00001b80       ?activateAccessibleHyperlink@AccessBridgeJavaEntryPoints@@QAEHPAV_jobject@@0@Z 10002b80 f   AccessBridgeJavaEntryPoints.obj
 0001:00001c04       ?addAccessibilityEventNotification@AccessBridgeJavaEntryPoints@@QAEH_J@Z 10002c04 f   AccessBridgeJavaEntryPoints.obj
 0001:00001ca0       ?addAccessibleSelectionFromContext@AccessBridgeJavaEntryPoints@@QAEXPAV_jobject@@H@Z 10002ca0 f   AccessBridgeJavaEntryPoints.obj
 0001:00001d18       ?addJavaEventNotification@AccessBridgeJavaEntryPoints@@QAEH_J@Z 10002d18 f   AccessBridgeJavaEntryPoints.obj
 0001:00001d98       ?clearAccessibleSelectionFromContext@AccessBridgeJavaEntryPoints@@QAEXPAV_jobject@@@Z 10002d98 f   AccessBridgeJavaEntryPoints.obj
 0001:00001e0c       ?doAccessibleActions@AccessBridgeJavaEntryPoints@@QAEHPAV_jobject@@PAUAccessibleActionsToDoTag@@PAJ@Z 10002e0c f   AccessBridgeJavaEntryPoints.obj
 0001:00001f33       ?getAccessibleActions@AccessBridgeJavaEntryPoints@@QAEHPAV_jobject@@PAUAccessibleActionsTag@@@Z 10002f33 f   AccessBridgeJavaEntryPoints.obj
 0001:00002148       ?getAccessibleChildFromContext@AccessBridgeJavaEntryPoints@@QAEPAV_jobject@@PAV2@J@Z 10003148 f   AccessBridgeJavaEntryPoints.obj
 0001:0000221c       ?getAccessibleContextAt@AccessBridgeJavaEntryPoints@@QAEPAV_jobject@@JJPAV2@@Z 1000321c f   AccessBridgeJavaEntryPoints.obj
 0001:000022d8       ?getAccessibleContextFromHWND@AccessBridgeJavaEntryPoints@@QAEPAV_jobject@@J@Z 100032d8 f   AccessBridgeJavaEntryPoints.obj
 0001:00002367       ?getAccessibleContextInfo@AccessBridgeJavaEntryPoints@@QAEHPAV_jobject@@PAUAccessibleContextInfoTag@@@Z 10003367 f   AccessBridgeJavaEntryPoints.obj
 0001:00003185       ?getAccessibleContextWithFocus@AccessBridgeJavaEntryPoints@@QAEPAV_jobject@@XZ 10004185 f   AccessBridgeJavaEntryPoints.obj
 0001:00003223       ?getAccessibleHyperlink@AccessBridgeJavaEntryPoints@@QAEHQAV_jobject@@JPAUAccessibleHyperlinkInfoTag@@@Z 10004223 f   AccessBridgeJavaEntryPoints.obj
 0001:0000348f       ?getAccessibleHyperlinkCount@AccessBridgeJavaEntryPoints@@QAEJQAV_jobject@@@Z 1000448f f   AccessBridgeJavaEntryPoints.obj
 0001:0000350f       ?getAccessibleHypertext@AccessBridgeJavaEntryPoints@@QAEHPAV_jobject@@PAUAccessibleHypertextInfoTag@@@Z 1000450f f   AccessBridgeJavaEntryPoints.obj
 0001:000038a2       ?getAccessibleHypertextExt@AccessBridgeJavaEntryPoints@@QAEHQAV_jobject@@JPAUAccessibleHypertextInfoTag@@@Z 100048a2 f   AccessBridgeJavaEntryPoints.obj
 0001:00003c46       ?getAccessibleHypertextLinkIndex@AccessBridgeJavaEntryPoints@@QAEJQAV_jobject@@J@Z 10004c46 f   AccessBridgeJavaEntryPoints.obj
 0001:00003ccf       ?getAccessibleIcons@AccessBridgeJavaEntryPoints@@QAEHPAV_jobject@@PAUAccessibleIconsTag@@@Z 10004ccf f   AccessBridgeJavaEntryPoints.obj
 0001:00003f92       ?getAccessibleKeyBindings@AccessBridgeJavaEntryPoints@@QAEHPAV_jobject@@PAUAccessibleKeyBindingsTag@@@Z 10004f92 f   AccessBridgeJavaEntryPoints.obj
 0001:000040d3       ?getAccessibleParentFromContext@AccessBridgeJavaEntryPoints@@QAEPAV_jobject@@PAV2@@Z 100050d3 f   AccessBridgeJavaEntryPoints.obj
 0001:0000419e       ?getAccessibleRelationSet@AccessBridgeJavaEntryPoints@@QAEHPAV_jobject@@PAUAccessibleRelationSetInfoTag@@@Z 1000519e f   AccessBridgeJavaEntryPoints.obj
 0001:00004493       ?getAccessibleSelectionCountFromContext@AccessBridgeJavaEntryPoints@@QAEHPAV_jobject@@@Z 10005493 f   AccessBridgeJavaEntryPoints.obj
 0001:00004519       ?getAccessibleSelectionFromContext@AccessBridgeJavaEntryPoints@@QAEPAV_jobject@@PAV2@H@Z 10005519 f   AccessBridgeJavaEntryPoints.obj
 0001:000045ea       ?getAccessibleTableCellInfo@AccessBridgeJavaEntryPoints@@QAEHPAV_jobject@@JJPAUAccessibleTableCellInfoTag@@@Z 100055ea f   AccessBridgeJavaEntryPoints.obj
 0001:00004815       ?getAccessibleTableColumn@AccessBridgeJavaEntryPoints@@QAEJPAV_jobject@@J@Z 10005815 f   AccessBridgeJavaEntryPoints.obj
 0001:000048a7       ?getAccessibleTableColumnDescription@AccessBridgeJavaEntryPoints@@QAEPAV_jobject@@PAV2@J@Z 100058a7 f   AccessBridgeJavaEntryPoints.obj
 0001:00004978       ?getAccessibleTableColumnHeader@AccessBridgeJavaEntryPoints@@QAEHPAV_jobject@@PAUAccessibleTableInfoTag@@@Z 10005978 f   AccessBridgeJavaEntryPoints.obj
 0001:00004adb       ?getAccessibleTableColumnSelectionCount@AccessBridgeJavaEntryPoints@@QAEJPAV_jobject@@@Z 10005adb f   AccessBridgeJavaEntryPoints.obj
 0001:00004b62       ?getAccessibleTableColumnSelections@AccessBridgeJavaEntryPoints@@QAEHPAV_jobject@@JPAJ@Z 10005b62 f   AccessBridgeJavaEntryPoints.obj
 0001:00004c13       ?getAccessibleTableIndex@AccessBridgeJavaEntryPoints@@QAEJPAV_jobject@@JJ@Z 10005c13 f   AccessBridgeJavaEntryPoints.obj
 0001:00004cab       ?getAccessibleTableInfo@AccessBridgeJavaEntryPoints@@QAEHPAV_jobject@@PAUAccessibleTableInfoTag@@@Z 10005cab f   AccessBridgeJavaEntryPoints.obj
 0001:00004e9b       ?getAccessibleTableRow@AccessBridgeJavaEntryPoints@@QAEJPAV_jobject@@J@Z 10005e9b f   AccessBridgeJavaEntryPoints.obj
 0001:00004f2d       ?getAccessibleTableRowDescription@AccessBridgeJavaEntryPoints@@QAEPAV_jobject@@PAV2@J@Z 10005f2d f   AccessBridgeJavaEntryPoints.obj
 0001:00004ffe       ?getAccessibleTableRowHeader@AccessBridgeJavaEntryPoints@@QAEHPAV_jobject@@PAUAccessibleTableInfoTag@@@Z 10005ffe f   AccessBridgeJavaEntryPoints.obj
 0001:00005161       ?getAccessibleTableRowSelectionCount@AccessBridgeJavaEntryPoints@@QAEJPAV_jobject@@@Z 10006161 f   AccessBridgeJavaEntryPoints.obj
 0001:000051e8       ?getAccessibleTableRowSelections@AccessBridgeJavaEntryPoints@@QAEHPAV_jobject@@JPAJ@Z 100061e8 f   AccessBridgeJavaEntryPoints.obj
 0001:00005299       ?getAccessibleTextAttributes@AccessBridgeJavaEntryPoints@@QAEHPAV_jobject@@JPAUAccessibleTextAttributesInfoTag@@@Z 10006299 f   AccessBridgeJavaEntryPoints.obj
 0001:00006481       ?getAccessibleTextInfo@AccessBridgeJavaEntryPoints@@QAEHPAV_jobject@@PAUAccessibleTextInfoTag@@JJ@Z 10007481 f   AccessBridgeJavaEntryPoints.obj
 0001:000065d7       ?getAccessibleTextItems@AccessBridgeJavaEntryPoints@@QAEHPAV_jobject@@PAUAccessibleTextItemsInfoTag@@J@Z 100075d7 f   AccessBridgeJavaEntryPoints.obj
 0001:00006a1a       ?getAccessibleTextLineBounds@AccessBridgeJavaEntryPoints@@QAEHPAV_jobject@@JPAJ1@Z 10007a1a f   AccessBridgeJavaEntryPoints.obj
 0001:00006b0b       ?getAccessibleTextRange@AccessBridgeJavaEntryPoints@@QAEHPAV_jobject@@JJPAGF@Z 10007b0b f   AccessBridgeJavaEntryPoints.obj
 0001:00006d09       ?getAccessibleTextRect@AccessBridgeJavaEntryPoints@@QAEHPAV_jobject@@PAUAccessibleTextRectInfoTag@@J@Z 10007d09 f   AccessBridgeJavaEntryPoints.obj
 0001:00006e9c       ?getAccessibleTextSelectionInfo@AccessBridgeJavaEntryPoints@@QAEHPAV_jobject@@PAUAccessibleTextSelectionInfoTag@@@Z 10007e9c f   AccessBridgeJavaEntryPoints.obj
 0001:000070e2       ?getActiveDescendent@AccessBridgeJavaEntryPoints@@QAEPAV_jobject@@QAV2@@Z 100080e2 f   AccessBridgeJavaEntryPoints.obj
 0001:0000719e       ?getCaretLocation@AccessBridgeJavaEntryPoints@@QAEHPAV_jobject@@PAUAccessibleTextRectInfoTag@@J@Z 1000819e f   AccessBridgeJavaEntryPoints.obj
 0001:00007331       ?getCurrentAccessibleValueFromContext@AccessBridgeJavaEntryPoints@@QAEHPAV_jobject@@PAGF@Z 10008331 f   AccessBridgeJavaEntryPoints.obj
 0001:000074cc       ?getHWNDFromAccessibleContext@AccessBridgeJavaEntryPoints@@QAEPAUHWND__@@PAV_jobject@@@Z 100084cc f   AccessBridgeJavaEntryPoints.obj
 0001:00007551       ?getMaximumAccessibleValueFromContext@AccessBridgeJavaEntryPoints@@QAEHPAV_jobject@@PAGF@Z 10008551 f   AccessBridgeJavaEntryPoints.obj
 0001:000076ec       ?getMinimumAccessibleValueFromContext@AccessBridgeJavaEntryPoints@@QAEHPAV_jobject@@PAGF@Z 100086ec f   AccessBridgeJavaEntryPoints.obj
 0001:00007887       ?getObjectDepth@AccessBridgeJavaEntryPoints@@QAEJQAV_jobject@@@Z 10008887 f   AccessBridgeJavaEntryPoints.obj
 0001:0000790f       ?getParentWithRole@AccessBridgeJavaEntryPoints@@QAEPAV_jobject@@QAV2@PBG@Z 1000890f f   AccessBridgeJavaEntryPoints.obj
 0001:000079f8       ?getParentWithRoleElseRoot@AccessBridgeJavaEntryPoints@@QAEPAV_jobject@@QAV2@PBG@Z 100089f8 f   AccessBridgeJavaEntryPoints.obj
 0001:00007ae1       ?getTextAttributesInRange@AccessBridgeJavaEntryPoints@@QAEHQAV_jobject@@HHPAUAccessibleTextAttributesInfoTag@@PAF@Z 10008ae1 f   AccessBridgeJavaEntryPoints.obj
 0001:00007d50       ?getTopLevelObject@AccessBridgeJavaEntryPoints@@QAEPAV_jobject@@QAV2@@Z 10008d50 f   AccessBridgeJavaEntryPoints.obj
 0001:00007e0c       ?getVersionInfo@AccessBridgeJavaEntryPoints@@QAEHPAUAccessBridgeVersionInfoTag@@@Z 10008e0c f   AccessBridgeJavaEntryPoints.obj
 0001:00007fff       ?getVirtualAccessibleName@AccessBridgeJavaEntryPoints@@QAEHQAV_jobject@@PAGH@Z 10008fff f   AccessBridgeJavaEntryPoints.obj
 0001:000081a7       ?getVisibleChildren@AccessBridgeJavaEntryPoints@@QAEHQAV_jobject@@HPAUVisibleChildenInfoTag@@@Z 100091a7 f   AccessBridgeJavaEntryPoints.obj
 0001:00008305       ?getVisibleChildrenCount@AccessBridgeJavaEntryPoints@@QAEHQAV_jobject@@@Z 10009305 f   AccessBridgeJavaEntryPoints.obj
 0001:00008378       ?isAccessibleChildSelectedFromContext@AccessBridgeJavaEntryPoints@@QAEHPAV_jobject@@H@Z 10009378 f   AccessBridgeJavaEntryPoints.obj
 0001:00008406       ?isAccessibleTableColumnSelected@AccessBridgeJavaEntryPoints@@QAEHPAV_jobject@@J@Z 10009406 f   AccessBridgeJavaEntryPoints.obj
 0001:00008497       ?isAccessibleTableRowSelected@AccessBridgeJavaEntryPoints@@QAEHPAV_jobject@@J@Z 10009497 f   AccessBridgeJavaEntryPoints.obj
 0001:00008528       ?isJavaWindow@AccessBridgeJavaEntryPoints@@QAEHJ@Z 10009528 f   AccessBridgeJavaEntryPoints.obj
 0001:000085a1       ?isSameObject@AccessBridgeJavaEntryPoints@@QAEHPAV_jobject@@0@Z 100095a1 f   AccessBridgeJavaEntryPoints.obj
 0001:00008615       ?removeAccessibilityEventNotification@AccessBridgeJavaEntryPoints@@QAEH_J@Z 10009615 f   AccessBridgeJavaEntryPoints.obj
 0001:00008695       ?removeAccessibleSelectionFromContext@AccessBridgeJavaEntryPoints@@QAEXPAV_jobject@@H@Z 10009695 f   AccessBridgeJavaEntryPoints.obj
 0001:0000870d       ?removeJavaEventNotification@AccessBridgeJavaEntryPoints@@QAEH_J@Z 1000970d f   AccessBridgeJavaEntryPoints.obj
 0001:0000878d       ?requestFocus@AccessBridgeJavaEntryPoints@@QAEHQAV_jobject@@@Z 1000978d f   AccessBridgeJavaEntryPoints.obj
 0001:00008815       ?selectAllAccessibleSelectionFromContext@AccessBridgeJavaEntryPoints@@QAEXPAV_jobject@@@Z 10009815 f   AccessBridgeJavaEntryPoints.obj
 0001:00008889       ?selectTextRange@AccessBridgeJavaEntryPoints@@QAEHQAV_jobject@@HH@Z 10009889 f   AccessBridgeJavaEntryPoints.obj
 0001:00008920       ?setCaretPosition@AccessBridgeJavaEntryPoints@@QAEHQAV_jobject@@H@Z 10009920 f   AccessBridgeJavaEntryPoints.obj
 0001:000089b1       ?setTextContents@AccessBridgeJavaEntryPoints@@QAEHQAV_jobject@@PBG@Z 100099b1 f   AccessBridgeJavaEntryPoints.obj
 0001:00008a6b       ?verifyAccessibleText@AccessBridgeJavaEntryPoints@@QAEHPAV_jobject@@@Z 10009a6b f   AccessBridgeJavaEntryPoints.obj
 0001:00008b56       ?initBroadcastMessageIDs@@YAHXZ 10009b56 f   AccessBridgeMessages.obj
 0001:00008b88       ??0JavaAccessBridge@@QAE@PAUHINSTANCE__@@@Z 10009b88 f   JavaAccessBridge.obj
 0001:00008bab       ??1JavaAccessBridge@@QAE@XZ 10009bab f   JavaAccessBridge.obj
 0001:00008c56       ?MemoryMappedFileCreated@JavaAccessBridge@@QAEJPAUHWND__@@PAD@Z 10009c56 f   JavaAccessBridge.obj
 0001:00008cd2       ?WindowsATDestroyed@JavaAccessBridge@@QAEXPAUHWND__@@@Z 10009cd2 f   JavaAccessBridge.obj
 0001:00008d5e       ?addAccessibilityEventNotification@JavaAccessBridge@@QAEX_JPAUHWND__@@@Z 10009d5e f   JavaAccessBridge.obj
 0001:00008df0       ?addJavaEventNotification@JavaAccessBridge@@QAEX_JPAUHWND__@@@Z 10009df0 f   JavaAccessBridge.obj
 0001:00008e82       ?fireCaretUpdate@JavaAccessBridge@@QAEXPAUJNIEnv_@@PAV_jobject@@11@Z 10009e82 f   JavaAccessBridge.obj
 0001:00008f71       ?fireFocusGained@JavaAccessBridge@@QAEXPAUJNIEnv_@@PAV_jobject@@11@Z 10009f71 f   JavaAccessBridge.obj
 0001:00009060       ?fireFocusLost@JavaAccessBridge@@QAEXPAUJNIEnv_@@PAV_jobject@@11@Z 1000a060 f   JavaAccessBridge.obj
 0001:0000914f       ?fireMenuCanceled@JavaAccessBridge@@QAEXPAUJNIEnv_@@PAV_jobject@@11@Z 1000a14f f   JavaAccessBridge.obj
 0001:0000924a       ?fireMenuDeselected@JavaAccessBridge@@QAEXPAUJNIEnv_@@PAV_jobject@@11@Z 1000a24a f   JavaAccessBridge.obj
 0001:00009345       ?fireMenuSelected@JavaAccessBridge@@QAEXPAUJNIEnv_@@PAV_jobject@@11@Z 1000a345 f   JavaAccessBridge.obj
 0001:00009440       ?fireMouseClicked@JavaAccessBridge@@QAEXPAUJNIEnv_@@PAV_jobject@@11@Z 1000a440 f   JavaAccessBridge.obj
 0001:0000952f       ?fireMouseEntered@JavaAccessBridge@@QAEXPAUJNIEnv_@@PAV_jobject@@11@Z 1000a52f f   JavaAccessBridge.obj
 0001:0000961e       ?fireMouseExited@JavaAccessBridge@@QAEXPAUJNIEnv_@@PAV_jobject@@11@Z 1000a61e f   JavaAccessBridge.obj
 0001:0000970d       ?fireMousePressed@JavaAccessBridge@@QAEXPAUJNIEnv_@@PAV_jobject@@11@Z 1000a70d f   JavaAccessBridge.obj
 0001:00009805       ?fireMouseReleased@JavaAccessBridge@@QAEXPAUJNIEnv_@@PAV_jobject@@11@Z 1000a805 f   JavaAccessBridge.obj
 0001:00009900       ?firePopupMenuCanceled@JavaAccessBridge@@QAEXPAUJNIEnv_@@PAV_jobject@@11@Z 1000a900 f   JavaAccessBridge.obj
 0001:000099fb       ?firePopupMenuWillBecomeInvisible@JavaAccessBridge@@QAEXPAUJNIEnv_@@PAV_jobject@@11@Z 1000a9fb f   JavaAccessBridge.obj
 0001:00009af6       ?firePopupMenuWillBecomeVisible@JavaAccessBridge@@QAEXPAUJNIEnv_@@PAV_jobject@@11@Z 1000aaf6 f   JavaAccessBridge.obj
 0001:00009bf1       ?firePropertyActiveDescendentChange@JavaAccessBridge@@QAEXPAUJNIEnv_@@PAV_jobject@@1111@Z 1000abf1 f   JavaAccessBridge.obj
 0001:00009cfa       ?firePropertyCaretChange@JavaAccessBridge@@QAEXPAUJNIEnv_@@PAV_jobject@@11JJ@Z 1000acfa f   JavaAccessBridge.obj
 0001:00009ddc       ?firePropertyChildChange@JavaAccessBridge@@QAEXPAUJNIEnv_@@PAV_jobject@@1111@Z 1000addc f   JavaAccessBridge.obj
 0001:00009ee5       ?firePropertyDescriptionChange@JavaAccessBridge@@QAEXPAUJNIEnv_@@PAV_jobject@@11PAV_jstring@@2@Z 1000aee5 f   JavaAccessBridge.obj
 0001:0000a0c4       ?firePropertyNameChange@JavaAccessBridge@@QAEXPAUJNIEnv_@@PAV_jobject@@11PAV_jstring@@2@Z 1000b0c4 f   JavaAccessBridge.obj
 0001:0000a2a3       ?firePropertySelectionChange@JavaAccessBridge@@QAEXPAUJNIEnv_@@PAV_jobject@@11@Z 1000b2a3 f   JavaAccessBridge.obj
 0001:0000a36d       ?firePropertyStateChange@JavaAccessBridge@@QAEXPAUJNIEnv_@@PAV_jobject@@11PAV_jstring@@2@Z 1000b36d f   JavaAccessBridge.obj
 0001:0000a54c       ?firePropertyTableModelChange@JavaAccessBridge@@QAEXPAUJNIEnv_@@PAV_jobject@@11PAV_jstring@@2@Z 1000b54c f   JavaAccessBridge.obj
 0001:0000a731       ?firePropertyTextChange@JavaAccessBridge@@QAEXPAUJNIEnv_@@PAV_jobject@@11@Z 1000b731 f   JavaAccessBridge.obj
 0001:0000a7fb       ?firePropertyValueChange@JavaAccessBridge@@QAEXPAUJNIEnv_@@PAV_jobject@@11PAV_jstring@@2@Z 1000b7fb f   JavaAccessBridge.obj
 0001:0000a9da       ?firePropertyVisibleDataChange@JavaAccessBridge@@QAEXPAUJNIEnv_@@PAV_jobject@@11@Z 1000b9da f   JavaAccessBridge.obj
 0001:0000aaa7       ?initWindow@JavaAccessBridge@@QAEHXZ 1000baa7 f   JavaAccessBridge.obj
 0001:0000aad3       ?javaRun@JavaAccessBridge@@QAEXPAUJNIEnv_@@PAV_jobject@@@Z 1000bad3 f   JavaAccessBridge.obj
 0001:0000ac42       ?javaShutdown@JavaAccessBridge@@QAEXPAUJNIEnv_@@PAV_jobject@@@Z 1000bc42 f   JavaAccessBridge.obj
 0001:0000acd3       ?postHelloToWindowsDLLMsg@JavaAccessBridge@@QAEXPAUHWND__@@@Z 1000bcd3 f   JavaAccessBridge.obj
 0001:0000ad17       ?processPackage@JavaAccessBridge@@QAEJPADH@Z 1000bd17 f   JavaAccessBridge.obj
 0001:0000bcf7       ?receiveMemoryPackage@JavaAccessBridge@@QAEHPAUHWND__@@J@Z 1000ccf7 f   JavaAccessBridge.obj
 0001:0000bd6a       ?releaseJavaObject@JavaAccessBridge@@QAEXPAV_jobject@@@Z 1000cd6a f   JavaAccessBridge.obj
 0001:0000bdb9       ?removeAccessibilityEventNotification@JavaAccessBridge@@QAEX_JPAUHWND__@@@Z 1000cdb9 f   JavaAccessBridge.obj
 0001:0000be4e       ?removeJavaEventNotification@JavaAccessBridge@@QAEX_JPAUHWND__@@@Z 1000ce4e f   JavaAccessBridge.obj
 0001:0000bee3       _AccessBridgeDialogProc@16 1000cee3 f   JavaAccessBridge.obj
 0001:0000bfe9       _DllMain@12                1000cfe9 f   JavaAccessBridge.obj
 0001:0000c052       _Java_com_sun_java_accessibility_internal_AccessBridge_caretUpdate@16 1000d052 f   JavaAccessBridge.obj
 0001:0000c05d       _Java_com_sun_java_accessibility_internal_AccessBridge_focusGained@16 1000d05d f   JavaAccessBridge.obj
 0001:0000c068       _Java_com_sun_java_accessibility_internal_AccessBridge_focusLost@16 1000d068 f   JavaAccessBridge.obj
 0001:0000c073       _Java_com_sun_java_accessibility_internal_AccessBridge_javaShutdown@8 1000d073 f   JavaAccessBridge.obj
 0001:0000c07e       _Java_com_sun_java_accessibility_internal_AccessBridge_jawtGetComponentFromNativeWindowHandle@12 1000d07e f   JavaAccessBridge.obj
 0001:0000c0ad       _Java_com_sun_java_accessibility_internal_AccessBridge_jawtGetNativeWindowHandleFromComponent@12 1000d0ad f   JavaAccessBridge.obj
 0001:0000c0f9       _Java_com_sun_java_accessibility_internal_AccessBridge_menuCanceled@16 1000d0f9 f   JavaAccessBridge.obj
 0001:0000c104       _Java_com_sun_java_accessibility_internal_AccessBridge_menuDeselected@16 1000d104 f   JavaAccessBridge.obj
 0001:0000c10f       _Java_com_sun_java_accessibility_internal_AccessBridge_menuSelected@16 1000d10f f   JavaAccessBridge.obj
 0001:0000c11a       _Java_com_sun_java_accessibility_internal_AccessBridge_mouseClicked@16 1000d11a f   JavaAccessBridge.obj
 0001:0000c125       _Java_com_sun_java_accessibility_internal_AccessBridge_mouseEntered@16 1000d125 f   JavaAccessBridge.obj
 0001:0000c130       _Java_com_sun_java_accessibility_internal_AccessBridge_mouseExited@16 1000d130 f   JavaAccessBridge.obj
 0001:0000c13b       _Java_com_sun_java_accessibility_internal_AccessBridge_mousePressed@16 1000d13b f   JavaAccessBridge.obj
 0001:0000c146       _Java_com_sun_java_accessibility_internal_AccessBridge_mouseReleased@16 1000d146 f   JavaAccessBridge.obj
 0001:0000c151       _Java_com_sun_java_accessibility_internal_AccessBridge_popupMenuCanceled@16 1000d151 f   JavaAccessBridge.obj
 0001:0000c15c       _Java_com_sun_java_accessibility_internal_AccessBridge_popupMenuWillBecomeInvisible@16 1000d15c f   JavaAccessBridge.obj
 0001:0000c167       _Java_com_sun_java_accessibility_internal_AccessBridge_popupMenuWillBecomeVisible@16 1000d167 f   JavaAccessBridge.obj
 0001:0000c172       _Java_com_sun_java_accessibility_internal_AccessBridge_propertyActiveDescendentChange@24 1000d172 f   JavaAccessBridge.obj
 0001:0000c181       _Java_com_sun_java_accessibility_internal_AccessBridge_propertyCaretChange@24 1000d181 f   JavaAccessBridge.obj
 0001:0000c190       _Java_com_sun_java_accessibility_internal_AccessBridge_propertyChildChange@24 1000d190 f   JavaAccessBridge.obj
 0001:0000c19f       _Java_com_sun_java_accessibility_internal_AccessBridge_propertyDescriptionChange@24 1000d19f f   JavaAccessBridge.obj
 0001:0000c1ae       _Java_com_sun_java_accessibility_internal_AccessBridge_propertyNameChange@24 1000d1ae f   JavaAccessBridge.obj
 0001:0000c1bd       _Java_com_sun_java_accessibility_internal_AccessBridge_propertySelectionChange@16 1000d1bd f   JavaAccessBridge.obj
 0001:0000c1c8       _Java_com_sun_java_accessibility_internal_AccessBridge_propertyStateChange@24 1000d1c8 f   JavaAccessBridge.obj
 0001:0000c1d7       _Java_com_sun_java_accessibility_internal_AccessBridge_propertyTableModelChange@24 1000d1d7 f   JavaAccessBridge.obj
 0001:0000c1e6       _Java_com_sun_java_accessibility_internal_AccessBridge_propertyTextChange@16 1000d1e6 f   JavaAccessBridge.obj
 0001:0000c1f1       _Java_com_sun_java_accessibility_internal_AccessBridge_propertyValueChange@24 1000d1f1 f   JavaAccessBridge.obj
 0001:0000c200       _Java_com_sun_java_accessibility_internal_AccessBridge_propertyVisibleDataChange@16 1000d200 f   JavaAccessBridge.obj
 0001:0000c20b       _Java_com_sun_java_accessibility_internal_AccessBridge_runDLL@8 1000d20b f   JavaAccessBridge.obj
 0001:0000c221       _Java_com_sun_java_accessibility_internal_AccessBridge_sendDebugString@12 1000d221 f   JavaAccessBridge.obj
 0001:0000c282       ??2@YAPAXI@Z               1000d282 f   LIBCMT:new_scalar.obj
 0001:0000c2b2       ??3@YAXPAXI@Z              1000d2b2 f   LIBCMT:delete_scalar_size.obj
 0001:0000c2c0       ??_U@YAPAXI@Z              1000d2c0 f   LIBCMT:new_array.obj
 0001:0000c2c9       ??_V@YAXPAX@Z              1000d2c9 f   LIBCMT:delete_array.obj
 0001:0000c2d0       __aulldiv                  1000d2d0 f   LIBCMT:ulldiv.obj
 0001:0000c338       @__security_check_cookie@4 1000d338 f   LIBCMT:secchk.obj
 0001:0000c689       __DllMainCRTStartup@12     1000d689 f   LIBCMT:dll_dllmain.obj
 0001:0000c6ac       ??0bad_alloc@std@@QAE@ABV01@@Z 1000d6ac f i LIBCMT:throw_bad_alloc.obj
 0001:0000c6c7       ??0bad_alloc@std@@QAE@XZ   1000d6c7 f i LIBCMT:throw_bad_alloc.obj
 0001:0000c6df       ??0bad_array_new_length@std@@QAE@ABV01@@Z 1000d6df f i LIBCMT:throw_bad_alloc.obj
 0001:0000c6fa       ??0bad_array_new_length@std@@QAE@XZ 1000d6fa f i LIBCMT:throw_bad_alloc.obj
 0001:0000c712       ??0exception@std@@QAE@ABV01@@Z 1000d712 f i LIBCMT:throw_bad_alloc.obj
 0001:0000c73e       ??1bad_array_new_length@std@@UAE@XZ 1000d73e f i LIBCMT:throw_bad_alloc.obj
 0001:0000c73e       ??1bad_alloc@std@@UAE@XZ   1000d73e f i LIBCMT:throw_bad_alloc.obj
 0001:0000c74f       ??_Ebad_alloc@std@@UAEPAXI@Z 1000d74f f i LIBCMT:throw_bad_alloc.obj
 0001:0000c74f       ??_Gbad_alloc@std@@UAEPAXI@Z 1000d74f f i LIBCMT:throw_bad_alloc.obj
 0001:0000c74f       ??_Gbad_array_new_length@std@@UAEPAXI@Z 1000d74f f i LIBCMT:throw_bad_alloc.obj
 0001:0000c74f       ??_Ebad_array_new_length@std@@UAEPAXI@Z 1000d74f f i LIBCMT:throw_bad_alloc.obj
 0001:0000c74f       ??_Eexception@std@@UAEPAXI@Z 1000d74f f i LIBCMT:throw_bad_alloc.obj
 0001:0000c74f       ??_Gexception@std@@UAEPAXI@Z 1000d74f f i LIBCMT:throw_bad_alloc.obj
 0001:0000c77c       ?__scrt_throw_std_bad_alloc@@YAXXZ 1000d77c f   LIBCMT:throw_bad_alloc.obj
 0001:0000c799       ?__scrt_throw_std_bad_array_new_length@@YAXXZ 1000d799 f   LIBCMT:throw_bad_alloc.obj
 0001:0000c7b6       ?what@exception@std@@UBEPBDXZ 1000d7b6 f i LIBCMT:throw_bad_alloc.obj
 0001:0000c7c3       ??3@YAXPAX@Z               1000d7c3 f   LIBCMT:delete_scalar.obj
 0001:0000c7c8       ___raise_securityfailure   1000d7c8 f   LIBCMT:gs_report.obj
 0001:0000c7f0       ___report_gsfailure        1000d7f0 f   LIBCMT:gs_report.obj
 0001:0000c936       ___security_init_cookie    1000d936 f   LIBCMT:gs_support.obj
 0001:0000c981       ?__scrt_initialize_type_info@@YAXXZ 1000d981 f   LIBCMT:tncleanup.obj
 0001:0000c98d       ?__scrt_uninitialize_type_info@@YAXXZ 1000d98d f   LIBCMT:tncleanup.obj
 0001:0000c999       ___local_stdio_scanf_options 1000d999 f i LIBCMT:default_local_stdio_options.obj
 0001:0000c99f       ___scrt_initialize_default_local_stdio_options 1000d99f f   LIBCMT:default_local_stdio_options.obj
 0001:0000ca00       ___scrt_acquire_startup_lock 1000da00 f   LIBCMT:utility.obj
 0001:0000ca32       ___scrt_dllmain_after_initialize_c 1000da32 f   LIBCMT:utility.obj
 0001:0000ca5d       ___scrt_dllmain_before_initialize_c 1000da5d f   LIBCMT:utility.obj
 0001:0000ca6b       ___scrt_dllmain_crt_thread_attach 1000da6b f   LIBCMT:utility.obj
 0001:0000ca8a       ___scrt_dllmain_crt_thread_detach 1000da8a f   LIBCMT:utility.obj
 0001:0000ca97       ___scrt_dllmain_exception_filter 1000da97 f   LIBCMT:utility.obj
 0001:0000cacb       ___scrt_dllmain_uninitialize_c 1000dacb f   LIBCMT:utility.obj
 0001:0000caee       ___scrt_dllmain_uninitialize_critical 1000daee f   LIBCMT:utility.obj
 0001:0000cafb       ___scrt_initialize_crt     1000dafb f   LIBCMT:utility.obj
 0001:0000cb34       ___scrt_initialize_onexit_tables 1000db34 f   LIBCMT:utility.obj
 0001:0000cbbb       ___scrt_is_nonwritable_in_current_image 1000dbbb f   LIBCMT:utility.obj
 0001:0000cc4f       ___scrt_release_startup_lock 1000dc4f f   LIBCMT:utility.obj
 0001:0000cc6c       ___scrt_uninitialize_crt   1000dc6c f   LIBCMT:utility.obj
 0001:0000cc94       ___scrt_get_dyn_tls_init_callback 1000dc94 f   LIBCMT:dyn_tls_init.obj
 0001:0000cc9a       ___scrt_fastfail           1000dc9a f   LIBCMT:utility_desktop.obj
 0001:0000cdb4       __crt_debugger_hook        1000ddb4 f   LIBCMT:utility_desktop.obj
 0001:0000cdbc       __RTC_Initialize           1000ddbc f   LIBCMT:initsect.obj
 0001:0000cde8       __RTC_Terminate            1000dde8 f   LIBCMT:initsect.obj
 0001:0000ce20       __SEH_prolog4              1000de20 f   LIBCMT:sehprolg4.obj
 0001:0000ce64       __SEH_epilog4              1000de64 f   LIBCMT:sehprolg4.obj
 0001:0000ce78       @_guard_check_icall_nop@4  1000de78 f i LIBCMT:guard_support.obj
 0001:0000ce7b       ??_Gtype_info@@UAEPAXI@Z   1000de7b f i LIBCMT:std_type_info_static.obj
 0001:0000ce7b       ??_Etype_info@@UAEPAXI@Z   1000de7b f i LIBCMT:std_type_info_static.obj
 0001:0000ce9e       ___isa_available_init      1000de9e f   LIBCMT:cpu_disp.obj
 0001:0000d06e       __get_startup_argv_mode    1000e06e f   LIBCMT:argv_mode.obj
 0001:0000d072       ___scrt_is_ucrt_dll_in_use 1000e072 f   LIBCMT:ucrt_detection.obj
 0001:0000d080       _memcpy                    1000e080 f   libvcruntime:memcpy.obj
 0001:0000d600       _memset                    1000e600 f   libvcruntime:memset.obj
 0001:0000d7a0       __except_handler4          1000e7a0 f   libvcruntime:chandler4.obj
 0001:0000d8fe       ___std_exception_copy      1000e8fe f   libvcruntime:std_exception.obj
 0001:0000d961       ___std_exception_destroy   1000e961 f   libvcruntime:std_exception.obj
 0001:0000d980       __CxxThrowException@8      1000e980 f   libvcruntime:throw.obj
 0001:0000d9ec       ___std_type_info_destroy_list 1000e9ec f   libvcruntime:std_type_info.obj
 0001:0000da0f       ___vcrt_initialize         1000ea0f f   libvcruntime:initialization.obj
 0001:0000da2e       ___vcrt_thread_attach      1000ea2e f   libvcruntime:initialization.obj
 0001:0000da39       ___vcrt_thread_detach      1000ea39 f   libvcruntime:initialization.obj
 0001:0000da44       ___vcrt_uninitialize       1000ea44 f   libvcruntime:initialization.obj
 0001:0000da5b       ___vcrt_uninitialize_critical 1000ea5b f   libvcruntime:initialization.obj
 0001:0000da63       ___DestructExceptionObject 1000ea63 f   libvcruntime:ehhelpers.obj
 0001:0000db04       ?_CallMemberFunction0@@YGXQAX0@Z 1000eb04 f i libvcruntime:ehhelpers.obj
 0001:0000db70       __local_unwind4            1000eb70 f   libvcruntime:exsup4.obj
 0001:0000dc44       __seh_longjmp_unwind4@4    1000ec44 f   libvcruntime:exsup4.obj
 0001:0000dc6c       @_EH4_CallFilterFunc@8     1000ec6c f   libvcruntime:exsup4.obj
 0001:0000dc84       @_EH4_TransferToHandler@8  1000ec84 f   libvcruntime:exsup4.obj
 0001:0000dca0       @_EH4_GlobalUnwind2@8      1000eca0 f   libvcruntime:exsup4.obj
 0001:0000dcbc       @_EH4_LocalUnwind@16       1000ecbc f   libvcruntime:exsup4.obj
 0001:0000dcd3       ___except_validate_context_record 1000ecd3 f   libvcruntime:jbcxrval.obj
 0001:0000dd03       ___except_validate_jump_buffer 1000ed03 f   libvcruntime:jbcxrval.obj
 0001:0000dd30       ___vcrt_freefls@4          1000ed30 f   libvcruntime:per_thread_data.obj
 0001:0000dd4c       ___vcrt_freeptd            1000ed4c f   libvcruntime:per_thread_data.obj
 0001:0000dd82       ___vcrt_getptd             1000ed82 f   libvcruntime:per_thread_data.obj
 0001:0000dd90       ___vcrt_getptd_noexit      1000ed90 f   libvcruntime:per_thread_data.obj
 0001:0000de22       ___vcrt_initialize_ptd     1000ee22 f   libvcruntime:per_thread_data.obj
 0001:0000de55       ___vcrt_uninitialize_ptd   1000ee55 f   libvcruntime:per_thread_data.obj
 0001:0000de70       ___vcrt_initialize_locks   1000ee70 f   libvcruntime:locks.obj
 0001:0000deac       ___vcrt_uninitialize_locks 1000eeac f   libvcruntime:locks.obj
 0001:0000def0       __global_unwind2           1000eef0 f   libvcruntime:exsup.obj
 0001:0000df56       __local_unwind2            1000ef56 f   libvcruntime:exsup.obj
 0001:0000dfda       __abnormal_termination     1000efda f   libvcruntime:exsup.obj
 0001:0000e000       __NLG_Notify1              1000f000 f   libvcruntime:exsup.obj
 0001:0000e00c       __NLG_Notify               1000f00c f   libvcruntime:exsup.obj
 0001:0000e023       __NLG_Dispatch             1000f023     libvcruntime:exsup.obj
 0001:0000e023       __NLG_Dispatch2            1000f023     libvcruntime:exsup.obj
 0001:0000e02b       __NLG_Call                 1000f02b f   libvcruntime:exsup.obj
 0001:0000e02d       __NLG_Return2              1000f02d     libvcruntime:exsup.obj
 0001:0000e111       ___vcrt_FlsAlloc           1000f111 f   libvcruntime:winapi_downlevel.obj
 0001:0000e14c       ___vcrt_FlsFree            1000f14c f   libvcruntime:winapi_downlevel.obj
 0001:0000e187       ___vcrt_FlsGetValue        1000f187 f   libvcruntime:winapi_downlevel.obj
 0001:0000e1c2       ___vcrt_FlsSetValue        1000f1c2 f   libvcruntime:winapi_downlevel.obj
 0001:0000e200       ___vcrt_InitializeCriticalSectionEx 1000f200 f   libvcruntime:winapi_downlevel.obj
 0001:0000e250       __CallSettingFrame@12      1000f250 f   libvcruntime:lowhelpr.obj
 0001:0000e277       __NLG_Return               1000f277     libvcruntime:lowhelpr.obj
 0001:0000e2a0       _memmove                   1000f2a0 f   libvcruntime:memmove.obj
 0001:0000e820       _strcmp                    1000f820 f   libucrt:strcmp.obj
 0001:0000e8b0       _strcpy                    1000f8b0 f   libucrt:strcat.obj
 0001:0000e8c0       _strcat                    1000f8c0 f   libucrt:strcat.obj
 0001:0000e9b0       _strncpy                   1000f9b0 f   libucrt:strncpy.obj
 0001:0000ec30       __beginthreadex            1000fc30 f   libucrt:thread.obj
 0001:0000ecb3       __endthreadex              1000fcb3 f   libucrt:thread.obj
 0001:0000ecd0       _strlen                    1000fcd0 f   libucrt:strlen.obj
 0001:0000ed60       _strncat                   1000fd60 f   libucrt:strncat.obj
 0001:0000ee95       ___acrt_initialize_stdio   1000fe95 f   libucrt:_file.obj
 0001:0000ef5d       ___acrt_iob_func           1000ff5d f   libucrt:_file.obj
 0001:0000ef6d       ___acrt_uninitialize_stdio 1000ff6d f   libucrt:_file.obj
 0001:0000efb9       __lock_file                1000ffb9 f   libucrt:_file.obj
 0001:0000efcd       __unlock_file              1000ffcd f   libucrt:_file.obj
 0001:0000f097       ??$count@D@formatting_buffer@__crt_stdio_output@@QBEIXZ 10010097 f i libucrt:output.obj
 0001:0000f0af       ??$count@_W@formatting_buffer@__crt_stdio_output@@QBEIXZ 100100af f i libucrt:output.obj
 0001:0000f0c8       ??$ensure_buffer_is_big_enough@D@formatting_buffer@__crt_stdio_output@@QAE_NI@Z 100100c8 f i libucrt:output.obj
 0001:0000f145       ??$ensure_buffer_is_big_enough@_W@formatting_buffer@__crt_stdio_output@@QAE_NI@Z 10010145 f i libucrt:output.obj
 0001:0000f1c3       ??$is_wide_character_specifier@D@__crt_stdio_output@@YA_N_KDW4length_modifier@0@@Z 100101c3 f i libucrt:output.obj
 0001:0000f1f4       ??$is_wide_character_specifier@_W@__crt_stdio_output@@YA_N_K_WW4length_modifier@0@@Z 100101f4 f i libucrt:output.obj
 0001:0000f242       ??$scratch_data@D@formatting_buffer@__crt_stdio_output@@QAEPADXZ 10010242 f i libucrt:output.obj
 0001:0000f260       ??$type_case_integer_parse_into_buffer@I@?$output_processor@DV?$stream_output_adapter@D@__crt_stdio_output@@V?$standard_base@DV?$stream_output_adapter@D@__crt_stdio_output@@@2@@__crt_stdio_output@@AAEXII_N@Z 10010260 f i libucrt:output.obj
 0001:0000f2d3       ??$type_case_integer_parse_into_buffer@I@?$output_processor@_WV?$stream_output_adapter@_W@__crt_stdio_output@@V?$standard_base@_WV?$stream_output_adapter@_W@__crt_stdio_output@@@2@@__crt_stdio_output@@AAEXII_N@Z 100102d3 f i libucrt:output.obj
 0001:0000f35a       ??$type_case_integer_parse_into_buffer@_K@?$output_processor@DV?$stream_output_adapter@D@__crt_stdio_output@@V?$standard_base@DV?$stream_output_adapter@D@__crt_stdio_output@@@2@@__crt_stdio_output@@AAEX_KI_N@Z 1001035a f i libucrt:output.obj
 0001:0000f3e8       ??$type_case_integer_parse_into_buffer@_K@?$output_processor@_WV?$stream_output_adapter@_W@__crt_stdio_output@@V?$standard_base@_WV?$stream_output_adapter@_W@__crt_stdio_output@@@2@@__crt_stdio_output@@AAEX_KI_N@Z 100103e8 f i libucrt:output.obj
 0001:0000f48a       ??$write_multiple_characters@V?$stream_output_adapter@D@__crt_stdio_output@@D@__crt_stdio_output@@YAXABV?$stream_output_adapter@D@0@DHQAH@Z 1001048a f i libucrt:output.obj
 0001:0000f4c5       ??$write_multiple_characters@V?$stream_output_adapter@_W@__crt_stdio_output@@D@__crt_stdio_output@@YAXABV?$stream_output_adapter@_W@0@DHQAH@Z 100104c5 f i libucrt:output.obj
 0001:0000f505       ??0?$common_data@D@__crt_stdio_output@@IAE@XZ 10010505 f i libucrt:output.obj
 0001:0000f54a       ??0?$common_data@_W@__crt_stdio_output@@IAE@XZ 1001054a f i libucrt:output.obj
 0001:0000f594       ??0?$output_adapter_data@DV?$stream_output_adapter@D@__crt_stdio_output@@@__crt_stdio_output@@IAE@ABV?$stream_output_adapter@D@1@_KQBDQAU__crt_locale_pointers@@QAD@Z 10010594 f i libucrt:output.obj
 0001:0000f5d0       ??0?$output_adapter_data@_WV?$stream_output_adapter@_W@__crt_stdio_output@@@__crt_stdio_output@@IAE@ABV?$stream_output_adapter@_W@1@_KQB_WQAU__crt_locale_pointers@@QAD@Z 100105d0 f i libucrt:output.obj
 0001:0000f60c       ??0_LocaleUpdate@@QAE@QAU__crt_locale_pointers@@@Z 1001060c f i libucrt:output.obj
 0001:0000f68f       ??1formatting_buffer@__crt_stdio_output@@QAE@XZ 1001068f f i libucrt:output.obj
 0001:0000f6a9       ??4?$__crt_unique_heap_ptr@DU__crt_internal_free_policy@@@@QAEAAV0@$$QAV0@@Z 100106a9 f i libucrt:output.obj
 0001:0000f84b       ?crop_zeroes@__crt_stdio_output@@YAXPADQAU__crt_locale_pointers@@@Z 1001084b f i libucrt:output.obj
 0001:0000f8ab       ?find_next_state@?$output_processor@DV?$stream_output_adapter@D@__crt_stdio_output@@V?$standard_base@DV?$stream_output_adapter@D@__crt_stdio_output@@@2@@__crt_stdio_output@@ABE?AW4state@2@DW432@@Z 100108ab f i libucrt:output.obj
 0001:0000f8e8       ?find_next_state@?$output_processor@_WV?$stream_output_adapter@_W@__crt_stdio_output@@V?$standard_base@_WV?$stream_output_adapter@_W@__crt_stdio_output@@@2@@__crt_stdio_output@@ABE?AW4state@2@_WW432@@Z 100108e8 f i libucrt:output.obj
 0001:0000f927       ?force_decimal_point@__crt_stdio_output@@YAXPADQAU__crt_locale_pointers@@@Z 10010927 f i libucrt:output.obj
 0001:0000f983       ?parse_int_from_format_string@?$output_processor@DV?$stream_output_adapter@D@__crt_stdio_output@@V?$standard_base@DV?$stream_output_adapter@D@__crt_stdio_output@@@2@@__crt_stdio_output@@AAE_NQAH@Z 10010983 f i libucrt:output.obj
 0001:0000f9f7       ?parse_int_from_format_string@?$output_processor@_WV?$stream_output_adapter@_W@__crt_stdio_output@@V?$standard_base@_WV?$stream_output_adapter@_W@__crt_stdio_output@@@2@@__crt_stdio_output@@AAE_NQAH@Z 100109f7 f i libucrt:output.obj
 0001:0000fa6d       ?process@?$output_processor@DV?$stream_output_adapter@D@__crt_stdio_output@@V?$standard_base@DV?$stream_output_adapter@D@__crt_stdio_output@@@2@@__crt_stdio_output@@QAEHXZ 10010a6d f i libucrt:output.obj
 0001:0000fb81       ?process@?$output_processor@_WV?$stream_output_adapter@_W@__crt_stdio_output@@V?$standard_base@_WV?$stream_output_adapter@_W@__crt_stdio_output@@@2@@__crt_stdio_output@@QAEHXZ 10010b81 f i libucrt:output.obj
 0001:0000fc9d       ?state_case_flag@?$output_processor@DV?$stream_output_adapter@D@__crt_stdio_output@@V?$standard_base@DV?$stream_output_adapter@D@__crt_stdio_output@@@2@@__crt_stdio_output@@AAE_NXZ 10010c9d f i libucrt:output.obj
 0001:0000fcda       ?state_case_flag@?$output_processor@_WV?$stream_output_adapter@_W@__crt_stdio_output@@V?$standard_base@_WV?$stream_output_adapter@_W@__crt_stdio_output@@@2@@__crt_stdio_output@@AAE_NXZ 10010cda f i libucrt:output.obj
 0001:0000fd17       ?state_case_normal@?$output_processor@DV?$stream_output_adapter@D@__crt_stdio_output@@V?$standard_base@DV?$stream_output_adapter@D@__crt_stdio_output@@@2@@__crt_stdio_output@@AAE_NXZ 10010d17 f i libucrt:output.obj
 0001:0000fd36       ?state_case_normal@?$output_processor@_WV?$stream_output_adapter@_W@__crt_stdio_output@@V?$standard_base@_WV?$stream_output_adapter@_W@__crt_stdio_output@@@2@@__crt_stdio_output@@AAE_NXZ 10010d36 f i libucrt:output.obj
 0001:0000fd55       ?state_case_normal_common@?$output_processor@DV?$stream_output_adapter@D@__crt_stdio_output@@V?$standard_base@DV?$stream_output_adapter@D@__crt_stdio_output@@@2@@__crt_stdio_output@@AAE_NXZ 10010d55 f i libucrt:output.obj
 0001:0000fd8f       ?state_case_normal_common@?$output_processor@_WV?$stream_output_adapter@_W@__crt_stdio_output@@V?$standard_base@_WV?$stream_output_adapter@_W@__crt_stdio_output@@@2@@__crt_stdio_output@@AAE_NXZ 10010d8f f i libucrt:output.obj
 0001:0000fdb9       ?state_case_normal_tchar@?$output_processor@DV?$stream_output_adapter@D@__crt_stdio_output@@V?$standard_base@DV?$stream_output_adapter@D@__crt_stdio_output@@@2@@__crt_stdio_output@@AAE_ND@Z 10010db9 f i libucrt:output.obj
 0001:0000fe26       ?state_case_precision@?$output_processor@DV?$stream_output_adapter@D@__crt_stdio_output@@V?$standard_base@DV?$stream_output_adapter@D@__crt_stdio_output@@@2@@__crt_stdio_output@@AAE_NXZ 10010e26 f i libucrt:output.obj
 0001:0000fe4c       ?state_case_precision@?$output_processor@_WV?$stream_output_adapter@_W@__crt_stdio_output@@V?$standard_base@_WV?$stream_output_adapter@_W@__crt_stdio_output@@@2@@__crt_stdio_output@@AAE_NXZ 10010e4c f i libucrt:output.obj
 0001:0000fe73       ?state_case_size@?$output_processor@DV?$stream_output_adapter@D@__crt_stdio_output@@V?$standard_base@DV?$stream_output_adapter@D@__crt_stdio_output@@@2@@__crt_stdio_output@@AAE_NXZ 10010e73 f i libucrt:output.obj
 0001:0000ffc1       ?state_case_size@?$output_processor@_WV?$stream_output_adapter@_W@__crt_stdio_output@@V?$standard_base@_WV?$stream_output_adapter@_W@__crt_stdio_output@@@2@@__crt_stdio_output@@AAE_NXZ 10010fc1 f i libucrt:output.obj
 0001:00010139       ?state_case_type@?$output_processor@DV?$stream_output_adapter@D@__crt_stdio_output@@V?$standard_base@DV?$stream_output_adapter@D@__crt_stdio_output@@@2@@__crt_stdio_output@@AAE_NXZ 10011139 f i libucrt:output.obj
 0001:0001036b       ?state_case_type@?$output_processor@_WV?$stream_output_adapter@_W@__crt_stdio_output@@V?$standard_base@_WV?$stream_output_adapter@_W@__crt_stdio_output@@@2@@__crt_stdio_output@@AAE_NXZ 1001136b f i libucrt:output.obj
 0001:000105d0       ?state_case_width@?$output_processor@DV?$stream_output_adapter@D@__crt_stdio_output@@V?$standard_base@DV?$stream_output_adapter@D@__crt_stdio_output@@@2@@__crt_stdio_output@@AAE_NXZ 100115d0 f i libucrt:output.obj
 0001:000105fb       ?state_case_width@?$output_processor@_WV?$stream_output_adapter@_W@__crt_stdio_output@@V?$standard_base@_WV?$stream_output_adapter@_W@__crt_stdio_output@@@2@@__crt_stdio_output@@AAE_NXZ 100115fb f i libucrt:output.obj
 0001:00010627       ?to_integer_size@__crt_stdio_output@@YAIW4length_modifier@1@@Z 10011627 f i libucrt:output.obj
 0001:0001067b       ?type_case_Z@?$output_processor@DV?$stream_output_adapter@D@__crt_stdio_output@@V?$standard_base@DV?$stream_output_adapter@D@__crt_stdio_output@@@2@@__crt_stdio_output@@AAE_NXZ 1001167b f i libucrt:output.obj
 0001:000106d5       ?type_case_Z@?$output_processor@_WV?$stream_output_adapter@_W@__crt_stdio_output@@V?$standard_base@_WV?$stream_output_adapter@_W@__crt_stdio_output@@@2@@__crt_stdio_output@@AAE_NXZ 100116d5 f i libucrt:output.obj
 0001:0001072f       ?type_case_a@?$output_processor@DV?$stream_output_adapter@D@__crt_stdio_output@@V?$standard_base@DV?$stream_output_adapter@D@__crt_stdio_output@@@2@@__crt_stdio_output@@AAE_NXZ 1001172f f i libucrt:output.obj
 0001:0001087e       ?type_case_a@?$output_processor@_WV?$stream_output_adapter@_W@__crt_stdio_output@@V?$standard_base@_WV?$stream_output_adapter@_W@__crt_stdio_output@@@2@@__crt_stdio_output@@AAE_NXZ 1001187e f i libucrt:output.obj
 0001:000109e3       ?type_case_c_tchar@?$output_processor@DV?$stream_output_adapter@D@__crt_stdio_output@@V?$standard_base@DV?$stream_output_adapter@D@__crt_stdio_output@@@2@@__crt_stdio_output@@AAE_ND@Z 100119e3 f i libucrt:output.obj
 0001:00010a73       ?type_case_c_tchar@?$output_processor@_WV?$stream_output_adapter@_W@__crt_stdio_output@@V?$standard_base@_WV?$stream_output_adapter@_W@__crt_stdio_output@@@2@@__crt_stdio_output@@AAE_N_W@Z 10011a73 f i libucrt:output.obj
 0001:00010b09       ?type_case_integer@?$output_processor@DV?$stream_output_adapter@D@__crt_stdio_output@@V?$standard_base@DV?$stream_output_adapter@D@__crt_stdio_output@@@2@@__crt_stdio_output@@AAE_NI_N@Z 10011b09 f i libucrt:output.obj
 0001:00010c5a       ?type_case_integer@?$output_processor@_WV?$stream_output_adapter@_W@__crt_stdio_output@@V?$standard_base@_WV?$stream_output_adapter@_W@__crt_stdio_output@@@2@@__crt_stdio_output@@AAE_NI_N@Z 10011c5a f i libucrt:output.obj
 0001:00010daf       ?type_case_n@?$output_processor@_WV?$stream_output_adapter@_W@__crt_stdio_output@@V?$standard_base@_WV?$stream_output_adapter@_W@__crt_stdio_output@@@2@@__crt_stdio_output@@AAE_NXZ 10011daf f i libucrt:output.obj
 0001:00010daf       ?type_case_n@?$output_processor@DV?$stream_output_adapter@D@__crt_stdio_output@@V?$standard_base@DV?$stream_output_adapter@D@__crt_stdio_output@@@2@@__crt_stdio_output@@AAE_NXZ 10011daf f i libucrt:output.obj
 0001:00010e23       ?type_case_o@?$output_processor@DV?$stream_output_adapter@D@__crt_stdio_output@@V?$standard_base@DV?$stream_output_adapter@D@__crt_stdio_output@@@2@@__crt_stdio_output@@AAE_NXZ 10011e23 f i libucrt:output.obj
 0001:00010e42       ?type_case_o@?$output_processor@_WV?$stream_output_adapter@_W@__crt_stdio_output@@V?$standard_base@_WV?$stream_output_adapter@_W@__crt_stdio_output@@@2@@__crt_stdio_output@@AAE_NXZ 10011e42 f i libucrt:output.obj
 0001:00010e61       ?type_case_p@?$output_processor@DV?$stream_output_adapter@D@__crt_stdio_output@@V?$standard_base@DV?$stream_output_adapter@D@__crt_stdio_output@@@2@@__crt_stdio_output@@AAE_NXZ 10011e61 f i libucrt:output.obj
 0001:00010e79       ?type_case_p@?$output_processor@_WV?$stream_output_adapter@_W@__crt_stdio_output@@V?$standard_base@_WV?$stream_output_adapter@_W@__crt_stdio_output@@@2@@__crt_stdio_output@@AAE_NXZ 10011e79 f i libucrt:output.obj
 0001:00010e91       ?type_case_s@?$output_processor@DV?$stream_output_adapter@D@__crt_stdio_output@@V?$standard_base@DV?$stream_output_adapter@D@__crt_stdio_output@@@2@@__crt_stdio_output@@AAE_NXZ 10011e91 f i libucrt:output.obj
 0001:00010f02       ?type_case_s@?$output_processor@_WV?$stream_output_adapter@_W@__crt_stdio_output@@V?$standard_base@_WV?$stream_output_adapter@_W@__crt_stdio_output@@@2@@__crt_stdio_output@@AAE_NXZ 10011f02 f i libucrt:output.obj
 0001:00010f75       ?type_case_s_compute_narrow_string_length@?$output_processor@_WV?$stream_output_adapter@_W@__crt_stdio_output@@V?$standard_base@_WV?$stream_output_adapter@_W@__crt_stdio_output@@@2@@__crt_stdio_output@@ABEHH_W@Z 10011f75 f i libucrt:output.obj
 0001:00010fbc       ?validate@?$stream_output_adapter@D@__crt_stdio_output@@QBE_NXZ 10011fbc f i libucrt:output.obj
 0001:00010fdd       ?validate@?$stream_output_adapter@_W@__crt_stdio_output@@QBE_NXZ 10011fdd f i libucrt:output.obj
 0001:00010fdd       ?validate@?$c_string_character_source@D@__crt_strtox@@QBE_NXZ 10011fdd f i libucrt:atox.obj
 0001:00010fdd       ?validate@?$c_string_character_source@_W@__crt_strtox@@QBE_NXZ 10011fdd f i libucrt:atox.obj
 0001:00010ff8       ?validate_stream_is_ansi_if_required@?$__acrt_stdio_char_traits@D@@SA_NQAU_iobuf@@@Z 10011ff8 f i libucrt:output.obj
 0001:0001107f       ?write_character_without_count_update@?$stream_output_adapter@D@__crt_stdio_output@@QBE_ND@Z 1001207f f i libucrt:output.obj
 0001:000110b5       ?write_character_without_count_update@?$stream_output_adapter@_W@__crt_stdio_output@@QBE_N_W@Z 100120b5 f i libucrt:output.obj
 0001:000110ee       ?write_stored_string_tchar@?$output_processor@DV?$stream_output_adapter@D@__crt_stdio_output@@V?$standard_base@DV?$stream_output_adapter@D@__crt_stdio_output@@@2@@__crt_stdio_output@@AAE_ND@Z 100120ee f i libucrt:output.obj
 0001:00011195       ?write_stored_string_tchar@?$output_processor@_WV?$stream_output_adapter@_W@__crt_stdio_output@@V?$standard_base@_WV?$stream_output_adapter@_W@__crt_stdio_output@@@2@@__crt_stdio_output@@AAE_N_W@Z 10012195 f i libucrt:output.obj
 0001:00011228       ?write_string@?$stream_output_adapter@D@__crt_stdio_output@@QBEXQBDHQAHAAV__crt_deferred_errno_cache@@@Z 10012228 f i libucrt:output.obj
 0001:00011254       ?write_string@?$stream_output_adapter@_W@__crt_stdio_output@@QBEXQB_WHQAHAAV__crt_deferred_errno_cache@@@Z 10012254 f i libucrt:output.obj
 0001:00011280       ?write_string_impl@?$output_adapter_common@DV?$stream_output_adapter@D@__crt_stdio_output@@@__crt_stdio_output@@IBEXQBDHQAHAAV__crt_deferred_errno_cache@@@Z 10012280 f i libucrt:output.obj
 0001:0001131e       ?write_string_impl@?$output_adapter_common@_WV?$stream_output_adapter@_W@__crt_stdio_output@@@__crt_stdio_output@@IBEXQB_WHQAHAAV__crt_deferred_errno_cache@@@Z 1001231e f i libucrt:output.obj
 0001:000113bf       ___acrt_locale_get_ctype_array_value 100123bf f i libucrt:output.obj
 0001:000113e1       ___stdio_common_vfprintf   100123e1 f   libucrt:output.obj
 0001:00011464       ___stdio_common_vfwprintf  10012464 f   libucrt:output.obj
 0001:000114e7       __fclose_nolock            100124e7 f   libucrt:fclose.obj
 0001:0001155e       _fclose                    1001255e f   libucrt:fclose.obj
 0001:00011699       _fopen                     10012699 f   libucrt:fopen.obj
 0001:0001179c       _getenv                    1001279c f   libucrt:getenv.obj
 0001:000117a7       _wcscmp                    100127a7 f   libucrt:wcscmp.obj
 0001:000117e7       _strnlen                   100127e7 f   libucrt:strnlen.obj
 0001:00011909       _wcslen                    10012909 f   libucrt:strnlen.obj
 0001:00011a31       _wcsnlen                   10012a31 f   libucrt:strnlen.obj
 0001:00011be1       _wcsncpy                   10012be1 f   libucrt:wcsncpy.obj
 0001:00011c24       ___acrt_initialize_new_handler 10012c24 f   libucrt:new_handler.obj
 0001:00011c33       __callnewh                 10012c33 f   libucrt:new_handler.obj
 0001:00011c60       __query_new_handler        10012c60 f   libucrt:new_handler.obj
 0001:00011cbc       _malloc                    10012cbc f   libucrt:malloc.obj
 0001:00011cc7       __initterm                 10012cc7 f   libucrt:initterm.obj
 0001:00011d0c       __initterm_e               10012d0c f   libucrt:initterm.obj
 0001:00011d3a       _free                      10012d3a f   libucrt:free.obj
 0001:00011d55       __seh_filter_dll           10012d55 f   libucrt:exception_filter.obj
 0001:00011d75       __seh_filter_exe           10012d75 f   libucrt:exception_filter.obj
 0001:00012143       ___acrt_initialize_thread_local_exit_callback 10013143 f   libucrt:exit.obj
 0001:00012152       __cexit                    10013152 f   libucrt:exit.obj
 0001:00012161       __exit                     10013161 f   libucrt:exit.obj
 0001:00012177       __is_c_termination_complete 10013177 f   libucrt:exit.obj
 0001:0001242b       ___acrt_allocate_buffer_for_argv 1001342b f   libucrt:argv_parsing.obj
 0001:0001247a       __configure_narrow_argv    1001347a f   libucrt:argv_parsing.obj
 0001:00012686       ??$uninitialize@A6AXAAPAPA_W@Z@?$dual_state_global@PAPA_W@__crt_state_management@@QAEXA6AXAAPAPA_W@Z@Z 10013686 f i libucrt:environment_initialization.obj
 0001:00012686       ??$uninitialize@A6AXAAPAPAD@Z@?$dual_state_global@PAPAD@__crt_state_management@@QAEXA6AXAAPAPAD@Z@Z 10013686 f i libucrt:environment_initialization.obj
 0001:000126e5       ___dcrt_get_or_create_narrow_environment_nolock 100136e5 f   libucrt:environment_initialization.obj
 0001:000126ea       ___dcrt_uninitialize_environments_nolock 100136ea f   libucrt:environment_initialization.obj
 0001:00012721       __initialize_narrow_environment 10013721 f   libucrt:environment_initialization.obj
 0001:0001285b       __execute_onexit_table     1001385b f   libucrt:onexit.obj
 0001:00012888       __initialize_onexit_table  10013888 f   libucrt:onexit.obj
 0001:000128b1       ___acrt_uninitialize_command_line 100138b1 f   libucrt:argv_data.obj
 0001:00012981       ??$__crt_fast_encode_pointer@PAX@@YAPAXQAX@Z 10013981 f i libucrt:initialization.obj
 0001:000129ce       ___acrt_initialize         100139ce f   libucrt:initialization.obj
 0001:000129e0       ___acrt_thread_attach      100139e0 f   libucrt:initialization.obj
 0001:000129eb       ___acrt_thread_detach      100139eb f   libucrt:initialization.obj
 0001:000129f3       ___acrt_uninitialize       100139f3 f   libucrt:initialization.obj
 0001:00012a23       ___acrt_uninitialize_critical 10013a23 f   libucrt:initialization.obj
 0001:00012a35       _terminate                 10013a35 f   libucrt:terminate.obj
 0001:00012a71       _strcpy_s                  10013a71 f   libucrt:strcpy_s.obj
 0001:00012acb       _abort                     10013acb f   libucrt:abort.obj
 0001:00012b0f       ??$is_overflow_condition@K@__crt_strtox@@YA_NIK@Z 10013b0f f i libucrt:atox.obj
 0001:00012b40       ??$parse_integer@KV?$c_string_character_source@D@__crt_strtox@@@__crt_strtox@@YAKQAU__crt_locale_pointers@@V?$c_string_character_source@D@0@H_N@Z 10013b40 f i libucrt:atox.obj
 0001:00012d65       ??$parse_integer@KV?$c_string_character_source@_W@__crt_strtox@@@__crt_strtox@@YAKQAU__crt_locale_pointers@@V?$c_string_character_source@_W@0@H_N@Z 10013d65 f i libucrt:atox.obj
 0001:0001336d       ?unget@?$c_string_character_source@D@__crt_strtox@@QAEXD@Z 1001436d f i libucrt:atox.obj
 0001:00013396       ?unget@?$c_string_character_source@_W@__crt_strtox@@QAEX_W@Z 10014396 f i libucrt:atox.obj
 0001:000133c4       __ischartype_l             100143c4 f i libucrt:atox.obj
 0001:00013420       _strncmp                   10014420 f   libucrt:strncmp.obj
 0001:00013498       _calloc                    10014498 f   libucrt:calloc.obj
 0001:000134a3       _wcsncmp                   100144a3 f   libucrt:wcsncmp.obj
 0001:000134dd       ___acrt_call_reportfault   100144dd f   libucrt:invalid_parameter.obj
 0001:00013616       ___acrt_initialize_invalid_parameter_handler 10014616 f   libucrt:invalid_parameter.obj
 0001:00013625       __invalid_parameter        10014625 f   libucrt:invalid_parameter.obj
 0001:00013689       __invalid_parameter_noinfo 10014689 f   libucrt:invalid_parameter.obj
 0001:00013699       __invoke_watson            10014699 f   libucrt:invalid_parameter.obj
 0001:000136cd       ___acrt_errno_from_os_error 100146cd f   libucrt:errno.obj
 0001:00013710       ___acrt_errno_map_os_error 10014710 f   libucrt:errno.obj
 0001:00013733       ___doserrno                10014733 f   libucrt:errno.obj
 0001:00013746       __errno                    10014746 f   libucrt:errno.obj
 0001:00013759       __calloc_base              10014759 f   libucrt:calloc_base.obj
 0001:000137b6       __free_base                100147b6 f   libucrt:free_base.obj
 0001:00013b2e       ___acrt_freeptd            10014b2e f   libucrt:per_thread_data.obj
 0001:00013b5a       ___acrt_getptd             10014b5a f   libucrt:per_thread_data.obj
 0001:00013c17       ___acrt_getptd_head        10014c17 f   libucrt:per_thread_data.obj
 0001:00013cb1       ___acrt_getptd_noexit      10014cb1 f   libucrt:per_thread_data.obj
 0001:00013d66       ___acrt_initialize_ptd     10014d66 f   libucrt:per_thread_data.obj
 0001:00013d92       ___acrt_uninitialize_ptd   10014d92 f   libucrt:per_thread_data.obj
 0001:00013f5e       ___acrt_AppPolicyGetProcessTerminationMethodInternal@4 10014f5e f   libucrt:winapi_thunks.obj
 0001:00013f9e       ___acrt_AppPolicyGetThreadInitializationTypeInternal@4 10014f9e f   libucrt:winapi_thunks.obj
 0001:00013fde       ___acrt_AreFileApisANSI@0  10014fde f   libucrt:winapi_thunks.obj
 0001:00013ffd       ___acrt_CompareStringEx@36 10014ffd f   libucrt:winapi_thunks.obj
 0001:0001405a       ___acrt_FlsAlloc@4         1001505a f   libucrt:winapi_thunks.obj
 0001:00014099       ___acrt_FlsFree@4          10015099 f   libucrt:winapi_thunks.obj
 0001:000140d8       ___acrt_FlsGetValue@4      100150d8 f   libucrt:winapi_thunks.obj
 0001:00014117       ___acrt_FlsSetValue@8      10015117 f   libucrt:winapi_thunks.obj
 0001:00014159       ___acrt_InitializeCriticalSectionEx@12 10015159 f   libucrt:winapi_thunks.obj
 0001:000141a4       ___acrt_LCMapStringEx@36   100151a4 f   libucrt:winapi_thunks.obj
 0001:00014201       ___acrt_LocaleNameToLCID@8 10015201 f   libucrt:winapi_thunks.obj
 0001:00014232       ___acrt_RoInitialize@4     10015232 f   libucrt:winapi_thunks.obj
 0001:0001426d       ___acrt_RoUninitialize@0   1001526d f   libucrt:winapi_thunks.obj
 0001:0001429b       ___acrt_initialize_winapi_thunks 1001529b f   libucrt:winapi_thunks.obj
 0001:000142c6       ___acrt_uninitialize_winapi_thunks 100152c6 f   libucrt:winapi_thunks.obj
 0001:000142fc       ___acrt_get_begin_thread_init_policy 100152fc f   libucrt:win_policies.obj
 0001:00014340       ___acrt_get_process_end_policy 10015340 f   libucrt:win_policies.obj
 0001:00014371       __fcloseall                10015371 f   libucrt:closeall.obj
 0001:000145f9       ___acrt_stdio_flush_nolock 100155f9 f   libucrt:fflush.obj
 0001:0001465e       __fflush_nolock            1001565e f   libucrt:fflush.obj
 0001:000146a6       __flushall                 100156a6 f   libucrt:fflush.obj
 0001:000146af       ___acrt_stdio_free_buffer_nolock 100156af f   libucrt:_freebuf.obj
 0001:00014859       ___acrt_initialize_lowio   10015859 f   libucrt:ioinit.obj
 0001:000148b9       ___acrt_uninitialize_lowio 100158b9 f   libucrt:ioinit.obj
 0001:000148e5       __malloc_base              100158e5 f   libucrt:malloc_base.obj
 0001:00014933       ??$make_c_string_character_source@_WPAPA_W@__crt_strtox@@YA?AV?$c_string_character_source@_W@0@QB_WQAPA_W@Z 10015933 f i libucrt:strtox.obj
 0001:00014933       ??$make_c_string_character_source@DPAPAD@__crt_strtox@@YA?AV?$c_string_character_source@D@0@QBDQAPAD@Z 10015933 f i libucrt:strtox.obj
 0001:0001494e       _strtol                    1001594e f   libucrt:strtox.obj
 0001:00014978       _wcstol                    10015978 f   libucrt:strtox.obj
 0001:000149a2       __mbtowc_l                 100159a2 f   libucrt:mbtowc.obj
 0001:00014ae4       _mbtowc                    10015ae4 f   libucrt:mbtowc.obj
 0001:00014afe       __wctomb_s_l               10015afe f   libucrt:wctomb.obj
 0001:00014c59       _wctomb_s                  10015c59 f   libucrt:wctomb.obj
 0001:00014c76       ___acrt_update_locale_info 10015c76 f   libucrt:locale_update.obj
 0001:00014ca3       ___acrt_update_multibyte_info 10015ca3 f   libucrt:locale_update.obj
 0001:00014cd0       ?__acrt_fp_classify@@YA?AW4__acrt_fp_class@@ABN@Z 10015cd0 f i libucrt:cvt.obj
 0001:0001551b       ___acrt_fp_format          1001651b f   libucrt:cvt.obj
 0001:00015686       __fputwc_nolock            10016686 f   libucrt:fputwc.obj
 0001:000157af       __fileno                   100167af f   libucrt:fileno.obj
 0001:000157d6       __fputc_nolock             100167d6 f   libucrt:fputc.obj
 0001:000157ff       __get_printf_count_output  100167ff f   libucrt:printf_count_output.obj
 0001:00015814       ___acrt_stdio_begin_temporary_buffering_nolock 10016814 f   libucrt:_sftbuf.obj
 0001:000158c7       ___acrt_stdio_end_temporary_buffering_nolock 100168c7 f   libucrt:_sftbuf.obj
 0001:0001596f       ___acrt_set_locale_changed 1001696f f   libucrt:wsetlocale.obj
 0001:0001597a       ___acrt_uninitialize_locale 1001697a f   libucrt:wsetlocale.obj
 0001:00015a2d       __close                    10016a2d f   libucrt:close.obj
 0001:00015aba       __close_nolock             10016aba f   libucrt:close.obj
 0001:00015b56       ?__acrt_stdio_allocate_stream@@YA?AV__crt_stdio_stream@@XZ 10016b56 f   libucrt:stream.obj
 0001:00015bbf       ?__acrt_stdio_free_stream@@YAXV__crt_stdio_stream@@@Z 10016bbf f   libucrt:stream.obj
 0001:00015cbc       ??$__acrt_stdio_parse_mode@D@@YA?AU__acrt_stdio_stream_mode@@QBD@Z 10016cbc f i libucrt:openfile.obj
 0001:00015f69       ?__acrt_stdio_parse_mode_D@@YA_NAAU__acrt_stdio_stream_mode@@@Z 10016f69 f i libucrt:openfile.obj
 0001:00015f84       ?__acrt_stdio_parse_mode_T@@YA_NAAU__acrt_stdio_stream_mode@@@Z 10016f84 f i libucrt:openfile.obj
 0001:00015fa3       ?__acrt_stdio_parse_mode_b@@YA_NAAU__acrt_stdio_stream_mode@@@Z 10016fa3 f i libucrt:openfile.obj
 0001:00015fc3       ?__acrt_stdio_parse_mode_c@@YA_NAAU__acrt_stdio_stream_mode@@AA_N@Z 10016fc3 f i libucrt:openfile.obj
 0001:00015fe5       ?__acrt_stdio_parse_mode_n@@YA_NAAU__acrt_stdio_stream_mode@@AA_N@Z 10016fe5 f i libucrt:openfile.obj
 0001:00016007       ?__acrt_stdio_parse_mode_plus@@YA_NAAU__acrt_stdio_stream_mode@@AA_N@Z 10017007 f i libucrt:openfile.obj
 0001:0001603d       ?__acrt_stdio_parse_mode_t@@YA_NAAU__acrt_stdio_stream_mode@@@Z 1001703d f i libucrt:openfile.obj
 0001:0001605d       ?__acrt_stdio_parse_mode_x@@YA_NAAU__acrt_stdio_stream_mode@@@Z 1001705d f i libucrt:openfile.obj
 0001:0001607d       __openfile                 1001707d f   libucrt:openfile.obj
 0001:00016088       __strnicoll                10017088 f   libucrt:strnicol.obj
 0001:000160b1       __strnicoll_l              100170b1 f   libucrt:strnicol.obj
 0001:00016179       ___acrt_initialize_locks   10017179 f   libucrt:locks.obj
 0001:000161ba       ___acrt_lock               100171ba f   libucrt:locks.obj
 0001:000161d1       ___acrt_uninitialize_locks 100171d1 f   libucrt:locks.obj
 0001:00016202       ___acrt_unlock             10017202 f   libucrt:locks.obj
 0001:000163b2       ??$__acrt_mbs_to_wcs_cp@U__crt_win32_buffer_internal_dynamic_resizing@@@@YAHQBDAAV?$__crt_win32_buffer@_WU__crt_win32_buffer_internal_dynamic_resizing@@@@I@Z 100173b2 f i libucrt:argv_wildcards.obj
 0001:000168c6       ?__acrt_get_utf8_acp_compatibility_codepage@@YAIXZ 100178c6 f i libucrt:argv_wildcards.obj
 0001:00016905       ?_deallocate@?$__crt_win32_buffer@DU__crt_win32_buffer_internal_dynamic_resizing@@@@AAEXXZ 10017905 f i libucrt:argv_wildcards.obj
 0001:00016905       ?_deallocate@?$__crt_win32_buffer@_WU__crt_win32_buffer_internal_dynamic_resizing@@@@AAEXXZ 10017905 f i libucrt:argv_wildcards.obj
 0001:0001691f       ?allocate@?$__crt_win32_buffer@DU__crt_win32_buffer_internal_dynamic_resizing@@@@QAEHI@Z 1001791f f i libucrt:argv_wildcards.obj
 0001:0001695b       ?allocate@?$__crt_win32_buffer@_WU__crt_win32_buffer_internal_dynamic_resizing@@@@QAEHI@Z 1001795b f i libucrt:argv_wildcards.obj
 0001:0001699a       ?allocate@__crt_win32_buffer_internal_dynamic_resizing@@SAHQAPAXIABV__crt_win32_buffer_empty_debug_info@@@Z 1001799a f i libucrt:argv_wildcards.obj
 0001:00016a40       ___acrt_expand_narrow_argv_wildcards 10017a40 f   libucrt:argv_wildcards.obj
 0001:00016b12       ?allocate@?$__crt_win32_buffer@DU__crt_win32_buffer_no_resizing@@@@QAEHI@Z 10017b12 f i libucrt:getmodulefilenamea.obj
 0001:00016b39       ?set_to_nullptr@?$__crt_win32_buffer@DU__crt_win32_buffer_no_resizing@@@@QAEXXZ 10017b39 f i libucrt:getmodulefilenamea.obj
 0001:00016b4d       ___acrt_GetModuleFileNameA 10017b4d f   libucrt:getmodulefilenamea.obj
 0001:0001710c       ___acrt_initialize_multibyte 1001810c f   libucrt:mbctype.obj
 0001:00017154       ___acrt_update_thread_multibyte_data 10018154 f   libucrt:mbctype.obj
 0001:00017167       __setmbcp_nolock           10018167 f   libucrt:mbctype.obj
 0001:00017432       __ismbblead                10018432 f   libucrt:ismbbyte.obj
 0001:0001744a       ___acrt_initialize_command_line 1001844a f   libucrt:argv_data.obj
 0001:00017463       ___acrt_MultiByteToWideChar 10018463 f   libucrt:multibytetowidechar.obj
 0001:000174df       ___acrt_WideCharToMultiByte 100184df f   libucrt:widechartomultibyte.obj
 0001:000175c3       ___dcrt_get_narrow_environment_from_os 100185c3 f   libucrt:get_environment_from_os.obj
 0001:000179a4       ___dcrt_set_variable_in_narrow_environment_nolock 100189a4 f   libucrt:setenv.obj
 0001:000179af       __recalloc_base            100189af f   libucrt:recalloc.obj
 0001:00017a1c       ___acrt_initialize_heap    10018a1c f   libucrt:heap_handle.obj
 0001:00017a2d       ___acrt_uninitialize_heap  10018a2d f   libucrt:heap_handle.obj
 0001:00017a37       ___acrt_execute_initializers 10018a37 f   libucrt:shared_initialization.obj
 0001:00017a9f       ___acrt_execute_uninitializers 10018a9f f   libucrt:shared_initialization.obj
 0001:00017b9e       ___acrt_get_sigabrt_handler 10018b9e f   libucrt:signal.obj
 0001:00017bc5       ___acrt_initialize_signal_handlers 10018bc5 f   libucrt:signal.obj
 0001:00017be3       ___fpecode                 10018be3 f   libucrt:signal.obj
 0001:00017bec       _raise                     10018bec f   libucrt:signal.obj
 0001:00017de7       ___acrt_has_user_matherr   10018de7 f   libucrt:matherr.obj
 0001:00017dff       ___acrt_initialize_user_matherr 10018dff f   libucrt:matherr.obj
 0001:00017e0e       ___acrt_invoke_user_matherr 10018e0e f   libucrt:matherr.obj
 0001:00017e40       ___pctype_func             10018e40 f   libucrt:ctype.obj
 0001:00017e64       _iswctype                  10018e64 f   libucrt:iswctype.obj
 0001:00017ecd       __isctype_l                10018ecd f   libucrt:isctype.obj
 0001:00017f98       __query_new_mode           10018f98 f   libucrt:new_mode.obj
 0001:00017f9f       ___acrt_add_locale_ref     10018f9f f   libucrt:locale_refcounting.obj
 0001:0001801c       ___acrt_free_locale        1001901c f   libucrt:locale_refcounting.obj
 0001:00018164       ___acrt_locale_add_lc_time_reference 10019164 f   libucrt:locale_refcounting.obj
 0001:0001818d       ___acrt_locale_free_lc_time_if_unreferenced 1001918d f   libucrt:locale_refcounting.obj
 0001:000181be       ___acrt_locale_release_lc_time_reference 100191be f   libucrt:locale_refcounting.obj
 0001:000181e7       ___acrt_release_locale_ref 100191e7 f   libucrt:locale_refcounting.obj
 0001:00018268       ___acrt_update_thread_locale_data 10019268 f   libucrt:locale_refcounting.obj
 0001:000182e9       __updatetlocinfoEx_nolock  100192e9 f   libucrt:locale_refcounting.obj
 0001:00018389       ___acrt_DownlevelLocaleNameToLCID 10019389 f   libucrt:lcidtoname_downlevel.obj
 0001:00018457       __commit                   10019457 f   libucrt:commit.obj
 0001:00018c4d       __write                    10019c4d f   libucrt:write.obj
 0001:00018d3f       __write_nolock             10019d3f f   libucrt:write.obj
 0001:00018f21       ___acrt_lowio_create_handle_array 10019f21 f   libucrt:osfinfo.obj
 0001:00018f9c       ___acrt_lowio_destroy_handle_array 10019f9c f   libucrt:osfinfo.obj
 0001:00018fd1       ___acrt_lowio_ensure_fh_exists 10019fd1 f   libucrt:osfinfo.obj
 0001:0001906f       ___acrt_lowio_lock_fh      1001a06f f   libucrt:osfinfo.obj
 0001:00019092       ___acrt_lowio_set_os_handle 1001a092 f   libucrt:osfinfo.obj
 0001:00019124       ___acrt_lowio_unlock_fh    1001a124 f   libucrt:osfinfo.obj
 0001:00019147       __alloc_osfhnd             1001a147 f   libucrt:osfinfo.obj
 0001:0001925a       __free_osfhnd              1001a25a f   libucrt:osfinfo.obj
 0001:000192eb       __get_osfhandle            1001a2eb f   libucrt:osfinfo.obj
 0001:00019355       __isleadbyte_l             1001a355 f i libucrt:_wctype.obj
 0001:000193bb       ?__mbrtowc_utf8@__crt_mbstring@@YAIPA_WPBDIPAU_Mbstatet@@@Z 1001a3bb f   libucrt:mbrtowc.obj
 0001:000193fb       ?__mbsrtowcs_utf8@__crt_mbstring@@YAIPA_WPAPBDIPAU_Mbstatet@@@Z 1001a3fb f   libucrt:mbrtowc.obj
 0001:000194f6       ?__c32rtomb_utf8@__crt_mbstring@@YAIPAD_UPAU_Mbstatet@@@Z 1001a4f6 f   libucrt:c32rtomb.obj
 0001:000195a1       ?return_illegal_sequence@__crt_mbstring@@YAIPAU_Mbstatet@@@Z 1001a5a1 f i libucrt:c32rtomb.obj
 0001:000195c0       ___acrt_fp_strflt_to_string 1001a5c0 f   libucrt:_fptostr.obj
 0001:00019680       ?divide@__crt_strtox@@YA_KAAUbig_integer@1@ABU21@@Z 1001a680 f i libucrt:cfout.obj
 0001:00019b18       ___acrt_fltout             1001ab18 f   libucrt:cfout.obj
 0001:0001b2af       ___acrt_stdio_flush_and_write_narrow_nolock 1001c2af f   libucrt:_flsbuf.obj
 0001:0001b2ba       ___acrt_stdio_flush_and_write_wide_nolock 1001c2ba f   libucrt:_flsbuf.obj
 0001:0001b2c5       __isatty                   1001c2c5 f   libucrt:isatty.obj
 0001:0001b31b       ___acrt_locale_free_monetary 1001c31b f   libucrt:initmon.obj
 0001:0001b419       ___acrt_locale_free_numeric 1001c419 f   libucrt:initnum.obj
 0001:0001b4ba       ___acrt_locale_free_time   1001c4ba f   libucrt:inittime.obj
 0001:0001b59e       ___acrt_GetStringTypeA     1001c59e f   libucrt:getstringtypea.obj
 0001:0001b6a1       __freea_crt                1001c6a1 f i libucrt:getstringtypea.obj
 0001:0001b6c1       ___ascii_wcsnicmp          1001c6c1 f   libucrt:wcsnicmp.obj
 0001:0001b710       __strnicmp                 1001c710 f   libucrt:strnicmp.obj
 0001:0001b77d       __strnicmp_l               1001c77d f   libucrt:strnicmp.obj
 0001:0001be13       __sopen_nolock             1001ce13 f   libucrt:open.obj
 0001:0001be81       __sopen_s                  1001ce81 f   libucrt:open.obj
 0001:0001bea4       __wsopen_nolock            1001cea4 f   libucrt:open.obj
 0001:0001c459       ___acrt_CompareStringA     1001d459 f   libucrt:comparestringa.obj
 0001:0001c4e0       _qsort                     1001d4e0 f   libucrt:qsort.obj
 0001:0001c9d7       _strncpy_s                 1001d9d7 f   libucrt:strncpy_s.obj
 0001:0001c9f0       _strpbrk                   1001d9f0 f   libucrt:strpbrk.obj
 0001:0001ca30       __mbsdec                   1001da30 f   libucrt:mbsdec.obj
 0001:0001ca47       __mbsdec_l                 1001da47 f   libucrt:mbsdec.obj
 0001:0001ccbe       ___acrt_LCMapStringA       1001dcbe f   libucrt:lcmapstringa.obj
 0001:0001cd16       ___acrt_SetEnvironmentVariableA 1001dd16 f   libucrt:setenvironmentvariablea.obj
 0001:0001cdab       __msize_base               1001ddab f   libucrt:msize.obj
 0001:0001cdde       __realloc_base             1001ddde f   libucrt:realloc_base.obj
 0001:0001ce47       ___acrt_GetStringTypeW     1001de47 f   libucrt:getstringtypew.obj
 0001:0001cfe8       __lseeki64                 1001dfe8 f   libucrt:lseek.obj
 0001:0001d003       __lseeki64_nolock          1001e003 f   libucrt:lseek.obj
 0001:0001d01e       __putwch_nolock            1001e01e f   libucrt:putwch.obj
 0001:0001d554       __read_nolock              1001e554 f   libucrt:read.obj
 0001:0001d904       __query_app_type           1001e904 f   libucrt:report_runtime_error.obj
 0001:0001d90a       ?__mbrtoc32_utf8@__crt_mbstring@@YAIPA_UPBDIPAU_Mbstatet@@@Z 1001e90a f   libucrt:mbrtoc32.obj
 0001:0001dab1       _fegetenv                  1001eab1 f   libucrt:fegetenv.obj
 0001:0001dace       _fesetenv                  1001eace f   libucrt:fesetenv.obj
 0001:0001db19       _feholdexcept              1001eb19 f   libucrt:feholdexcept.obj
 0001:0001db70       __CIlog10                  1001eb70 f   libucrt:log10_impl.obj
 0001:0001dbab       __CIlog10_default          1001ebab f   libucrt:log10_impl.obj
 0001:0001dbbf       __log10_default            1001ebbf     libucrt:log10_impl.obj
 0001:0001dc80       _ceil                      1001ec80 f   libucrt:ceil_pentium4.obj
 0001:0001dcc0       __ceil_pentium4            1001ecc0 f   libucrt:ceil_pentium4.obj
 0001:0001dd9d       ___acrt_stdio_allocate_buffer_nolock 1001ed9d f   libucrt:_getbuf.obj
 0001:0001de00       ___ascii_strnicmp          1001ee00 f   libucrt:_strnicm.obj
 0001:0001de61       __get_fmode                1001ee61 f   libucrt:setmode.obj
 0001:0001de8e       __setmode_nolock           1001ee8e f   libucrt:setmode.obj
 0001:0001df5d       ??0__crt_seek_guard@@QAE@H_J@Z 1001ef5d f i libucrt:chsize.obj
 0001:0001dfaa       __chsize_nolock            1001efaa f   libucrt:chsize.obj
 0001:0001e11a       ___strncnt                 1001f11a f   libucrt:strncnt.obj
 0001:0001e155       ___dcrt_lowio_ensure_console_output_initialized 1001f155 f   libucrt:initcon.obj
 0001:0001e174       ___dcrt_terminate_console_output 1001f174 f   libucrt:initcon.obj
 0001:0001e18b       ___dcrt_write_console      1001f18b f   libucrt:initcon.obj
 0001:0001e4ed       ___acrt_fenv_get_control   1001f4ed f   libucrt:_fenvutils.obj
 0001:0001e56d       ___acrt_fenv_get_status    1001f56d f   libucrt:_fenvutils.obj
 0001:0001e625       ___acrt_fenv_set_control   1001f625 f   libucrt:_fenvutils.obj
 0001:0001e68d       ___acrt_fenv_set_status    1001f68d f   libucrt:_fenvutils.obj
 0001:0001e784       __clearfp                  1001f784 f   libucrt:ieee87.obj
 0001:0001e862       ___acrt_initialize_sse2    1001f862 f   libucrt:mathfcns.obj
 0001:0001e880       __CIlog10_pentium4         1001f880 f   libucrt:log10_pentium4.obj
 0001:0001e898       __log10_pentium4           1001f898     libucrt:log10_pentium4.obj
 0001:0001eb30       __fFEXP                    1001fb30 f   libucrt:87tran.obj
 0001:0001eb87       __rtinfpopse               1001fb87     libucrt:87tran.obj
 0001:0001eb89       __rtinfnpopse              1001fb89     libucrt:87tran.obj
 0001:0001eb99       __fFLN                     1001fb99     libucrt:87tran.obj
 0001:0001ec4e       __rtinfpop                 1001fc4e     libucrt:87tran.obj
 0001:0001ec50       __rtinfnpop                1001fc50     libucrt:87tran.obj
 0001:0001ec60       __rtforexpinf              1001fc60 f   libucrt:87tran.obj
 0001:0001ec6d       __ffexpm1                  1001fc6d     libucrt:87tran.obj
 0001:0001ed20       __trandisp1                1001fd20 f   libucrt:87disp.obj
 0001:0001ed95       __trandisp2                1001fd95 f   libucrt:87disp.obj
 0001:0001ee2f       __rttospopde               1001fe2f     libucrt:87disp.obj
 0001:0001ee34       __rttospop                 1001fe34     libucrt:87disp.obj
 0001:0001ee40       __rtnospop                 1001fe40 f   libucrt:87disp.obj
 0001:0001ee50       __rttosnpop                1001fe50 f   libucrt:87disp.obj
 0001:0001ee51       __rtnospopde               1001fe51     libucrt:87disp.obj
 0001:0001ee58       __rtzeropop                1001fe58     libucrt:87disp.obj
 0001:0001ee5a       __rtzeronpop               1001fe5a     libucrt:87disp.obj
 0001:0001ee60       __rtzerospop               1001fe60 f   libucrt:87disp.obj
 0001:0001ee6d       __rtonepop                 1001fe6d     libucrt:87disp.obj
 0001:0001ee70       __rtonenpop                1001fe70 f   libucrt:87disp.obj
 0001:0001ee80       __tosnan1                  1001fe80 f   libucrt:87disp.obj
 0001:0001eeb0       __nosnan2                  1001feb0 f   libucrt:87disp.obj
 0001:0001eec0       __tosnan2                  1001fec0 f   libucrt:87disp.obj
 0001:0001eef0       __nan2                     1001fef0 f   libucrt:87disp.obj
 0001:0001ef30       __rtindfpop                1001ff30 f   libucrt:87disp.obj
 0001:0001ef32       __rtindfnpop               1001ff32     libucrt:87disp.obj
 0001:0001ef43       __rttosnpopde              1001ff43     libucrt:87disp.obj
 0001:0001ef50       __rtatan2inf               1001ff50 f   libucrt:87disp.obj
 0001:0001ef6d       __rtchsifneg               1001ff6d     libucrt:87disp.obj
 0001:0001ef80       __twoToTOS                 1001ff80 f   libucrt:common.obj
 0001:0001ef95       __load_CW                  1001ff95 f   libucrt:common.obj
 0001:0001efac       __convertTOStoQNaN         1001ffac f   libucrt:common.obj
 0001:0001efc5       __fload_withFB             1001ffc5 f   libucrt:common.obj
 0001:0001f008       __checkTOS_withFB          10020008 f   libucrt:common.obj
 0001:0001f01e       __fast_exit                1002001e f   libucrt:common.obj
 0001:0001f02b       __math_exit                1002002b f   libucrt:common.obj
 0001:0001f055       __check_overflow_exit      10020055 f   libucrt:common.obj
 0001:0001f069       __check_range_exit         10020069 f   libucrt:common.obj
 0001:0001f110       __startTwoArgErrorHandling 10020110 f   libucrt:genexcep.obj
 0001:0001f127       __startOneArgErrorHandling 10020127 f   libucrt:genexcep.obj
 0001:0001f163       ___libm_error_support      10020163 f   libucrt:libm_error.obj
 0001:0001f357       __ceil_default             10020357 f   libucrt:ceil.obj
 0001:0001f40c       __clrfp                    1002040c f   libucrt:fpctrl.obj
 0001:0001f41d       __ctrlfp                   1002041d f   libucrt:fpctrl.obj
 0001:0001f447       __set_statfp               10020447 f   libucrt:fpctrl.obj
 0001:0001f4a0       __statfp                   100204a0 f   libucrt:fpctrl.obj
 0001:0001f4b0       __d_inttype                100204b0 f   libucrt:powhlp.obj
 0001:0001f518       __powhlp                   10020518 f   libucrt:powhlp.obj
 0001:0001f643       __87except                 10020643 f   libucrt:87except.obj
 0001:0001f74d       __frnd                     1002074d f   libucrt:frnd.obj
 0001:0001f761       __errcode                  10020761 f   libucrt:fpexcept.obj
 0001:0001f795       __except1                  10020795 f   libucrt:fpexcept.obj
 0001:0001f863       __handle_exc               10020863 f   libucrt:fpexcept.obj
 0001:0001fa4e       __raise_exc                10020a4e f   libucrt:fpexcept.obj
 0001:0001fa71       __raise_exc_ex             10020a71 f   libucrt:fpexcept.obj
 0001:0001fd67       __set_errno_from_matherr   10020d67 f   libucrt:fpexcept.obj
 0001:0001fd96       __umatherr                 10020d96 f   libucrt:fpexcept.obj
 0001:0001fe36       __decomp                   10020e36 f   libucrt:util.obj
 0001:0001ff08       __set_exp                  10020f08 f   libucrt:util.obj
 0001:0001ff35       __sptype                   10020f35 f   libucrt:util.obj
 0001:0001ff93       __fpclass                  10020f93 f   libucrt:ieeemisc.obj
 0001:00020037       _IsProcessorFeaturePresent@4 10021037 f   kernel32:KERNEL32.dll
 0001:00020040       __FindPESection            10021040 f   LIBCMT:pesect.obj
 0001:00020090       __IsNonwritableInCurrentImage 10021090 f   LIBCMT:pesect.obj
 0001:00020150       __ValidateImageBase        10021150 f   LIBCMT:pesect.obj
 0001:00020190       __aulldvrm                 10021190 f   LIBCMT:ulldvrm.obj
 0001:00020230       __allmul                   10021230 f   LIBCMT:llmul.obj
 0001:00020270       __alldvrm                  10021270 f   LIBCMT:lldvrm.obj
 0001:00020350       __aullshr                  10021350 f   LIBCMT:ullshr.obj
 0001:00020370       __chkstk                   10021370 f   LIBCMT:chkstk.obj
 0001:00020370       __alloca_probe             10021370 f   LIBCMT:chkstk.obj
 0001:000203a0       __allshl                   100213a0 f   LIBCMT:llshl.obj
 0001:000203c0       __ftol2_sse                100213c0     LIBCMT:ftol2.obj
 0001:000203c0       __ftol2_sse_excpt          100213c0     LIBCMT:ftol2.obj
 0001:000203c0       __ftoi2                    100213c0 f   LIBCMT:ftol2.obj
 0001:00020440       __ftoui2                   10021440 f   LIBCMT:ftol2.obj
 0001:000204f0       __ftol2                    100214f0 f   LIBCMT:ftol2.obj
 0001:000205a0       __ftoul2                   100215a0 f   LIBCMT:ftol2.obj
 0001:00020660       __alloca_probe_16          10021660 f   LIBCMT:alloca16.obj
 0001:00020676       __alloca_probe_8           10021676     LIBCMT:alloca16.obj
 0001:00020690       _strrchr                   10021690 f   libvcruntime:strrchr.obj
 0001:000207d0       _strchr                    100217d0 f   libvcruntime:strchr.obj
 0001:0002083e       ___from_strstr_to_strchr   1002183e     libvcruntime:strchr.obj
 0001:000208fb       __filter_x86_sse2_floating_point_exception 100218fb f   LIBCMT:x86_exception_filter.obj
 0001:000208fb       __filter_x86_sse2_floating_point_exception_default 100218fb f   LIBCMT:x86_exception_filter.obj
 0002:00000000       __imp__CloseHandle@4       10022000     kernel32:KERNEL32.dll
 0002:00000004       __imp__GetLastError@0      10022004     kernel32:KERNEL32.dll
 0002:00000008       __imp__MapViewOfFile@20    10022008     kernel32:KERNEL32.dll
 0002:0000000c       __imp__UnmapViewOfFile@4   1002200c     kernel32:KERNEL32.dll
 0002:00000010       __imp__OpenFileMappingA@12 10022010     kernel32:KERNEL32.dll
 0002:00000014       __imp__GetSystemTimeAsFileTime@4 10022014     kernel32:KERNEL32.dll
 0002:00000018       __imp__InitializeCriticalSection@4 10022018     kernel32:KERNEL32.dll
 0002:0000001c       __imp__EnterCriticalSection@4 1002201c     kernel32:KERNEL32.dll
 0002:00000020       __imp__LeaveCriticalSection@4 10022020     kernel32:KERNEL32.dll
 0002:00000024       __imp__DeleteCriticalSection@4 10022024     kernel32:KERNEL32.dll
 0002:00000028       __imp__Sleep@4             10022028     kernel32:KERNEL32.dll
 0002:0000002c       __imp__WriteConsoleW@20    1002202c     kernel32:KERNEL32.dll
 0002:00000030       __imp__SetEndOfFile@4      10022030     kernel32:KERNEL32.dll
 0002:00000034       __imp__ReadConsoleW@20     10022034     kernel32:KERNEL32.dll
 0002:00000038       __imp__ReadFile@20         10022038     kernel32:KERNEL32.dll
 0002:0000003c       __imp__HeapReAlloc@16      1002203c     kernel32:KERNEL32.dll
 0002:00000040       __imp__HeapSize@12         10022040     kernel32:KERNEL32.dll
 0002:00000044       __imp__CreateFileW@28      10022044     kernel32:KERNEL32.dll
 0002:00000048       __imp__GetStringTypeW@16   10022048     kernel32:KERNEL32.dll
 0002:0000004c       __imp__SetFilePointerEx@20 1002204c     kernel32:KERNEL32.dll
 0002:00000050       __imp__GetFileSizeEx@8     10022050     kernel32:KERNEL32.dll
 0002:00000054       __imp__SetStdHandle@8      10022054     kernel32:KERNEL32.dll
 0002:00000058       __imp__GetConsoleMode@8    10022058     kernel32:KERNEL32.dll
 0002:0000005c       __imp__UnhandledExceptionFilter@4 1002205c     kernel32:KERNEL32.dll
 0002:00000060       __imp__SetUnhandledExceptionFilter@4 10022060     kernel32:KERNEL32.dll
 0002:00000064       __imp__GetCurrentProcess@0 10022064     kernel32:KERNEL32.dll
 0002:00000068       __imp__TerminateProcess@8  10022068     kernel32:KERNEL32.dll
 0002:0000006c       __imp__IsProcessorFeaturePresent@4 1002206c     kernel32:KERNEL32.dll
 0002:00000070       __imp__QueryPerformanceCounter@4 10022070     kernel32:KERNEL32.dll
 0002:00000074       __imp__GetCurrentProcessId@0 10022074     kernel32:KERNEL32.dll
 0002:00000078       __imp__GetCurrentThreadId@0 10022078     kernel32:KERNEL32.dll
 0002:0000007c       __imp__InitializeSListHead@4 1002207c     kernel32:KERNEL32.dll
 0002:00000080       __imp__IsDebuggerPresent@0 10022080     kernel32:KERNEL32.dll
 0002:00000084       __imp__GetStartupInfoW@4   10022084     kernel32:KERNEL32.dll
 0002:00000088       __imp__GetModuleHandleW@4  10022088     kernel32:KERNEL32.dll
 0002:0000008c       __imp__RaiseException@16   1002208c     kernel32:KERNEL32.dll
 0002:00000090       __imp__InterlockedFlushSList@4 10022090     kernel32:KERNEL32.dll
 0002:00000094       __imp__RtlUnwind@16        10022094     kernel32:KERNEL32.dll
 0002:00000098       __imp__SetLastError@4      10022098     kernel32:KERNEL32.dll
 0002:0000009c       __imp__InitializeCriticalSectionAndSpinCount@8 1002209c     kernel32:KERNEL32.dll
 0002:000000a0       __imp__TlsAlloc@0          100220a0     kernel32:KERNEL32.dll
 0002:000000a4       __imp__TlsGetValue@4       100220a4     kernel32:KERNEL32.dll
 0002:000000a8       __imp__TlsSetValue@8       100220a8     kernel32:KERNEL32.dll
 0002:000000ac       __imp__TlsFree@4           100220ac     kernel32:KERNEL32.dll
 0002:000000b0       __imp__FreeLibrary@4       100220b0     kernel32:KERNEL32.dll
 0002:000000b4       __imp__GetProcAddress@8    100220b4     kernel32:KERNEL32.dll
 0002:000000b8       __imp__LoadLibraryExW@12   100220b8     kernel32:KERNEL32.dll
 0002:000000bc       __imp__CreateThread@24     100220bc     kernel32:KERNEL32.dll
 0002:000000c0       __imp__ExitThread@4        100220c0     kernel32:KERNEL32.dll
 0002:000000c4       __imp__FreeLibraryAndExitThread@8 100220c4     kernel32:KERNEL32.dll
 0002:000000c8       __imp__GetModuleHandleExW@12 100220c8     kernel32:KERNEL32.dll
 0002:000000cc       __imp__ExitProcess@4       100220cc     kernel32:KERNEL32.dll
 0002:000000d0       __imp__GetModuleFileNameW@12 100220d0     kernel32:KERNEL32.dll
 0002:000000d4       __imp__HeapAlloc@12        100220d4     kernel32:KERNEL32.dll
 0002:000000d8       __imp__HeapFree@12         100220d8     kernel32:KERNEL32.dll
 0002:000000dc       __imp__CompareStringW@24   100220dc     kernel32:KERNEL32.dll
 0002:000000e0       __imp__LCMapStringW@24     100220e0     kernel32:KERNEL32.dll
 0002:000000e4       __imp__GetStdHandle@4      100220e4     kernel32:KERNEL32.dll
 0002:000000e8       __imp__GetFileType@4       100220e8     kernel32:KERNEL32.dll
 0002:000000ec       __imp__FindClose@4         100220ec     kernel32:KERNEL32.dll
 0002:000000f0       __imp__FindFirstFileExW@24 100220f0     kernel32:KERNEL32.dll
 0002:000000f4       __imp__FindNextFileW@8     100220f4     kernel32:KERNEL32.dll
 0002:000000f8       __imp__IsValidCodePage@4   100220f8     kernel32:KERNEL32.dll
 0002:000000fc       __imp__GetACP@0            100220fc     kernel32:KERNEL32.dll
 0002:00000100       __imp__GetOEMCP@0          10022100     kernel32:KERNEL32.dll
 0002:00000104       __imp__GetCPInfo@8         10022104     kernel32:KERNEL32.dll
 0002:00000108       __imp__GetCommandLineA@0   10022108     kernel32:KERNEL32.dll
 0002:0000010c       __imp__GetCommandLineW@0   1002210c     kernel32:KERNEL32.dll
 0002:00000110       __imp__MultiByteToWideChar@24 10022110     kernel32:KERNEL32.dll
 0002:00000114       __imp__WideCharToMultiByte@32 10022114     kernel32:KERNEL32.dll
 0002:00000118       __imp__GetEnvironmentStringsW@0 10022118     kernel32:KERNEL32.dll
 0002:0000011c       __imp__FreeEnvironmentStringsW@4 1002211c     kernel32:KERNEL32.dll
 0002:00000120       __imp__SetEnvironmentVariableW@8 10022120     kernel32:KERNEL32.dll
 0002:00000124       __imp__GetProcessHeap@0    10022124     kernel32:KERNEL32.dll
 0002:00000128       __imp__FlushFileBuffers@4  10022128     kernel32:KERNEL32.dll
 0002:0000012c       __imp__WriteFile@20        1002212c     kernel32:KERNEL32.dll
 0002:00000130       __imp__GetConsoleCP@0      10022130     kernel32:KERNEL32.dll
 0002:00000134       __imp__DecodePointer@4     10022134     kernel32:KERNEL32.dll
 0002:00000138       \177KERNEL32_NULL_THUNK_DATA 10022138     kernel32:KERNEL32.dll
 0002:0000013c       __imp__GetMessageA@16      1002213c     user32:USER32.dll
 0002:00000140       __imp__CreateDialogParamA@20 10022140     user32:USER32.dll
 0002:00000144       __imp__PostMessageA@16     10022144     user32:USER32.dll
 0002:00000148       __imp__DispatchMessageA@4  10022148     user32:USER32.dll
 0002:0000014c       __imp__TranslateMessage@4  1002214c     user32:USER32.dll
 0002:00000150       __imp__RegisterWindowMessageA@4 10022150     user32:USER32.dll
 0002:00000154       __imp__PostQuitMessage@4   10022154     user32:USER32.dll
 0002:00000158       __imp__PostThreadMessageA@16 10022158     user32:USER32.dll
 0002:0000015c       __imp__SendMessageA@16     1002215c     user32:USER32.dll
 0002:00000160       \177USER32_NULL_THUNK_DATA 10022160     user32:USER32.dll
 0002:00000164       __imp__JAWT_GetAWT@8       10022164     jawt:jawt.dll
 0002:00000168       \177jawt_NULL_THUNK_DATA   10022168     jawt:jawt.dll
 0002:0000016c       ___guard_check_icall_fptr  1002216c     LIBCMT:guard_support.obj
 0002:00000170       ___xc_a                    10022170     LIBCMT:initializers.obj
 0002:00000174       ___xc_z                    10022174     LIBCMT:initializers.obj
 0002:00000178       ___xi_a                    10022178     LIBCMT:initializers.obj
 0002:0000017c       ___acrt_stdio_initializer  1002217c     libucrt:stdio_initializer.obj
 0002:00000180       ___acrt_multibyte_initializer 10022180     libucrt:multibyte_initializer.obj
 0002:00000184       ___acrt_tran_sse2_initializer 10022184     libucrt:sse2_initializer.obj
 0002:00000188       ___xi_z                    10022188     LIBCMT:initializers.obj
 0002:0000018c       ___xp_a                    1002218c     LIBCMT:initializers.obj
 0002:00000190       ___acrt_locale_terminator  10022190     libucrt:locale_initializer.obj
 0002:00000194       ___dcrt_console_output_terminator 10022194     libucrt:console_output_initializer.obj
 0002:00000198       ___acrt_stdio_terminator   10022198     libucrt:stdio_initializer.obj
 0002:0000019c       ___xp_z                    1002219c     LIBCMT:initializers.obj
 0002:000001a0       ___xt_a                    100221a0     LIBCMT:initializers.obj
 0002:000001a4       ___xt_z                    100221a4     LIBCMT:initializers.obj
 0002:000001b0       ??_C@_0DL@PNCLIPJM@?$FLINFO?$FN?3?5in?5AccessBridgeATInstan@ 100221b0     AccessBridgeATInstance.obj
 0002:000001ec       ??_C@_0DA@ILNDDPNA@?$FLINFO?$FN?3?5?5?5unmapping?5memoryMappe@ 100221ec     AccessBridgeATInstance.obj
 0002:0000021c       ??_C@_0DJ@FCAPEKK@?$FLINFO?$FN?3?5?5?5closing?5memoryMappedF@ 1002221c     AccessBridgeATInstance.obj
 0002:00000258       ??_C@_0DB@BBBKEEOJ@?$FLINFO?$FN?3?5In?5AccessBridgeATInstan@ 10022258     AccessBridgeATInstance.obj
 0002:0000028c       ??_C@_0DJ@HCNGCGLH@?$FLERROR?$FN?3?5?5?5Failed?5to?5CreateFile@ 1002228c     AccessBridgeATInstance.obj
 0002:000002c8       ??_C@_0DC@INNGAKAO@?$FLINFO?$FN?3?5?5?5CreateFileMapping?5wor@ 100222c8     AccessBridgeATInstance.obj
 0002:000002fc       ??_C@_0DF@EKLGABNF@?$FLERROR?$FN?3?5?5?5Failed?5to?5MapViewOfF@ 100222fc     AccessBridgeATInstance.obj
 0002:00000334       ??_C@_0CK@LMLFEIHL@?$FLINFO?$FN?3?5?5?5MapViewOfFile?5worked?5@ 10022334     AccessBridgeATInstance.obj
 0002:00000360       ??_C@_03DJNNCAJF@OK?$DP@   10022360     AccessBridgeATInstance.obj
 0002:00000364       ??_C@_0DL@FPNEIEFH@?$FLERROR?$FN?3?5?5?5JavaVM?5failed?5to?5wri@ 10022364     AccessBridgeATInstance.obj
 0002:000003a0       ??_C@_0CN@CCHCHAPN@?$FLINFO?$FN?3?5?5?5JavaVM?5successfully?5w@ 100223a0     AccessBridgeATInstance.obj
 0002:000003d0       ??_C@_03ONJMBPEK@OK?$CB@   100223d0     AccessBridgeATInstance.obj
 0002:000003d8       ??_C@_0EE@MNPDBEBN@?$FLINFO?$FN?3?5AccessBridgeATInstance?3@ 100223d8     AccessBridgeATInstance.obj
 0002:00000420       ??_C@_0FI@KACFLKHC@?$FLINFO?$FN?3?5AccessBridgeATInstance?3@ 10022420     AccessBridgeATInstance.obj
 0002:00000478       ??_C@_0EN@DDCKACNO@?$FLINFO?$FN?3?5AccessBridgeATInstance?3@ 10022478     AccessBridgeATInstance.obj
 0002:000004c8       ??_C@_0BJ@FKCDJFDK@JAVA_ACCESSBRIDGE_LOGDIR@ 100224c8     AccessBridgeDebug.obj
 0002:000004e4       ??_C@_04FPOLKAEB@?4log@    100224e4     AccessBridgeDebug.obj
 0002:000004ec       ??_C@_01NOFIACDB@w@        100224ec     AccessBridgeDebug.obj
 0002:000004f0       ??_C@_04EINJHBMM@?6?$CFs?6@ 100224f0     AccessBridgeDebug.obj
 0002:000004f8       ??_C@_0BH@PPBGFLKL@Could?5not?5open?5file?5?$CFs@ 100224f8     AccessBridgeDebug.obj
 0002:00000510       ??_C@_07IBOBEFLP@?$FL?$CFllu?$FN?5@ 10022510     AccessBridgeDebug.obj
 0002:00000518       ??_C@_02PCIJFNDE@?$AN?6@   10022518     AccessBridgeDebug.obj
 0002:0000051c       ??_C@_0DD@HABIDLLD@?$FLINFO?$FN?3?5AccessBridgeJavaEntryPo@ 1002251c     AccessBridgeJavaEntryPoints.obj
 0002:00000550       ??_C@_0CI@FJHGEAOO@?$FLINFO?$FN?3?5Calling?5BuildJavaEntryP@ 10022550     AccessBridgeJavaEntryPoints.obj
 0002:00000578       ??_C@_0DB@PHGNIPBB@com?1sun?1java?1accessibility?1inte@ 10022578     AccessBridgeJavaEntryPoints.obj
 0002:000005ac       ??_C@_0CP@OJHOIDNH@?$FLERROR?$FN?3?5?5FindClass?$CI?$CFs?$CJ?5failed?$CB@ 100225ac     AccessBridgeJavaEntryPoints.obj
 0002:000005dc       ??_C@_0DE@FJPDGHPE@?$FLERROR?$FN?3?5FindClass?$CI?$CFs?$CJ?5failed?$CB?5@ 100225dc     AccessBridgeJavaEntryPoints.obj
 0002:00000610       ??_C@_0BG@JLFLBLJI@?$CILjava?1lang?1Object?$DL?$CJV@ 10022610     AccessBridgeJavaEntryPoints.obj
 0002:00000628       ??_C@_0BD@PAIEAHIF@decrementReference@ 10022628     AccessBridgeJavaEntryPoints.obj
 0002:0000063c       ??_C@_0DP@BBIEPKKN@?$FLERROR?$FN?3?5GetMethodID?$CI?$CFs?$CJ?5failed@ 1002263c     AccessBridgeJavaEntryPoints.obj
 0002:0000067c       ??_C@_0BF@FOHFOJOB@?$CI?$CJLjava?1lang?1String?$DL@ 1002267c     AccessBridgeJavaEntryPoints.obj
 0002:00000694       ??_C@_0BH@KKNMIJGK@getJavaVersionProperty@ 10022694     AccessBridgeJavaEntryPoints.obj
 0002:000006ac       ??_C@_04FJLILDCB@?$CII?$CJZ@ 100226ac     AccessBridgeJavaEntryPoints.obj
 0002:000006b4       ??_C@_0N@MHDJENGP@isJavaWindow@ 100226b4     AccessBridgeJavaEntryPoints.obj
 0002:000006c4       ??_C@_0CL@DDDHKJEI@?$CII?$CJLjavax?1accessibility?1Accessi@ 100226c4     AccessBridgeJavaEntryPoints.obj
 0002:000006f0       ??_C@_0CB@JPFPCEPL@getContextFromNativeWindowHandl@ 100226f0     AccessBridgeJavaEntryPoints.obj
 0002:00000714       ??_C@_0CL@LNFAHLDN@?$CILjavax?1accessibility?1Accessibl@ 10022714     AccessBridgeJavaEntryPoints.obj
 0002:00000740       ??_C@_0CB@OGDNEJKI@getNativeWindowHandleFromContex@ 10022740     AccessBridgeJavaEntryPoints.obj
 0002:00000768       ??_C@_0FB@EAOFMHCM@?$CILjavax?1accessibility?1Accessibl@ 10022768     AccessBridgeJavaEntryPoints.obj
 0002:000007bc       ??_C@_0BP@OKMFCEDC@getAccessibleParentFromContext@ 100227bc     AccessBridgeJavaEntryPoints.obj
 0002:000007dc       ??_C@_0DN@EHCPLCMJ@?$CILjavax?1accessibility?1Accessibl@ 100227dc     AccessBridgeJavaEntryPoints.obj
 0002:0000081c       ??_C@_0BA@NNDOMDNC@setTextContents@ 1002281c     AccessBridgeJavaEntryPoints.obj
 0002:00000830       ??_C@_0GD@DBHMDOGO@?$CILjavax?1accessibility?1Accessibl@ 10022830     AccessBridgeJavaEntryPoints.obj
 0002:00000894       ??_C@_0BC@EHMJEOIE@getParentWithRole@ 10022894     AccessBridgeJavaEntryPoints.obj
 0002:000008a8       ??_C@_0BC@CBIPDOMM@getTopLevelObject@ 100228a8     AccessBridgeJavaEntryPoints.obj
 0002:000008bc       ??_C@_0BK@KAMHKCND@getParentWithRoleElseRoot@ 100228bc     AccessBridgeJavaEntryPoints.obj
 0002:000008d8       ??_C@_0P@POFHEAF@getObjectDepth@ 100228d8     AccessBridgeJavaEntryPoints.obj
 0002:000008e8       ??_C@_0BE@CDLLPKAM@getActiveDescendent@ 100228e8     AccessBridgeJavaEntryPoints.obj
 0002:00000900       ??_C@_0FD@CINPJKCJ@?$CIIILjavax?1accessibility?1Accessi@ 10022900     AccessBridgeJavaEntryPoints.obj
 0002:00000954       ??_C@_0BH@BIEKBJIN@getAccessibleContextAt@ 10022954     AccessBridgeJavaEntryPoints.obj
 0002:0000096c       ??_C@_0CK@DOBCJGDO@?$CI?$CJLjavax?1accessibility?1Accessib@ 1002296c     AccessBridgeJavaEntryPoints.obj
 0002:00000998       ??_C@_0BO@BAFCPPBG@getAccessibleContextWithFocus@ 10022998     AccessBridgeJavaEntryPoints.obj
 0002:000009b8       ??_C@_0DM@JMIIJMDP@?$CILjavax?1accessibility?1Accessibl@ 100229b8     AccessBridgeJavaEntryPoints.obj
 0002:000009f4       ??_C@_0BN@DPBDCOIO@getAccessibleNameFromContext@ 100229f4     AccessBridgeJavaEntryPoints.obj
 0002:00000a14       ??_C@_0CE@IOFJICIE@getAccessibleDescriptionFromCon@ 10022a14     AccessBridgeJavaEntryPoints.obj
 0002:00000a38       ??_C@_0CD@DDGCACMP@getAccessibleRoleStringFromCont@ 10022a38     AccessBridgeJavaEntryPoints.obj
 0002:00000a5c       ??_C@_0CJ@OOFFKIOD@getAccessibleRoleStringFromCont@ 10022a5c     AccessBridgeJavaEntryPoints.obj
 0002:00000a88       ??_C@_0CF@JIKEBCCK@getAccessibleStatesStringFromCo@ 10022a88     AccessBridgeJavaEntryPoints.obj
 0002:00000ab0       ??_C@_0CL@EODHLGAL@getAccessibleStatesStringFromCo@ 10022ab0     AccessBridgeJavaEntryPoints.obj
 0002:00000adc       ??_C@_0CG@LAIPJCLP@getAccessibleIndexInParentFromC@ 10022adc     AccessBridgeJavaEntryPoints.obj
 0002:00000b04       ??_C@_0CG@KMCKGMOL@getAccessibleChildrenCountFromC@ 10022b04     AccessBridgeJavaEntryPoints.obj
 0002:00000b30       ??_C@_0FC@MAPACPFB@?$CILjavax?1accessibility?1Accessibl@ 10022b30     AccessBridgeJavaEntryPoints.obj
 0002:00000b84       ??_C@_0BO@BJCAFAFF@getAccessibleChildFromContext@ 10022b84     AccessBridgeJavaEntryPoints.obj
 0002:00000ba4       ??_C@_0DO@DCCADJME@?$CILjavax?1accessibility?1Accessibl@ 10022ba4     AccessBridgeJavaEntryPoints.obj
 0002:00000be4       ??_C@_0CH@EEFIDNHA@getAccessibleBoundsOnScreenFrom@ 10022be4     AccessBridgeJavaEntryPoints.obj
 0002:00000c0c       ??_C@_0BP@FJIKBALD@getAccessibleXcoordFromContext@ 10022c0c     AccessBridgeJavaEntryPoints.obj
 0002:00000c2c       ??_C@_0BP@LGNIKGFC@getAccessibleYcoordFromContext@ 10022c2c     AccessBridgeJavaEntryPoints.obj
 0002:00000c4c       ??_C@_0BP@EMIHBOON@getAccessibleHeightFromContext@ 10022c4c     AccessBridgeJavaEntryPoints.obj
 0002:00000c6c       ??_C@_0BO@OAEOJGNL@getAccessibleWidthFromContext@ 10022c6c     AccessBridgeJavaEntryPoints.obj
 0002:00000c90       ??_C@_0FD@DOBAJOLJ@?$CILjavax?1accessibility?1Accessibl@ 10022c90     AccessBridgeJavaEntryPoints.obj
 0002:00000ce4       ??_C@_0CC@MHPILDJI@getAccessibleComponentFromConte@ 10022ce4     AccessBridgeJavaEntryPoints.obj
 0002:00000d08       ??_C@_0FA@DEIINAGF@?$CILjavax?1accessibility?1Accessibl@ 10022d08     AccessBridgeJavaEntryPoints.obj
 0002:00000d58       ??_C@_0BP@PKDLLPIG@getAccessibleActionFromContext@ 10022d58     AccessBridgeJavaEntryPoints.obj
 0002:00000d78       ??_C@_0FD@KNPEAGPM@?$CILjavax?1accessibility?1Accessibl@ 10022d78     AccessBridgeJavaEntryPoints.obj
 0002:00000dcc       ??_C@_0CC@BHJMNIGA@getAccessibleSelectionFromConte@ 10022dcc     AccessBridgeJavaEntryPoints.obj
 0002:00000df0       ??_C@_0EO@JMGLFFGI@?$CILjavax?1accessibility?1Accessibl@ 10022df0     AccessBridgeJavaEntryPoints.obj
 0002:00000e40       ??_C@_0BN@CMHLOCAB@getAccessibleTextFromContext@ 10022e40     AccessBridgeJavaEntryPoints.obj
 0002:00000e60       ??_C@_0EP@DILHGLKF@?$CILjavax?1accessibility?1Accessibl@ 10022e60     AccessBridgeJavaEntryPoints.obj
 0002:00000eb0       ??_C@_0BO@BFBIPFI@getAccessibleValueFromContext@ 10022eb0     AccessBridgeJavaEntryPoints.obj
 0002:00000ed0       ??_C@_0EP@DNAJNMPI@?$CILjavax?1accessibility?1Accessibl@ 10022ed0     AccessBridgeJavaEntryPoints.obj
 0002:00000f20       ??_C@_0BO@PAPKMEMG@getAccessibleTableFromContext@ 10022f20     AccessBridgeJavaEntryPoints.obj
 0002:00000f40       ??_C@_0EP@HGIIMPLK@?$CILjavax?1accessibility?1Accessibl@ 10022f40     AccessBridgeJavaEntryPoints.obj
 0002:00000f90       ??_C@_0BO@PDGALDAF@getContextFromAccessibleTable@ 10022f90     AccessBridgeJavaEntryPoints.obj
 0002:00000fb0       ??_C@_0BM@FOJGHDMD@getAccessibleTableRowHeader@ 10022fb0     AccessBridgeJavaEntryPoints.obj
 0002:00000fcc       ??_C@_0BP@FNCIHNLO@getAccessibleTableColumnHeader@ 10022fcc     AccessBridgeJavaEntryPoints.obj
 0002:00000fec       ??_C@_0BL@FHMDFDAE@getAccessibleTableRowCount@ 10022fec     AccessBridgeJavaEntryPoints.obj
 0002:00001008       ??_C@_0BO@FPCPCCIG@getAccessibleTableColumnCount@ 10023008     AccessBridgeJavaEntryPoints.obj
 0002:00001028       ??_C@_0FB@MHAEKEPL@?$CILjavax?1accessibility?1Accessibl@ 10023028     AccessBridgeJavaEntryPoints.obj
 0002:0000107c       ??_C@_0CI@CIBBMNLI@getAccessibleTableCellAccessibl@ 1002307c     AccessBridgeJavaEntryPoints.obj
 0002:000010a4       ??_C@_0CL@HMHFCPKO@?$CILjavax?1accessibility?1Accessibl@ 100230a4     AccessBridgeJavaEntryPoints.obj
 0002:000010d0       ??_C@_0BM@BBCGJJGP@getAccessibleTableCellIndex@ 100230d0     AccessBridgeJavaEntryPoints.obj
 0002:000010ec       ??_C@_0CA@MEOFLNBC@getAccessibleTableCellRowExtent@ 100230ec     AccessBridgeJavaEntryPoints.obj
 0002:0000110c       ??_C@_0CD@GOAKABO@getAccessibleTableCellColumnExt@ 1002310c     AccessBridgeJavaEntryPoints.obj
 0002:00001130       ??_C@_0CL@BNJKGODM@?$CILjavax?1accessibility?1Accessibl@ 10023130     AccessBridgeJavaEntryPoints.obj
 0002:0000115c       ??_C@_0BO@KIDDCDEB@isAccessibleTableCellSelected@ 1002315c     AccessBridgeJavaEntryPoints.obj
 0002:0000117c       ??_C@_0CE@NOEAKJPM@getAccessibleTableRowHeaderRowC@ 1002317c     AccessBridgeJavaEntryPoints.obj
 0002:000011a0       ??_C@_0CH@NOEKFODF@getAccessibleTableColumnHeaderR@ 100231a0     AccessBridgeJavaEntryPoints.obj
 0002:000011c8       ??_C@_0CH@HOBKNLMK@getAccessibleTableRowHeaderColu@ 100231c8     AccessBridgeJavaEntryPoints.obj
 0002:000011f0       ??_C@_0CK@FLEMOIGB@getAccessibleTableColumnHeaderC@ 100231f0     AccessBridgeJavaEntryPoints.obj
 0002:00001220       ??_C@_0FA@NJKKHECI@?$CILjavax?1accessibility?1Accessibl@ 10023220     AccessBridgeJavaEntryPoints.obj
 0002:00001270       ??_C@_0CB@KCKFJBAJ@getAccessibleTableRowDescriptio@ 10023270     AccessBridgeJavaEntryPoints.obj
 0002:00001294       ??_C@_0CE@KHNFECJN@getAccessibleTableColumnDescrip@ 10023294     AccessBridgeJavaEntryPoints.obj
 0002:000012b8       ??_C@_0CJ@HGNCMOOJ@?$CILjavax?1accessibility?1Accessibl@ 100232b8     AccessBridgeJavaEntryPoints.obj
 0002:000012e4       ??_C@_0CE@CDNGIBEK@getAccessibleTableRowSelectionC@ 100232e4     AccessBridgeJavaEntryPoints.obj
 0002:00001308       ??_C@_0CK@OKAFABOP@?$CILjavax?1accessibility?1Accessibl@ 10023308     AccessBridgeJavaEntryPoints.obj
 0002:00001334       ??_C@_0BN@PCLDBBIG@isAccessibleTableRowSelected@ 10023334     AccessBridgeJavaEntryPoints.obj
 0002:00001354       ??_C@_0CK@ILOKEAHN@?$CILjavax?1accessibility?1Accessibl@ 10023354     AccessBridgeJavaEntryPoints.obj
 0002:00001380       ??_C@_0CA@CNAAIKJJ@getAccessibleTableRowSelections@ 10023380     AccessBridgeJavaEntryPoints.obj
 0002:000013a0       ??_C@_0CH@CDNMHGID@getAccessibleTableColumnSelecti@ 100233a0     AccessBridgeJavaEntryPoints.obj
 0002:000013c8       ??_C@_0CA@NFOBJKJN@isAccessibleTableColumnSelected@ 100233c8     AccessBridgeJavaEntryPoints.obj
 0002:000013e8       ??_C@_0CD@FNIEANFO@getAccessibleTableColumnSelecti@ 100233e8     AccessBridgeJavaEntryPoints.obj
 0002:0000140c       ??_C@_0BG@JNIAKEE@getAccessibleTableRow@ 1002340c     AccessBridgeJavaEntryPoints.obj
 0002:00001424       ??_C@_0BJ@DEHNOIGE@getAccessibleTableColumn@ 10023424     AccessBridgeJavaEntryPoints.obj
 0002:00001440       ??_C@_0BI@MLOHLDGL@getAccessibleTableIndex@ 10023440     AccessBridgeJavaEntryPoints.obj
 0002:00001458       ??_C@_0BL@NLFDIBPJ@getAccessibleRelationCount@ 10023458     AccessBridgeJavaEntryPoints.obj
 0002:00001474       ??_C@_0DN@BLNOMAFI@?$CILjavax?1accessibility?1Accessibl@ 10023474     AccessBridgeJavaEntryPoints.obj
 0002:000014b4       ??_C@_0BJ@DOGHLHFJ@getAccessibleRelationKey@ 100234b4     AccessBridgeJavaEntryPoints.obj
 0002:000014d0       ??_C@_0CM@KJPNEAF@?$CILjavax?1accessibility?1Accessibl@ 100234d0     AccessBridgeJavaEntryPoints.obj
 0002:000014fc       ??_C@_0CB@ONJFHOJM@getAccessibleRelationTargetCoun@ 100234fc     AccessBridgeJavaEntryPoints.obj
 0002:00001520       ??_C@_0FD@OOMEDHDI@?$CILjavax?1accessibility?1Accessibl@ 10023520     AccessBridgeJavaEntryPoints.obj
 0002:00001574       ??_C@_0BM@MFFGDMCG@getAccessibleRelationTarget@ 10023574     AccessBridgeJavaEntryPoints.obj
 0002:00001590       ??_C@_0FD@IPGDKGIL@?$CILjavax?1accessibility?1Accessibl@ 10023590     AccessBridgeJavaEntryPoints.obj
 0002:000015e4       ??_C@_0BH@IPNEFMCF@getAccessibleHypertext@ 100235e4     AccessBridgeJavaEntryPoints.obj
 0002:00001600       ??_C@_0FE@PMDDAMJI@?$CILjavax?1accessibility?1Accessibl@ 10023600     AccessBridgeJavaEntryPoints.obj
 0002:00001654       ??_C@_0BM@JMCFFMCN@activateAccessibleHyperlink@ 10023654     AccessBridgeJavaEntryPoints.obj
 0002:00001670       ??_C@_0BM@IADLHNKN@getAccessibleHyperlinkCount@ 10023670     AccessBridgeJavaEntryPoints.obj
 0002:00001690       ??_C@_0FG@JAOELFOA@?$CILjavax?1accessibility?1Accessibl@ 10023690     AccessBridgeJavaEntryPoints.obj
 0002:000016e8       ??_C@_0BH@EAGDOOIC@getAccessibleHyperlink@ 100236e8     AccessBridgeJavaEntryPoints.obj
 0002:00001700       ??_C@_0DO@OBGKICOI@?$CILjavax?1accessibility?1Accessibl@ 10023700     AccessBridgeJavaEntryPoints.obj
 0002:00001740       ??_C@_0BL@MPKBBMO@getAccessibleHyperlinkText@ 10023740     AccessBridgeJavaEntryPoints.obj
 0002:0000175c       ??_C@_0BK@DJNACEGJ@getAccessibleHyperlinkURL@ 1002375c     AccessBridgeJavaEntryPoints.obj
 0002:00001778       ??_C@_0CN@CAHDBMA@?$CILjavax?1accessibility?1Accessibl@ 10023778     AccessBridgeJavaEntryPoints.obj
 0002:000017a8       ??_C@_0CB@LKDEDAHI@getAccessibleHyperlinkStartInde@ 100237a8     AccessBridgeJavaEntryPoints.obj
 0002:000017cc       ??_C@_0BP@KJGEOOIO@getAccessibleHyperlinkEndIndex@ 100237cc     AccessBridgeJavaEntryPoints.obj
 0002:000017ec       ??_C@_0CO@HPBFOBHC@?$CILjavax?1accessibility?1Accessibl@ 100237ec     AccessBridgeJavaEntryPoints.obj
 0002:0000181c       ??_C@_0CA@FBPINCJA@getAccessibleHypertextLinkIndex@ 1002381c     AccessBridgeJavaEntryPoints.obj
 0002:0000183c       ??_C@_0BO@KGNEMCMH@getAccessibleKeyBindingsCount@ 1002383c     AccessBridgeJavaEntryPoints.obj
 0002:0000185c       ??_C@_0CM@PAHADMIP@?$CILjavax?1accessibility?1Accessibl@ 1002385c     AccessBridgeJavaEntryPoints.obj
 0002:00001888       ??_C@_0BM@HBNEDKIN@getAccessibleKeyBindingChar@ 10023888     AccessBridgeJavaEntryPoints.obj
 0002:000018a4       ??_C@_0CB@CIMFEKNG@getAccessibleKeyBindingModifier@ 100238a4     AccessBridgeJavaEntryPoints.obj
 0002:000018c8       ??_C@_0BI@MJKKDJIF@getAccessibleIconsCount@ 100238c8     AccessBridgeJavaEntryPoints.obj
 0002:000018e0       ??_C@_0BN@CJEBMOD@getAccessibleIconDescription@ 100238e0     AccessBridgeJavaEntryPoints.obj
 0002:00001900       ??_C@_0BI@MDOGDIAA@getAccessibleIconHeight@ 10023900     AccessBridgeJavaEntryPoints.obj
 0002:00001918       ??_C@_0BH@GGKEIMGD@getAccessibleIconWidth@ 10023918     AccessBridgeJavaEntryPoints.obj
 0002:00001930       ??_C@_0BK@PKOFGGNC@getAccessibleActionsCount@ 10023930     AccessBridgeJavaEntryPoints.obj
 0002:0000194c       ??_C@_0BI@DODALGBC@getAccessibleActionName@ 1002394c     AccessBridgeJavaEntryPoints.obj
 0002:00001964       ??_C@_0BE@CCPKEBNJ@doAccessibleActions@ 10023964     AccessBridgeJavaEntryPoints.obj
 0002:00001978       ??_C@_0CC@JCBADKJK@getAccessibleCharCountFromConte@ 10023978     AccessBridgeJavaEntryPoints.obj
 0002:0000199c       ??_C@_0CG@KPDPNIKI@getAccessibleCaretPositionFromC@ 1002399c     AccessBridgeJavaEntryPoints.obj
 0002:000019c4       ??_C@_0CN@CCCKKDDE@?$CILjavax?1accessibility?1Accessibl@ 100239c4     AccessBridgeJavaEntryPoints.obj
 0002:000019f4       ??_C@_0CF@IPJFBKEC@getAccessibleIndexAtPointFromCo@ 100239f4     AccessBridgeJavaEntryPoints.obj
 0002:00001a1c       ??_C@_0CG@CGEAMPNI@getAccessibleLetterAtIndexFromC@ 10023a1c     AccessBridgeJavaEntryPoints.obj
 0002:00001a44       ??_C@_0CE@CLNANFEE@getAccessibleWordAtIndexFromCon@ 10023a44     AccessBridgeJavaEntryPoints.obj
 0002:00001a68       ??_C@_0CI@BJNPGKMI@getAccessibleSentenceAtIndexFro@ 10023a68     AccessBridgeJavaEntryPoints.obj
 0002:00001a90       ??_C@_0CL@HGHPNDH@getAccessibleTextSelectionStart@ 10023a90     AccessBridgeJavaEntryPoints.obj
 0002:00001abc       ??_C@_0CJ@IPEBCNBB@getAccessibleTextSelectionEndFr@ 10023abc     AccessBridgeJavaEntryPoints.obj
 0002:00001ae8       ??_C@_0CJ@IBCLFAFA@getAccessibleTextSelectedTextFr@ 10023ae8     AccessBridgeJavaEntryPoints.obj
 0002:00001b14       ??_C@_0CK@JLPCFBLN@getAccessibleAttributesAtIndexF@ 10023b14     AccessBridgeJavaEntryPoints.obj
 0002:00001b40       ??_C@_0EK@JEPLCIJI@?$CILjavax?1accessibility?1Accessibl@ 10023b40     AccessBridgeJavaEntryPoints.obj
 0002:00001b8c       ??_C@_0CM@LKNKHCB@getAccessibleAttributeSetAtInde@ 10023b8c     AccessBridgeJavaEntryPoints.obj
 0002:00001bb8       ??_C@_0DP@HKEBFOCN@?$CILjavax?1accessibility?1Accessibl@ 10023bb8     AccessBridgeJavaEntryPoints.obj
 0002:00001bf8       ??_C@_0CI@IIHCGONP@getAccessibleTextRectAtIndexFro@ 10023bf8     AccessBridgeJavaEntryPoints.obj
 0002:00001c20       ??_C@_0CO@OMLKOFDL@getAccessibleXcoordTextRectAtIn@ 10023c20     AccessBridgeJavaEntryPoints.obj
 0002:00001c50       ??_C@_0CO@NKEIHFMI@getAccessibleYcoordTextRectAtIn@ 10023c50     AccessBridgeJavaEntryPoints.obj
 0002:00001c80       ??_C@_0CO@JHFMLGGO@getAccessibleHeightTextRectAtIn@ 10023c80     AccessBridgeJavaEntryPoints.obj
 0002:00001cb0       ??_C@_0CN@COKFHFFE@getAccessibleWidthTextRectAtInd@ 10023cb0     AccessBridgeJavaEntryPoints.obj
 0002:00001ce0       ??_C@_0BC@NPONPPPN@getCaretLocationX@ 10023ce0     AccessBridgeJavaEntryPoints.obj
 0002:00001cf4       ??_C@_0BC@MGPGMOLM@getCaretLocationY@ 10023cf4     AccessBridgeJavaEntryPoints.obj
 0002:00001d08       ??_C@_0BH@MJJIPGPF@getCaretLocationHeight@ 10023d08     AccessBridgeJavaEntryPoints.obj
 0002:00001d20       ??_C@_0BG@BIMEFOON@getCaretLocationWidth@ 10023d20     AccessBridgeJavaEntryPoints.obj
 0002:00001d38       ??_C@_0CL@JPPFAPAC@getAccessibleTextLineLeftBounds@ 10023d38     AccessBridgeJavaEntryPoints.obj
 0002:00001d64       ??_C@_0CM@IBNKHADJ@getAccessibleTextLineRightBound@ 10023d64     AccessBridgeJavaEntryPoints.obj
 0002:00001d90       ??_C@_0DO@MIIPGCPP@?$CILjavax?1accessibility?1Accessibl@ 10023d90     AccessBridgeJavaEntryPoints.obj
 0002:00001dd0       ??_C@_0CC@CIBLKPOK@getAccessibleTextRangeFromConte@ 10023dd0     AccessBridgeJavaEntryPoints.obj
 0002:00001df4       ??_C@_0CF@CJIJHKPD@getCurrentAccessibleValueFromCo@ 10023df4     AccessBridgeJavaEntryPoints.obj
 0002:00001e1c       ??_C@_0CF@PMHBGBIN@getMaximumAccessibleValueFromCo@ 10023e1c     AccessBridgeJavaEntryPoints.obj
 0002:00001e44       ??_C@_0CF@MEICJJIC@getMinimumAccessibleValueFromCo@ 10023e44     AccessBridgeJavaEntryPoints.obj
 0002:00001e6c       ??_C@_0CM@MHMFNKJL@?$CILjavax?1accessibility?1Accessibl@ 10023e6c     AccessBridgeJavaEntryPoints.obj
 0002:00001e98       ??_C@_0CC@OHDKMAMO@addAccessibleSelectionFromConte@ 10023e98     AccessBridgeJavaEntryPoints.obj
 0002:00001ebc       ??_C@_0CL@HAAKHFKD@?$CILjavax?1accessibility?1Accessibl@ 10023ebc     AccessBridgeJavaEntryPoints.obj
 0002:00001ee8       ??_C@_0CE@JAJNKBKJ@clearAccessibleSelectionFromCon@ 10023ee8     AccessBridgeJavaEntryPoints.obj
 0002:00001f0c       ??_C@_0CH@GOOENNPE@getAccessibleSelectionCountFrom@ 10023f0c     AccessBridgeJavaEntryPoints.obj
 0002:00001f34       ??_C@_0CM@GLHAJFJH@?$CILjavax?1accessibility?1Accessibl@ 10023f34     AccessBridgeJavaEntryPoints.obj
 0002:00001f60       ??_C@_0CF@PFGNJKHP@isAccessibleChildSelectedFromCo@ 10023f60     AccessBridgeJavaEntryPoints.obj
 0002:00001f88       ??_C@_0CF@LNEMJFKL@removeAccessibleSelectionFromCo@ 10023f88     AccessBridgeJavaEntryPoints.obj
 0002:00001fb0       ??_C@_0CI@GIPFHPKO@selectAllAccessibleSelectionFro@ 10023fb0     AccessBridgeJavaEntryPoints.obj
 0002:00001fd8       ??_C@_04OHLIFDMD@?$CIJ?$CJV@ 10023fd8     AccessBridgeJavaEntryPoints.obj
 0002:00001fe0       ??_C@_0BJ@MPIBKFAO@addJavaEventNotification@ 10023fe0     AccessBridgeJavaEntryPoints.obj
 0002:00001ffc       ??_C@_0BM@FNBBPCEJ@removeJavaEventNotification@ 10023ffc     AccessBridgeJavaEntryPoints.obj
 0002:00002018       ??_C@_0CC@MPLKGCBM@addAccessibilityEventNotificati@ 10024018     AccessBridgeJavaEntryPoints.obj
 0002:0000203c       ??_C@_0CF@JFMMDHHJ@removeAccessibilityEventNotific@ 1002403c     AccessBridgeJavaEntryPoints.obj
 0002:00002064       ??_C@_0CD@PFBLKFGD@?$CILjavax?1swing?1text?1AttributeSet@ 10024064     AccessBridgeJavaEntryPoints.obj
 0002:00002088       ??_C@_0BI@PMOBPKB@getBoldFromAttributeSet@ 10024088     AccessBridgeJavaEntryPoints.obj
 0002:000020a0       ??_C@_0BK@HMLEJNMA@getItalicFromAttributeSet@ 100240a0     AccessBridgeJavaEntryPoints.obj
 0002:000020bc       ??_C@_0BN@BGEODKID@getUnderlineFromAttributeSet@ 100240bc     AccessBridgeJavaEntryPoints.obj
 0002:000020dc       ??_C@_0CB@BICMGOJK@getStrikethroughFromAttributeSe@ 100240dc     AccessBridgeJavaEntryPoints.obj
 0002:00002100       ??_C@_0BP@BNLEAGAN@getSuperscriptFromAttributeSet@ 10024100     AccessBridgeJavaEntryPoints.obj
 0002:00002120       ??_C@_0BN@FENOLEGG@getSubscriptFromAttributeSet@ 10024120     AccessBridgeJavaEntryPoints.obj
 0002:00002140       ??_C@_0DE@PFGGMCPM@?$CILjavax?1swing?1text?1AttributeSet@ 10024140     AccessBridgeJavaEntryPoints.obj
 0002:00002174       ??_C@_0CD@MGNACFJA@getBackgroundColorFromAttribute@ 10024174     AccessBridgeJavaEntryPoints.obj
 0002:00002198       ??_C@_0CD@JFAEMBOF@getForegroundColorFromAttribute@ 10024198     AccessBridgeJavaEntryPoints.obj
 0002:000021bc       ??_C@_0BO@JFHBDDGD@getFontFamilyFromAttributeSet@ 100241bc     AccessBridgeJavaEntryPoints.obj
 0002:000021dc       ??_C@_0CD@JEPEOEPB@?$CILjavax?1swing?1text?1AttributeSet@ 100241dc     AccessBridgeJavaEntryPoints.obj
 0002:00002200       ??_C@_0BM@OMIOBJPB@getFontSizeFromAttributeSet@ 10024200     AccessBridgeJavaEntryPoints.obj
 0002:0000221c       ??_C@_0BN@BAFOGOJK@getAlignmentFromAttributeSet@ 1002421c     AccessBridgeJavaEntryPoints.obj
 0002:0000223c       ??_C@_0BN@DEDFHCOP@getBidiLevelFromAttributeSet@ 1002423c     AccessBridgeJavaEntryPoints.obj
 0002:0000225c       ??_C@_0CD@BDGMPIDO@?$CILjavax?1swing?1text?1AttributeSet@ 1002425c     AccessBridgeJavaEntryPoints.obj
 0002:00002280       ??_C@_0CD@EJOOBJDB@getFirstLineIndentFromAttribute@ 10024280     AccessBridgeJavaEntryPoints.obj
 0002:000022a4       ??_C@_0BO@KCBIJLNO@getLeftIndentFromAttributeSet@ 100242a4     AccessBridgeJavaEntryPoints.obj
 0002:000022c4       ??_C@_0BP@KEIFBKEA@getRightIndentFromAttributeSet@ 100242c4     AccessBridgeJavaEntryPoints.obj
 0002:000022e4       ??_C@_0BP@ICDNCHPN@getLineSpacingFromAttributeSet@ 100242e4     AccessBridgeJavaEntryPoints.obj
 0002:00002304       ??_C@_0BO@CHPMHCHE@getSpaceAboveFromAttributeSet@ 10024304     AccessBridgeJavaEntryPoints.obj
 0002:00002324       ??_C@_0BO@DOLMIFOK@getSpaceBelowFromAttributeSet@ 10024324     AccessBridgeJavaEntryPoints.obj
 0002:00002344       ??_C@_0CL@NMLPDKKP@?$CILjavax?1accessibility?1Accessibl@ 10024344     AccessBridgeJavaEntryPoints.obj
 0002:00002370       ??_C@_0N@CEMKNPGL@requestFocus@ 10024370     AccessBridgeJavaEntryPoints.obj
 0002:00002380       ??_C@_0CN@EDMFOCKG@?$CILjavax?1accessibility?1Accessibl@ 10024380     AccessBridgeJavaEntryPoints.obj
 0002:000023b0       ??_C@_0BA@JKPGAJFL@selectTextRange@ 100243b0     AccessBridgeJavaEntryPoints.obj
 0002:000023c0       ??_C@_0BI@IIOLCPFK@getVisibleChildrenCount@ 100243c0     AccessBridgeJavaEntryPoints.obj
 0002:000023d8       ??_C@_0BA@JIDLMKH@getVisibleChild@ 100243d8     AccessBridgeJavaEntryPoints.obj
 0002:000023e8       ??_C@_0BB@ENIAPGBO@setCaretPosition@ 100243e8     AccessBridgeJavaEntryPoints.obj
 0002:000023fc       ??_C@_0CE@MELACKPN@getVirtualAccessibleNameFromCon@ 100243fc     AccessBridgeJavaEntryPoints.obj
 0002:00002420       ??_C@_0DP@ODHDIMGL@?$FLINFO?$FN?3?5Calling?5AccessBridgeJav@ 10024420     AccessBridgeJavaEntryPoints.obj
 0002:00002460       ??_C@_0DD@INJPOCHE@Getting?5isJavaWindow?5?9?5call?5to?5@ 10024460     AccessBridgeJavaEntryPoints.obj
 0002:00002494       ??_C@_0DN@ENCLOLFG@?$FLERROR?$FN?3?5?$CK?$CK?$CK?5Exception?5occured?5@ 10024494     AccessBridgeJavaEntryPoints.obj
 0002:000024d4       ??_C@_0DH@DHJJKMLN@?$FLERROR?$FN?3?5either?5jniEnv?5?$DN?$DN?50?5or?5@ 100244d4     AccessBridgeJavaEntryPoints.obj
 0002:0000250c       ??_C@_0DN@GKGIBPBO@?$FLINFO?$FN?3?5In?5AccessBridgeJavaEntr@ 1002450c     AccessBridgeJavaEntryPoints.obj
 0002:0000254c       ??_C@_0BF@LOIOEBHF@Calling?5IsSameObject@ 1002454c     AccessBridgeJavaEntryPoints.obj
 0002:00002564       ??_C@_0CE@PJOLBDKG@?$FLINFO?$FN?3?5?5?5isSameObject?5returnin@ 10024564     AccessBridgeJavaEntryPoints.obj
 0002:00002588       ??_C@_0EK@MPPKLDGH@?$FLINFO?$FN?3?5In?5AccessBridgeJavaEntr@ 10024588     AccessBridgeJavaEntryPoints.obj
 0002:000025d4       ??_C@_0DP@INBKCEII@Getting?5AccessibleContextFromHW@ 100245d4     AccessBridgeJavaEntryPoints.obj
 0002:00002618       ??_C@_0EI@POHJNOIF@?$FLERROR?$FN?3?5?5either?5jniEnv?5?$DN?$DN?50?5or@ 10024618     AccessBridgeJavaEntryPoints.obj
 0002:00002660       ??_C@_0EK@KGPHBKLN@?$FLINFO?$FN?3?5In?5AccessBridgeJavaEntr@ 10024660     AccessBridgeJavaEntryPoints.obj
 0002:000026ac       ??_C@_0DM@OPKABADC@Getting?5HWNDFromAccessibleConte@ 100246ac     AccessBridgeJavaEntryPoints.obj
 0002:000026e8       ??_C@_0BD@NKFEMHLM@?$FLINFO?$FN?3?5rHWND?5?$DN?5?$CFX@ 100246e8     AccessBridgeJavaEntryPoints.obj
 0002:00002700       ??_C@_0EH@MFPOIGJN@?$FLERROR?$FN?3?5either?5jniEnv?5?$DN?$DN?50?5or?5@ 10024700     AccessBridgeJavaEntryPoints.obj
 0002:00002748       ??_C@_0EC@BPPANMDJ@?$FLINFO?$FN?3?5In?5AccessBridgeJavaEntr@ 10024748     AccessBridgeJavaEntryPoints.obj
 0002:0000278c       ??_C@_0BN@LGGMDMGD@?$FLERROR?$FN?3?5?5?5?5NewString?5failed@ 1002478c     AccessBridgeJavaEntryPoints.obj
 0002:000027ac       ??_C@_0CO@NCDGKPGB@setTextContents?5?9?5call?5to?5CallB@ 100247ac     AccessBridgeJavaEntryPoints.obj
 0002:000027dc       ??_C@_0BI@IMHMFAIB@?$FLINFO?$FN?3?5?5?5?5?5result?5?$DN?5?$CFd@ 100247dc     AccessBridgeJavaEntryPoints.obj
 0002:000027f4       ??_C@_0DK@MGDAPF@?$FLERROR?$FN?3?5either?5jniEnv?5?$DN?$DN?50?5or?5@ 100247f4     AccessBridgeJavaEntryPoints.obj
 0002:00002830       ??_C@_0DP@LHNNHOD@?$FLINFO?$FN?3?5In?5AccessBridgeJavaEntr@ 10024830     AccessBridgeJavaEntryPoints.obj
 0002:00002870       ??_C@_0BO@LLFKIHLA@?$FLERROR?$FN?3?5?5?5?5?5NewString?5failed@ 10024870     AccessBridgeJavaEntryPoints.obj
 0002:00002890       ??_C@_0DE@KBFMBJPI@Getting?5ParentWithRole?5?9?5call?5t@ 10024890     AccessBridgeJavaEntryPoints.obj
 0002:000028c4       ??_C@_0CE@LNEDINGM@?$FLINFO?$FN?3?5?5?5?5?5rAccessibleContext?5@ 100248c4     AccessBridgeJavaEntryPoints.obj
 0002:000028e8       ??_C@_0DA@OMNPGENP@Getting?5ParentWithRole?5?9?5call?5t@ 100248e8     AccessBridgeJavaEntryPoints.obj
 0002:00002918       ??_C@_0EF@LHAMKGPK@?$FLINFO?$FN?3?5?5?5Returning?5?9?5returnedA@ 10024918     AccessBridgeJavaEntryPoints.obj
 0002:00002960       ??_C@_0DM@OLEIFDLG@?$FLERROR?$FN?3?5either?5jniEnv?5?$DN?$DN?50?5or?5@ 10024960     AccessBridgeJavaEntryPoints.obj
 0002:0000299c       ??_C@_0DP@EPHBFJKE@?$FLINFO?$FN?3?5In?5AccessBridgeJavaEntr@ 1002499c     AccessBridgeJavaEntryPoints.obj
 0002:000029dc       ??_C@_0DE@FDIFCLEM@Getting?5TopLevelObject?5?9?5call?5t@ 100249dc     AccessBridgeJavaEntryPoints.obj
 0002:00002a10       ??_C@_0CB@GDMCCFCK@?$FLINFO?$FN?3?5?5rAccessibleContext?5?$DN?5?$CF@ 10024a10     AccessBridgeJavaEntryPoints.obj
 0002:00002a34       ??_C@_0DA@ELIJHKN@Getting?5TopLevelObject?5?9?5call?5t@ 10024a34     AccessBridgeJavaEntryPoints.obj
 0002:00002a64       ??_C@_0DM@MKIGPNDF@?$FLERROR?$FN?3?5either?5jniEnv?5?$DN?$DN?50?5or?5@ 10024a64     AccessBridgeJavaEntryPoints.obj
 0002:00002aa0       ??_C@_0EH@MCHGGFNF@?$FLINFO?$FN?3?5In?5AccessBridgeJavaEntr@ 10024aa0     AccessBridgeJavaEntryPoints.obj
 0002:00002ae8       ??_C@_0DM@IKNMPPHI@Getting?5ParentWithRoleElseRoot?5@ 10024ae8     AccessBridgeJavaEntryPoints.obj
 0002:00002b24       ??_C@_0DI@CDJCPAOF@Getting?5ParentWithRoleElseRoot?5@ 10024b24     AccessBridgeJavaEntryPoints.obj
 0002:00002b60       ??_C@_0EF@MODADMKL@?$FLERROR?$FN?3?5?5either?5jniEnv?5?$DN?$DN?50?5or@ 10024b60     AccessBridgeJavaEntryPoints.obj
 0002:00002ba8       ??_C@_0DM@EBONPKNN@?$FLINFO?$FN?3?5In?5AccessBridgeJavaEntr@ 10024ba8     AccessBridgeJavaEntryPoints.obj
 0002:00002be4       ??_C@_0CO@CCBFEFG@Getting?5ObjectDepth?5?9?5call?5to?5C@ 10024be4     AccessBridgeJavaEntryPoints.obj
 0002:00002c14       ??_C@_0BJ@KJFHIGKC@?$FLINFO?$FN?3?5?5?5?5?5rResult?5?$DN?5?$CFd@ 10024c14     AccessBridgeJavaEntryPoints.obj
 0002:00002c30       ??_C@_0DJ@NCMDONA@?$FLERROR?$FN?3?5either?5jniEnv?5?$DN?$DN?50?5or?5@ 10024c30     AccessBridgeJavaEntryPoints.obj
 0002:00002c70       ??_C@_0EB@OJAHMNKI@?$FLINFO?$FN?3?5In?5AccessBridgeJavaEntr@ 10024c70     AccessBridgeJavaEntryPoints.obj
 0002:00002cb4       ??_C@_0DG@FKCKDOAD@Getting?5ActiveDescendent?5?9?5call@ 10024cb4     AccessBridgeJavaEntryPoints.obj
 0002:00002cec       ??_C@_0DC@DOJHNKHC@Getting?5ActiveDescendant?5?9?5call@ 10024cec     AccessBridgeJavaEntryPoints.obj
 0002:00002d20       ??_C@_0DO@FBKMCPK@?$FLERROR?$FN?3?5either?5jniEnv?5?$DN?$DN?50?5or?5@ 10024d20     AccessBridgeJavaEntryPoints.obj
 0002:00002d60       ??_C@_0CK@IFAHAOG@?$FLINFO?$FN?3?5?5getVirtualAccessibleNa@ 10024d60     AccessBridgeJavaEntryPoints.obj
 0002:00002d8c       ??_C@_0DE@GLGPLDPG@Getting?5AccessibleName?5?9?5call?5t@ 10024d8c     AccessBridgeJavaEntryPoints.obj
 0002:00002dc0       ??_C@_0DC@LMABNHGH@Getting?5AccessibleName?5?9?5call?5t@ 10024dc0     AccessBridgeJavaEntryPoints.obj
 0002:00002df4       ??_C@_0DD@FODFLNBM@Getting?5AccessibleName?5?9?5call?5t@ 10024df4     AccessBridgeJavaEntryPoints.obj
 0002:00002e28       ??_C@_0DG@LKNGBJAO@Getting?5AccessibleName?5?9?5call?5t@ 10024e28     AccessBridgeJavaEntryPoints.obj
 0002:00002e60       ??_C@_0DC@MBCPGFEL@Getting?5AccessibleName?5?9?5call?5t@ 10024e60     AccessBridgeJavaEntryPoints.obj
 0002:00002e94       ??_C@_1DA@BACBNKJB@?$AA?5?$AA?5?$AAA?$AAc?$AAc?$AAe?$AAs?$AAs?$AAi?$AAb?$AAl?$AAe?$AA?5?$AAN?$AAa@ 10024e94     AccessBridgeJavaEntryPoints.obj
 0002:00002ec4       ??_C@_0DC@HCPEBFPJ@Getting?5AccessibleName?5?9?5call?5t@ 10024ec4     AccessBridgeJavaEntryPoints.obj
 0002:00002ef8       ??_C@_0CD@JNOMKFNM@?$FLINFO?$FN?3?5?5?5Accessible?5Name?5is?5nu@ 10024ef8     AccessBridgeJavaEntryPoints.obj
 0002:00002f20       ??_C@_0EN@LBGKPBFG@?$FLINFO?$FN?3?5either?5jniEnv?5?$DN?$DN?50?5or?5g@ 10024f20     AccessBridgeJavaEntryPoints.obj
 0002:00002f70       ??_C@_0DK@COLMCNJL@?$FLINFO?$FN?3?5In?5AccessBridgeJavaEntr@ 10024f70     AccessBridgeJavaEntryPoints.obj
 0002:00002fac       ??_C@_0CL@OHFNFEAE@requestFocus?5?9?5call?5to?5CallBool@ 10024fac     AccessBridgeJavaEntryPoints.obj
 0002:00002fd8       ??_C@_0BH@JOKEJIHH@?$FLINFO?$FN?3?5?5?5?5result?5?$DN?5?$CFd@ 10024fd8     AccessBridgeJavaEntryPoints.obj
 0002:00002ff0       ??_C@_0DH@OADKFKDG@?$FLERROR?$FN?3?5either?5jniEnv?5?$DN?$DN?50?5or?5@ 10024ff0     AccessBridgeJavaEntryPoints.obj
 0002:00003028       ??_C@_0FB@HEEEBDKB@?$FLINFO?$FN?3?5In?5AccessBridgeJavaEntr@ 10025028     AccessBridgeJavaEntryPoints.obj
 0002:0000307c       ??_C@_0CO@NOPLEGNC@selectTextRange?5?9?5call?5to?5CallB@ 1002507c     AccessBridgeJavaEntryPoints.obj
 0002:000030ac       ??_C@_0DK@EDLAMPCD@?$FLERROR?$FN?3?5either?5jniEnv?5?$DN?$DN?50?5or?5@ 100250ac     AccessBridgeJavaEntryPoints.obj
 0002:000030e8       ??_C@_0FK@CBBPCLFD@?$FLINFO?$FN?3?5In?5AccessBridgeJavaEntr@ 100250e8     AccessBridgeJavaEntryPoints.obj
 0002:00003144       ??_C@_0DN@CIOOGMLK@?$FLINFO?$FN?3?5?5Getting?5full?5test_attr@ 10025144     AccessBridgeJavaEntryPoints.obj
 0002:00003188       ??_C@_0EB@FNOCJLAN@Getting?5AccessibleAttributesAtI@ 10025188     AccessBridgeJavaEntryPoints.obj
 0002:000031cc       ??_C@_0DE@NPIJKEOK@?$FLINFO?$FN?3?5?5?5returned?5from?5CallObj@ 100251cc     AccessBridgeJavaEntryPoints.obj
 0002:00003200       ??_C@_0DP@GAODIEPK@Getting?5AccessibleAttributesAtI@ 10025200     AccessBridgeJavaEntryPoints.obj
 0002:00003240       ??_C@_0EA@NAFHLALG@Getting?5AccessibleAttributesAtI@ 10025240     AccessBridgeJavaEntryPoints.obj
 0002:00003280       ??_C@_0ED@HICLLPAP@Getting?5AccessibleAttributesAtI@ 10025280     AccessBridgeJavaEntryPoints.obj
 0002:000032c4       ??_C@_0DP@BNMNDGNG@Getting?5AccessibleAttributesAtI@ 100252c4     AccessBridgeJavaEntryPoints.obj
 0002:00003308       ??_C@_1FE@NAFGNNMA@?$AA?$FL?$AAI?$AAN?$AAF?$AAO?$AA?$FN?$AA?3?$AA?5?$AA?5?$AAA?$AAc?$AAc?$AAe?$AAs?$AAs@ 10025308     AccessBridgeJavaEntryPoints.obj
 0002:0000335c       ??_C@_0DP@KOBGEGGE@Getting?5AccessibleAttributesAtI@ 1002535c     AccessBridgeJavaEntryPoints.obj
 0002:0000339c       ??_C@_0CO@GBFCDBDB@?$FLWARN?$FN?3?5?5?5Accessible?5Text?5attri@ 1002539c     AccessBridgeJavaEntryPoints.obj
 0002:000033d0       ??_C@_0FB@DKHOICMI@?$FLERROR?$FN?3?5either?5env?5?$DN?$DN?50?5or?5get@ 100253d0     AccessBridgeJavaEntryPoints.obj
 0002:00003428       ??_C@_0EH@KKFBHMJC@?$FLINFO?$FN?3?5?$CD?$CD?$CD?$CD?$CD?5AccessBridgeJavaE@ 10025428     AccessBridgeJavaEntryPoints.obj
 0002:00003470       ??_C@_0DP@MHLDKAGF@?$CD?$CD?$CD?$CD?$CD?5Getting?5visible?5children?5@ 10025470     AccessBridgeJavaEntryPoints.obj
 0002:000034b0       ??_C@_0CM@JAPBNGLO@?$FLINFO?$FN?3?5?5?5?$CD?$CD?$CD?$CD?$CD?5visible?5childre@ 100254b0     AccessBridgeJavaEntryPoints.obj
 0002:000034e0       ??_C@_0FD@GLIPOPHN@?$FLINFO?$FN?3?5?$CD?$CD?$CD?$CD?$CD?5AccessBridgeJavaE@ 100254e0     AccessBridgeJavaEntryPoints.obj
 0002:00003534       ??_C@_0CH@ONKDDCMN@?$FLINFO?$FN?3?5?5?5getting?5visible?5child@ 10025534     AccessBridgeJavaEntryPoints.obj
 0002:0000355c       ??_C@_0DJ@HGPLCHEB@?$CD?$CD?$CD?$CD?$CD?5getVisibleChildMethod?5?9?5c@ 1002555c     AccessBridgeJavaEntryPoints.obj
 0002:00003598       ??_C@_0DF@JHJIJJH@?$CD?$CD?$CD?$CD?$CD?5getVisibleChildMethod?5?9?5c@ 10025598     AccessBridgeJavaEntryPoints.obj
 0002:000035d0       ??_C@_0CD@ECMHOCH@?$FLINFO?$FN?3?5?5?5?$CD?$CD?$CD?$CD?$CD?5visible?5child?5?$DN@ 100255d0     AccessBridgeJavaEntryPoints.obj
 0002:000035f8       ??_C@_0EK@GNPPBBMN@?$FLINFO?$FN?3?5?5?5?$CD?$CD?$CD?$CD?$CD?5AccessBridgeJav@ 100255f8     AccessBridgeJavaEntryPoints.obj
 0002:00003648       ??_C@_0EL@OPKFGOFA@?$FLINFO?$FN?3?5In?5AccessBridgeJavaEntr@ 10025648     AccessBridgeJavaEntryPoints.obj
 0002:00003694       ??_C@_0CO@BDNAFHGG@setCaretPostion?5?9?5call?5to?5CallB@ 10025694     AccessBridgeJavaEntryPoints.obj
 0002:000036c4       ??_C@_0BJ@PGHBDIPI@?$FLERROR?$FN?3?5?5?5?5?5result?5?$DN?5?$CFd@ 100256c4     AccessBridgeJavaEntryPoints.obj
 0002:000036e0       ??_C@_0DL@CBEPMOL@?$FLERROR?$FN?3?5either?5jniEnv?5?$DN?$DN?50?5or?5@ 100256e0     AccessBridgeJavaEntryPoints.obj
 0002:0000371c       ??_C@_0DP@DPLDEGDE@?$FLINFO?$FN?3?5Calling?5AccessBridgeJav@ 1002571c     AccessBridgeJavaEntryPoints.obj
 0002:0000375c       ??_C@_0DJ@EBEOKJAG@Getting?5JavaVersionProperty?5?9?5c@ 1002575c     AccessBridgeJavaEntryPoints.obj
 0002:00003798       ??_C@_0FC@KFJABCDE@?$FLERROR?$FN?3?5?5?$CK?$CK?$CK?5Exception?5when?5ge@ 10025798     AccessBridgeJavaEntryPoints.obj
 0002:000037ec       ??_C@_0DL@FDAICLOI@Getting?5JavaVersionProperty?5?9?5c@ 100257ec     AccessBridgeJavaEntryPoints.obj
 0002:00003828       ??_C@_0DH@PEMIMKKJ@Getting?5JavaVersionProperty?5?9?5c@ 10025828     AccessBridgeJavaEntryPoints.obj
 0002:00003860       ??_C@_1CK@PFPDBLJ@?$AA?5?$AA?5?$AAJ?$AAa?$AAv?$AAa?$AA?5?$AAv?$AAe?$AAr?$AAs?$AAi?$AAo?$AAn?$AA?5@ 10025860     AccessBridgeJavaEntryPoints.obj
 0002:0000388c       ??_C@_0DH@EHBDLKBL@Getting?5JavaVersionProperty?5?9?5c@ 1002588c     AccessBridgeJavaEntryPoints.obj
 0002:000038c4       ??_C@_0CA@KOJKOLB@?$FLWARN?$FN?3?5?5?5Java?5version?5is?5null?4@ 100258c4     AccessBridgeJavaEntryPoints.obj
 0002:000038e4       ??_C@_0DP@FHBJPJDO@?$FLERROR?$FN?3?5?5either?5env?5?$DN?$DN?50?5or?5ge@ 100258e4     AccessBridgeJavaEntryPoints.obj
 0002:00003928       ??_C@_0EC@OAJCCJEK@?$FLINFO?$FN?3?5Calling?5AccessBridgeJav@ 10025928     AccessBridgeJavaEntryPoints.obj
 0002:0000396c       ??_C@_0BF@MJCCCBHB@?$FLERROR?$FN?3?5?5No?5Java?5VM@ 1002596c     AccessBridgeJavaEntryPoints.obj
 0002:00003984       ??_C@_0BH@PCLEJECO@?$FLERROR?$FN?3?5?5Null?5jobject@ 10025984     AccessBridgeJavaEntryPoints.obj
 0002:0000399c       ??_C@_0DE@FOOENAKM@Getting?5AccessibleText?5?9?5call?5t@ 1002599c     AccessBridgeJavaEntryPoints.obj
 0002:000039d0       ??_C@_0BP@NHKMDDHI@?$FLERROR?$FN?3?5?5?5AccessibleText?5?$DN?5?$CFp@ 100259d0     AccessBridgeJavaEntryPoints.obj
 0002:000039f0       ??_C@_0DC@NHCDOGBO@Getting?5AccessibleText?5?9?5call?5t@ 100259f0     AccessBridgeJavaEntryPoints.obj
 0002:00003a28       ??_C@_0EF@KPMHECBJ@?$FLERROR?$FN?3?5?5either?5env?5?$DN?$DN?50?5or?5ge@ 10025a28     AccessBridgeJavaEntryPoints.obj
 0002:00003a70       ??_C@_0CL@OMBEMJIM@?$FLERROR?$FN?3?5?5jobject?5is?5not?5an?5Acc@ 10025a70     AccessBridgeJavaEntryPoints.obj
 0002:00003aa0       ??_C@_0FB@IMPDGAOD@?$FLINFO?$FN?3?5Calling?5AccessBridgeJav@ 10025aa0     AccessBridgeJavaEntryPoints.obj
 0002:00003af4       ??_C@_0DJ@CBKJGOIB@Getting?5AccessibleContextAt?5?9?5c@ 10025af4     AccessBridgeJavaEntryPoints.obj
 0002:00003b30       ??_C@_0DF@PJCJKGPI@Getting?5AccessibleContextAt?5?9?5c@ 10025b30     AccessBridgeJavaEntryPoints.obj
 0002:00003b68       ??_C@_0DP@LFOACNJN@?$FLERROR?$FN?3?5?5either?5env?5?$DN?$DN?50?5or?5ge@ 10025b68     AccessBridgeJavaEntryPoints.obj
 0002:00003ba8       ??_C@_0EN@LHFHLFOC@?$FLINFO?$FN?3?5Calling?5AccessBridgeJav@ 10025ba8     AccessBridgeJavaEntryPoints.obj
 0002:00003bf8       ??_C@_0EA@NLINILPH@Getting?5AccessibleContextWithFo@ 10025bf8     AccessBridgeJavaEntryPoints.obj
 0002:00003c38       ??_C@_0DM@IJDJLPBO@Getting?5AccessibleContextWithFo@ 10025c38     AccessBridgeJavaEntryPoints.obj
 0002:00003c78       ??_C@_0EJ@KBIILIHA@?$FLERROR?$FN?3?5?5either?5jniEnv?5?$DN?$DN?50?5or@ 10025c78     AccessBridgeJavaEntryPoints.obj
 0002:00003cc8       ??_C@_0FB@NNGDGCK@?$FLINFO?$FN?3?5?$CD?$CD?$CD?$CD?$CD?5Calling?5AccessBri@ 10025cc8     AccessBridgeJavaEntryPoints.obj
 0002:00003d1c       ??_C@_0DF@BABIDEMG@?$FLWARN?$FN?3?5?5passed?5in?5AccessibleCo@ 10025d1c     AccessBridgeJavaEntryPoints.obj
 0002:00003d58       ??_C@_1EA@IPHAHEJA@?$AA?$FL?$AAI?$AAN?$AAF?$AAO?$AA?$FN?$AA?3?$AA?5?$AA?5?$AA?5?$AAA?$AAc?$AAc?$AAe?$AAs@ 10025d58     AccessBridgeJavaEntryPoints.obj
 0002:00003d98       ??_C@_0CD@BCDIDKCI@?$FLWARN?$FN?3?5?5?5Accessible?5Name?5is?5nu@ 10025d98     AccessBridgeJavaEntryPoints.obj
 0002:00003dc0       ??_C@_0EF@DMNCHIBL@?$FLERROR?$FN?3?5?5either?5env?5?$DN?$DN?50?5or?5ge@ 10025dc0     AccessBridgeJavaEntryPoints.obj
 0002:00003e08       ??_C@_0DL@IPNAGHCP@Getting?5AccessibleDescription?5?9@ 10025e08     AccessBridgeJavaEntryPoints.obj
 0002:00003e48       ??_C@_1EO@NBFBPIFN@?$AA?$FL?$AAI?$AAN?$AAF?$AAO?$AA?$FN?$AA?3?$AA?5?$AA?5?$AA?5?$AAA?$AAc?$AAc?$AAe?$AAs@ 10025e48     AccessBridgeJavaEntryPoints.obj
 0002:00003e98       ??_C@_0CK@KNEKOBNE@?$FLWARN?$FN?3?5?5?5Accessible?5Descriptio@ 10025e98     AccessBridgeJavaEntryPoints.obj
 0002:00003ec8       ??_C@_0EM@LPILGNDD@?$FLERROR?$FN?3?5?5either?5env?5?$DN?$DN?50?5or?5ge@ 10025ec8     AccessBridgeJavaEntryPoints.obj
 0002:00003f14       ??_C@_0DE@IKDIHCF@Getting?5AccessibleRole?5?9?5call?5t@ 10025f14     AccessBridgeJavaEntryPoints.obj
 0002:00003f48       ??_C@_0DC@FOMJEAJG@Getting?5AccessibleRole?5?9?5call?5t@ 10025f48     AccessBridgeJavaEntryPoints.obj
 0002:00003f7c       ??_C@_0DD@JEGNLHAB@Getting?5AccessibleRole?5?9?5call?5t@ 10025f7c     AccessBridgeJavaEntryPoints.obj
 0002:00003fb0       ??_C@_0DG@DBHHBIKL@Getting?5AccessibleRole?5?9?5call?5t@ 10025fb0     AccessBridgeJavaEntryPoints.obj
 0002:00003fe8       ??_C@_0DC@CDOHPCLK@Getting?5AccessibleRole?5?9?5call?5t@ 10025fe8     AccessBridgeJavaEntryPoints.obj
 0002:00004020       ??_C@_1EA@DFMPHGFH@?$AA?$FL?$AAI?$AAN?$AAF?$AAO?$AA?$FN?$AA?3?$AA?5?$AA?5?$AA?5?$AAA?$AAc?$AAc?$AAe?$AAs@ 10026020     AccessBridgeJavaEntryPoints.obj
 0002:00004060       ??_C@_0DC@JADMICAI@Getting?5AccessibleRole?5?9?5call?5t@ 10026060     AccessBridgeJavaEntryPoints.obj
 0002:00004094       ??_C@_0CD@DPDMNHLG@?$FLWARN?$FN?3?5?5?5Accessible?5Role?5is?5nu@ 10026094     AccessBridgeJavaEntryPoints.obj
 0002:000040b8       ??_C@_0EL@ENOHPPLP@?$FLERROR?$FN?3?5?5either?5env?5?$DN?$DN?50?5or?5ge@ 100260b8     AccessBridgeJavaEntryPoints.obj
 0002:00004104       ??_C@_0DK@OPAANMJH@Getting?5AccessibleRole_en_US?5?9?5@ 10026104     AccessBridgeJavaEntryPoints.obj
 0002:00004140       ??_C@_0DI@CJNJDFMD@Getting?5AccessibleRole_en_US?5?9?5@ 10026140     AccessBridgeJavaEntryPoints.obj
 0002:00004178       ??_C@_0DJ@IPBLACAP@Getting?5AccessibleRole_en_US?5?9?5@ 10026178     AccessBridgeJavaEntryPoints.obj
 0002:000041b4       ??_C@_0DM@BLDNLLEO@Getting?5AccessibleRole_en_US?5?9?5@ 100261b4     AccessBridgeJavaEntryPoints.obj
 0002:000041f0       ??_C@_0DI@FEPHIHOP@Getting?5AccessibleRole_en_US?5?9?5@ 100261f0     AccessBridgeJavaEntryPoints.obj
 0002:00004228       ??_C@_1EM@ICLLIBMO@?$AA?$FL?$AAI?$AAN?$AAF?$AAO?$AA?$FN?$AA?3?$AA?5?$AA?5?$AA?5?$AAA?$AAc?$AAc?$AAe?$AAs@ 10026228     AccessBridgeJavaEntryPoints.obj
 0002:00004274       ??_C@_0DI@OHCMPHFN@Getting?5AccessibleRole_en_US?5?9?5@ 10026274     AccessBridgeJavaEntryPoints.obj
 0002:000042ac       ??_C@_0CJ@JHFOCCMF@?$FLWARN?$FN?3?5?5?5Accessible?5Role?5en_US@ 100262ac     AccessBridgeJavaEntryPoints.obj
 0002:000042d8       ??_C@_0FA@EDCBAJIO@?$FLERROR?$FN?3?5either?5env?5?$DN?$DN?50?5or?5get@ 100262d8     AccessBridgeJavaEntryPoints.obj
 0002:00004328       ??_C@_0DF@HNCNCNCA@Getting?5AccessibleState?5?9?5call?5@ 10026328     AccessBridgeJavaEntryPoints.obj
 0002:00004360       ??_C@_0DD@FJJPIJBK@Getting?5AccessibleState?5?9?5call?5@ 10026360     AccessBridgeJavaEntryPoints.obj
 0002:00004394       ??_C@_0DE@HAGECOMD@Getting?5AccessibleState?5?9?5call?5@ 10026394     AccessBridgeJavaEntryPoints.obj
 0002:000043c8       ??_C@_0DH@HKADNDJG@Getting?5AccessibleState?5?9?5call?5@ 100263c8     AccessBridgeJavaEntryPoints.obj
 0002:00004400       ??_C@_0DD@CELBDLDG@Getting?5AccessibleState?5?9?5call?5@ 10026400     AccessBridgeJavaEntryPoints.obj
 0002:00004438       ??_C@_1EE@DCJFHGCM@?$AA?$FL?$AAI?$AAN?$AAF?$AAO?$AA?$FN?$AA?3?$AA?5?$AA?5?$AA?5?$AAA?$AAc?$AAc?$AAe?$AAs@ 10026438     AccessBridgeJavaEntryPoints.obj
 0002:0000447c       ??_C@_0DD@JHGKELIE@Getting?5AccessibleState?5?9?5call?5@ 1002647c     AccessBridgeJavaEntryPoints.obj
 0002:000044b0       ??_C@_0CF@EJIKBPCF@?$FLWARN?$FN?3?5?5?5Accessible?5States?5is?5@ 100264b0     AccessBridgeJavaEntryPoints.obj
 0002:000044d8       ??_C@_0EN@PLJCLDAI@?$FLERROR?$FN?3?5?5either?5env?5?$DN?$DN?50?5or?5ge@ 100264d8     AccessBridgeJavaEntryPoints.obj
 0002:00004528       ??_C@_0DL@NKOGKBKA@Getting?5AccessibleState_en_US?5?9@ 10026528     AccessBridgeJavaEntryPoints.obj
 0002:00004564       ??_C@_0DJ@EPIHCNDB@Getting?5AccessibleState_en_US?5?9@ 10026564     AccessBridgeJavaEntryPoints.obj
 0002:000045a0       ??_C@_0DK@NMMOMPCH@Getting?5AccessibleState_en_US?5?9@ 100265a0     AccessBridgeJavaEntryPoints.obj
 0002:000045dc       ??_C@_0DN@KFIOCDBN@Getting?5AccessibleState_en_US?5?9@ 100265dc     AccessBridgeJavaEntryPoints.obj
 0002:0000461c       ??_C@_0DJ@DCKJJPBN@Getting?5AccessibleState_en_US?5?9@ 1002661c     AccessBridgeJavaEntryPoints.obj
 0002:00004658       ??_C@_1FA@BNDENPHM@?$AA?$FL?$AAI?$AAN?$AAF?$AAO?$AA?$FN?$AA?3?$AA?5?$AA?5?$AA?5?$AAA?$AAc?$AAc?$AAe?$AAs@ 10026658     AccessBridgeJavaEntryPoints.obj
 0002:000046a8       ??_C@_0DJ@IBHCOPKP@Getting?5AccessibleState_en_US?5?9@ 100266a8     AccessBridgeJavaEntryPoints.obj
 0002:000046e4       ??_C@_0CL@LNKMOAJG@?$FLWARN?$FN?3?5?5?5Accessible?5States?5en_@ 100266e4     AccessBridgeJavaEntryPoints.obj
 0002:00004710       ??_C@_0FC@KNGBOCJI@?$FLERROR?$FN?3?5either?5env?5?$DN?$DN?50?5or?5get@ 10026710     AccessBridgeJavaEntryPoints.obj
 0002:00004764       ??_C@_0DK@NAACLIEE@Getting?5AccessibleIndexInParent@ 10026764     AccessBridgeJavaEntryPoints.obj
 0002:000047a0       ??_C@_0BP@LDKDBFNM@?$FLINFO?$FN?3?5?5?5Index?5in?5Parent?5?$DN?5?$CFd@ 100267a0     AccessBridgeJavaEntryPoints.obj
 0002:000047c0       ??_C@_0EO@FMBHNIPI@?$FLERROR?$FN?3?5?5either?5env?5?$DN?$DN?50?5or?5ge@ 100267c0     AccessBridgeJavaEntryPoints.obj
 0002:00004810       ??_C@_0EK@BLALEJAL@?$FLINFO?$FN?3?5?$CK?$CK?$CK?5jniEnv?3?5?$CFp?$DL?5accessB@ 10026810     AccessBridgeJavaEntryPoints.obj
 0002:0000485c       ??_C@_0DK@HBEJENLO@Getting?5AccessibleChildrenCount@ 1002685c     AccessBridgeJavaEntryPoints.obj
 0002:00004898       ??_C@_0BO@INNKBLPE@?$FLINFO?$FN?3?5?5?5Children?5count?5?$DN?5?$CFd@ 10026898     AccessBridgeJavaEntryPoints.obj
 0002:000048b8       ??_C@_0EO@BPNCCJLD@?$FLERROR?$FN?3?5?5either?5env?5?$DN?$DN?50?5or?5ge@ 100268b8     AccessBridgeJavaEntryPoints.obj
 0002:00004908       ??_C@_0EK@PAPEMOFA@?$FLINFO?$FN?3?5?$CK?$CK?$CK?5jniEnv?3?5?$CFp?$DL?5accessB@ 10026908     AccessBridgeJavaEntryPoints.obj
 0002:00004954       ??_C@_0DD@EIHALEFK@Getting?5AccessibleXcoord?5?9?5call@ 10026954     AccessBridgeJavaEntryPoints.obj
 0002:00004988       ??_C@_0BH@EMDFCPBA@?$FLINFO?$FN?3?5?5?5X?5coord?5?$DN?5?$CFd@ 10026988     AccessBridgeJavaEntryPoints.obj
 0002:000049a0       ??_C@_0EH@EAAFBPMN@?$FLERROR?$FN?3?5?5either?5env?5?$DN?$DN?50?5or?5ge@ 100269a0     AccessBridgeJavaEntryPoints.obj
 0002:000049e8       ??_C@_0EK@PIPPCCAB@?$FLINFO?$FN?3?5?$CK?$CK?$CK?5jniEnv?3?5?$CFX?$DL?5accessB@ 100269e8     AccessBridgeJavaEntryPoints.obj
 0002:00004a34       ??_C@_0DD@HOICCEKJ@Getting?5AccessibleYcoord?5?9?5call@ 10026a34     AccessBridgeJavaEntryPoints.obj
 0002:00004a68       ??_C@_0BH@JBKDPGJF@?$FLINFO?$FN?3?5?5?5Y?5coord?5?$DN?5?$CFd@ 10026a68     AccessBridgeJavaEntryPoints.obj
 0002:00004a80       ??_C@_0EH@CDACMGOJ@?$FLERROR?$FN?3?5?5either?5env?5?$DN?$DN?50?5or?5ge@ 10026a80     AccessBridgeJavaEntryPoints.obj
 0002:00004ac8       ??_C@_0DC@IECDLNHB@Getting?5AccessibleWidth?5?9?5call?5@ 10026ac8     AccessBridgeJavaEntryPoints.obj
 0002:00004afc       ??_C@_0BF@EEAFCLIB@?$FLINFO?$FN?3?5?5?5Width?5?$DN?5?$CFd@ 10026afc     AccessBridgeJavaEntryPoints.obj
 0002:00004b18       ??_C@_0EG@HOHNFBDJ@?$FLERROR?$FN?3?5?5either?5env?5?$DN?$DN?50?5or?5ge@ 10026b18     AccessBridgeJavaEntryPoints.obj
 0002:00004b60       ??_C@_0DD@DDJGOHAP@Getting?5AccessibleHeight?5?9?5call@ 10026b60     AccessBridgeJavaEntryPoints.obj
 0002:00004b94       ??_C@_0BG@DJGLJFGH@?$FLINFO?$FN?3?5?5?5Height?5?$DN?5?$CFd@ 10026b94     AccessBridgeJavaEntryPoints.obj
 0002:00004bb0       ??_C@_0EH@LBBAABEE@?$FLERROR?$FN?3?5?5either?5env?5?$DN?$DN?50?5or?5ge@ 10026bb0     AccessBridgeJavaEntryPoints.obj
 0002:00004bf8       ??_C@_0DJ@LNCBBGOH@Getting?5AccessibleComponent?5?9?5c@ 10026bf8     AccessBridgeJavaEntryPoints.obj
 0002:00004c34       ??_C@_0CD@PFGFGKFI@?$FLINFO?$FN?3?5?5?5AccessibleComponent?5?$DN@ 10026c34     AccessBridgeJavaEntryPoints.obj
 0002:00004c58       ??_C@_0DH@KGCNAJLL@Getting?5AccessibleComponent?5?9?5c@ 10026c58     AccessBridgeJavaEntryPoints.obj
 0002:00004c90       ??_C@_0EK@MOFEFKAP@?$FLERROR?$FN?3?5?5either?5env?5?$DN?$DN?50?5or?5ge@ 10026c90     AccessBridgeJavaEntryPoints.obj
 0002:00004cdc       ??_C@_0DG@DACOODAE@Getting?5AccessibleAction?5?9?5call@ 10026cdc     AccessBridgeJavaEntryPoints.obj
 0002:00004d14       ??_C@_0CA@PJFDOLN@?$FLINFO?$FN?3?5?5?5AccessibleAction?5?$DN?5?$CFp@ 10026d14     AccessBridgeJavaEntryPoints.obj
 0002:00004d34       ??_C@_0DE@DDPPAPLP@Getting?5AccessibleAction?5?9?5call@ 10026d34     AccessBridgeJavaEntryPoints.obj
 0002:00004d68       ??_C@_0EH@DKLGJNHO@?$FLERROR?$FN?3?5?5either?5env?5?$DN?$DN?50?5or?5ge@ 10026d68     AccessBridgeJavaEntryPoints.obj
 0002:00004db0       ??_C@_0DJ@CGHCFMLP@Getting?5AccessibleSelection?5?9?5c@ 10026db0     AccessBridgeJavaEntryPoints.obj
 0002:00004dec       ??_C@_0CD@PJLLNPAJ@?$FLINFO?$FN?3?5?5?5AccessibleSelection?5?$DN@ 10026dec     AccessBridgeJavaEntryPoints.obj
 0002:00004e10       ??_C@_0DH@PGPODJFA@Getting?5AccessibleSelection?5?9?5c@ 10026e10     AccessBridgeJavaEntryPoints.obj
 0002:00004e48       ??_C@_0EK@NDMBIFBF@?$FLERROR?$FN?3?5?5either?5env?5?$DN?$DN?50?5or?5ge@ 10026e48     AccessBridgeJavaEntryPoints.obj
 0002:00004e94       ??_C@_0DO@EELLKHNA@?$FLINFO?$FN?3?5?$CD?$CD?$CD?$CD?$CD?5Calling?5getAccess@ 10026e94     AccessBridgeJavaEntryPoints.obj
 0002:00004ed8       ??_C@_0EE@BBNKAGDP@?$FLINFO?$FN?3?5?$CD?$CD?$CD?$CD?$CD?5?4?4?4?5Returned?5from@ 10026ed8     AccessBridgeJavaEntryPoints.obj
 0002:00004f1c       ??_C@_0DL@DIOKBKHD@?$CD?$CD?$CD?$CD?$CD?5Getting?5AccessibleTable?5?9@ 10026f1c     AccessBridgeJavaEntryPoints.obj
 0002:00004f58       ??_C@_0CF@KFOMFGJG@?$FLINFO?$FN?3?5?5?5?$CD?$CD?$CD?$CD?$CD?5AccessibleTable@ 10026f58     AccessBridgeJavaEntryPoints.obj
 0002:00004f80       ??_C@_0DJ@ELALBBFD@?$CD?$CD?$CD?$CD?$CD?5Getting?5AccessibleTable?5?9@ 10026f80     AccessBridgeJavaEntryPoints.obj
 0002:00004fc0       ??_C@_0EF@MKDIKDJP@?$FLERROR?$FN?3?5either?5env?5?$DN?$DN?50?5or?5get@ 10026fc0     AccessBridgeJavaEntryPoints.obj
 0002:00005008       ??_C@_0BO@PJMPGGKG@?$FLINFO?$FN?3?5?5?5AccessibleText?5?$DN?5?$CFp@ 10027008     AccessBridgeJavaEntryPoints.obj
 0002:00005028       ??_C@_0DF@NJBDDCEL@Getting?5AccessibleValue?5?9?5call?5@ 10027028     AccessBridgeJavaEntryPoints.obj
 0002:00005060       ??_C@_0BP@BANALONE@?$FLINFO?$FN?3?5?5?5AccessibleValue?5?$DN?5?$CFp@ 10027060     AccessBridgeJavaEntryPoints.obj
 0002:00005080       ??_C@_0DD@JJHMAHMH@Getting?5AccessibleValue?5?9?5call?5@ 10027080     AccessBridgeJavaEntryPoints.obj
 0002:000050b8       ??_C@_0EG@HHMGAANK@?$FLERROR?$FN?3?5?5either?5env?5?$DN?$DN?50?5or?5ge@ 100270b8     AccessBridgeJavaEntryPoints.obj
 0002:00005100       ??_C@_0DJ@EACHBMMF@Getting?5AccessibleHypertext?5?9?5c@ 10027100     AccessBridgeJavaEntryPoints.obj
 0002:0000513c       ??_C@_0CD@DNELEHHF@?$FLINFO?$FN?3?5?5?5AccessibleHypertext?5?$DN@ 1002713c     AccessBridgeJavaEntryPoints.obj
 0002:00005160       ??_C@_0DH@DONNNDKC@Getting?5AccessibleHypertext?5?9?5c@ 10027160     AccessBridgeJavaEntryPoints.obj
 0002:00005198       ??_C@_0FA@DGBOEHHP@?$FLINFO?$FN?3?5Calling?5AccessBridgeJav@ 10027198     AccessBridgeJavaEntryPoints.obj
 0002:000051e8       ??_C@_0DF@OGEEIIFE@Getting?5AccessibleChild?5?9?5call?5@ 100271e8     AccessBridgeJavaEntryPoints.obj
 0002:00005220       ??_C@_0DB@OOCPCHE@Getting?5AccessibleChild?5?9?5call?5@ 10027220     AccessBridgeJavaEntryPoints.obj
 0002:00005254       ??_C@_0DD@JNMELFAO@Getting?5AccessibleChild?5?9?5call?5@ 10027254     AccessBridgeJavaEntryPoints.obj
 0002:00005288       ??_C@_0EC@MDNHELGM@?$FLERROR?$FN?3?5?5either?5env?5?$DN?$DN?50?5or?5ge@ 10027288     AccessBridgeJavaEntryPoints.obj
 0002:000052d0       ??_C@_0FB@PNLEIBEF@?$FLINFO?$FN?3?5Calling?5AccessBridgeJav@ 100272d0     AccessBridgeJavaEntryPoints.obj
 0002:00005324       ??_C@_0DG@BJCEEHCN@Getting?5AccessibleParent?5?9?5call@ 10027324     AccessBridgeJavaEntryPoints.obj
 0002:0000535c       ??_C@_0DC@MKLJMCBC@Getting?5AccessibleParent?5?9?5call@ 1002735c     AccessBridgeJavaEntryPoints.obj
 0002:00005390       ??_C@_0DE@IILKINNI@Getting?5AccessibleParent?5?9?5call@ 10027390     AccessBridgeJavaEntryPoints.obj
 0002:000053c8       ??_C@_0EH@MOCAMKEC@?$FLERROR?$FN?3?5?5either?5env?5?$DN?$DN?50?5or?5ge@ 100273c8     AccessBridgeJavaEntryPoints.obj
 0002:00005410       ??_C@_0EP@IDGNPODK@?$FLINFO?$FN?3?5?$CD?$CD?$CD?$CD?$CD?5Calling?5AccessBri@ 10027410     AccessBridgeJavaEntryPoints.obj
 0002:00005460       ??_C@_0EA@HDPDLION@?$CD?$CD?$CD?$CD?$CD?5Getting?5AccessibleTableRo@ 10027460     AccessBridgeJavaEntryPoints.obj
 0002:000054a0       ??_C@_0CF@OMEBMMOI@?$FLINFO?$FN?3?5?5?5?$CD?$CD?$CD?$CD?$CD?5table?5row?5count@ 100274a0     AccessBridgeJavaEntryPoints.obj
 0002:000054c8       ??_C@_0DN@MNMKPHBJ@?$FLERROR?$FN?3?5either?5env?5?$DN?$DN?50?5or?5get@ 100274c8     AccessBridgeJavaEntryPoints.obj
 0002:00005508       ??_C@_0DN@LHDBHOOP@Getting?5AccessibleTableColumnCo@ 10027508     AccessBridgeJavaEntryPoints.obj
 0002:00005548       ??_C@_0CI@GJGENPPF@?$FLINFO?$FN?3?5?5?5?$CD?$CD?$CD?$CD?$CD?5table?5column?5co@ 10027548     AccessBridgeJavaEntryPoints.obj
 0002:00005570       ??_C@_0EF@LHBDGBA@?$FLERROR?$FN?3?5either?5env?5?$DN?$DN?50?5or?5get@ 10027570     AccessBridgeJavaEntryPoints.obj
 0002:000055b8       ??_C@_0DH@GFGBCDOC@?$CD?$CD?$CD?$CD?$CD?5Getting?5AccessibleTable?5?9@ 100275b8     AccessBridgeJavaEntryPoints.obj
 0002:000055f0       ??_C@_0CF@DCCEHDEO@?$FLINFO?$FN?3?5?5?5?$CD?$CD?$CD?$CD?$CD?5accessibleTable@ 100275f0     AccessBridgeJavaEntryPoints.obj
 0002:00005618       ??_C@_0DP@FLHLIILD@?$FLINFO?$FN?3?5?$CD?$CD?$CD?$CD?$CD?5Calling?5getContex@ 10027618     AccessBridgeJavaEntryPoints.obj
 0002:00005658       ??_C@_0EF@JOJDMPNM@?$FLINFO?$FN?3?5?$CD?$CD?$CD?$CD?$CD?5?4?4?4?5Returned?5from@ 10027658     AccessBridgeJavaEntryPoints.obj
 0002:000056a0       ??_C@_0CH@GEKEKGKL@?$FLINFO?$FN?3?5?5?5?$CD?$CD?$CD?$CD?$CD?5accessibleConte@ 100276a0     AccessBridgeJavaEntryPoints.obj
 0002:000056c8       ??_C@_0EG@CNEBJJDJ@?$FLERROR?$FN?3?5either?5env?5?$DN?$DN?50?5or?5get@ 100276c8     AccessBridgeJavaEntryPoints.obj
 0002:00005710       ??_C@_0FE@GFOFNDOE@?$FLINFO?$FN?3?5?$CD?$CD?$CD?$CD?$CD?5Calling?5AccessBri@ 10027710     AccessBridgeJavaEntryPoints.obj
 0002:00005768       ??_C@_0GF@GDALOMIB@?$FLINFO?$FN?3?5?$CD?$CD?$CD?$CD?$CD?5Calling?5AccessBri@ 10027768     AccessBridgeJavaEntryPoints.obj
 0002:000057d0       ??_C@_0EB@IFJOCDDE@?$CD?$CD?$CD?$CD?$CD?5Getting?5AccessibleTableCe@ 100277d0     AccessBridgeJavaEntryPoints.obj
 0002:00005814       ??_C@_0CG@KKOMOEPJ@?$FLINFO?$FN?3?5?5?5?$CD?$CD?$CD?$CD?$CD?5table?5cell?5inde@ 10027814     AccessBridgeJavaEntryPoints.obj
 0002:00005840       ??_C@_0ED@MJPDAFIJ@?$FLERROR?$FN?3?5either?5env?5?$DN?$DN?50?5or?5get@ 10027840     AccessBridgeJavaEntryPoints.obj
 0002:00005888       ??_C@_0EK@HFAIKGKI@?$CD?$CD?$CD?$CD?$CD?5Getting?5AccessibleTableCe@ 10027888     AccessBridgeJavaEntryPoints.obj
 0002:000058d4       ??_C@_0CL@CDCOGIJD@?$FLINFO?$FN?3?5?5?5?$CD?$CD?$CD?$CD?$CD?5table?5cell?5row?5@ 100278d4     AccessBridgeJavaEntryPoints.obj
 0002:00005900       ??_C@_0EH@MFABNFMJ@?$FLERROR?$FN?3?5either?5env?5?$DN?$DN?50?5or?5get@ 10027900     AccessBridgeJavaEntryPoints.obj
 0002:00005948       ??_C@_0EN@GIPGNDGO@?$CD?$CD?$CD?$CD?$CD?5Getting?5AccessibleTableCe@ 10027948     AccessBridgeJavaEntryPoints.obj
 0002:00005998       ??_C@_0CN@JHPAHOLB@?$FLINFO?$FN?3?5?5?$CD?$CD?$CD?$CD?$CD?5table?5cell?5colum@ 10027998     AccessBridgeJavaEntryPoints.obj
 0002:000059c8       ??_C@_0EK@MCJJFMIG@?$FLERROR?$FN?3?5either?5env?5?$DN?$DN?50?5or?5get@ 100279c8     AccessBridgeJavaEntryPoints.obj
 0002:00005a18       ??_C@_0EK@OAKDMNFI@?$CD?$CD?$CD?$CD?$CD?5Getting?5isAccessibleTable@ 10027a18     AccessBridgeJavaEntryPoints.obj
 0002:00005a64       ??_C@_0CL@FGJJGBAG@?$FLINFO?$FN?3?5?5?5?$CD?$CD?$CD?$CD?$CD?5table?5cell?5isSe@ 10027a64     AccessBridgeJavaEntryPoints.obj
 0002:00005a90       ??_C@_0EF@NDHLMIOL@?$FLERROR?$FN?3?5either?5env?5?$DN?$DN?50?5or?5isA@ 10027a90     AccessBridgeJavaEntryPoints.obj
 0002:00005ad8       ??_C@_0FA@PNFLEDNO@?$CD?$CD?$CD?$CD?$CD?5Getting?5AccessibleTableCe@ 10027ad8     AccessBridgeJavaEntryPoints.obj
 0002:00005b28       ??_C@_0EM@CCOLAKIM@?$CD?$CD?$CD?$CD?$CD?5Getting?5AccessibleTableCe@ 10027b28     AccessBridgeJavaEntryPoints.obj
 0002:00005b74       ??_C@_0DC@NHIEBBHC@?$FLINFO?$FN?3?5?5?5?$CD?$CD?$CD?$CD?$CD?5table?5cell?5Acce@ 10027b74     AccessBridgeJavaEntryPoints.obj
 0002:00005ba8       ??_C@_0EP@BAKELAEL@?$FLERROR?$FN?3?5either?5env?5?$DN?$DN?50?5or?5get@ 10027ba8     AccessBridgeJavaEntryPoints.obj
 0002:00005bf8       ??_C@_0FJ@JCFFKNHH@?$FLINFO?$FN?3?5?5?$CD?$CD?$CD?$CD?$CD?5Calling?5AccessBr@ 10027bf8     AccessBridgeJavaEntryPoints.obj
 0002:00005c58       ??_C@_0FE@DGILOPPB@?$FLINFO?$FN?3?5?$CD?$CD?$CD?$CD?$CD?5Calling?5AccessBri@ 10027c58     AccessBridgeJavaEntryPoints.obj
 0002:00005cb0       ??_C@_0EJ@OONHAJKO@?$CD?$CD?$CD?$CD?$CD?5Getting?5AccessibleTableRo@ 10027cb0     AccessBridgeJavaEntryPoints.obj
 0002:00005d00       ??_C@_0EG@NDBCAEFO@?$FLERROR?$FN?3?5either?5env?5?$DN?$DN?50?5or?5get@ 10027d00     AccessBridgeJavaEntryPoints.obj
 0002:00005d48       ??_C@_0EG@DALLPPNJ@Getting?5AccessibleTableRowHeade@ 10027d48     AccessBridgeJavaEntryPoints.obj
 0002:00005d90       ??_C@_0EO@OOHGOEEK@?$FLERROR?$FN?3?5either?5env?5?$DN?$DN?50?5or?5get@ 10027d90     AccessBridgeJavaEntryPoints.obj
 0002:00005de0       ??_C@_0EE@GCIECGJK@?$CD?$CD?$CD?$CD?$CD?5Getting?5AccessibleTableRo@ 10027de0     AccessBridgeJavaEntryPoints.obj
 0002:00005e28       ??_C@_0EA@OEOKKCMN@?$CD?$CD?$CD?$CD?$CD?5Getting?5AccessibleTableRo@ 10027e28     AccessBridgeJavaEntryPoints.obj
 0002:00005e68       ??_C@_0DA@BEAKBEEG@?$FLINFO?$FN?3?5?5?5?$CD?$CD?$CD?$CD?$CD?5row?5header?5Acce@ 10027e68     AccessBridgeJavaEntryPoints.obj
 0002:00005e98       ??_C@_0ED@KKINKAGC@?$FLERROR?$FN?3?5either?5env?5?$DN?$DN?50?5or?5get@ 10027e98     AccessBridgeJavaEntryPoints.obj
 0002:00005ee0       ??_C@_0FL@PPBJDPIL@?$FLINFO?$FN?3?5?5?5?$CD?$CD?$CD?$CD?$CD?5Calling?5AccessB@ 10027ee0     AccessBridgeJavaEntryPoints.obj
 0002:00005f40       ??_C@_0FH@EJOHBEGH@?$FLINFO?$FN?3?5?$CD?$CD?$CD?$CD?$CD?5Calling?5AccessBri@ 10027f40     AccessBridgeJavaEntryPoints.obj
 0002:00005f98       ??_C@_0EM@ILKGOFLG@?$CD?$CD?$CD?$CD?$CD?5Getting?5AccessibleTableCo@ 10027f98     AccessBridgeJavaEntryPoints.obj
 0002:00005fe8       ??_C@_0EK@LPGMLANE@?$FLERROR?$FN?3?5?5either?5env?5?$DN?$DN?50?5or?5ge@ 10027fe8     AccessBridgeJavaEntryPoints.obj
 0002:00006038       ??_C@_0EJ@CKEIFDID@Getting?5AccessibleTableColumnHe@ 10028038     AccessBridgeJavaEntryPoints.obj
 0002:00006088       ??_C@_0FB@LHNIAEHP@?$FLERROR?$FN?3?5either?5env?5?$DN?$DN?50?5or?5get@ 10028088     AccessBridgeJavaEntryPoints.obj
 0002:000060e0       ??_C@_0EH@JIOGAIC@?$CD?$CD?$CD?$CD?$CD?5Getting?5AccessibleTableCo@ 100280e0     AccessBridgeJavaEntryPoints.obj
 0002:00006128       ??_C@_0ED@DCBGPFPL@?$CD?$CD?$CD?$CD?$CD?5Getting?5AccessibleTableCo@ 10028128     AccessBridgeJavaEntryPoints.obj
 0002:0000616c       ??_C@_0DD@JPNBDACB@?$FLINFO?$FN?3?5?5?5?$CD?$CD?$CD?$CD?$CD?5column?5header?5A@ 1002816c     AccessBridgeJavaEntryPoints.obj
 0002:000061a0       ??_C@_0EG@EHCJNLHA@?$FLERROR?$FN?3?5either?5env?5?$DN?$DN?50?5or?5get@ 100281a0     AccessBridgeJavaEntryPoints.obj
 0002:000061e8       ??_C@_0FO@DKAHOFOA@?$FLINFO?$FN?3?5?5?5?$CD?$CD?$CD?$CD?$CD?5Calling?5AccessB@ 100281e8     AccessBridgeJavaEntryPoints.obj
 0002:00006248       ??_C@_0FJ@IPEPPO@?$FLINFO?$FN?3?5?$CD?$CD?$CD?$CD?$CD?5Calling?5AccessBri@ 10028248     AccessBridgeJavaEntryPoints.obj
 0002:000062a8       ??_C@_0ED@ECGPKBKB@Getting?5AccessibleTableRowDescr@ 100282a8     AccessBridgeJavaEntryPoints.obj
 0002:000062ec       ??_C@_0DP@MGPIFPGE@Getting?5AccessibleTableRowDescr@ 100282ec     AccessBridgeJavaEntryPoints.obj
 0002:00006330       ??_C@_0EB@HPGBLABA@Getting?5AccessibleTableRowDescr@ 10028330     AccessBridgeJavaEntryPoints.obj
 0002:00006378       ??_C@_0EI@FALMFIJI@?$FLERROR?$FN?3?5either?5env?5?$DN?$DN?50?5or?5get@ 10028378     AccessBridgeJavaEntryPoints.obj
 0002:000063c0       ??_C@_0FM@OGMEFLJF@?$FLINFO?$FN?3?5?$CD?$CD?$CD?$CD?$CD?5Calling?5AccessBri@ 100283c0     AccessBridgeJavaEntryPoints.obj
 0002:00006420       ??_C@_0EG@HNHAKGAA@Getting?5AccessibleTableColumnDe@ 10028420     AccessBridgeJavaEntryPoints.obj
 0002:00006468       ??_C@_0EC@OOIBKPKB@Getting?5AccessibleTableColumnDe@ 10028468     AccessBridgeJavaEntryPoints.obj
 0002:000064b0       ??_C@_0EE@HEFBEJHO@Getting?5AccessibleTableColumnDe@ 100284b0     AccessBridgeJavaEntryPoints.obj
 0002:000064f8       ??_C@_0EL@MDADMDPK@?$FLERROR?$FN?3?5either?5env?5?$DN?$DN?50?5or?5get@ 100284f8     AccessBridgeJavaEntryPoints.obj
 0002:00006548       ??_C@_0FD@NONCILOI@?$FLINFO?$FN?3?5?$CD?$CD?$CD?$CD?$CD?5AccessBridgeJavaE@ 10028548     AccessBridgeJavaEntryPoints.obj
 0002:000065a0       ??_C@_0EJ@CONOFLFI@?$CD?$CD?$CD?$CD?$CD?5Getting?5AccessibleTableRo@ 100285a0     AccessBridgeJavaEntryPoints.obj
 0002:000065ec       ??_C@_0CP@GJAEEGNO@?$FLINFO?$FN?3?5?5?5?$CD?$CD?$CD?$CD?$CD?5table?5row?5selec@ 100285ec     AccessBridgeJavaEntryPoints.obj
 0002:00006620       ??_C@_0EL@JIBDDMIF@?$FLERROR?$FN?3?5either?5env?5?$DN?$DN?50?5or?5get@ 10028620     AccessBridgeJavaEntryPoints.obj
 0002:00006670       ??_C@_0FA@LAKDEELL@?$FLINFO?$FN?3?5?$CD?$CD?$CD?$CD?$CD?5AccessBridgeJavaE@ 10028670     AccessBridgeJavaEntryPoints.obj
 0002:000066c0       ??_C@_0EJ@PAIANDP@?$CD?$CD?$CD?$CD?$CD?5Getting?5isAccessibleTable@ 100286c0     AccessBridgeJavaEntryPoints.obj
 0002:0000670c       ??_C@_0CK@ENCKDAKJ@?$FLINFO?$FN?3?5?5?5?$CD?$CD?$CD?$CD?$CD?5table?5row?5isSel@ 1002870c     AccessBridgeJavaEntryPoints.obj
 0002:00006738       ??_C@_0EE@OPDECGCG@?$FLERROR?$FN?3?5either?5env?5?$DN?$DN?50?5or?5isA@ 10028738     AccessBridgeJavaEntryPoints.obj
 0002:00006780       ??_C@_0FG@BNGDNOAB@?$FLINFO?$FN?3?5?$CD?$CD?$CD?$CD?$CD?5AccessBridgeJavaE@ 10028780     AccessBridgeJavaEntryPoints.obj
 0002:000067d8       ??_C@_0EF@MANEDMPN@?$CD?$CD?$CD?$CD?$CD?5Getting?5AccessibleTableRo@ 100287d8     AccessBridgeJavaEntryPoints.obj
 0002:00006820       ??_C@_0CN@EGDPALEC@?$FLINFO?$FN?3?5?5?5?$CD?$CD?$CD?$CD?$CD?5table?5row?5selec@ 10028820     AccessBridgeJavaEntryPoints.obj
 0002:00006850       ??_C@_0FH@IBIGBELL@?$FLINFO?$FN?3?5?5?5?$CD?$CD?$CD?$CD?$CD?5AccessBridgeJav@ 10028850     AccessBridgeJavaEntryPoints.obj
 0002:000068a8       ??_C@_0FG@LAILABJF@?$FLINFO?$FN?3?5?$CD?$CD?$CD?$CD?$CD?5AccessBridgeJavaE@ 100288a8     AccessBridgeJavaEntryPoints.obj
 0002:00006900       ??_C@_0EM@ELKPLHEA@?$CD?$CD?$CD?$CD?$CD?5Getting?5AccessibleTableCo@ 10028900     AccessBridgeJavaEntryPoints.obj
 0002:0000694c       ??_C@_0DC@EFKBJLFF@?$FLINFO?$FN?3?5?5?5?$CD?$CD?$CD?$CD?$CD?5table?5column?5se@ 1002894c     AccessBridgeJavaEntryPoints.obj
 0002:00006980       ??_C@_0FD@ODFPPIDD@?$FLINFO?$FN?3?5?$CD?$CD?$CD?$CD?$CD?5AccessBridgeJavaE@ 10028980     AccessBridgeJavaEntryPoints.obj
 0002:000069d8       ??_C@_0EM@HPIPAKED@?$CD?$CD?$CD?$CD?$CD?5Getting?5isAccessibleTable@ 100289d8     AccessBridgeJavaEntryPoints.obj
 0002:00006a24       ??_C@_0CN@OPIEHDOO@?$FLINFO?$FN?3?5?5?5?$CD?$CD?$CD?$CD?$CD?5table?5column?5is@ 10028a24     AccessBridgeJavaEntryPoints.obj
 0002:00006a58       ??_C@_0EI@CBBNNOEE@?$FLERROR?$FN?3?5?5either?5env?5?$DN?$DN?50?5or?5is@ 10028a58     AccessBridgeJavaEntryPoints.obj
 0002:00006aa0       ??_C@_0FK@KHEECFFC@?$FLINFO?$FN?3?5?$CD?$CD?$CD?$CD?$CD?5AccessBridgeJavaE@ 10028aa0     AccessBridgeJavaEntryPoints.obj
 0002:00006b00       ??_C@_0EI@NDNDKOON@?$CD?$CD?$CD?$CD?$CD?5Getting?5AccessibleTableCo@ 10028b00     AccessBridgeJavaEntryPoints.obj
 0002:00006b48       ??_C@_0DA@FGAFLCDN@?$FLINFO?$FN?3?5?5?5?$CD?$CD?$CD?$CD?$CD?5table?5Column?5se@ 10028b48     AccessBridgeJavaEntryPoints.obj
 0002:00006b78       ??_C@_0FK@PECCMPIL@?$FLINFO?$FN?3?5?5?5?$CD?$CD?$CD?$CD?$CD?5AccessBridgeJav@ 10028b78     AccessBridgeJavaEntryPoints.obj
 0002:00006bd8       ??_C@_0EP@DEKNIMFA@?$FLINFO?$FN?3?5?$CD?$CD?$CD?$CD?$CD?5AccessBridgeJavaE@ 10028bd8     AccessBridgeJavaEntryPoints.obj
 0002:00006c28       ??_C@_0DL@DELNDLCL@?$CD?$CD?$CD?$CD?$CD?5Getting?5AccessibleTableRo@ 10028c28     AccessBridgeJavaEntryPoints.obj
 0002:00006c64       ??_C@_0BP@MEJOIGMM@?$FLINFO?$FN?3?5?5?5?$CD?$CD?$CD?$CD?$CD?5table?5row?5?$DN?5?$CFd@ 10028c64     AccessBridgeJavaEntryPoints.obj
 0002:00006c84       ??_C@_0DN@DIFOEGJK@?$FLERROR?$FN?3?5either?5env?5?$DN?$DN?50?5or?5get@ 10028c84     AccessBridgeJavaEntryPoints.obj
 0002:00006cc8       ??_C@_0FC@BFBAOEGI@?$FLINFO?$FN?3?5?$CD?$CD?$CD?$CD?$CD?5AccessBridgeJavaE@ 10028cc8     AccessBridgeJavaEntryPoints.obj
 0002:00006d1c       ??_C@_0DO@MBGEOOOH@?$CD?$CD?$CD?$CD?$CD?5Getting?5AccessibleTableCo@ 10028d1c     AccessBridgeJavaEntryPoints.obj
 0002:00006d5c       ??_C@_0CC@CJBEHFKG@?$FLINFO?$FN?3?5?5?5?$CD?$CD?$CD?$CD?$CD?5table?5column?5?$DN?5@ 10028d5c     AccessBridgeJavaEntryPoints.obj
 0002:00006d80       ??_C@_0EA@IFBLPNLC@?$FLERROR?$FN?3?5either?5env?5?$DN?$DN?50?5or?5get@ 10028d80     AccessBridgeJavaEntryPoints.obj
 0002:00006dc0       ??_C@_0FH@GMMGKHHK@?$FLINFO?$FN?3?5?$CD?$CD?$CD?$CD?$CD?5AccessBridgeJavaE@ 10028dc0     AccessBridgeJavaEntryPoints.obj
 0002:00006e18       ??_C@_0EA@IDLLLJIK@?$CD?$CD?$CD?$CD?$CD?5Getting?5getAccessibleTabl@ 10028e18     AccessBridgeJavaEntryPoints.obj
 0002:00006e58       ??_C@_0CB@JIHDIDBK@?$FLINFO?$FN?3?5?5?5?$CD?$CD?$CD?$CD?$CD?5table?5index?5?$DN?5?$CF@ 10028e58     AccessBridgeJavaEntryPoints.obj
 0002:00006e7c       ??_C@_0DP@EPGMKJOF@?$FLERROR?$FN?3?5either?5env?5?$DN?$DN?50?5or?5get@ 10028e7c     AccessBridgeJavaEntryPoints.obj
 0002:00006ec0       ??_C@_0EM@OMNMKDMF@?$FLINFO?$FN?3?5?$CD?$CD?$CD?$CD?$CD?5AccessBridgeJavaE@ 10028ec0     AccessBridgeJavaEntryPoints.obj
 0002:00006f10       ??_C@_0EA@LPBOBAAO@?$CD?$CD?$CD?$CD?$CD?5Getting?5AccessibleRelatio@ 10028f10     AccessBridgeJavaEntryPoints.obj
 0002:00006f50       ??_C@_0CO@JNBGELMK@?$FLINFO?$FN?3?5?5?5?$CD?$CD?$CD?$CD?$CD?5AccessibleRelat@ 10028f50     AccessBridgeJavaEntryPoints.obj
 0002:00006f80       ??_C@_0DL@KJPPMLJK@Getting?5AccessibleRelationKey?5?9@ 10028f80     AccessBridgeJavaEntryPoints.obj
 0002:00006fbc       ??_C@_0DK@CJPLLCPL@Getting?5AccessibleRelation?5key?5@ 10028fbc     AccessBridgeJavaEntryPoints.obj
 0002:00006ff8       ??_C@_0DL@KHBJJIBG@Getting?5AccessibleRelation?5key?5@ 10028ff8     AccessBridgeJavaEntryPoints.obj
 0002:00007034       ??_C@_0DO@GNGKCACF@Getting?5AccessibleRelation?5key?5@ 10029034     AccessBridgeJavaEntryPoints.obj
 0002:00007074       ??_C@_0CL@LKNHIIFA@?$FLINFO?$FN?3?5?$CD?$CD?$CD?$CD?$CD?5AccessibleRelatio@ 10029074     AccessBridgeJavaEntryPoints.obj
 0002:000070a0       ??_C@_0DK@OHAOHAGF@Getting?5AccessibleRelation?5key?5@ 100290a0     AccessBridgeJavaEntryPoints.obj
 0002:000070dc       ??_C@_0CK@FLLDFIHJ@?$FLWARN?$FN?3?5?5?5AccessibleRelation?5ke@ 100290dc     AccessBridgeJavaEntryPoints.obj
 0002:00007108       ??_C@_0DL@FOJGEEOM@Getting?5AccessibleRelationSet?5?9@ 10029108     AccessBridgeJavaEntryPoints.obj
 0002:00007144       ??_C@_0DH@OOCHFOKL@Getting?5AccessibleRelationSet?5?9@ 10029144     AccessBridgeJavaEntryPoints.obj
 0002:0000717c       ??_C@_0CA@NHODALDJ@?$FLINFO?$FN?3?5?5?5relation?5set?5item?3?5?$CFp@ 1002917c     AccessBridgeJavaEntryPoints.obj
 0002:000071a0       ??_C@_0FA@NBCFFMGI@?$FLINFO?$FN?3?5?5?5?$CD?$CD?$CD?$CD?$CD?5AccessBridgeJav@ 100291a0     AccessBridgeJavaEntryPoints.obj
 0002:000071f0       ??_C@_0EK@KKPLDFBH@?$FLINFO?$FN?3?5?$CD?$CD?$CD?$CD?$CD?5AccessBridgeJavaE@ 100291f0     AccessBridgeJavaEntryPoints.obj
 0002:0000723c       ??_C@_0DP@KAHCJAMC@?$CD?$CD?$CD?$CD?$CD?5Getting?5AccessibleHyperte@ 1002923c     AccessBridgeJavaEntryPoints.obj
 0002:0000727c       ??_C@_0DL@BCGGEGFO@?$CD?$CD?$CD?$CD?$CD?5Getting?5AccessibleHyperte@ 1002927c     AccessBridgeJavaEntryPoints.obj
 0002:000072b8       ??_C@_0CJ@KAIOACGL@?$FLINFO?$FN?3?5?5?5?$CD?$CD?$CD?$CD?$CD?5AccessibleHyper@ 100292b8     AccessBridgeJavaEntryPoints.obj
 0002:000072e4       ??_C@_0DK@IMJHJIPP@?$FLWARN?$FN?3?5?5?5?$CD?$CD?$CD?$CD?$CD?5null?5Accessible@ 100292e4     AccessBridgeJavaEntryPoints.obj
 0002:00007320       ??_C@_0DI@FEBHIMOE@?$CD?$CD?$CD?$CD?$CD?5Getting?5hyperlink?5count?5?9@ 10029320     AccessBridgeJavaEntryPoints.obj
 0002:00007358       ??_C@_0CF@OFPNIMKK@?$FLINFO?$FN?3?5?5?5?$CD?$CD?$CD?$CD?$CD?5hyperlink?5count@ 10029358     AccessBridgeJavaEntryPoints.obj
 0002:00007380       ??_C@_0DP@CIGIOMPM@?$CD?$CD?$CD?$CD?$CD?5Getting?5AccessibleHyperli@ 10029380     AccessBridgeJavaEntryPoints.obj
 0002:000073c0       ??_C@_0DL@PDIOCHOJ@?$CD?$CD?$CD?$CD?$CD?5Getting?5AccessibleHyperli@ 100293c0     AccessBridgeJavaEntryPoints.obj
 0002:000073fc       ??_C@_0CJ@FJIBOEOI@?$FLINFO?$FN?3?5?5?5?$CD?$CD?$CD?$CD?$CD?5AccessibleHyper@ 100293fc     AccessBridgeJavaEntryPoints.obj
 0002:00007428       ??_C@_0DE@FAMBBMPD@Getting?5hyperlink?5text?5?9?5call?5t@ 10029428     AccessBridgeJavaEntryPoints.obj
 0002:0000745c       ??_C@_0DM@FFPIAIEA@Getting?5AccessibleHyperlink?5tex@ 1002945c     AccessBridgeJavaEntryPoints.obj
 0002:00007498       ??_C@_0DN@PLNGPBKI@Getting?5AccessibleHyperlink?5tex@ 10029498     AccessBridgeJavaEntryPoints.obj
 0002:000074d8       ??_C@_0EA@BNEOPMKM@Getting?5AccessibleHyperlink?5tex@ 100294d8     AccessBridgeJavaEntryPoints.obj
 0002:00007518       ??_C@_0CN@IIHGCCLN@?$FLINFO?$FN?3?5?$CD?$CD?$CD?$CD?$CD?5AccessibleHyperli@ 10029518     AccessBridgeJavaEntryPoints.obj
 0002:00007548       ??_C@_0DM@JLANMKNO@Getting?5AccessibleHyperlink?5tex@ 10029548     AccessBridgeJavaEntryPoints.obj
 0002:00007584       ??_C@_0CM@DKPAOLF@?$FLWARN?$FN?3?5?5?5AccessibleHyperlink?5t@ 10029584     AccessBridgeJavaEntryPoints.obj
 0002:000075b0       ??_C@_0DO@DJICJOGB@?$CD?$CD?$CD?$CD?$CD?5Getting?5hyperlink?5start?5i@ 100295b0     AccessBridgeJavaEntryPoints.obj
 0002:000075f0       ??_C@_0CL@GNKIIEKN@?$FLINFO?$FN?3?5?5?5?$CD?$CD?$CD?$CD?$CD?5hyperlink?5start@ 100295f0     AccessBridgeJavaEntryPoints.obj
 0002:0000761c       ??_C@_0DM@MGHLFEBK@?$CD?$CD?$CD?$CD?$CD?5Getting?5hyperlink?5end?5ind@ 1002961c     AccessBridgeJavaEntryPoints.obj
 0002:00007658       ??_C@_0CJ@POHPAAGA@?$FLINFO?$FN?3?5?5?5?$CD?$CD?$CD?$CD?$CD?5hyperlink?5end?5i@ 10029658     AccessBridgeJavaEntryPoints.obj
 0002:00007688       ??_C@_0EO@MCEJOGLJ@?$FLINFO?$FN?3?5?5?5?$CD?$CD?$CD?$CD?$CD?5AccessBridgeJav@ 10029688     AccessBridgeJavaEntryPoints.obj
 0002:000076d8       ??_C@_0FC@PJEJEFPL@?$FLINFO?$FN?3?5Calling?5AccessBridgeJav@ 100296d8     AccessBridgeJavaEntryPoints.obj
 0002:0000772c       ??_C@_0DK@IAFPEHK@activateAccessibleHyperlink?5?9?5c@ 1002972c     AccessBridgeJavaEntryPoints.obj
 0002:00007768       ??_C@_0EG@NBDJGANF@?$FLERROR?$FN?3?5either?5jniEnv?5?$DN?$DN?50?5or?5@ 10029768     AccessBridgeJavaEntryPoints.obj
 0002:000077b0       ??_C@_0FO@LCEKGOMG@?$FLINFO?$FN?3?5?$CD?$CD?$CD?$CD?$CD?5AccessBridgeJavaE@ 100297b0     AccessBridgeJavaEntryPoints.obj
 0002:00007810       ??_C@_0CD@FKJEEIHP@?$FLINFO?$FN?3?5?5?5getting?5hyperlink?5?$CFd?5@ 10029810     AccessBridgeJavaEntryPoints.obj
 0002:00007838       ??_C@_0FB@LIBMBPHJ@?$FLINFO?$FN?3?5?5?5?$CD?$CD?$CD?$CD?$CD?5AccessBridgeJav@ 10029838     AccessBridgeJavaEntryPoints.obj
 0002:00007890       ??_C@_0EL@OJOFGNCE@?$FLINFO?$FN?3?5?$CD?$CD?$CD?$CD?$CD?5AccessBridgeJavaE@ 10029890     AccessBridgeJavaEntryPoints.obj
 0002:000078e0       ??_C@_0FL@JFFPJPNI@?$FLINFO?$FN?3?5?$CD?$CD?$CD?$CD?$CD?5AccessBridgeJavaE@ 100298e0     AccessBridgeJavaEntryPoints.obj
 0002:0000793c       ??_C@_0DI@MNABDACM@?$CD?$CD?$CD?$CD?$CD?5Getting?5hyperlink?5index?5?9@ 1002993c     AccessBridgeJavaEntryPoints.obj
 0002:00007974       ??_C@_0CF@MJOBJPAA@?$FLINFO?$FN?3?5?5?5?$CD?$CD?$CD?$CD?$CD?5hyperlink?5index@ 10029974     AccessBridgeJavaEntryPoints.obj
 0002:000079a0       ??_C@_0FC@MDIFEEKA@?$FLINFO?$FN?3?5?$CD?$CD?$CD?$CD?$CD?5AccessBridgeJavaE@ 100299a0     AccessBridgeJavaEntryPoints.obj
 0002:000079f8       ??_C@_0EM@DFNHGKKP@?$FLINFO?$FN?3?5?$CD?$CD?$CD?$CD?$CD?5AccessBridgeJavaE@ 100299f8     AccessBridgeJavaEntryPoints.obj
 0002:00007a44       ??_C@_0DL@CLKJJKNH@?$CD?$CD?$CD?$CD?$CD?5Getting?5key?5bindings?5coun@ 10029a44     AccessBridgeJavaEntryPoints.obj
 0002:00007a80       ??_C@_0CI@OKJNHPKA@?$FLINFO?$FN?3?5?5?5?$CD?$CD?$CD?$CD?$CD?5key?5bindings?5co@ 10029a80     AccessBridgeJavaEntryPoints.obj
 0002:00007aa8       ??_C@_0DP@FMCKMBKC@?$CD?$CD?$CD?$CD?$CD?5Getting?5key?5binding?5chara@ 10029aa8     AccessBridgeJavaEntryPoints.obj
 0002:00007ae8       ??_C@_0FN@DCEDCNML@?$FLINFO?$FN?3?5?5?5?$CD?$CD?$CD?$CD?$CD?5key?5binding?5cha@ 10029ae8     AccessBridgeJavaEntryPoints.obj
 0002:00007b48       ??_C@_0DO@HKGJEFDO@?$CD?$CD?$CD?$CD?$CD?5Getting?5key?5binding?5modif@ 10029b48     AccessBridgeJavaEntryPoints.obj
 0002:00007b88       ??_C@_0CK@OFBJGPDI@?$FLINFO?$FN?3?5?5?$CD?$CD?$CD?$CD?$CD?5key?5binding?5modi@ 10029b88     AccessBridgeJavaEntryPoints.obj
 0002:00007bb8       ??_C@_0EG@MKCABNJD@?$FLINFO?$FN?3?5?$CD?$CD?$CD?$CD?$CD?5AccessBridgeJavaE@ 10029bb8     AccessBridgeJavaEntryPoints.obj
 0002:00007c00       ??_C@_0CG@IDHCCFPM@?$FLWARN?$FN?3?5?5?5?$CD?$CD?$CD?$CD?$CD?5missing?5method?$CI@ 10029c00     AccessBridgeJavaEntryPoints.obj
 0002:00007c28       ??_C@_0DE@JDHACCPK@?$CD?$CD?$CD?$CD?$CD?5Getting?5icons?5count?5?9?5cal@ 10029c28     AccessBridgeJavaEntryPoints.obj
 0002:00007c5c       ??_C@_0CB@DPKCEABK@?$FLINFO?$FN?3?5?5?5?$CD?$CD?$CD?$CD?$CD?5icons?5count?5?$DN?5?$CF@ 10029c5c     AccessBridgeJavaEntryPoints.obj
 0002:00007c80       ??_C@_0DG@HKLCCMCD@Getting?5icon?5description?5?9?5call@ 10029c80     AccessBridgeJavaEntryPoints.obj
 0002:00007cb8       ??_C@_0DO@JICPIJF@Getting?5AccessibleIcon?5descript@ 10029cb8     AccessBridgeJavaEntryPoints.obj
 0002:00007cf8       ??_C@_0DP@NDDKNAD@Getting?5AccessibleIcon?5descript@ 10029cf8     AccessBridgeJavaEntryPoints.obj
 0002:00007d38       ??_C@_0EC@OANEKHE@Getting?5AccessibleIcon?5descript@ 10029d38     AccessBridgeJavaEntryPoints.obj
 0002:00007d7c       ??_C@_0CP@OGEOHJKD@?$FLINFO?$FN?3?5?$CD?$CD?$CD?$CD?$CD?5AccessibleIcon?5de@ 10029d7c     AccessBridgeJavaEntryPoints.obj
 0002:00007dac       ??_C@_0DO@MHHHDKAL@Getting?5AccessibleIcon?5descript@ 10029dac     AccessBridgeJavaEntryPoints.obj
 0002:00007dec       ??_C@_0CO@EGEFBBBG@?$FLWARN?$FN?3?5?5?5AccessibleIcon?5descri@ 10029dec     AccessBridgeJavaEntryPoints.obj
 0002:00007e1c       ??_C@_0DE@GOAGCEO@?$CD?$CD?$CD?$CD?$CD?5Getting?5icon?5height?5?9?5cal@ 10029e1c     AccessBridgeJavaEntryPoints.obj
 0002:00007e50       ??_C@_0CB@BMHPADNP@?$FLINFO?$FN?3?5?5?5?$CD?$CD?$CD?$CD?$CD?5icon?5height?5?$DN?5?$CF@ 10029e50     AccessBridgeJavaEntryPoints.obj
 0002:00007e74       ??_C@_0DD@EHAOAGFJ@?$CD?$CD?$CD?$CD?$CD?5Getting?5icon?5width?5?9?5call@ 10029e74     AccessBridgeJavaEntryPoints.obj
 0002:00007ea8       ??_C@_0CA@DPEBDDDD@?$FLINFO?$FN?3?5?5?5?$CD?$CD?$CD?$CD?$CD?5icon?5width?5?$DN?5?$CFd@ 10029ea8     AccessBridgeJavaEntryPoints.obj
 0002:00007ec8       ??_C@_0DG@DLFAKGJK@?$CD?$CD?$CD?$CD?$CD?5Getting?5actions?5count?5?9?5c@ 10029ec8     AccessBridgeJavaEntryPoints.obj
 0002:00007f00       ??_C@_0CH@EOBAHIJB@?$FLINFO?$FN?3?5?5?5?$CD?$CD?$CD?$CD?$CD?5key?5actions?5cou@ 10029f00     AccessBridgeJavaEntryPoints.obj
 0002:00007f28       ??_C@_0DC@LHBGBJKA@Getting?5Action?5Name?5?5?9?5call?5to?5@ 10029f28     AccessBridgeJavaEntryPoints.obj
 0002:00007f5c       ??_C@_0DK@MCEEGDOO@Getting?5AccessibleAction?5Name?5?5@ 10029f5c     AccessBridgeJavaEntryPoints.obj
 0002:00007f98       ??_C@_0DL@IBEDPAGK@Getting?5AccessibleAction?5name?5?5@ 10029f98     AccessBridgeJavaEntryPoints.obj
 0002:00007fd4       ??_C@_0DO@BGBLOIHC@Getting?5AccessibleAction?5name?5?5@ 10029fd4     AccessBridgeJavaEntryPoints.obj
 0002:00008014       ??_C@_0CL@LDPKEJLA@?$FLINFO?$FN?3?5?$CD?$CD?$CD?$CD?$CD?5AccessibleAction?5@ 1002a014     AccessBridgeJavaEntryPoints.obj
 0002:00008040       ??_C@_0DK@GEFGKAFF@Getting?5AccessibleAction?5name?5?5@ 1002a040     AccessBridgeJavaEntryPoints.obj
 0002:0000807c       ??_C@_0CK@GFGPDCKK@?$FLWARN?$FN?3?5?5?5AccessibleAction?5name@ 1002a07c     AccessBridgeJavaEntryPoints.obj
 0002:000080a8       ??_C@_0FG@HPHLKACM@?$FLINFO?$FN?3?5Calling?5AccessBridgeJav@ 1002a0a8     AccessBridgeJavaEntryPoints.obj
 0002:00008100       ??_C@_0CB@NAFFMPJL@?$FLINFO?$FN?3?5?5?5?5?5doing?5?$CFd?5actions?5?4?4@ 1002a100     AccessBridgeJavaEntryPoints.obj
 0002:00008124       ??_C@_0CE@MIPOFJEF@?$FLINFO?$FN?3?5?5?5?5?5doing?5action?5?$CFd?3?5?$CFs@ 1002a124     AccessBridgeJavaEntryPoints.obj
 0002:00008148       ??_C@_0DC@PKIFPAKH@doAccessibleActions?5?9?5call?5to?5C@ 1002a148     AccessBridgeJavaEntryPoints.obj
 0002:0000817c       ??_C@_0BO@OONLHHCL@?$FLERROR?$FN?3?5?5?5?5?5Action?5?$CFd?5failed@ 1002a17c     AccessBridgeJavaEntryPoints.obj
 0002:000081a0       ??_C@_0FA@KEPHMGGF@?$FLINFO?$FN?3?5Calling?5AccessBridgeJav@ 1002a1a0     AccessBridgeJavaEntryPoints.obj
 0002:000081f0       ??_C@_0DG@GCJDNJFK@Getting?5AccessibleCharCount?5?9?5c@ 1002a1f0     AccessBridgeJavaEntryPoints.obj
 0002:00008228       ??_C@_0BK@OIDALDPI@?$FLINFO?$FN?3?5?5?5Char?5count?5?$DN?5?$CFd@ 1002a228     AccessBridgeJavaEntryPoints.obj
 0002:00008248       ??_C@_0EJ@JKPJJPMH@?$FLERROR?$FN?3?5either?5env?5?$DN?$DN?50?5or?5get@ 1002a248     AccessBridgeJavaEntryPoints.obj
 0002:00008294       ??_C@_0DK@EFHALPMO@Getting?5AccessibleCaretPosition@ 1002a294     AccessBridgeJavaEntryPoints.obj
 0002:000082d0       ??_C@_0BO@CCCENNB@?$FLINFO?$FN?3?5?5?5Index?5at?5caret?5?$DN?5?$CFd@ 1002a2d0     AccessBridgeJavaEntryPoints.obj
 0002:000082f0       ??_C@_0EN@DJGOBIMD@?$FLERROR?$FN?3?5either?5env?5?$DN?$DN?50?5or?5get@ 1002a2f0     AccessBridgeJavaEntryPoints.obj
 0002:00008340       ??_C@_0DJ@MLOJKMJI@Getting?5AccessibleIndexAtPoint?5@ 1002a340     AccessBridgeJavaEntryPoints.obj
 0002:0000837c       ??_C@_0BO@FIAABPFC@?$FLINFO?$FN?3?5?5?5Index?5at?5point?5?$DN?5?$CFd@ 1002a37c     AccessBridgeJavaEntryPoints.obj
 0002:000083a0       ??_C@_0EM@ENNBLMPC@?$FLERROR?$FN?3?5either?5env?5?$DN?$DN?50?5or?5get@ 1002a3a0     AccessBridgeJavaEntryPoints.obj
 0002:000083f0       ??_C@_0EJ@KDHBNGHD@?$FLINFO?$FN?3?5Calling?5AccessBridgeJav@ 1002a3f0     AccessBridgeJavaEntryPoints.obj
 0002:0000843c       ??_C@_0DK@CALJAPAO@Getting?5AccessibleLetterAtIndex@ 1002a43c     AccessBridgeJavaEntryPoints.obj
 0002:00008478       ??_C@_0DL@JDJLEMDG@Getting?5AccessibleLetterAtIndex@ 1002a478     AccessBridgeJavaEntryPoints.obj
 0002:000084b4       ??_C@_0DP@BIFOHJBB@Getting?5AccessibleLetterAtIndex@ 1002a4b4     AccessBridgeJavaEntryPoints.obj
 0002:000084f4       ??_C@_0DL@OOLFPOBK@Getting?5AccessibleLetterAtIndex@ 1002a4f4     AccessBridgeJavaEntryPoints.obj
 0002:00008530       ??_C@_0CG@BAFOKJKC@?$FLINFO?$FN?3?5?5?5Accessible?5Text?5lette@ 1002a530     AccessBridgeJavaEntryPoints.obj
 0002:00008558       ??_C@_0DL@FNGOIOKI@Getting?5AccessibleLetterAtIndex@ 1002a558     AccessBridgeJavaEntryPoints.obj
 0002:00008594       ??_C@_0CK@KNLDNGDN@?$FLWARN?$FN?3?5?5?5Accessible?5Text?5lette@ 1002a594     AccessBridgeJavaEntryPoints.obj
 0002:000085c0       ??_C@_0EN@GBFAECFE@?$FLERROR?$FN?3?5either?5env?5?$DN?$DN?50?5or?5get@ 1002a5c0     AccessBridgeJavaEntryPoints.obj
 0002:00008610       ??_C@_0DI@DFJMLOME@Getting?5AccessibleWordAtIndex?5?9@ 1002a610     AccessBridgeJavaEntryPoints.obj
 0002:00008648       ??_C@_0DJ@OIDPECCJ@Getting?5AccessibleWordAtIndex?5?9@ 1002a648     AccessBridgeJavaEntryPoints.obj
 0002:00008684       ??_C@_0DK@MPAFOPBO@Getting?5AccessibleWordAtIndex?5?9@ 1002a684     AccessBridgeJavaEntryPoints.obj
 0002:000086c0       ??_C@_0DN@BHAGMCIL@Getting?5AccessibleWordAtIndex?5?9@ 1002a6c0     AccessBridgeJavaEntryPoints.obj
 0002:00008700       ??_C@_0DJ@JFBBPAAF@Getting?5AccessibleWordAtIndex?5?9@ 1002a700     AccessBridgeJavaEntryPoints.obj
 0002:00008740       ??_C@_1EK@ODCBDMFL@?$AA?$FL?$AAI?$AAN?$AAF?$AAO?$AA?$FN?$AA?3?$AA?5?$AA?5?$AA?5?$AAA?$AAc?$AAc?$AAe?$AAs@ 1002a740     AccessBridgeJavaEntryPoints.obj
 0002:0000878c       ??_C@_0DJ@CGMKIALH@Getting?5AccessibleWordAtIndex?5?9@ 1002a78c     AccessBridgeJavaEntryPoints.obj
 0002:000087c8       ??_C@_0CI@JLGHFNHI@?$FLWARN?$FN?3?5?5?5Accessible?5Text?5word?5@ 1002a7c8     AccessBridgeJavaEntryPoints.obj
 0002:000087f0       ??_C@_0EL@NKGFFDIO@?$FLERROR?$FN?3?5either?5env?5?$DN?$DN?50?5or?5get@ 1002a7f0     AccessBridgeJavaEntryPoints.obj
 0002:0000883c       ??_C@_0DP@OGFHHBKC@Getting?5AccessibleSentenceAtInd@ 1002a83c     AccessBridgeJavaEntryPoints.obj
 0002:0000887c       ??_C@_0DN@MGFPCBII@Getting?5AccessibleSentenceAtInd@ 1002a87c     AccessBridgeJavaEntryPoints.obj
 0002:000088bc       ??_C@_0DO@GOPKBMAD@Getting?5AccessibleSentenceAtInd@ 1002a8bc     AccessBridgeJavaEntryPoints.obj
 0002:00008900       ??_C@_0EB@BBGLKPPK@Getting?5AccessibleSentenceAtInd@ 1002a900     AccessBridgeJavaEntryPoints.obj
 0002:00008944       ??_C@_0DN@LLHBJDKE@Getting?5AccessibleSentenceAtInd@ 1002a944     AccessBridgeJavaEntryPoints.obj
 0002:00008988       ??_C@_1FC@FOIECOHK@?$AA?$FL?$AAI?$AAN?$AAF?$AAO?$AA?$FN?$AA?3?$AA?5?$AA?5?$AA?5?$AAA?$AAc?$AAc?$AAe?$AAs@ 1002a988     AccessBridgeJavaEntryPoints.obj
 0002:000089dc       ??_C@_0DN@IKKODBG@Getting?5AccessibleSentenceAtInd@ 1002a9dc     AccessBridgeJavaEntryPoints.obj
 0002:00008a1c       ??_C@_0CM@EBOEJDBD@?$FLWARN?$FN?3?5?5?5Accessible?5Text?5sente@ 1002aa1c     AccessBridgeJavaEntryPoints.obj
 0002:00008a48       ??_C@_0EP@JMGAHICJ@?$FLERROR?$FN?3?5either?5env?5?$DN?$DN?50?5or?5get@ 1002aa48     AccessBridgeJavaEntryPoints.obj
 0002:00008a98       ??_C@_0FB@DGBDAMEN@?$FLINFO?$FN?3?5Calling?5AccessBridgeJav@ 1002aa98     AccessBridgeJavaEntryPoints.obj
 0002:00008aec       ??_C@_0DP@BBIGIAAH@Getting?5AccessibleTextSelection@ 1002aaec     AccessBridgeJavaEntryPoints.obj
 0002:00008b2c       ??_C@_0BP@MPEDAFPO@?$FLINFO?$FN?3?5?5?5Selection?5start?5?$DN?5?$CFd@ 1002ab2c     AccessBridgeJavaEntryPoints.obj
 0002:00008b50       ??_C@_0FD@EDCFOMDB@?$FLERROR?$FN?3?5?5either?5env?5?$DN?$DN?50?5or?5ge@ 1002ab50     AccessBridgeJavaEntryPoints.obj
 0002:00008ba4       ??_C@_0DN@MBOJJHKP@Getting?5AccessibleTextSelection@ 1002aba4     AccessBridgeJavaEntryPoints.obj
 0002:00008be4       ??_C@_0BN@JAKAFPAN@?$FLINFO?$FN?3?5?5?5Selection?5end?5?$DN?5?$CFd@ 1002abe4     AccessBridgeJavaEntryPoints.obj
 0002:00008c08       ??_C@_0FA@HPMPKGDO@?$FLERROR?$FN?3?5either?5env?5?$DN?$DN?50?5or?5get@ 1002ac08     AccessBridgeJavaEntryPoints.obj
 0002:00008c58       ??_C@_0EA@KGAPFINL@Getting?5AccessibleTextSelectedT@ 1002ac58     AccessBridgeJavaEntryPoints.obj
 0002:00008c98       ??_C@_0DO@OMODBJBJ@Getting?5AccessibleTextSelectedT@ 1002ac98     AccessBridgeJavaEntryPoints.obj
 0002:00008cd8       ??_C@_0DP@OJNIADOJ@Getting?5AccessibleTextSelectedT@ 1002acd8     AccessBridgeJavaEntryPoints.obj
 0002:00008d18       ??_C@_0EC@KNCELFHB@Getting?5AccessibleTextSelectedT@ 1002ad18     AccessBridgeJavaEntryPoints.obj
 0002:00008d5c       ??_C@_0DO@JBMNKLDF@Getting?5AccessibleTextSelectedT@ 1002ad5c     AccessBridgeJavaEntryPoints.obj
 0002:00008d9c       ??_C@_0CK@DDDAABEG@?$FLINFO?$FN?3?5?5?5Accessible?8s?5selected@ 1002ad9c     AccessBridgeJavaEntryPoints.obj
 0002:00008dc8       ??_C@_0DO@CCBGNLIH@Getting?5AccessibleTextSelectedT@ 1002adc8     AccessBridgeJavaEntryPoints.obj
 0002:00008e08       ??_C@_0CO@GAOLMCL@?$FLWARN?$FN?3?5?5?5Accessible?8s?5selected@ 1002ae08     AccessBridgeJavaEntryPoints.obj
 0002:00008e38       ??_C@_0EP@FNBFNNLO@?$FLWARN?$FN?3?5either?5env?5?$DN?$DN?50?5or?5getA@ 1002ae38     AccessBridgeJavaEntryPoints.obj
 0002:00008e88       ??_C@_0EO@HEMIPALC@?$FLINFO?$FN?3?5Calling?5AccessBridgeJav@ 1002ae88     AccessBridgeJavaEntryPoints.obj
 0002:00008ed8       ??_C@_0CK@OGCGGLCF@?$FLINFO?$FN?3?5?5Getting?5AttributeSet?5a@ 1002aed8     AccessBridgeJavaEntryPoints.obj
 0002:00008f08       ??_C@_0ED@CGONELLD@Getting?5AccessibleAttributeSetA@ 1002af08     AccessBridgeJavaEntryPoints.obj
 0002:00008f50       ??_C@_0FD@BNPBOBD@?$FLERROR?$FN?3?5either?5env?5?$DN?$DN?50?5or?5get@ 1002af50     AccessBridgeJavaEntryPoints.obj
 0002:00008fa8       ??_C@_0FG@OPHHFMC@?$FLWARN?$FN?3?5?5AttributeSet?5returned?5@ 1002afa8     AccessBridgeJavaEntryPoints.obj
 0002:00009000       ??_C@_0CL@BFGDEBIA@?$FLINFO?$FN?3?5?5Getting?5bold?5from?5Attr@ 1002b000     AccessBridgeJavaEntryPoints.obj
 0002:0000902c       ??_C@_0DL@NGCGOJOD@Getting?5BoldFromAttributeSet?5?9?5@ 1002b02c     AccessBridgeJavaEntryPoints.obj
 0002:00009068       ??_C@_0DP@GPLAEKHL@?$FLERROR?$FN?3?5either?5env?5?$DN?$DN?50?5or?5get@ 1002b068     AccessBridgeJavaEntryPoints.obj
 0002:000090a8       ??_C@_0DI@GHAHHMIG@Getting?5BoldFromAttributeSet?5?9?5@ 1002b0a8     AccessBridgeJavaEntryPoints.obj
 0002:000090e0       ??_C@_0DI@NENMAMDE@Getting?5BoldFromAttributeSet?5?9?5@ 1002b0e0     AccessBridgeJavaEntryPoints.obj
 0002:00009118       ??_C@_0CN@DLPNJKCI@?$FLINFO?$FN?3?5?5Getting?5italic?5from?5At@ 1002b118     AccessBridgeJavaEntryPoints.obj
 0002:00009148       ??_C@_0DN@FALJGLGH@Getting?5ItalicFromAttributeSet?5@ 1002b148     AccessBridgeJavaEntryPoints.obj
 0002:00009188       ??_C@_0EC@PFKOONOF@?$FLERROR?$FN?3?5either?5env?5?$DN?$DN?50?5or?5get@ 1002b188     AccessBridgeJavaEntryPoints.obj
 0002:000091cc       ??_C@_0DK@CEDKJPGF@Getting?5ItalicFromAttributeSet?5@ 1002b1cc     AccessBridgeJavaEntryPoints.obj
 0002:00009208       ??_C@_0DK@JHOBOPNH@Getting?5ItalicFromAttributeSet?5@ 1002b208     AccessBridgeJavaEntryPoints.obj
 0002:00009244       ??_C@_0DA@HJAHPBCP@?$FLINFO?$FN?3?5?5Getting?5underline?5from@ 1002b244     AccessBridgeJavaEntryPoints.obj
 0002:00009278       ??_C@_0EA@LFOJMIBN@Getting?5UnderlineFromAttributeS@ 1002b278     AccessBridgeJavaEntryPoints.obj
 0002:000092b8       ??_C@_0EF@LMCHMLNC@?$FLERROR?$FN?3?5?5either?5env?5?$DN?$DN?50?5or?5ge@ 1002b2b8     AccessBridgeJavaEntryPoints.obj
 0002:00009300       ??_C@_0DN@GEOGGPCN@Getting?5UnderlineFromAttributeS@ 1002b300     AccessBridgeJavaEntryPoints.obj
 0002:00009340       ??_C@_0DN@NHDNBPJP@Getting?5UnderlineFromAttributeS@ 1002b340     AccessBridgeJavaEntryPoints.obj
 0002:00009380       ??_C@_0DE@MIAPKOHI@?$FLINFO?$FN?3?5?5Getting?5strikethrough?5@ 1002b380     AccessBridgeJavaEntryPoints.obj
 0002:000093b8       ??_C@_0EE@DDJIBELI@Getting?5StrikethroughFromAttrib@ 1002b3b8     AccessBridgeJavaEntryPoints.obj
 0002:00009400       ??_C@_0EI@HMMOGEKC@?$FLERROR?$FN?3?5either?5env?5?$DN?$DN?50?5or?5get@ 1002b400     AccessBridgeJavaEntryPoints.obj
 0002:00009448       ??_C@_0EB@GCIGLCLO@Getting?5StrikethroughFromAttrib@ 1002b448     AccessBridgeJavaEntryPoints.obj
 0002:00009490       ??_C@_0EB@NBFNMCAM@Getting?5StrikethroughFromAttrib@ 1002b490     AccessBridgeJavaEntryPoints.obj
 0002:000094d4       ??_C@_0DC@ENJFOBHI@?$FLINFO?$FN?3?5?5Getting?5superscript?5fr@ 1002b4d4     AccessBridgeJavaEntryPoints.obj
 0002:00009508       ??_C@_0EC@BAJDPNIO@Getting?5SuperscriptFromAttribut@ 1002b508     AccessBridgeJavaEntryPoints.obj
 0002:00009550       ??_C@_0EH@EIIKEOA@?$FLERROR?$FN?3?5either?5env?5?$DN?$DN?50?5or?5get@ 1002b550     AccessBridgeJavaEntryPoints.obj
 0002:00009598       ??_C@_0DP@LNAJFDKJ@Getting?5SuperscriptFromAttribut@ 1002b598     AccessBridgeJavaEntryPoints.obj
 0002:000095d8       ??_C@_0DP@ONCCDBL@Getting?5SuperscriptFromAttribut@ 1002b5d8     AccessBridgeJavaEntryPoints.obj
 0002:00009618       ??_C@_0DA@KLOJONPP@?$FLINFO?$FN?3?5?5Getting?5subscript?5from@ 1002b618     AccessBridgeJavaEntryPoints.obj
 0002:00009648       ??_C@_0EA@NMFFGPLI@Getting?5SubscriptFromAttributeS@ 1002b648     AccessBridgeJavaEntryPoints.obj
 0002:00009688       ??_C@_0EE@EGHOMMOM@?$FLERROR?$FN?3?5either?5env?5?$DN?$DN?50?5or?5get@ 1002b688     AccessBridgeJavaEntryPoints.obj
 0002:000096cc       ??_C@_0DN@NJLPKKJA@Getting?5SubscriptFromAttributeS@ 1002b6cc     AccessBridgeJavaEntryPoints.obj
 0002:0000970c       ??_C@_0DN@GKGENKCC@Getting?5SubscriptFromAttributeS@ 1002b70c     AccessBridgeJavaEntryPoints.obj
 0002:0000974c       ??_C@_0DG@JDMMILDN@?$FLINFO?$FN?3?5?5Getting?5backgroundColo@ 1002b74c     AccessBridgeJavaEntryPoints.obj
 0002:00009788       ??_C@_0EF@CPKEHGFF@Getting?5BackgroundColorFromAttr@ 1002b788     AccessBridgeJavaEntryPoints.obj
 0002:000097d0       ??_C@_0ED@OOEECCFB@Getting?5BackgroundColorFromAttr@ 1002b7d0     AccessBridgeJavaEntryPoints.obj
 0002:00009818       ??_C@_0EE@JBNNGNHA@Getting?5BackgroundColorFromAttr@ 1002b818     AccessBridgeJavaEntryPoints.obj
 0002:00009860       ??_C@_0EH@NEPCIENA@Getting?5BackgroundColorFromAttr@ 1002b860     AccessBridgeJavaEntryPoints.obj
 0002:000098a8       ??_C@_0ED@JDGKJAHN@Getting?5BackgroundColorFromAttr@ 1002b8a8     AccessBridgeJavaEntryPoints.obj
 0002:000098f0       ??_C@_1GA@PMLMKIMP@?$AA?$FL?$AAI?$AAN?$AAF?$AAO?$AA?$FN?$AA?3?$AA?5?$AA?5?$AA?5?$AAA?$AAt?$AAt?$AAr?$AAi@ 1002b8f0     AccessBridgeJavaEntryPoints.obj
 0002:00009950       ??_C@_0ED@CALBOAMP@Getting?5BackgroundColorFromAttr@ 1002b950     AccessBridgeJavaEntryPoints.obj
 0002:00009994       ??_C@_0DD@DIMBBLFG@?$FLWARN?$FN?3?5?5?5AttributeSet?8s?5backgr@ 1002b994     AccessBridgeJavaEntryPoints.obj
 0002:000099c8       ??_C@_0EK@LDLFAHLP@?$FLERROR?$FN?3?5either?5env?5?$DN?$DN?50?5or?5get@ 1002b9c8     AccessBridgeJavaEntryPoints.obj
 0002:00009a14       ??_C@_0DG@OAPFKBJG@?$FLINFO?$FN?3?5?5Getting?5foregroundColo@ 1002ba14     AccessBridgeJavaEntryPoints.obj
 0002:00009a50       ??_C@_0EF@CFMCBGOA@Getting?5ForegroundColorFromAttr@ 1002ba50     AccessBridgeJavaEntryPoints.obj
 0002:00009a98       ??_C@_0ED@CGONGGIL@Getting?5ForegroundColorFromAttr@ 1002ba98     AccessBridgeJavaEntryPoints.obj
 0002:00009ae0       ??_C@_0EE@PHBDPPPO@Getting?5ForegroundColorFromAttr@ 1002bae0     AccessBridgeJavaEntryPoints.obj
 0002:00009b28       ??_C@_0EH@PCLFBD@Getting?5ForegroundColorFromAttr@ 1002bb28     AccessBridgeJavaEntryPoints.obj
 0002:00009b70       ??_C@_0ED@FLMDNEKH@Getting?5ForegroundColorFromAttr@ 1002bb70     AccessBridgeJavaEntryPoints.obj
 0002:00009bb8       ??_C@_1GA@DDCOJJLA@?$AA?$FL?$AAI?$AAN?$AAF?$AAO?$AA?$FN?$AA?3?$AA?5?$AA?5?$AA?5?$AAA?$AAt?$AAt?$AAr?$AAi@ 1002bbb8     AccessBridgeJavaEntryPoints.obj
 0002:00009c18       ??_C@_0ED@OIBIKEBF@Getting?5ForegroundColorFromAttr@ 1002bc18     AccessBridgeJavaEntryPoints.obj
 0002:00009c5c       ??_C@_0DD@EGLIFJNP@?$FLWARN?$FN?3?5?5?5AttributeSet?8s?5foregr@ 1002bc5c     AccessBridgeJavaEntryPoints.obj
 0002:00009c90       ??_C@_0EK@JAILLABF@?$FLERROR?$FN?3?5either?5env?5?$DN?$DN?50?5or?5get@ 1002bc90     AccessBridgeJavaEntryPoints.obj
 0002:00009cdc       ??_C@_0DB@NPCHLNMB@?$FLINFO?$FN?3?5?5Getting?5fontFamily?5fro@ 1002bcdc     AccessBridgeJavaEntryPoints.obj
 0002:00009d10       ??_C@_0EA@OFLFMJOA@Getting?5FontFamilyFromAttribute@ 1002bd10     AccessBridgeJavaEntryPoints.obj
 0002:00009d50       ??_C@_0DO@ECEGIKHO@Getting?5FontFamilyFromAttribute@ 1002bd50     AccessBridgeJavaEntryPoints.obj
 0002:00009d90       ??_C@_0DP@DKKAFCIB@Getting?5FontFamilyFromAttribute@ 1002bd90     AccessBridgeJavaEntryPoints.obj
 0002:00009dd0       ??_C@_0EC@BGJOLKCB@Getting?5FontFamilyFromAttribute@ 1002bdd0     AccessBridgeJavaEntryPoints.obj
 0002:00009e14       ??_C@_0DO@DPGIDIFC@Getting?5FontFamilyFromAttribute@ 1002be14     AccessBridgeJavaEntryPoints.obj
 0002:00009e58       ??_C@_1FE@LCMANMIC@?$AA?$FL?$AAI?$AAN?$AAF?$AAO?$AA?$FN?$AA?3?$AA?5?$AA?5?$AA?5?$AAA?$AAt?$AAt?$AAr?$AAi@ 1002be58     AccessBridgeJavaEntryPoints.obj
 0002:00009eac       ??_C@_0DO@IMLDEIOA@Getting?5FontFamilyFromAttribute@ 1002beac     AccessBridgeJavaEntryPoints.obj
 0002:00009eec       ??_C@_0CN@DFPIBNDO@?$FLWARN?$FN?3?5?5?5AttributeSet?8s?5fontFa@ 1002beec     AccessBridgeJavaEntryPoints.obj
 0002:00009f20       ??_C@_0EF@MEIJBCDI@?$FLERROR?$FN?3?5either?5env?5?$DN?$DN?50?5or?5get@ 1002bf20     AccessBridgeJavaEntryPoints.obj
 0002:00009f68       ??_C@_0DA@NKBCCHCB@?$FLINFO?$FN?3?5?5Getting?5font?5size?5from@ 1002bf68     AccessBridgeJavaEntryPoints.obj
 0002:00009f98       ??_C@_0DL@OGKGFGCH@Getting?5FontSizeFromAttributeSe@ 1002bf98     AccessBridgeJavaEntryPoints.obj
 0002:00009fd4       ??_C@_0CI@MMDBDPDB@?$FLINFO?$FN?3?5?5?5AttributeSet?8s?5font?5s@ 1002bfd4     AccessBridgeJavaEntryPoints.obj
 0002:0000a000       ??_C@_0EE@EGBGOKJP@?$FLERROR?$FN?3?5either?5env?5?$DN?$DN?50?5or?5get@ 1002c000     AccessBridgeJavaEntryPoints.obj
 0002:0000a044       ??_C@_0DM@KMMBHJCP@Getting?5FontSizeFromAttributeSe@ 1002c044     AccessBridgeJavaEntryPoints.obj
 0002:0000a080       ??_C@_0DM@BPBKAJJN@Getting?5FontSizeFromAttributeSe@ 1002c080     AccessBridgeJavaEntryPoints.obj
 0002:0000a0bc       ??_C@_0CI@DPJLKBCH@?5Getting?5alignment?5from?5Attribu@ 1002c0bc     AccessBridgeJavaEntryPoints.obj
 0002:0000a0e4       ??_C@_0DM@IEKBPPGN@Getting?5AlignmentFromAttributeS@ 1002c0e4     AccessBridgeJavaEntryPoints.obj
 0002:0000a120       ??_C@_0DN@DKKKNGAI@Getting?5AlignmentFromAttributeS@ 1002c120     AccessBridgeJavaEntryPoints.obj
 0002:0000a160       ??_C@_0DN@IJHBKGLK@Getting?5AlignmentFromAttributeS@ 1002c160     AccessBridgeJavaEntryPoints.obj
 0002:0000a1a0       ??_C@_0DA@IEHDNKCA@?$FLINFO?$FN?3?5?5Getting?5bidiLevel?5from@ 1002c1a0     AccessBridgeJavaEntryPoints.obj
 0002:0000a1d0       ??_C@_0DM@HHHEIBLO@Getting?5BidiLevelFromAttributeS@ 1002c1d0     AccessBridgeJavaEntryPoints.obj
 0002:0000a210       ??_C@_0EE@FHPLAGJN@?$FLERROR?$FN?3?5either?5env?5?$DN?$DN?50?5or?5get@ 1002c210     AccessBridgeJavaEntryPoints.obj
 0002:0000a254       ??_C@_0DN@CFIDIABI@Getting?5BidiLevelFromAttributeS@ 1002c254     AccessBridgeJavaEntryPoints.obj
 0002:0000a294       ??_C@_0DN@JGFIPAKK@Getting?5BidiLevelFromAttributeS@ 1002c294     AccessBridgeJavaEntryPoints.obj
 0002:0000a2d4       ??_C@_0DH@CAJPMJAH@?$FLERROR?$FN?3?5?5Getting?5firstLineInde@ 1002c2d4     AccessBridgeJavaEntryPoints.obj
 0002:0000a310       ??_C@_0EC@GDNCLBBP@Getting?5FirstLineIndentFromAttr@ 1002c310     AccessBridgeJavaEntryPoints.obj
 0002:0000a358       ??_C@_0EK@JNGBIMLH@?$FLERROR?$FN?3?5either?5env?5?$DN?$DN?50?5or?5get@ 1002c358     AccessBridgeJavaEntryPoints.obj
 0002:0000a3a8       ??_C@_0ED@IEEGLFFG@Getting?5FirstLineIndentFromAttr@ 1002c3a8     AccessBridgeJavaEntryPoints.obj
 0002:0000a3f0       ??_C@_0ED@DHJNMFOE@Getting?5FirstLineIndentFromAttr@ 1002c3f0     AccessBridgeJavaEntryPoints.obj
 0002:0000a434       ??_C@_0DB@GIKOBABF@?$FLINFO?$FN?3?5?5Getting?5leftIndent?5fro@ 1002c434     AccessBridgeJavaEntryPoints.obj
 0002:0000a468       ??_C@_0DN@GGPJCLGF@Getting?5LeftIndentFromAttribute@ 1002c468     AccessBridgeJavaEntryPoints.obj
 0002:0000a4a8       ??_C@_0EF@JFNBAGAC@?$FLERROR?$FN?3?5either?5env?5?$DN?$DN?50?5or?5get@ 1002c4a8     AccessBridgeJavaEntryPoints.obj
 0002:0000a4f0       ??_C@_0DO@DEJDAGOO@Getting?5LeftIndentFromAttribute@ 1002c4f0     AccessBridgeJavaEntryPoints.obj
 0002:0000a530       ??_C@_0DO@IHEIHGFM@Getting?5LeftIndentFromAttribute@ 1002c530     AccessBridgeJavaEntryPoints.obj
 0002:0000a570       ??_C@_0DC@OHJHAPPB@?$FLINFO?$FN?3?5?5Getting?5rightIndent?5fr@ 1002c570     AccessBridgeJavaEntryPoints.obj
 0002:0000a5a4       ??_C@_0DO@GPANPNCO@Getting?5RightIndentFromAttribut@ 1002c5a4     AccessBridgeJavaEntryPoints.obj
 0002:0000a5e8       ??_C@_0EG@FKGIOCMJ@?$FLERROR?$FN?3?5either?5env?5?$DN?$DN?50?5or?5get@ 1002c5e8     AccessBridgeJavaEntryPoints.obj
 0002:0000a630       ??_C@_0DP@NFJEGKCA@Getting?5RightIndentFromAttribut@ 1002c630     AccessBridgeJavaEntryPoints.obj
 0002:0000a670       ??_C@_0DP@GGEPBKJC@Getting?5RightIndentFromAttribut@ 1002c670     AccessBridgeJavaEntryPoints.obj
 0002:0000a6b0       ??_C@_0DC@FBCMPKE@?$FLINFO?$FN?3?5?5Getting?5lineSpacing?5fr@ 1002c6b0     AccessBridgeJavaEntryPoints.obj
 0002:0000a6e4       ??_C@_0DO@OLMNNFJE@Getting?5LineSpacingFromAttribut@ 1002c6e4     AccessBridgeJavaEntryPoints.obj
 0002:0000a728       ??_C@_0EH@DJGGHDHL@?$FLERROR?$FN?3?5?5either?5env?5?$DN?$DN?50?5or?5ge@ 1002c728     AccessBridgeJavaEntryPoints.obj
 0002:0000a770       ??_C@_0DP@POKEPAJK@Getting?5LineSpacingFromAttribut@ 1002c770     AccessBridgeJavaEntryPoints.obj
 0002:0000a7b0       ??_C@_0DP@ENHPIACI@Getting?5LineSpacingFromAttribut@ 1002c7b0     AccessBridgeJavaEntryPoints.obj
 0002:0000a7f0       ??_C@_0DB@BBFBINOC@?$FLINFO?$FN?3?5?5Getting?5spaceAbove?5fro@ 1002c7f0     AccessBridgeJavaEntryPoints.obj
 0002:0000a824       ??_C@_0DN@LICNMEPC@Getting?5SpaceAboveFromAttribute@ 1002c824     AccessBridgeJavaEntryPoints.obj
 0002:0000a868       ??_C@_0EG@DEAABEIJ@?$FLERROR?$FN?3?5?5either?5env?5?$DN?$DN?50?5or?5ge@ 1002c868     AccessBridgeJavaEntryPoints.obj
 0002:0000a8b0       ??_C@_0DO@FKCGNEOG@Getting?5SpaceAboveFromAttribute@ 1002c8b0     AccessBridgeJavaEntryPoints.obj
 0002:0000a8f0       ??_C@_0DO@OJPNKEFE@Getting?5SpaceAboveFromAttribute@ 1002c8f0     AccessBridgeJavaEntryPoints.obj
 0002:0000a930       ??_C@_0DB@IPEMBOFF@?$FLINFO?$FN?3?5?5Getting?5spaceBelow?5fro@ 1002c930     AccessBridgeJavaEntryPoints.obj
 0002:0000a964       ??_C@_0DN@KGEHENNL@Getting?5SpaceBelowFromAttribute@ 1002c964     AccessBridgeJavaEntryPoints.obj
 0002:0000a9a8       ??_C@_0EG@PAJHHADM@?$FLERROR?$FN?3?5?5either?5env?5?$DN?$DN?50?5or?5ge@ 1002c9a8     AccessBridgeJavaEntryPoints.obj
 0002:0000a9f0       ??_C@_0DO@BIIKCGAD@Getting?5SpaceBelowFromAttribute@ 1002c9f0     AccessBridgeJavaEntryPoints.obj
 0002:0000aa30       ??_C@_0DO@KLFBFGLB@Getting?5SpaceBelowFromAttribute@ 1002ca30     AccessBridgeJavaEntryPoints.obj
 0002:0000aa70       ??_C@_0DD@NEPODHGJ@?$FLINFO?$FN?3?5?5Decrementing?5reference@ 1002ca70     AccessBridgeJavaEntryPoints.obj
 0002:0000aaa4       ??_C@_0DJ@KDCCLHCF@Releasing?5AttributeSet?5object?5?9@ 1002caa4     AccessBridgeJavaEntryPoints.obj
 0002:0000aae0       ??_C@_0DF@KOJHMOGM@?$FLERROR?$FN?3?5?5either?5env?5?$DN?$DN?50?5or?5ac@ 1002cae0     AccessBridgeJavaEntryPoints.obj
 0002:0000ab18       ??_C@_0DJ@BAPJMHJH@Releasing?5AttributeSet?5object?5?9@ 1002cb18     AccessBridgeJavaEntryPoints.obj
 0002:0000ab54       ??_C@_0DI@FAAGAOKI@?$FLINFO?$FN?3?5?5Getting?5full?5attribute@ 1002cb54     AccessBridgeJavaEntryPoints.obj
 0002:0000ab8c       ??_C@_0DD@BPFGOEDD@?$FLINFO?$FN?3?5?5returned?5from?5CallObje@ 1002cb8c     AccessBridgeJavaEntryPoints.obj
 0002:0000abc0       ??_C@_1FG@IBEGPOLG@?$AA?$FL?$AAI?$AAN?$AAF?$AAO?$AA?$FN?$AA?3?$AA?5?$AA?5?$AA?5?$AAA?$AAc?$AAc?$AAe?$AAs@ 1002cbc0     AccessBridgeJavaEntryPoints.obj
 0002:0000ac18       ??_C@_0FC@NKKMDLMK@?$FLERROR?$FN?3?5?5either?5env?5?$DN?$DN?50?5or?5ge@ 1002cc18     AccessBridgeJavaEntryPoints.obj
 0002:0000ac70       ??_C@_0EB@FOBGJMBG@Getting?5AccessibleAttributeSetA@ 1002cc70     AccessBridgeJavaEntryPoints.obj
 0002:0000acb8       ??_C@_0FD@ONBHOKNL@?$FLINFO?$FN?3?5Calling?5AccessBridgeJav@ 1002ccb8     AccessBridgeJavaEntryPoints.obj
 0002:0000ad0c       ??_C@_0DL@PJLLEMMJ@Getting?5AccessibleXcoordTextRec@ 1002cd0c     AccessBridgeJavaEntryPoints.obj
 0002:0000ad48       ??_C@_0BG@CDBEIJEJ@?$FLINFO?$FN?3?5?5X?5coord?5?$DN?5?$CFd@ 1002cd48     AccessBridgeJavaEntryPoints.obj
 0002:0000ad60       ??_C@_0FF@CICHONC@?$FLERROR?$FN?3?5either?5env?5?$DN?$DN?50?5or?5get@ 1002cd60     AccessBridgeJavaEntryPoints.obj
 0002:0000adb8       ??_C@_0DL@BBKMNMGI@Getting?5AccessibleYcoordTextRec@ 1002cdb8     AccessBridgeJavaEntryPoints.obj
 0002:0000adf8       ??_C@_0FF@LPGHAKKN@?$FLINFO?$FN?3?5?5either?5env?5?$DN?$DN?50?5or?5get@ 1002cdf8     AccessBridgeJavaEntryPoints.obj
 0002:0000ae50       ??_C@_0DK@GOMAAIJJ@Getting?5AccessibleWidthTextRect@ 1002ce50     AccessBridgeJavaEntryPoints.obj
 0002:0000ae8c       ??_C@_0BD@PFFPBFHC@?$FLINFO?$FN?3?5Width?5?$DN?5?$CFd@ 1002ce8c     AccessBridgeJavaEntryPoints.obj
 0002:0000aea0       ??_C@_0FD@LFKJAPPJ@?$FLINFO?$FN?3?5either?5env?5?$DN?$DN?50?5or?5getA@ 1002cea0     AccessBridgeJavaEntryPoints.obj
 0002:0000aef4       ??_C@_0DL@LIFPGLAA@Getting?5AccessibleHeightTextRec@ 1002cef4     AccessBridgeJavaEntryPoints.obj
 0002:0000af30       ??_C@_0BE@BNGOGMPP@?$FLINFO?$FN?3?5Height?5?$DN?5?$CFd@ 1002cf30     AccessBridgeJavaEntryPoints.obj
 0002:0000af48       ??_C@_0FG@JCNMAPKJ@?$FLERROR?$FN?3?5?5either?5env?5?$DN?$DN?50?5or?5ge@ 1002cf48     AccessBridgeJavaEntryPoints.obj
 0002:0000afa0       ??_C@_0EO@GAEGCFMP@?$FLINFO?$FN?3?5Calling?5AccessBridgeJav@ 1002cfa0     AccessBridgeJavaEntryPoints.obj
 0002:0000aff0       ??_C@_0DF@JPKJOLBB@Getting?5caret?5X?5coordinate?5?9?5ca@ 1002cff0     AccessBridgeJavaEntryPoints.obj
 0002:0000b028       ??_C@_0DK@INHGMNIG@?$FLERROR?$FN?3?5?5either?5env?5?$DN?$DN?50?5or?5ge@ 1002d028     AccessBridgeJavaEntryPoints.obj
 0002:0000b064       ??_C@_0DF@NBCAOALI@Getting?5caret?5Y?5coordinate?5?9?5ca@ 1002d064     AccessBridgeJavaEntryPoints.obj
 0002:0000b09c       ??_C@_0DK@FAOABEAD@?$FLERROR?$FN?3?5?5either?5env?5?$DN?$DN?50?5or?5ge@ 1002d09c     AccessBridgeJavaEntryPoints.obj
 0002:0000b0d8       ??_C@_0CO@LPKJFNHN@Getting?5caret?5width?5?9?5call?5to?5C@ 1002d0d8     AccessBridgeJavaEntryPoints.obj
 0002:0000b108       ??_C@_0DO@KCIKCBGA@?$FLERROR?$FN?3?5?5either?5env?5?$DN?$DN?50?5or?5ge@ 1002d108     AccessBridgeJavaEntryPoints.obj
 0002:0000b148       ??_C@_0CP@DKBLCBME@Getting?5caret?5height?5?9?5call?5to?5@ 1002d148     AccessBridgeJavaEntryPoints.obj
 0002:0000b178       ??_C@_0DP@MHKONHOK@?$FLERROR?$FN?3?5?5either?5env?5?$DN?$DN?50?5or?5ge@ 1002d178     AccessBridgeJavaEntryPoints.obj
 0002:0000b1b8       ??_C@_0EO@OPGMODFN@?$FLINFO?$FN?3?5Calling?5AccessBridgeJav@ 1002d1b8     AccessBridgeJavaEntryPoints.obj
 0002:0000b208       ??_C@_0DP@HIDGMFDD@Getting?5AccessibleTextLineLeftB@ 1002d208     AccessBridgeJavaEntryPoints.obj
 0002:0000b248       ??_C@_0BK@INECDNLO@?$FLINFO?$FN?3?5?5?5startIndex?5?$DN?5?$CFd@ 1002d248     AccessBridgeJavaEntryPoints.obj
 0002:0000b268       ??_C@_0FD@BGKHJCDH@?$FLERROR?$FN?3?5?5either?5env?5?$DN?$DN?50?5or?5ge@ 1002d268     AccessBridgeJavaEntryPoints.obj
 0002:0000b2c0       ??_C@_0EA@OJGAJNKG@Getting?5AccessibleTextLineRight@ 1002d2c0     AccessBridgeJavaEntryPoints.obj
 0002:0000b300       ??_C@_0BI@NAKKCMDP@?$FLINFO?$FN?3?5?5?5endIndex?5?$DN?5?$CFd@ 1002d300     AccessBridgeJavaEntryPoints.obj
 0002:0000b318       ??_C@_0FE@HOJFBBNL@?$FLERROR?$FN?3?5?5either?5env?5?$DN?$DN?50?5or?5ge@ 1002d318     AccessBridgeJavaEntryPoints.obj
 0002:0000b370       ??_C@_0FM@PBOJPFBI@?$FLINFO?$FN?3?5Calling?5AccessBridgeJav@ 1002d370     AccessBridgeJavaEntryPoints.obj
 0002:0000b3cc       ??_C@_0BH@GCPBFEO@?$FLERROR?$FN?3?5?5end?5?$DM?5start?$CB@ 1002d3cc     AccessBridgeJavaEntryPoints.obj
 0002:0000b3e4       ??_C@_0DJ@OHJBLKEE@Getting?5AccessibleTextRange?5?9?5c@ 1002d3e4     AccessBridgeJavaEntryPoints.obj
 0002:0000b420       ??_C@_0DH@MLKPAEJI@Getting?5AccessibleTextRange?5?9?5c@ 1002d420     AccessBridgeJavaEntryPoints.obj
 0002:0000b458       ??_C@_1HO@MOIAIALP@?$AA?$FL?$AAI?$AAN?$AAF?$AAO?$AA?$FN?$AA?3?$AA?5?$AA?5?$AA?5?$AAA?$AAc?$AAc?$AAe?$AAs@ 1002d458     AccessBridgeJavaEntryPoints.obj
 0002:0000b4d8       ??_C@_0DB@GEMONLMO@?$FLINFO?$FN?3?5?5Accessible?5Text?5string@ 1002d4d8     AccessBridgeJavaEntryPoints.obj
 0002:0000b510       ??_C@_1HM@KJDBDPH@?$AA?$FL?$AAI?$AAN?$AAF?$AAO?$AA?$FN?$AA?3?$AA?5?$AA?5?$AA?5?$AAA?$AAc?$AAc?$AAe?$AAs@ 1002d510     AccessBridgeJavaEntryPoints.obj
 0002:0000b58c       ??_C@_0DI@HDEAPMEC@Getting?5AccessibleTextRange?5?9?5c@ 1002d58c     AccessBridgeJavaEntryPoints.obj
 0002:0000b5c4       ??_C@_0DL@BFPJOBGO@Getting?5AccessibleTextRange?5?9?5c@ 1002d5c4     AccessBridgeJavaEntryPoints.obj
 0002:0000b600       ??_C@_0DH@LGIBLGLE@Getting?5AccessibleTextRange?5?9?5c@ 1002d600     AccessBridgeJavaEntryPoints.obj
 0002:0000b638       ??_C@_1EM@MAOOPBBK@?$AA?$FL?$AAI?$AAN?$AAF?$AAO?$AA?$FN?$AA?3?$AA?5?$AA?5?$AA?5?$AAA?$AAc?$AAc?$AAe?$AAs@ 1002d638     AccessBridgeJavaEntryPoints.obj
 0002:0000b684       ??_C@_0DH@FFKMGAG@Getting?5AccessibleTextRange?5?9?5c@ 1002d684     AccessBridgeJavaEntryPoints.obj
 0002:0000b6bc       ??_C@_0DB@ENPGLEMN@?$FLWARN?$FN?3?5?5?5current?5Accessible?5Te@ 1002d6bc     AccessBridgeJavaEntryPoints.obj
 0002:0000b6f0       ??_C@_0EJ@IGDKNKCL@?$FLERROR?$FN?3?5either?5env?5?$DN?$DN?50?5or?5get@ 1002d6f0     AccessBridgeJavaEntryPoints.obj
 0002:0000b740       ??_C@_0FH@DFGPJEBI@?$FLINFO?$FN?3?5Calling?5AccessBridgeJav@ 1002d740     AccessBridgeJavaEntryPoints.obj
 0002:0000b798       ??_C@_0DM@FMEJNEAF@Getting?5CurrentAccessibleValue?5@ 1002d798     AccessBridgeJavaEntryPoints.obj
 0002:0000b7d4       ??_C@_0DK@DEBJEKPP@Getting?5CurrentAccessibleValue?5@ 1002d7d4     AccessBridgeJavaEntryPoints.obj
 0002:0000b810       ??_C@_0DL@KAGJLOPH@Getting?5CurrentAccessibleValue?5@ 1002d810     AccessBridgeJavaEntryPoints.obj
 0002:0000b84c       ??_C@_0DO@FGJBGIKN@Getting?5CurrentAccessibleValue?5@ 1002d84c     AccessBridgeJavaEntryPoints.obj
 0002:0000b88c       ??_C@_0DK@EJDHPIND@Getting?5CurrentAccessibleValue?5@ 1002d88c     AccessBridgeJavaEntryPoints.obj
 0002:0000b8c8       ??_C@_0CI@LHBKPIPL@?$FLINFO?$FN?3?5?5?5current?5Accessible?5Va@ 1002d8c8     AccessBridgeJavaEntryPoints.obj
 0002:0000b8f0       ??_C@_0DK@PKOMIIGB@Getting?5CurrentAccessibleValue?5@ 1002d8f0     AccessBridgeJavaEntryPoints.obj
 0002:0000b92c       ??_C@_0CM@JBCHBMHL@?$FLWARN?$FN?3?5?5?5current?5Accessible?5Va@ 1002d92c     AccessBridgeJavaEntryPoints.obj
 0002:0000b958       ??_C@_0EN@CEFCJCHP@?$FLERROR?$FN?3?5?5either?5env?5?$DN?$DN?50?5or?5ge@ 1002d958     AccessBridgeJavaEntryPoints.obj
 0002:0000b9a8       ??_C@_0FH@LDANAJBK@?$FLINFO?$FN?3?5Calling?5AccessBridgeJav@ 1002d9a8     AccessBridgeJavaEntryPoints.obj
 0002:0000ba00       ??_C@_0DM@CNMGLEAD@Getting?5MaximumAccessibleValue?5@ 1002da00     AccessBridgeJavaEntryPoints.obj
 0002:0000ba3c       ??_C@_0DK@LPOBNFBI@Getting?5MaximumAccessibleValue?5@ 1002da3c     AccessBridgeJavaEntryPoints.obj
 0002:0000ba78       ??_C@_0DL@JOIMDBLD@Getting?5MaximumAccessibleValue?5@ 1002da78     AccessBridgeJavaEntryPoints.obj
 0002:0000bab4       ??_C@_0DO@ENHJNPPM@Getting?5MaximumAccessibleValue?5@ 1002dab4     AccessBridgeJavaEntryPoints.obj
 0002:0000baf4       ??_C@_0DK@MCMPGHDE@Getting?5MaximumAccessibleValue?5@ 1002daf4     AccessBridgeJavaEntryPoints.obj
 0002:0000bb30       ??_C@_0CI@MOLFAIEC@?$FLINFO?$FN?3?5?5?5maximum?5Accessible?5Va@ 1002db30     AccessBridgeJavaEntryPoints.obj
 0002:0000bb58       ??_C@_0DK@HBBEBHIG@Getting?5MaximumAccessibleValue?5@ 1002db58     AccessBridgeJavaEntryPoints.obj
 0002:0000bb94       ??_C@_0CM@EENPAHAF@?$FLWARN?$FN?3?5?5?5maximum?5Accessible?5Va@ 1002db94     AccessBridgeJavaEntryPoints.obj
 0002:0000bbc0       ??_C@_0EM@DECMFMLP@?$FLERROR?$FN?3?5either?5env?5?$DN?$DN?50?5or?5get@ 1002dbc0     AccessBridgeJavaEntryPoints.obj
 0002:0000bc10       ??_C@_0FH@NCJCNBPB@?$FLINFO?$FN?3?5Calling?5AccessBridgeJav@ 1002dc10     AccessBridgeJavaEntryPoints.obj
 0002:0000bc68       ??_C@_0DM@EKOMNNCH@Getting?5MinimumAccessibleValue?5@ 1002dc68     AccessBridgeJavaEntryPoints.obj
 0002:0000bca4       ??_C@_0DK@POFOBDIM@Getting?5MinimumAccessibleValue?5@ 1002dca4     AccessBridgeJavaEntryPoints.obj
 0002:0000bce0       ??_C@_0DL@GJKPNJCI@Getting?5MinimumAccessibleValue?5@ 1002dce0     AccessBridgeJavaEntryPoints.obj
 0002:0000bd1c       ??_C@_0DO@IIPPIAIM@Getting?5MinimumAccessibleValue?5@ 1002dd1c     AccessBridgeJavaEntryPoints.obj
 0002:0000bd5c       ??_C@_0DK@IDHAKBKA@Getting?5MinimumAccessibleValue?5@ 1002dd5c     AccessBridgeJavaEntryPoints.obj
 0002:0000bd98       ??_C@_0CI@HMFEBFFJ@?$FLINFO?$FN?3?5?5?5mimimum?5Accessible?5Va@ 1002dd98     AccessBridgeJavaEntryPoints.obj
 0002:0000bdc0       ??_C@_0DK@DAKLNBBC@Getting?5MinimumAccessibleValue?5@ 1002ddc0     AccessBridgeJavaEntryPoints.obj
 0002:0000bdfc       ??_C@_0CM@LFDDPHLF@?$FLWARN?$FN?3?5?5?5mimimum?5Accessible?5Va@ 1002ddfc     AccessBridgeJavaEntryPoints.obj
 0002:0000be28       ??_C@_0EM@FNBMNDID@?$FLERROR?$FN?3?5either?5env?5?$DN?$DN?50?5or?5get@ 1002de28     AccessBridgeJavaEntryPoints.obj
 0002:0000be78       ??_C@_0FE@GLAEHJLA@?$FLINFO?$FN?3?5Calling?5AccessBridgeJav@ 1002de78     AccessBridgeJavaEntryPoints.obj
 0002:0000becc       ??_C@_0DI@HFNIIMHH@Doing?5addAccessibleSelection?5?9?5@ 1002decc     AccessBridgeJavaEntryPoints.obj
 0002:0000bf04       ??_C@_0CP@EBNEHGHB@?$FLERROR?$FN?3?5?$CK?$CK?$CK?5Exception?5occured?5@ 1002df04     AccessBridgeJavaEntryPoints.obj
 0002:0000bf34       ??_C@_0CL@OKIJNCBD@?$FLINFO?$FN?3?5?5?5returned?5from?5CallObj@ 1002df34     AccessBridgeJavaEntryPoints.obj
 0002:0000bf60       ??_C@_0EK@CMGGDKGL@?$FLERROR?$FN?3?5?5either?5env?5?$DN?$DN?50?5or?5ad@ 1002df60     AccessBridgeJavaEntryPoints.obj
 0002:0000bfb0       ??_C@_0FG@JICCBONC@?$FLINFO?$FN?3?5Calling?5AccessBridgeJav@ 1002dfb0     AccessBridgeJavaEntryPoints.obj
 0002:0000c008       ??_C@_0DK@GPKPKKON@Doing?5clearAccessibleSelection?5@ 1002e008     AccessBridgeJavaEntryPoints.obj
 0002:0000c048       ??_C@_0EM@NKPDGGGN@?$FLERROR?$FN?3?5?5either?5env?5?$DN?$DN?50?5or?5cl@ 1002e048     AccessBridgeJavaEntryPoints.obj
 0002:0000c098       ??_C@_0FE@PIPHOHFI@?$FLINFO?$FN?3?5Calling?5AccessBridgeJav@ 1002e098     AccessBridgeJavaEntryPoints.obj
 0002:0000c0f0       ??_C@_0EA@EDHDCMHP@Getting?5AccessibleSelectionCont@ 1002e0f0     AccessBridgeJavaEntryPoints.obj
 0002:0000c130       ??_C@_0DM@IFLFNJN@Getting?5AccessibleSelectionCont@ 1002e130     AccessBridgeJavaEntryPoints.obj
 0002:0000c16c       ??_C@_0DO@FEBBEFGL@Getting?5AccessibleSelectionCont@ 1002e16c     AccessBridgeJavaEntryPoints.obj
 0002:0000c1b0       ??_C@_0FA@KGJFECGD@?$FLERROR?$FN?3?5either?5env?5?$DN?$DN?50?5or?5get@ 1002e1b0     AccessBridgeJavaEntryPoints.obj
 0002:0000c200       ??_C@_0FJ@KDCCHMFP@?$FLINFO?$FN?3?5Calling?5AccessBridgeJav@ 1002e200     AccessBridgeJavaEntryPoints.obj
 0002:0000c25c       ??_C@_0DL@JPLKCOEB@Getting?5AccessibleSelectionCoun@ 1002e25c     AccessBridgeJavaEntryPoints.obj
 0002:0000c298       ??_C@_0EO@LLPLNNDE@?$FLERROR?$FN?3?5either?5env?5?$DN?$DN?50?5or?5get@ 1002e298     AccessBridgeJavaEntryPoints.obj
 0002:0000c2e8       ??_C@_0FH@BEGAHKNM@?$FLINFO?$FN?3?5Calling?5AccessBridgeJav@ 1002e2e8     AccessBridgeJavaEntryPoints.obj
 0002:0000c340       ??_C@_0DO@DGOGEINB@Doing?5isAccessibleChildSelected@ 1002e340     AccessBridgeJavaEntryPoints.obj
 0002:0000c380       ??_C@_0EM@FIJEFPDC@?$FLERROR?$FN?3?5either?5env?5?$DN?$DN?50?5or?5isA@ 1002e380     AccessBridgeJavaEntryPoints.obj
 0002:0000c3d0       ??_C@_0FH@DBFJFKMJ@?$FLINFO?$FN?3?5Calling?5AccessBridgeJav@ 1002e3d0     AccessBridgeJavaEntryPoints.obj
 0002:0000c428       ??_C@_0DL@BHDCMLKI@Doing?5removeAccessibleSelection@ 1002e428     AccessBridgeJavaEntryPoints.obj
 0002:0000c468       ??_C@_0EN@HJFMAEOO@?$FLERROR?$FN?3?5?5either?5env?5?$DN?$DN?50?5or?5re@ 1002e468     AccessBridgeJavaEntryPoints.obj
 0002:0000c4b8       ??_C@_0FK@MANGNIPE@?$FLINFO?$FN?3?5Calling?5AccessBridgeJav@ 1002e4b8     AccessBridgeJavaEntryPoints.obj
 0002:0000c514       ??_C@_0DO@JHGLNKHC@Doing?5selectAllAccessibleSelect@ 1002e514     AccessBridgeJavaEntryPoints.obj
 0002:0000c558       ??_C@_0EP@JCKDPHMN@?$FLERROR?$FN?3?5either?5env?5?$DN?$DN?50?5or?5sel@ 1002e558     AccessBridgeJavaEntryPoints.obj
 0002:0000c5a8       ??_C@_0EO@IEPNANKM@?$FLINFO?$FN?3?5?5?5in?5AccessBridgeJavaEn@ 1002e5a8     AccessBridgeJavaEntryPoints.obj
 0002:0000c5f8       ??_C@_0DK@GPMPKEMH@Doing?5addJavaEventNotification?5@ 1002e5f8     AccessBridgeJavaEntryPoints.obj
 0002:0000c638       ??_C@_0EA@IOOHIHIM@?$FLERROR?$FN?3?5either?5env?5?$DN?$DN?50?5or?5add@ 1002e638     AccessBridgeJavaEntryPoints.obj
 0002:0000c678       ??_C@_0FA@BBNLJKAK@?$FLINFO?$FN?3?5?5in?5AccessBridgeJavaEnt@ 1002e678     AccessBridgeJavaEntryPoints.obj
 0002:0000c6c8       ??_C@_0DN@IBNHMLMO@Doing?5removeJavaEventNotificati@ 1002e6c8     AccessBridgeJavaEntryPoints.obj
 0002:0000c708       ??_C@_0ED@LKLPMFCD@?$FLERROR?$FN?3?5either?5env?5?$DN?$DN?50?5or?5rem@ 1002e708     AccessBridgeJavaEntryPoints.obj
 0002:0000c750       ??_C@_0FH@ICFBIMPG@?$FLINFO?$FN?3?5?5?5in?5AccessBridgeJavaEn@ 1002e750     AccessBridgeJavaEntryPoints.obj
 0002:0000c7a8       ??_C@_0FL@OCFIPKDP@?$FLINFO?$FN?3?5?5?5?5addAccessibilityEven@ 1002e7a8     AccessBridgeJavaEntryPoints.obj
 0002:0000c804       ??_C@_0DH@DNDEHAJF@Doing?5addAccessibilityEvent?5?9?5c@ 1002e804     AccessBridgeJavaEntryPoints.obj
 0002:0000c840       ??_C@_0EJ@BAMHEIMC@?$FLERROR?$FN?3?5either?5env?5?$DN?$DN?50?5or?5add@ 1002e840     AccessBridgeJavaEntryPoints.obj
 0002:0000c890       ??_C@_0ED@BCNEMPCF@?$FLINFO?$FN?3?5?5?5?5?5addAccessibilityEve@ 1002e890     AccessBridgeJavaEntryPoints.obj
 0002:0000c8d8       ??_C@_0FJ@JPJKPKP@?$FLINFO?$FN?3?5?5in?5AccessBridgeJavaEnt@ 1002e8d8     AccessBridgeJavaEntryPoints.obj
 0002:0000c934       ??_C@_0DK@KGOHAMJ@Doing?5removeAccessibilityEvent?5@ 1002e934     AccessBridgeJavaEntryPoints.obj
 0002:0000c970       ??_C@_0EM@MPLDCCAE@?$FLERROR?$FN?3?5either?5env?5?$DN?$DN?50?5or?5rem@ 1002e970     AccessBridgeJavaEntryPoints.obj
 0002:0000c9bc       ??_C@_0BM@BIAOFPJG@AccessBridge?9FromJava?9Hello@ 1002e9bc     AccessBridgeMessages.obj
 0002:0000c9d8       ??_C@_0BP@OELHMMDF@AccessBridge?9FromWindows?9Hello@ 1002e9d8     AccessBridgeMessages.obj
 0002:0000c9f8       ??_C@_0CN@HNEPECB@?$FLINFO?$FN?3?5JavaAccessBridge?4DLL?5ru@ 1002e9f8     JavaAccessBridge.obj
 0002:0000ca28       ??_C@_0CN@OBDABACD@?$FLINFO?$FN?3?5In?5AccessBridgeDialog?5?9@ 1002ea28     JavaAccessBridge.obj
 0002:0000ca58       ??_C@_0DM@LEGKGBDC@?$FLINFO?$FN?3?5In?5AccessBridgeDialog?5?9@ 1002ea58     JavaAccessBridge.obj
 0002:0000ca94       ??_C@_0DP@KFGJNONL@?$FLINFO?$FN?3?5In?5AccessBridgeDialog?5?9@ 1002ea94     JavaAccessBridge.obj
 0002:0000cad4       ??_C@_0DN@BOPHDCMF@?$FLINFO?$FN?3?5In?5AccessBridgeDialog?5?9@ 1002ead4     JavaAccessBridge.obj
 0002:0000cb18       ??_C@_0EG@LODLDNEL@?$FLINFO?$FN?3?5In?5AccessBridgeDialog?5?9@ 1002eb18     JavaAccessBridge.obj
 0002:0000cb60       ??_C@_0EE@OLIPFHDH@?$FLINFO?$FN?3?5In?5AccessBridgeDialog?5?9@ 1002eb60     JavaAccessBridge.obj
 0002:0000cba4       ??_C@_0DO@KFBCLDPM@?$FLINFO?$FN?3?5In?5AccessBridgeDialog?5?9@ 1002eba4     JavaAccessBridge.obj
 0002:0000cbe8       ??_C@_0EF@PPOLOLIM@?$FLINFO?$FN?3?5In?5AccessBridgeDialog?5?9@ 1002ebe8     JavaAccessBridge.obj
 0002:0000cc30       ??_C@_0BD@BOAKDBCO@java_access_bridge@ 1002ec30     JavaAccessBridge.obj
 0002:0000cc44       ??_C@_0DB@JHKNDMME@?$FLINFO?$FN?3?5in?5JavaAccessBridge?3?3?$HOJ@ 1002ec44     JavaAccessBridge.obj
 0002:0000cc78       ??_C@_0CF@DJNKIAAH@?$FLINFO?$FN?3?5?5telling?5?$CFp?5we?8re?5going@ 1002ec78     JavaAccessBridge.obj
 0002:0000cca0       ??_C@_0CP@BKDEGDJC@?$FLINFO?$FN?3?5?5finished?5telling?5ATs?5a@ 1002eca0     JavaAccessBridge.obj
 0002:0000ccd0       ??_C@_0CA@EIEOEDOI@?$FLINFO?$FN?3?5?5?5finished?5deleting?5ATs@ 1002ecd0     JavaAccessBridge.obj
 0002:0000ccf0       ??_C@_0BP@EBFMIPOK@?$FLINFO?$FN?3?5GOODBYE?5CRUEL?5WORLD?4?4?4@ 1002ecf0     JavaAccessBridge.obj
 0002:0000cd10       ??_C@_0DB@BKKBMMIL@?$FLINFO?$FN?3?5JavaAccessBridge?3?3javaR@ 1002ed10     JavaAccessBridge.obj
 0002:0000cd44       ??_C@_0BJ@CDAHIMFI@?$FLINFO?$FN?3?5?5?5?9?$DO?5javaVM?5?$DN?5?$CFp@ 1002ed44     JavaAccessBridge.obj
 0002:0000cd60       ??_C@_0CF@HBJLLMBP@?$FLINFO?$FN?3?5?5?9?$DO?5windowsThreadJNIEnv@ 1002ed60     JavaAccessBridge.obj
 0002:0000cd88       ??_C@_0DL@EDCIECNK@?$FLINFO?$FN?3?5?5?5all?5Java?5thread?5entry@ 1002ed88     JavaAccessBridge.obj
 0002:0000cdc4       ??_C@_0DO@DHHHOLPH@?$FLINFO?$FN?3?5?5?5all?5Windows?5thread?5en@ 1002edc4     JavaAccessBridge.obj
 0002:0000ce04       ??_C@_0CF@FINMKFHO@?$FLINFO?$FN?3?5?5?5Window?5created?4?5?5HWND@ 1002ee04     JavaAccessBridge.obj
 0002:0000ce2c       ??_C@_0CG@KCHIBPOJ@?$FLERROR?$FN?3?5?5?5FAILED?5TO?5CREATE?5WIN@ 1002ee2c     JavaAccessBridge.obj
 0002:0000ce54       ??_C@_0BJ@LMONFDOG@ACCESSBRIDGESTATUSWINDOW@ 1002ee54     JavaAccessBridge.obj
 0002:0000ce70       ??_C@_0DG@HAJICJFK@?$FLINFO?$FN?3?5In?5JavaAccessBridge?3?3po@ 1002ee70     JavaAccessBridge.obj
 0002:0000cea8       ??_C@_0CO@FLLNHCIG@?$FLINFO?$FN?3?5?5?5calling?5PostMessage?$CI?$CF@ 1002eea8     JavaAccessBridge.obj
 0002:0000ced8       ??_C@_0CM@DCNJAPPO@?$FLERROR?$FN?3?5ATs?5?$DN?$DN?50?$CB?5?$CIshouldn?8t?5h@ 1002eed8     JavaAccessBridge.obj
 0002:0000cf04       ??_C@_0DH@JMPJBGDF@?$FLINFO?$FN?3?5JavaAccessBridge?3?3recei@ 1002ef04     JavaAccessBridge.obj
 0002:0000cf40       ??_C@_0EB@GECAJJE@?$FLERROR?$FN?3?5?9?5ATs?5?$DN?$DN?50?5?$CIshouldn?8t?5@ 1002ef40     JavaAccessBridge.obj
 0002:0000cf84       ??_C@_0DL@FAPEODKG@?$FLERROR?$FN?3?5receiving?5memory?5packa@ 1002ef84     JavaAccessBridge.obj
 0002:0000cfc0       ??_C@_0DM@MJCPMIJG@?$FLINFO?$FN?3?5Processing?5package?5sent@ 1002efc0     JavaAccessBridge.obj
 0002:0000cffc       ??_C@_0BL@EFABEHOK@?$FLINFO?$FN?3?5?5PackageType?5?$DN?5?$CFX?3@ 1002effc     JavaAccessBridge.obj
 0002:0000d018       ??_C@_0DC@HOEDKHHL@?$FLINFO?$FN?3?5?5?5type?5?$DN?$DN?5cMemoryMapped@ 1002f018     JavaAccessBridge.obj
 0002:0000d050       ??_C@_0EC@JELBKKLB@?$FLERROR?$FN?3?5?5?5?5processing?5FAILED?$CB?$CB@ 1002f050     JavaAccessBridge.obj
 0002:0000d094       ??_C@_0CM@EGHIFACB@?$FLINFO?$FN?3?5?5?5type?5?$DN?$DN?5cReleaseJavaO@ 1002f094     JavaAccessBridge.obj
 0002:0000d0c0       ??_C@_0EB@PCOLNIOI@?$FLERROR?$FN?3?5?5?5processing?5FAILED?$CB?$CB?5@ 1002f0c0     JavaAccessBridge.obj
 0002:0000d104       ??_C@_0DB@HJBBLNK@?$FLINFO?$FN?3?5?5?5type?5?$DN?$DN?5cGetAccessBri@ 1002f104     JavaAccessBridge.obj
 0002:0000d138       ??_C@_0CH@OGPNINNH@?$FLINFO?$FN?3?5?5?5type?5?$DN?$DN?5cIsJavaWindow@ 1002f138     JavaAccessBridge.obj
 0002:0000d160       ??_C@_0CF@KCGBFLNL@?$FLINFO?$FN?3?5?5?5?5?5?9?$DO?5returning?5result@ 1002f160     JavaAccessBridge.obj
 0002:0000d188       ??_C@_0CH@FFMGBMGP@?$FLINFO?$FN?3?5?5?5type?5?$DN?$DN?5cIsSameObject@ 1002f188     JavaAccessBridge.obj
 0002:0000d1b0       ??_C@_0DI@FGDPIMOI@?$FLINFO?$FN?3?5?5?5?5type?5?$DN?$DN?5cGetAccessib@ 1002f1b0     JavaAccessBridge.obj
 0002:0000d1e8       ??_C@_0CN@KFALDIEC@?$FLINFO?$FN?3?5?5?5?5?5?5?9?$DO?5returning?5AC?5?$DN?5@ 1002f1e8     JavaAccessBridge.obj
 0002:0000d218       ??_C@_0DI@ICOCNDDM@?$FLINFO?$FN?3?5?5?5?5type?5?$DN?$DN?5cGetHWNDFrom@ 1002f218     JavaAccessBridge.obj
 0002:0000d250       ??_C@_0CD@DNCFKFDK@?$FLINFO?$FN?3?5?5?5?5?5?9?$DO?5returning?5HWND?5?$DN@ 1002f250     JavaAccessBridge.obj
 0002:0000d274       ??_C@_0CK@DBBKGOKJ@?$FLINFO?$FN?3?5?5?5type?5?$DN?$DN?5cSetTextConte@ 1002f274     JavaAccessBridge.obj
 0002:0000d2a0       ??_C@_0JK@BDICEONN@?$FLINFO?$FN?3?5?5?5type?5?$DN?$DN?5cGetParentWit@ 1002f2a0     JavaAccessBridge.obj
 0002:0000d33c       ??_C@_0CM@FMGIHPCP@?$FLINFO?$FN?3?5?5?5type?5?$DN?$DN?5cGetTopLevelO@ 1002f33c     JavaAccessBridge.obj
 0002:0000d368       ??_C@_0DC@EMOAFCHE@?$FLINFO?$FN?3?5?5?5?5?5?5?9?$DO?5returning?5rAcce@ 1002f368     JavaAccessBridge.obj
 0002:0000d39c       ??_C@_0DE@EHPIAHAD@?$FLINFO?$FN?3?5?5?5type?5?$DN?$DN?5cGetParentWit@ 1002f39c     JavaAccessBridge.obj
 0002:0000d3d0       ??_C@_0CJ@CIIOKEJA@?$FLINFO?$FN?3?5?5?5type?5?$DN?$DN?5cGetObjectDep@ 1002f3d0     JavaAccessBridge.obj
 0002:0000d3fc       ??_C@_0CG@CCMHCDED@?$FLINFO?$FN?3?5?5?5?5?5?9?$DO?5returning?5rResul@ 1002f3fc     JavaAccessBridge.obj
 0002:0000d424       ??_C@_0CO@HPDBNII@?$FLINFO?$FN?3?5?5?5type?5?$DN?$DN?5cGetActiveDes@ 1002f424     JavaAccessBridge.obj
 0002:0000d454       ??_C@_0CO@EEGIDCBJ@?$FLINFO?$FN?3?5?5?9?$DO?5returning?5rAccessib@ 1002f454     JavaAccessBridge.obj
 0002:0000d484       ??_C@_0DB@BLNOEMHA@?$FLINFO?$FN?3?5?5?5type?5?$DN?$DN?5cGetAccessibl@ 1002f484     JavaAccessBridge.obj
 0002:0000d4b8       ??_C@_0DI@BBJPLAPN@?$FLINFO?$FN?3?5?5?5type?5?$DN?$DN?5cGetAccessibl@ 1002f4b8     JavaAccessBridge.obj
 0002:0000d4f0       ??_C@_0DD@EKFFDOAF@?$FLINFO?$FN?3?5?5?5type?5?$DN?$DN?5cGetAccessibl@ 1002f4f0     JavaAccessBridge.obj
 0002:0000d524       ??_C@_0DI@HCCMIAAH@?$FLINFO?$FN?3?5?5?5type?5?$DN?$DN?5cGetAccessibl@ 1002f524     JavaAccessBridge.obj
 0002:0000d55c       ??_C@_0DK@EHNJMPFO@?$FLINFO?$FN?3?5?5?5?5type?5?$DN?$DN?5cGetAccessib@ 1002f55c     JavaAccessBridge.obj
 0002:0000d598       ??_C@_0DI@DNENMOMG@?$FLINFO?$FN?3?5?5?5?5?$CD?$CD?$CD?$CD?$CD?5type?5?$DN?$DN?5cGetAc@ 1002f598     JavaAccessBridge.obj
 0002:0000d5d0       ??_C@_0CG@KFAMLONA@?$FLINFO?$FN?3?5?5?5?5?$CD?$CD?$CD?$CD?$CD?5processing?5suc@ 1002f5d0     JavaAccessBridge.obj
 0002:0000d5f8       ??_C@_0EI@KKCFGLCL@?$FLERROR?$FN?3?5?5?5?5?$CD?$CD?$CD?$CD?$CD?5processing?5FA@ 1002f5f8     JavaAccessBridge.obj
 0002:0000d640       ??_C@_0DM@ONBKHFBE@?$FLINFO?$FN?3?5?5?5?5?$CD?$CD?$CD?$CD?$CD?5type?5?$DN?$DN?5cGetAc@ 1002f640     JavaAccessBridge.obj
 0002:0000d67c       ??_C@_0DN@MOEKMKGM@?$FLINFO?$FN?3?5?5?5?5?$CD?$CD?$CD?$CD?$CD?5type?5?$DN?$DN?5cGetAc@ 1002f67c     JavaAccessBridge.obj
 0002:0000d6c0       ??_C@_0EA@CAKJDHMA@?$FLINFO?$FN?3?5?5?5?5?$CD?$CD?$CD?$CD?$CD?5type?5?$DN?$DN?5cGetAc@ 1002f6c0     JavaAccessBridge.obj
 0002:0000d700       ??_C@_0EC@JLIHGBEM@?$FLINFO?$FN?3?5?5?5?5?$CD?$CD?$CD?$CD?$CD?5type?5?$DN?$DN?5cGetAc@ 1002f700     JavaAccessBridge.obj
 0002:0000d748       ??_C@_0EF@DBAFGNDK@?$FLINFO?$FN?3?5?5?5?5?$CD?$CD?$CD?$CD?$CD?5type?5?$DN?$DN?5cGetAc@ 1002f748     JavaAccessBridge.obj
 0002:0000d790       ??_C@_0EI@BCPJNOBP@?$FLINFO?$FN?3?5?5?5?5?$CD?$CD?$CD?$CD?$CD?5type?5?$DN?$DN?5cGetAc@ 1002f790     JavaAccessBridge.obj
 0002:0000d7d8       ??_C@_0EF@ONIGGHFH@?$FLINFO?$FN?3?5?5?5?5?$CD?$CD?$CD?$CD?$CD?5type?5?$DN?$DN?5cGetAc@ 1002f7d8     JavaAccessBridge.obj
 0002:0000d820       ??_C@_0DO@ENBHEGBB@?$FLINFO?$FN?3?5?5?5?5?$CD?$CD?$CD?$CD?$CD?5type?5?$DN?$DN?5cIsAcc@ 1002f820     JavaAccessBridge.obj
 0002:0000d860       ??_C@_0EB@PMALJKOF@?$FLINFO?$FN?3?5?5?5?5?$CD?$CD?$CD?$CD?$CD?5type?5?$DN?$DN?5cIsAcc@ 1002f860     JavaAccessBridge.obj
 0002:0000d8a8       ??_C@_0EE@NFLEEFCE@?$FLINFO?$FN?3?5?5?5?5?$CD?$CD?$CD?$CD?$CD?5type?5?$DN?$DN?5cGetAc@ 1002f8a8     JavaAccessBridge.obj
 0002:0000d8f0       ??_C@_0EH@DNDNECPC@?$FLINFO?$FN?3?5?5?5?5?5?5?$CD?$CD?$CD?$CD?$CD?5cGetAccessib@ 1002f8f0     JavaAccessBridge.obj
 0002:0000d938       ??_C@_0EF@PFDKDHMH@?$FLINFO?$FN?3?5?5?5?5?5?5?$CD?$CD?$CD?$CD?$CD?5cGetAccessib@ 1002f938     JavaAccessBridge.obj
 0002:0000d980       ??_C@_0EB@FNPEGMEK@?$FLINFO?$FN?3?5?5?5?5?$CD?$CD?$CD?$CD?$CD?5type?5?$DN?$DN?5cGetAc@ 1002f980     JavaAccessBridge.obj
 0002:0000d9c4       ??_C@_0DH@HGKABJI@?$FLINFO?$FN?3?5?5?5?5?$CD?$CD?$CD?$CD?$CD?5type?5?$DN?$DN?5cGetAc@ 1002f9c4     JavaAccessBridge.obj
 0002:0000d9fc       ??_C@_0DK@PHHNIBJB@?$FLINFO?$FN?3?5?5?5?5?$CD?$CD?$CD?$CD?$CD?5type?5?$DN?$DN?5cGetAc@ 1002f9fc     JavaAccessBridge.obj
 0002:0000da38       ??_C@_0DJ@ECCDOPKO@?$FLINFO?$FN?3?5?5?5?5?$CD?$CD?$CD?$CD?$CD?5type?5?$DN?$DN?5cGetAc@ 1002fa38     JavaAccessBridge.obj
 0002:0000da74       ??_C@_0DK@GDIGFCLP@?$FLINFO?$FN?3?5?5?5?5?$CD?$CD?$CD?$CD?$CD?5type?5?$DN?$DN?5cGetAc@ 1002fa74     JavaAccessBridge.obj
 0002:0000dab0       ??_C@_0DI@BPKDDCHO@?$FLINFO?$FN?3?5?5?5?5?$CD?$CD?$CD?$CD?$CD?5type?5?$DN?$DN?5cGetAc@ 1002fab0     JavaAccessBridge.obj
 0002:0000dae8       ??_C@_0DN@OAAMPEIM@?$FLINFO?$FN?3?5?5?5?5?$CD?$CD?$CD?$CD?$CD?5type?5?$DN?$DN?5cActiv@ 1002fae8     JavaAccessBridge.obj
 0002:0000db28       ??_C@_0DN@GBPFAJCJ@?$FLINFO?$FN?3?5?5?5?5?$CD?$CD?$CD?$CD?$CD?5type?5?$DN?$DN?5cGetAc@ 1002fb28     JavaAccessBridge.obj
 0002:0000db68       ??_C@_0DM@HFKCAKHD@?$FLINFO?$FN?3?5?5?5?5?$CD?$CD?$CD?$CD?$CD?5processing?5suc@ 1002fb68     JavaAccessBridge.obj
 0002:0000dba4       ??_C@_0DL@BKPFGPAI@?$FLINFO?$FN?3?5?5?5?5?$CD?$CD?$CD?$CD?$CD?5type?5?$DN?$DN?5cGetAc@ 1002fba4     JavaAccessBridge.obj
 0002:0000dbe0       ??_C@_0EB@HBBMKHLL@?$FLINFO?$FN?3?5?5?5?5?$CD?$CD?$CD?$CD?$CD?5type?5?$DN?$DN?5cGetAc@ 1002fbe0     JavaAccessBridge.obj
 0002:0000dc24       ??_C@_0DI@EGGEEHLE@?$FLINFO?$FN?3?5?5?5?5?$CD?$CD?$CD?$CD?$CD?5type?5?$DN?$DN?5cGetAc@ 1002fc24     JavaAccessBridge.obj
 0002:0000dc5c       ??_C@_0DK@LOBFOEFG@?$FLINFO?$FN?3?5?5?5?5?$CD?$CD?$CD?$CD?$CD?5type?5?$DN?$DN?5cGetAc@ 1002fc5c     JavaAccessBridge.obj
 0002:0000dc98       ??_C@_0DE@NCPKKLJG@?$FLINFO?$FN?3?5?5?5?5?$CD?$CD?$CD?$CD?$CD?5type?5?$DN?$DN?5cGetAc@ 1002fc98     JavaAccessBridge.obj
 0002:0000dcd0       ??_C@_0EH@OKFMNJOP@?$FLERROR?$FN?3?5?5?5?$CD?$CD?$CD?$CD?$CD?5processing?5FAI@ 1002fcd0     JavaAccessBridge.obj
 0002:0000dd18       ??_C@_0DG@CDFKKFMN@?$FLINFO?$FN?3?5?5?5?5?$CD?$CD?$CD?$CD?$CD?5type?5?$DN?$DN?5cGetAc@ 1002fd18     JavaAccessBridge.obj
 0002:0000dd50       ??_C@_0DF@GOCDLFHO@?$FLINFO?$FN?3?5?5?5?5?$CD?$CD?$CD?$CD?$CD?5type?5?$DN?$DN?5cDoAcc@ 1002fd50     JavaAccessBridge.obj
 0002:0000dd88       ??_C@_0DJ@FOPNGHK@?$FLINFO?$FN?3?5?5?5?5?$CD?$CD?$CD?$CD?$CD?5type?5?$DN?$DN?5GetVir@ 1002fd88     JavaAccessBridge.obj
 0002:0000ddc4       ??_C@_0CN@KKAHFJLP@?$FLINFO?$FN?3?5?5?5?5?$CD?$CD?$CD?$CD?$CD?5type?5?$DN?$DN?5Reques@ 1002fdc4     JavaAccessBridge.obj
 0002:0000ddf4       ??_C@_0DA@BDJNNLOI@?$FLINFO?$FN?3?5?5?5?5?$CD?$CD?$CD?$CD?$CD?5type?5?$DN?$DN?5Select@ 1002fdf4     JavaAccessBridge.obj
 0002:0000de24       ??_C@_0DJ@JNPDLANK@?$FLINFO?$FN?3?5?5?5?5?$CD?$CD?$CD?$CD?$CD?5type?5?$DN?$DN?5GetTex@ 1002fe24     JavaAccessBridge.obj
 0002:0000de60       ??_C@_0DI@KCHGBBIN@?$FLINFO?$FN?3?5?5?5?5?$CD?$CD?$CD?$CD?$CD?5type?5?$DN?$DN?5GetVis@ 1002fe60     JavaAccessBridge.obj
 0002:0000de98       ??_C@_0DD@HFEKHIPA@?$FLINFO?$FN?3?5?5?5?5?$CD?$CD?$CD?$CD?$CD?5type?5?$DN?$DN?5GetVis@ 1002fe98     JavaAccessBridge.obj
 0002:0000decc       ??_C@_0DB@HDPFDIKC@?$FLINFO?$FN?3?5?5?5?5?$CD?$CD?$CD?$CD?$CD?5type?5?$DN?$DN?5SetCar@ 1002fecc     JavaAccessBridge.obj
 0002:0000df00       ??_C@_0DB@MBKJOFKA@?$FLINFO?$FN?3?5?5?5?5type?5?$DN?$DN?5cGetAccessib@ 1002ff00     JavaAccessBridge.obj
 0002:0000df34       ??_C@_0DC@FACNMLJM@?$FLINFO?$FN?3?5?5?5?5type?5?$DN?$DN?5cGetAccessib@ 1002ff34     JavaAccessBridge.obj
 0002:0000df68       ??_C@_0DK@BMAJHBGM@?$FLINFO?$FN?3?5?5?5?5type?5?$DN?$DN?5cGetAccessib@ 1002ff68     JavaAccessBridge.obj
 0002:0000dfa4       ??_C@_0DK@KLKIIEMH@?$FLINFO?$FN?3?5?5?5?5type?5?$DN?$DN?5cGetAccessib@ 1002ffa4     JavaAccessBridge.obj
 0002:0000dfe0       ??_C@_0DF@LJIJJCFL@?$FLINFO?$FN?3?5?5?5?5type?5?$DN?$DN?5cGetAccessib@ 1002ffe0     JavaAccessBridge.obj
 0002:0000e018       ??_C@_0CM@DKHFKJOD@?$FLINFO?$FN?3?5?5?5?5type?5?$DN?$DN?5cGetCaretLoc@ 10030018     JavaAccessBridge.obj
 0002:0000e044       ??_C@_0DH@CHPJDHJL@?$FLINFO?$FN?3?5?5?5?5type?5?$DN?$DN?5cGetAccessib@ 10030044     JavaAccessBridge.obj
 0002:0000e07c       ??_C@_0DC@HMIBGEHP@?$FLINFO?$FN?3?5?5?5?5type?5?$DN?$DN?5cGetAccessib@ 1003007c     JavaAccessBridge.obj
 0002:0000e0b0       ??_C@_0EA@OJBBPFCG@?$FLINFO?$FN?3?5?5?5?5type?5?$DN?$DN?5cGetCurrentA@ 100300b0     JavaAccessBridge.obj
 0002:0000e0f0       ??_C@_0EA@FFJJPODP@?$FLINFO?$FN?3?5?5?5?5type?5?$DN?$DN?5cGetMaximumA@ 100300f0     JavaAccessBridge.obj
 0002:0000e130       ??_C@_0EA@GABLOPGB@?$FLINFO?$FN?3?5?5?5?5type?5?$DN?$DN?5cGetMinimumA@ 10030130     JavaAccessBridge.obj
 0002:0000e170       ??_C@_0DN@NHMKNOBO@?$FLINFO?$FN?3?5?5?5?5type?5?$DN?$DN?5cAddAccessib@ 10030170     JavaAccessBridge.obj
 0002:0000e1b0       ??_C@_0DP@CDAIIOJL@?$FLINFO?$FN?3?5?5?5?5type?5?$DN?$DN?5cClearAccess@ 100301b0     JavaAccessBridge.obj
 0002:0000e1f0       ??_C@_0DN@FGNKIKEK@?$FLINFO?$FN?3?5?5?5?5type?5?$DN?$DN?5cGetAccessib@ 100301f0     JavaAccessBridge.obj
 0002:0000e230       ??_C@_0EC@JGIFJEAP@?$FLINFO?$FN?3?5?5?5?5type?5?$DN?$DN?5cGetAccessib@ 10030230     JavaAccessBridge.obj
 0002:0000e278       ??_C@_0EA@BDFAJBM@?$FLINFO?$FN?3?5?5?5?5type?5?$DN?$DN?5cIsAccessibl@ 10030278     JavaAccessBridge.obj
 0002:0000e2b8       ??_C@_0EA@NOOOKPJ@?$FLINFO?$FN?3?5?5?5?5type?5?$DN?$DN?5cRemoveAcces@ 100302b8     JavaAccessBridge.obj
 0002:0000e2f8       ??_C@_0ED@CNEBOKEO@?$FLINFO?$FN?3?5?5?5?5type?5?$DN?$DN?5cSelectAllAc@ 100302f8     JavaAccessBridge.obj
 0002:0000e33c       ??_C@_0DD@FDABBAIG@?$FLINFO?$FN?3?5?5?5?5type?5?$DN?5cAddJavaEvent@ 1003033c     JavaAccessBridge.obj
 0002:0000e370       ??_C@_0DG@CJJGFHBD@?$FLINFO?$FN?3?5?5?5?5type?5?$DN?5cRemoveJavaEv@ 10030370     JavaAccessBridge.obj
 0002:0000e3a8       ??_C@_0DM@IHHPMOM@?$FLINFO?$FN?3?5?5?5?5type?5?$DN?5cAddAccessibi@ 100303a8     JavaAccessBridge.obj
 0002:0000e3e4       ??_C@_0DP@CLPLFGHM@?$FLINFO?$FN?3?5?5?5?5type?5?$DN?5cRemoveAccess@ 100303e4     JavaAccessBridge.obj
 0002:0000e428       ??_C@_0EG@DADDGPDA@?$FLERROR?$FN?3?5?5?5?5processing?5FAILED?$CB?$CB@ 10030428     JavaAccessBridge.obj
 0002:0000e470       ??_C@_0CI@PMGDCMNI@?$FLINFO?$FN?3?5?5?5?5package?5processing?5c@ 10030470     JavaAccessBridge.obj
 0002:0000e498       ??_C@_0CO@NOIJCKLH@?$FLINFO?$FN?3?5?5?5in?5MemoryMappedFileCr@ 10030498     JavaAccessBridge.obj
 0002:0000e4c8       ??_C@_0DJ@MGBOAEHL@?$FLINFO?$FN?3?5?5?5?5?5just?5created?5a?5new?5@ 100304c8     JavaAccessBridge.obj
 0002:0000e504       ??_C@_0DA@PCLBAGKL@?$FLINFO?$FN?3?5?5?5Successfully?5initiate@ 10030504     JavaAccessBridge.obj
 0002:0000e534       ??_C@_0CL@IAFANAPB@?$FLERROR?$FN?3?5Failed?5to?5initiate?5IPC@ 10030534     JavaAccessBridge.obj
 0002:0000e560       ??_C@_0DE@FDNKAIDO@?$FLINFO?$FN?3?5in?5JavaAccessBridge?3?3Wi@ 10030560     JavaAccessBridge.obj
 0002:0000e594       ??_C@_0CO@DDCCLLBJ@?$FLERROR?$FN?3?5?9?$DO?5ATs?5?$DN?$DN?50?$CB?5?$CIshouldn?8@ 10030594     JavaAccessBridge.obj
 0002:0000e5c4       ??_C@_0CP@IIHJFGGB@?$FLINFO?$FN?3?5?5?5data?5structures?5succe@ 100305c4     JavaAccessBridge.obj
 0002:0000e5f4       ??_C@_0DB@JABMCGEJ@?$FLERROR?$FN?3?5couldn?8t?5find?5matching@ 100305f4     JavaAccessBridge.obj
 0002:0000e628       ??_C@_0CP@LEPCODGO@?$FLINFO?$FN?3?5In?5JavaAccessBridge?3?3re@ 10030628     JavaAccessBridge.obj
 0002:0000e658       ??_C@_0BH@GNOIGMFE@?$FLINFO?$FN?3?5?5?5object?5X?3?5?$CFp@ 10030658     JavaAccessBridge.obj
 0002:0000e670       ??_C@_0CE@NAEKPPND@?$FLINFO?$FN?3?5?5?5global?5reference?5dele@ 10030670     JavaAccessBridge.obj
 0002:0000e694       ??_C@_0CC@DPMNCGAA@?$FLERROR?$FN?3?5windowsThreadJNIEnv?5?$DN?$DN@ 10030694     JavaAccessBridge.obj
 0002:0000e6b8       ??_C@_0DF@HMNKBJGB@?$FLINFO?$FN?3?5?5?5adding?5Java?5event?5typ@ 100306b8     JavaAccessBridge.obj
 0002:0000e6f0       ??_C@_0CO@OPGCCICC@?$FLINFO?$FN?3?5?5?5found?5HWND?0?5javaEvent@ 100306f0     JavaAccessBridge.obj
 0002:0000e720       ??_C@_0CP@MJMPLPDN@?$FLINFO?$FN?3?5?5?5union?5of?5all?5Java?5AT?5@ 10030720     JavaAccessBridge.obj
 0002:0000e750       ??_C@_0FO@PMMLAHPF@?$FLINFO?$FN?3?5?5?5no?5other?5AT?5wanted?5th@ 10030750     JavaAccessBridge.obj
 0002:0000e7b0       ??_C@_0DJ@DFJLLFAC@?$FLINFO?$FN?3?5?5?5removing?5Java?5event?5t@ 100307b0     JavaAccessBridge.obj
 0002:0000e7f0       ??_C@_0FO@LBFBGKHJ@?$FLINFO?$FN?3?5?5?5no?5other?5AT?5wanted?5th@ 100307f0     JavaAccessBridge.obj
 0002:0000e850       ??_C@_0DN@PDHOAFNL@?$FLINFO?$FN?3?5?5?5adding?5Accesibility?5e@ 10030850     JavaAccessBridge.obj
 0002:0000e890       ??_C@_0DH@EPKDBDGJ@?$FLINFO?$FN?3?5?5?5found?5HWND?0?5accessibi@ 10030890     JavaAccessBridge.obj
 0002:0000e8c8       ??_C@_0DI@IJKEHAJM@?$FLINFO?$FN?3?5?5?5union?5of?5all?5Accessib@ 100308c8     JavaAccessBridge.obj
 0002:0000e900       ??_C@_0GG@CGBBDJFJ@?$FLINFO?$FN?3?5?5?5no?5other?5AT?5wanted?5th@ 10030900     JavaAccessBridge.obj
 0002:0000e968       ??_C@_0EB@PJLIMJAJ@?$FLINFO?$FN?3?5?5?5removing?5Accesibility@ 10030968     JavaAccessBridge.obj
 0002:0000e9b0       ??_C@_0GH@FGGMCIOE@?$FLINFO?$FN?3?5?5?5no?5other?5AT?5wanted?5th@ 100309b0     JavaAccessBridge.obj
 0002:0000ea18       ??_C@_0GL@DLLNHKDB@?$FLINFO?$FN?3?5Java_com_sun_java_acces@ 10030a18     JavaAccessBridge.obj
 0002:0000ea84       ??_C@_0BI@GOJFHMPI@?$FLINFO?$FN?3?5?5?5sending?5to?5AT@ 10030a84     JavaAccessBridge.obj
 0002:0000eaa0       ??_C@_0EA@HDPEOOCD@?$FLINFO?$FN?3?5?5?5GlobalRef?8d?5Event?3?5?$CFp@ 10030aa0     JavaAccessBridge.obj
 0002:0000eae0       ??_C@_0CN@HLLEMELD@?$FLINFO?$FN?3?5?5done?5with?5propertyCare@ 10030ae0     JavaAccessBridge.obj
 0002:0000eb10       ??_C@_0HB@FIEPPBDD@?$FLINFO?$FN?3?5Java_com_sun_java_acces@ 10030b10     JavaAccessBridge.obj
 0002:0000eb84       ??_C@_0BL@ENCPOIKC@java?1lang?1OutOfMemoryError@ 10030b84     JavaAccessBridge.obj
 0002:0000eba0       ??_C@_1O@CEDCILHN@?$AA?$CI?$AAn?$AAu?$AAl?$AAl?$AA?$CJ@ 10030ba0     JavaAccessBridge.obj
 0002:0000ebb0       ??_C@_0DE@IIPLELBE@?$FLINFO?$FN?3?5?5?5done?5with?5propertyDes@ 10030bb0     JavaAccessBridge.obj
 0002:0000ebe8       ??_C@_0GK@FGEOELMA@?$FLINFO?$FN?3?5Java_com_sun_java_acces@ 10030be8     JavaAccessBridge.obj
 0002:0000ec54       ??_C@_0CM@LHIINGJI@?$FLINFO?$FN?3?5?5done?5with?5propertyName@ 10030c54     JavaAccessBridge.obj
 0002:0000ec80       ??_C@_0GH@NDFIEILD@?$FLINFO?$FN?3?5Java_com_sun_java_acces@ 10030c80     JavaAccessBridge.obj
 0002:0000ece8       ??_C@_0DC@IDEPNPKP@?$FLINFO?$FN?3?5?5?5done?5with?5propertySel@ 10030ce8     JavaAccessBridge.obj
 0002:0000ed20       ??_C@_0GL@LHHKNKCF@?$FLINFO?$FN?3?5Java_com_sun_java_acces@ 10030d20     JavaAccessBridge.obj
 0002:0000ed8c       ??_C@_0DI@HBGABKPB@?$FLINFO?$FN?3?5?5?5GlobalRef?8d?5Event?3?5?$CFp@ 10030d8c     JavaAccessBridge.obj
 0002:0000edc4       ??_C@_0CN@HPCDPOIL@?$FLINFO?$FN?3?5?5done?5with?5propertyStat@ 10030dc4     JavaAccessBridge.obj
 0002:0000edf8       ??_C@_0GC@GKPNHBKM@?$FLINFO?$FN?3?5Java_com_sun_java_acces@ 10030df8     JavaAccessBridge.obj
 0002:0000ee5c       ??_C@_0CM@MKJMCAOF@?$FLINFO?$FN?3?5?5done?5with?5propertyText@ 10030e5c     JavaAccessBridge.obj
 0002:0000ee88       ??_C@_0GL@LMHLMBIC@?$FLINFO?$FN?3?5Java_com_sun_java_acces@ 10030e88     JavaAccessBridge.obj
 0002:0000eef4       ??_C@_0CO@LJOPOKFE@?$FLINFO?$FN?3?5?5?5done?5with?5propertyVal@ 10030ef4     JavaAccessBridge.obj
 0002:0000ef28       ??_C@_0GJ@PEJPEKID@?$FLINFO?$FN?3?5Java_com_sun_java_acces@ 10030f28     JavaAccessBridge.obj
 0002:0000ef94       ??_C@_0DD@LNFBPAKO@?$FLINFO?$FN?3?5?5done?5with?5propertyVisi@ 10030f94     JavaAccessBridge.obj
 0002:0000efc8       ??_C@_0HD@JKCIIIAC@?$FLINFO?$FN?3?5Java_com_sun_java_acces@ 10030fc8     JavaAccessBridge.obj
 0002:0000f03c       ??_C@_0BH@HMENLEAO@?$FLINFO?$FN?3?5?5sending?5to?5AT@ 1003103c     JavaAccessBridge.obj
 0002:0000f058       ??_C@_0GP@GEKEHDBB@?$FLINFO?$FN?3?5?5GlobalRef?8d?5Event?3?5?$CFp?5@ 10031058     JavaAccessBridge.obj
 0002:0000f0c8       ??_C@_0CN@LGDOHOEO@?$FLINFO?$FN?3?5?5done?5with?5propertyChil@ 100310c8     JavaAccessBridge.obj
 0002:0000f0f8       ??_C@_0HO@MNNKGDDP@?$FLINFO?$FN?3?5Java_com_sun_java_acces@ 100310f8     JavaAccessBridge.obj
 0002:0000f178       ??_C@_0IG@DNLGNOND@?$FLINFO?$FN?3?5?5?5GlobalRef?8d?5Event?3?5?$CFp@ 10031178     JavaAccessBridge.obj
 0002:0000f200       ??_C@_0CO@GOOPPCJH@?$FLINFO?$FN?3?5?5done?5with?5propertyActi@ 10031200     JavaAccessBridge.obj
 0002:0000f230       ??_C@_0GP@NILNKGMP@?$FLINFO?$FN?3?5Java_com_sun_java_acces@ 10031230     JavaAccessBridge.obj
 0002:0000f2a0       ??_C@_0BA@KOMOFG@?5?5sending?5to?5AT@ 100312a0     JavaAccessBridge.obj
 0002:0000f2b0       ??_C@_0DC@FMNGEBKI@?$FLINFO?$FN?3?5?5done?5with?5propertyTabl@ 100312b0     JavaAccessBridge.obj
 0002:0000f2e4       ??_C@_0DA@ODJJOIDA@?$FLINFO?$FN?3?5Firing?5event?5id?5?$DN?5?$CFd?$CI?$CFp@ 100312e4     JavaAccessBridge.obj
 0002:0000f314       ??_C@_0CF@EPNHEIBO@?$FLINFO?$FN?3?5?5?5done?5with?5firing?5AWT?5@ 10031314     JavaAccessBridge.obj
 0002:0000f33c       ??_C@_0DI@NNGMMOBO@?$FLINFO?$FN?3?5Firing?5event?5id?5?$DN?5?$CFd?$CI?$CFp@ 1003133c     JavaAccessBridge.obj
 0002:0000f374       ??_C@_0DJ@GLLLDFPO@?$FLINFO?$FN?3?5javaEventMask?5?$DN?5?$CFX?5even@ 10031374     JavaAccessBridge.obj
 0002:0000f3b0       ??_C@_1CO@CCIONPKC@?$AAA?$AAc?$AAc?$AAe?$AAs?$AAs?$AAB?$AAr?$AAi?$AAd?$AAg?$AAe?$AA?4?$AAj?$AAa@ 100313b0     JavaAccessBridge.obj
 0002:0000f3e0       __pDefaultRawDllMain       100313e0     LIBCMT:dll_dllmain.obj
 0002:0000f3e0       __pRawDllMain              100313e0     LIBCMT:dll_dllmain.obj
 0002:0000f3e8       ??_7exception@std@@6B@     100313e8     LIBCMT:throw_bad_alloc.obj
 0002:0000f3f0       ??_C@_0BC@EOODALEL@Unknown?5exception@ 100313f0     LIBCMT:throw_bad_alloc.obj
 0002:0000f408       ??_7bad_alloc@std@@6B@     10031408     LIBCMT:throw_bad_alloc.obj
 0002:0000f410       ??_C@_0P@GHFPNOJB@bad?5allocation@ 10031410     LIBCMT:throw_bad_alloc.obj
 0002:0000f424       ??_7bad_array_new_length@std@@6B@ 10031424     LIBCMT:throw_bad_alloc.obj
 0002:0000f42c       ??_C@_0BF@KINCDENJ@bad?5array?5new?5length@ 1003142c     LIBCMT:throw_bad_alloc.obj
 0002:0000f450       ??_7type_info@@6B@         10031450     LIBCMT:std_type_info_static.obj
 0002:0000f454       __pDestructExceptionObject 10031454     libvcruntime:ehhelpers.obj
 0002:0000f7d8       ??_C@_08EHJDFFNH@__based?$CI@ 100317d8     libvcruntime:undname.obj
 0002:0000f7e4       ??_C@_07KOLFKCDI@__cdecl@  100317e4     libvcruntime:undname.obj
 0002:0000f7ec       ??_C@_08GHMPAG@__pascal@   100317ec     libvcruntime:undname.obj
 0002:0000f7f8       ??_C@_09IFJBGAPI@__stdcall@ 100317f8     libvcruntime:undname.obj
 0002:0000f804       ??_C@_0L@NPHFGOKO@__thiscall@ 10031804     libvcruntime:undname.obj
 0002:0000f810       ??_C@_0L@JMKHOMEK@__fastcall@ 10031810     libvcruntime:undname.obj
 0002:0000f81c       ??_C@_0N@BCKKPABJ@__vectorcall@ 1003181c     libvcruntime:undname.obj
 0002:0000f82c       ??_C@_09HIJEGCPM@__clrcall@ 1003182c     libvcruntime:undname.obj
 0002:0000f838       ??_C@_06GHPCKEAG@__eabi@   10031838     libvcruntime:undname.obj
 0002:0000f840       ??_C@_09IOPIDJLG@__swift_1@ 10031840     libvcruntime:undname.obj
 0002:0000f84c       ??_C@_09KFNFGKHF@__swift_2@ 1003184c     libvcruntime:undname.obj
 0002:0000f858       ??_C@_07JOMMBBKO@__ptr64@  10031858     libvcruntime:undname.obj
 0002:0000f860       ??_C@_0L@PILCLIHE@__restrict@ 10031860     libvcruntime:undname.obj
 0002:0000f86c       ??_C@_0M@GFIIJFMG@__unaligned@ 1003186c     libvcruntime:undname.obj
 0002:0000f878       ??_C@_09DHDLOLLB@restrict?$CI@ 10031878     libvcruntime:undname.obj
 0002:0000f882       ??_C@_00CNPNBAHC@@         10031882     libvcruntime:undname.obj
 0002:0000f884       ??_C@_04NIHEBCM@?5new@     10031884     libvcruntime:undname.obj
 0002:0000f88c       ??_C@_07FPCDHGMM@?5delete@ 1003188c     libvcruntime:undname.obj
 0002:0000f894       ??_C@_01NEMOKFLO@?$DN@     10031894     libvcruntime:undname.obj
 0002:0000f898       ??_C@_02GPIOPFAK@?$DO?$DO@ 10031898     libvcruntime:undname.obj
 0002:0000f89c       ??_C@_02FODMEDOG@?$DM?$DM@ 1003189c     libvcruntime:undname.obj
 0002:0000f8a0       ??_C@_01DCLJPIOD@?$CB@     100318a0     libvcruntime:undname.obj
 0002:0000f8a4       ??_C@_02EGOFBIJA@?$DN?$DN@ 100318a4     libvcruntime:undname.obj
 0002:0000f8a8       ??_C@_02FDNJECIE@?$CB?$DN@ 100318a8     libvcruntime:undname.obj
 0002:0000f8ac       ??_C@_02GPECMEKF@?$FL?$FN@ 100318ac     libvcruntime:undname.obj
 0002:0000f8b0       ??_C@_08LHJFAFGD@operator@ 100318b0     libvcruntime:undname.obj
 0002:0000f8bc       ??_C@_02HBOOOICD@?9?$DO@   100318bc     libvcruntime:undname.obj
 0002:0000f8c0       ??_C@_01NBENCBCI@?$CK@     100318c0     libvcruntime:undname.obj
 0002:0000f8c4       ??_C@_02ECNGHCIF@?$CL?$CL@ 100318c4     libvcruntime:undname.obj
 0002:0000f8c8       ??_C@_02BAABKJLB@?9?9@     100318c8     libvcruntime:undname.obj
 0002:0000f8cc       ??_C@_01JOAMLHOP@?9@       100318cc     libvcruntime:undname.obj
 0002:0000f8d0       ??_C@_01MIFGBAGJ@?$CL@     100318d0     libvcruntime:undname.obj
 0002:0000f8d4       ??_C@_01HNPIGOCE@?$CG@     100318d4     libvcruntime:undname.obj
 0002:0000f8d8       ??_C@_03MNHNFDLC@?9?$DO?$CK@ 100318d8     libvcruntime:undname.obj
 0002:0000f8dc       ??_C@_01KMDKNFGN@?1@       100318dc     libvcruntime:undname.obj
 0002:0000f8e0       ??_C@_01FGNFDNOH@?$CF@     100318e0     libvcruntime:undname.obj
 0002:0000f8e4       ??_C@_01MNNFJEPP@?$DM@     100318e4     libvcruntime:undname.obj
 0002:0000f8e8       ??_C@_02EHCHHCKH@?$DM?$DN@ 100318e8     libvcruntime:undname.obj
 0002:0000f8ec       ??_C@_01PPODPGHN@?$DO@     100318ec     libvcruntime:undname.obj
 0002:0000f8f0       ??_C@_02EEKDKGMJ@?$DO?$DN@ 100318f0     libvcruntime:undname.obj
 0002:0000f8f4       ??_C@_01IHBHIGKO@?0@       100318f4     libvcruntime:undname.obj
 0002:0000f8f8       ??_C@_02HCKGKOFO@?$CI?$CJ@ 100318f8     libvcruntime:undname.obj
 0002:0000f8fc       ??_C@_01PJKLJHI@?$HO@      100318fc     libvcruntime:undname.obj
 0002:0000f900       ??_C@_01JKBOJNNK@?$FO@     10031900     libvcruntime:undname.obj
 0002:0000f904       ??_C@_01DNKMNLPK@?$HM@     10031904     libvcruntime:undname.obj
 0002:0000f908       ??_C@_02PPKAJPJL@?$CG?$CG@ 10031908     libvcruntime:undname.obj
 0002:0000f90c       ??_C@_02NONPIBCD@?$HM?$HM@ 1003190c     libvcruntime:undname.obj
 0002:0000f910       ??_C@_02FPIMKNGF@?$CK?$DN@ 10031910     libvcruntime:undname.obj
 0002:0000f914       ??_C@_02FOEOMHFC@?$CL?$DN@ 10031914     libvcruntime:undname.obj
 0002:0000f918       ??_C@_02FKMDLLOA@?9?$DN@   10031918     libvcruntime:undname.obj
 0002:0000f91c       ??_C@_02FJEHGPIO@?1?$DN@   1003191c     libvcruntime:undname.obj
 0002:0000f920       ??_C@_02FENAOKFI@?$CF?$DN@ 10031920     libvcruntime:undname.obj
 0002:0000f924       ??_C@_03IKFCCPFF@?$DO?$DO?$DN@ 10031924     libvcruntime:undname.obj
 0002:0000f928       ??_C@_03CDNPDDLA@?$DM?$DM?$DN@ 10031928     libvcruntime:undname.obj
 0002:0000f92c       ??_C@_02FGJGFEAB@?$CG?$DN@ 1003192c     libvcruntime:undname.obj
 0002:0000f930       ??_C@_02DHLNPPGH@?$HM?$DN@ 10031930     libvcruntime:undname.obj
 0002:0000f934       ??_C@_02MHEGNOJ@?$FO?$DN@  10031934     libvcruntime:undname.obj
 0002:0000f938       ??_C@_09IFPLHPGF@?$GAvftable?8@ 10031938     libvcruntime:undname.obj
 0002:0000f944       ??_C@_09BLBHBJP@?$GAvbtable?8@ 10031944     libvcruntime:undname.obj
 0002:0000f950       ??_C@_07FEEIOKP@?$GAvcall?8@ 10031950     libvcruntime:undname.obj
 0002:0000f958       ??_C@_08LLFFHHDJ@?$GAtypeof?8@ 10031958     libvcruntime:undname.obj
 0002:0000f964       ??_C@_0BF@KDPPACIK@?$GAlocal?5static?5guard?8@ 10031964     libvcruntime:undname.obj
 0002:0000f97c       ??_C@_08OBABFOLI@?$GAstring?8@ 1003197c     libvcruntime:undname.obj
 0002:0000f988       ??_C@_0BD@JDLKDPAB@?$GAvbase?5destructor?8@ 10031988     libvcruntime:undname.obj
 0002:0000f99c       ??_C@_0BN@DEGPLNFK@?$GAvector?5deleting?5destructor?8@ 1003199c     libvcruntime:undname.obj
 0002:0000f9bc       ??_C@_0BO@OBMKPJIG@?$GAdefault?5constructor?5closure?8@ 100319bc     libvcruntime:undname.obj
 0002:0000f9dc       ??_C@_0BN@IMDCHIKM@?$GAscalar?5deleting?5destructor?8@ 100319dc     libvcruntime:undname.obj
 0002:0000f9fc       ??_C@_0BO@PFGOCPJJ@?$GAvector?5constructor?5iterator?8@ 100319fc     libvcruntime:undname.obj
 0002:0000fa1c       ??_C@_0BN@LFPFMEDL@?$GAvector?5destructor?5iterator?8@ 10031a1c     libvcruntime:undname.obj
 0002:0000fa3c       ??_C@_0CE@IKBNEHA@?$GAvector?5vbase?5constructor?5itera@ 10031a3c     libvcruntime:undname.obj
 0002:0000fa60       ??_C@_0BL@NILFHHPC@?$GAvirtual?5displacement?5map?8@ 10031a60     libvcruntime:undname.obj
 0002:0000fa7c       ??_C@_0CB@JONCMFFK@?$GAeh?5vector?5constructor?5iterator@ 10031a7c     libvcruntime:undname.obj
 0002:0000faa0       ??_C@_0CA@GCEOPDGL@?$GAeh?5vector?5destructor?5iterator?8@ 10031aa0     libvcruntime:undname.obj
 0002:0000fac0       ??_C@_0CH@OOJPLCPH@?$GAeh?5vector?5vbase?5constructor?5it@ 10031ac0     libvcruntime:undname.obj
 0002:0000fae8       ??_C@_0BL@LLKPOHJI@?$GAcopy?5constructor?5closure?8@ 10031ae8     libvcruntime:undname.obj
 0002:0000fb04       ??_C@_0BA@KBCDOMBN@?$GAudt?5returning?8@ 10031b04     libvcruntime:undname.obj
 0002:0000fb14       ??_C@_03KLGMFNMG@?$GAEH@   10031b14     libvcruntime:undname.obj
 0002:0000fb18       ??_C@_05KHLCHHI@?$GARTTI@  10031b18     libvcruntime:undname.obj
 0002:0000fb20       ??_C@_0BA@KKLDJDLB@?$GAlocal?5vftable?8@ 10031b20     libvcruntime:undname.obj
 0002:0000fb30       ??_C@_0CE@IIHCMGGL@?$GAlocal?5vftable?5constructor?5clos@ 10031b30     libvcruntime:undname.obj
 0002:0000fb54       ??_C@_06FHBGPFGH@?5new?$FL?$FN@ 10031b54     libvcruntime:undname.obj
 0002:0000fb5c       ??_C@_09LBNFPBCA@?5delete?$FL?$FN@ 10031b5c     libvcruntime:undname.obj
 0002:0000fb68       ??_C@_0P@HJKNJFNN@?$GAomni?5callsig?8@ 10031b68     libvcruntime:undname.obj
 0002:0000fb78       ??_C@_0BL@CNOONJFP@?$GAplacement?5delete?5closure?8@ 10031b78     libvcruntime:undname.obj
 0002:0000fb94       ??_C@_0BN@CKNJLHMB@?$GAplacement?5delete?$FL?$FN?5closure?8@ 10031b94     libvcruntime:undname.obj
 0002:0000fbb4       ??_C@_0CG@CFDHKGGD@?$GAmanaged?5vector?5constructor?5ite@ 10031bb4     libvcruntime:undname.obj
 0002:0000fbdc       ??_C@_0CF@IMGKMJNO@?$GAmanaged?5vector?5destructor?5iter@ 10031bdc     libvcruntime:undname.obj
 0002:0000fc04       ??_C@_0CG@HLDDJMAG@?$GAeh?5vector?5copy?5constructor?5ite@ 10031c04     libvcruntime:undname.obj
 0002:0000fc2c       ??_C@_0CM@FCBBDIGB@?$GAeh?5vector?5vbase?5copy?5construct@ 10031c2c     libvcruntime:undname.obj
 0002:0000fc58       ??_C@_0BL@CLIPGLGB@?$GAdynamic?5initializer?5for?5?8@ 10031c58     libvcruntime:undname.obj
 0002:0000fc74       ??_C@_0CB@PDBIFEP@?$GAdynamic?5atexit?5destructor?5for?5@ 10031c74     libvcruntime:undname.obj
 0002:0000fc98       ??_C@_0CD@CGAJBKEJ@?$GAvector?5copy?5constructor?5iterat@ 10031c98     libvcruntime:undname.obj
 0002:0000fcbc       ??_C@_0CJ@GJELGAMM@?$GAvector?5vbase?5copy?5constructor?5@ 10031cbc     libvcruntime:undname.obj
 0002:0000fce8       ??_C@_0CL@FGIJHLCE@?$GAmanaged?5vector?5copy?5constructo@ 10031ce8     libvcruntime:undname.obj
 0002:0000fd14       ??_C@_0BM@PMGGMLDN@?$GAlocal?5static?5thread?5guard?8@ 10031d14     libvcruntime:undname.obj
 0002:0000fd30       ??_C@_0N@BDNMDMOL@operator?5?$CC?$CC?5@ 10031d30     libvcruntime:undname.obj
 0002:0000fd40       ??_C@_0BC@GGEBGALA@operator?5co_await@ 10031d40     libvcruntime:undname.obj
 0002:0000fd54       ??_C@_0M@GAAIMMOH@operator?$DM?$DN?$DO@ 10031d54     libvcruntime:undname.obj
 0002:0000fd60       ??_C@_0BC@DAFEJGAK@?5Type?5Descriptor?8@ 10031d60     libvcruntime:undname.obj
 0002:0000fd74       ??_C@_0BM@LDKODKLH@?5Base?5Class?5Descriptor?5at?5?$CI@ 10031d74     libvcruntime:undname.obj
 0002:0000fd90       ??_C@_0BD@LGICGFMM@?5Base?5Class?5Array?8@ 10031d90     libvcruntime:undname.obj
 0002:0000fda4       ??_C@_0BN@MECKDCOJ@?5Class?5Hierarchy?5Descriptor?8@ 10031da4     libvcruntime:undname.obj
 0002:0000fdc4       ??_C@_0BK@CFCOFLF@?5Complete?5Object?5Locator?8@ 10031dc4     libvcruntime:undname.obj
 0002:0000fde0       ??_C@_0BG@JNJLAMPM@?$GAanonymous?5namespace?8@ 10031de0     libvcruntime:undname.obj
 0002:0000fe04       ??_C@_1DM@KHCHBNEB@?$AAa?$AAp?$AAi?$AA?9?$AAm?$AAs?$AA?9?$AAw?$AAi?$AAn?$AA?9?$AAc?$AAo?$AAr?$AAe@ 10031e04     libvcruntime:winapi_downlevel.obj
 0002:0000fe40       ??_C@_1DK@LPPGFMPP@?$AAa?$AAp?$AAi?$AA?9?$AAm?$AAs?$AA?9?$AAw?$AAi?$AAn?$AA?9?$AAc?$AAo?$AAr?$AAe@ 10031e40     libvcruntime:winapi_downlevel.obj
 0002:0000fe7c       ??_C@_1BC@GDMECMAK@?$AAk?$AAe?$AAr?$AAn?$AAe?$AAl?$AA3?$AA2@ 10031e7c     libvcruntime:winapi_downlevel.obj
 0002:0000fe90       ??_C@_1BA@PFFKHIOG@?$AAa?$AAp?$AAi?$AA?9?$AAm?$AAs?$AA?9@ 10031e90     libvcruntime:winapi_downlevel.obj
 0002:0000fea8       ??_C@_08KNHFBNJ@FlsAlloc@  10031ea8     libvcruntime:winapi_downlevel.obj
 0002:0000febc       ??_C@_07PEJMOBNF@FlsFree@  10031ebc     libvcruntime:winapi_downlevel.obj
 0002:0000fecc       ??_C@_0M@GDNOONDI@FlsGetValue@ 10031ecc     libvcruntime:winapi_downlevel.obj
 0002:0000fee0       ??_C@_0M@JCPCPOEF@FlsSetValue@ 10031ee0     libvcruntime:winapi_downlevel.obj
 0002:0000fef4       ??_C@_0BM@HCFOFFN@InitializeCriticalSectionEx@ 10031ef4     libvcruntime:winapi_downlevel.obj
 0002:0000ff10       _standard_lookup_table     10031f10     libucrt:output.obj
 0002:0000ff6c       ??_C@_06OJHGLDPL@?$CInull?$CJ@ 10031f6c     libucrt:output.obj
 0002:0000ff78       ___acrt_exception_action_table 10031f78     libucrt:exception_filter.obj
 0002:00010008       ___acrt_signal_action_table_count 10032008     libucrt:exception_filter.obj
 0002:0001000c       ___acrt_signal_action_first_fpe_index 1003200c     libucrt:exception_filter.obj
 0002:00010010       ___acrt_signal_action_fpe_count 10032010     libucrt:exception_filter.obj
 0002:00010014       ??_C@_1BI@BGOHAHKC@?$AAm?$AAs?$AAc?$AAo?$AAr?$AAe?$AAe?$AA?4?$AAd?$AAl?$AAl@ 10032014     libucrt:exit.obj
 0002:0001002c       ??_C@_0P@MIGLKIOC@CorExitProcess@ 1003202c     libucrt:exit.obj
 0002:00010278       ??_C@_1EA@JGEFHKEI@?$AAa?$AAp?$AAi?$AA?9?$AAm?$AAs?$AA?9?$AAw?$AAi?$AAn?$AA?9?$AAc?$AAo?$AAr?$AAe@ 10032278     libucrt:winapi_thunks.obj
 0002:000102b8       ??_C@_1DI@IJCEHOCB@?$AAa?$AAp?$AAi?$AA?9?$AAm?$AAs?$AA?9?$AAw?$AAi?$AAn?$AA?9?$AAc?$AAo?$AAr?$AAe@ 100322b8     libucrt:winapi_thunks.obj
 0002:000102f0       ??_C@_1EI@MPIAOHOC@?$AAa?$AAp?$AAi?$AA?9?$AAm?$AAs?$AA?9?$AAw?$AAi?$AAn?$AA?9?$AAc?$AAo?$AAr?$AAe@ 100322f0     libucrt:winapi_thunks.obj
 0002:00010338       ??_C@_1FK@FPHCKFIE@?$AAa?$AAp?$AAi?$AA?9?$AAm?$AAs?$AA?9?$AAw?$AAi?$AAn?$AA?9?$AAc?$AAo?$AAr?$AAe@ 10032338     libucrt:winapi_thunks.obj
 0002:00010398       ??_C@_1EM@DILCGIIO@?$AAa?$AAp?$AAi?$AA?9?$AAm?$AAs?$AA?9?$AAw?$AAi?$AAn?$AA?9?$AAc?$AAo?$AAr?$AAe@ 10032398     libucrt:winapi_thunks.obj
 0002:000103e4       ??_C@_1DM@LNCGDDPN@?$AAa?$AAp?$AAi?$AA?9?$AAm?$AAs?$AA?9?$AAw?$AAi?$AAn?$AA?9?$AAc?$AAo?$AAr?$AAe@ 100323e4     libucrt:winapi_thunks.obj
 0002:00010420       ??_C@_1DO@FPAPJEMD@?$AAa?$AAp?$AAi?$AA?9?$AAm?$AAs?$AA?9?$AAw?$AAi?$AAn?$AA?9?$AAc?$AAo?$AAr?$AAe@ 10032420     libucrt:winapi_thunks.obj
 0002:00010460       ??_C@_1DK@NDHNAHIO@?$AAa?$AAp?$AAi?$AA?9?$AAm?$AAs?$AA?9?$AAw?$AAi?$AAn?$AA?9?$AAc?$AAo?$AAr?$AAe@ 10032460     libucrt:winapi_thunks.obj
 0002:0001049c       ??_C@_1DM@KGHDGBCM@?$AAa?$AAp?$AAi?$AA?9?$AAm?$AAs?$AA?9?$AAw?$AAi?$AAn?$AA?9?$AAc?$AAo?$AAr?$AAe@ 1003249c     libucrt:winapi_thunks.obj
 0002:000104d8       ??_C@_1EO@IJIOEFOH@?$AAa?$AAp?$AAi?$AA?9?$AAm?$AAs?$AA?9?$AAw?$AAi?$AAn?$AA?9?$AAr?$AAt?$AAc?$AAo@ 100324d8     libucrt:winapi_thunks.obj
 0002:00010528       ??_C@_1FG@HHGEKANL@?$AAa?$AAp?$AAi?$AA?9?$AAm?$AAs?$AA?9?$AAw?$AAi?$AAn?$AA?9?$AAs?$AAe?$AAc?$AAu@ 10032528     libucrt:winapi_thunks.obj
 0002:00010580       ??_C@_1EG@DBIOJECG@?$AAe?$AAx?$AAt?$AA?9?$AAm?$AAs?$AA?9?$AAw?$AAi?$AAn?$AA?9?$AAn?$AAt?$AAu?$AAs@ 10032580     libucrt:winapi_thunks.obj
 0002:000105c8       ??_C@_1EO@FIHMJCLF@?$AAe?$AAx?$AAt?$AA?9?$AAm?$AAs?$AA?9?$AAw?$AAi?$AAn?$AA?9?$AAn?$AAt?$AAu?$AAs@ 100325c8     libucrt:winapi_thunks.obj
 0002:00010618       ??_C@_1BC@DNHGCMLG@?$AAa?$AAd?$AAv?$AAa?$AAp?$AAi?$AA3?$AA2@ 10032618     libucrt:winapi_thunks.obj
 0002:0001062c       ??_C@_1M@OAIMIKLP@?$AAn?$AAt?$AAd?$AAl?$AAl@ 1003262c     libucrt:winapi_thunks.obj
 0002:00010638       ??_C@_1EG@DPGNFKGC@?$AAa?$AAp?$AAi?$AA?9?$AAm?$AAs?$AA?9?$AAw?$AAi?$AAn?$AA?9?$AAa?$AAp?$AAp?$AAm@ 10032638     libucrt:winapi_thunks.obj
 0002:00010680       ??_C@_1O@BCCLBEOE@?$AAu?$AAs?$AAe?$AAr?$AA3?$AA2@ 10032680     libucrt:winapi_thunks.obj
 0002:00010690       ??_C@_1BA@IAIFMGEF@?$AAe?$AAx?$AAt?$AA?9?$AAm?$AAs?$AA?9@ 10032690     libucrt:winapi_thunks.obj
 0002:000106a4       ??_C@_0BA@FHFNEAED@AreFileApisANSI@ 100326a4     libucrt:winapi_thunks.obj
 0002:000106bc       ??_C@_0BA@IHGNDAEB@CompareStringEx@ 100326bc     libucrt:winapi_thunks.obj
 0002:000106fc       ??_C@_0O@KKBNKAPF@LCMapStringEx@ 100326fc     libucrt:winapi_thunks.obj
 0002:00010714       ??_C@_0BB@HBDEELFH@LocaleNameToLCID@ 10032714     libucrt:winapi_thunks.obj
 0002:0001072c       ??_C@_0N@PPOMPGGK@RoInitialize@ 1003272c     libucrt:winapi_thunks.obj
 0002:00010740       ??_C@_0P@LLFHBIJD@RoUninitialize@ 10032740     libucrt:winapi_thunks.obj
 0002:00010754       ??_C@_0CF@OJOFEIGO@AppPolicyGetProcessTerminationM@ 10032754     libucrt:winapi_thunks.obj
 0002:00010780       ??_C@_0CF@NNDFDCOC@AppPolicyGetThreadInitializatio@ 10032780     libucrt:winapi_thunks.obj
 0002:000107e8       ??_C@_03OEIAHPBN@INF@      100327e8     libucrt:cvt.obj
 0002:000107ec       ??_C@_03OJHLLCGB@inf@      100327ec     libucrt:cvt.obj
 0002:000107f0       ??_C@_03LKNCIKJB@NAN@      100327f0     libucrt:cvt.obj
 0002:000107f4       ??_C@_03LHCJEHON@nan@      100327f4     libucrt:cvt.obj
 0002:000107f8       ??_C@_09OFJJIMPC@NAN?$CISNAN?$CJ@ 100327f8     libucrt:cvt.obj
 0002:00010804       ??_C@_09IPFBKMDL@nan?$CIsnan?$CJ@ 10032804     libucrt:cvt.obj
 0002:00010810       ??_C@_08IKHNHAJ@NAN?$CIIND?$CJ@ 10032810     libucrt:cvt.obj
 0002:0001081c       ??_C@_08OFCDMILK@nan?$CIind?$CJ@ 1003281c     libucrt:cvt.obj
 0002:00010828       ??_C@_05KLBDPFGC@e?$CL000@ 10032828     libucrt:cvt.obj
 0002:00010830       ___lc_time_c               10032830     libucrt:nlsdata.obj
 0002:00010994       ??_C@_03KOEHGMDN@Sun@      10032994     libucrt:nlsdata.obj
 0002:00010998       ??_C@_03PDAGKDH@Mon@       10032998     libucrt:nlsdata.obj
 0002:0001099c       ??_C@_03NAGEINEP@Tue@      1003299c     libucrt:nlsdata.obj
 0002:000109a0       ??_C@_03MHOMLAJA@Wed@      100329a0     libucrt:nlsdata.obj
 0002:000109a4       ??_C@_03IOFIKPDN@Thu@      100329a4     libucrt:nlsdata.obj
 0002:000109a8       ??_C@_03IDIOELNC@Fri@      100329a8     libucrt:nlsdata.obj
 0002:000109ac       ??_C@_03FEFJNEK@Sat@       100329ac     libucrt:nlsdata.obj
 0002:000109b0       ??_C@_06OOPIFAJ@Sunday@    100329b0     libucrt:nlsdata.obj
 0002:000109b8       ??_C@_06JLEDEDGH@Monday@   100329b8     libucrt:nlsdata.obj
 0002:000109c0       ??_C@_07BAAGCFCM@Tuesday@  100329c0     libucrt:nlsdata.obj
 0002:000109c8       ??_C@_09DLIGFAKA@Wednesday@ 100329c8     libucrt:nlsdata.obj
 0002:000109d4       ??_C@_08HACCIKIA@Thursday@ 100329d4     libucrt:nlsdata.obj
 0002:000109e0       ??_C@_06JECMNKMI@Friday@   100329e0     libucrt:nlsdata.obj
 0002:000109e8       ??_C@_08INBOOONO@Saturday@ 100329e8     libucrt:nlsdata.obj
 0002:000109f4       ??_C@_03JIHJHPIE@Jan@      100329f4     libucrt:nlsdata.obj
 0002:000109f8       ??_C@_03HJBDCHOM@Feb@      100329f8     libucrt:nlsdata.obj
 0002:000109fc       ??_C@_03ODNJBKGA@Mar@      100329fc     libucrt:nlsdata.obj
 0002:00010a00       ??_C@_03LEOLGMJP@Apr@      10032a00     libucrt:nlsdata.obj
 0002:00010a04       ??_C@_03CNMDKL@May@        10032a04     libucrt:nlsdata.obj
 0002:00010a08       ??_C@_03IDFGHECI@Jun@      10032a08     libucrt:nlsdata.obj
 0002:00010a0c       ??_C@_03LBGABGKK@Jul@      10032a0c     libucrt:nlsdata.obj
 0002:00010a10       ??_C@_03IFJFEIGA@Aug@      10032a10     libucrt:nlsdata.obj
 0002:00010a14       ??_C@_03GGCAPAJC@Sep@      10032a14     libucrt:nlsdata.obj
 0002:00010a18       ??_C@_03BMAOKBAD@Oct@      10032a18     libucrt:nlsdata.obj
 0002:00010a1c       ??_C@_03JPJOFNIA@Nov@      10032a1c     libucrt:nlsdata.obj
 0002:00010a20       ??_C@_03MKABNOCG@Dec@      10032a20     libucrt:nlsdata.obj
 0002:00010a24       ??_C@_07CGJPFGJA@January@  10032a24     libucrt:nlsdata.obj
 0002:00010a2c       ??_C@_08GNJGEPFN@February@ 10032a2c     libucrt:nlsdata.obj
 0002:00010a38       ??_C@_05HPCKOFNC@March@    10032a38     libucrt:nlsdata.obj
 0002:00010a40       ??_C@_05DMJDNLEJ@April@    10032a40     libucrt:nlsdata.obj
 0002:00010a48       ??_C@_04CNLMGBGM@June@     10032a48     libucrt:nlsdata.obj
 0002:00010a50       ??_C@_04MIEPOIFP@July@     10032a50     libucrt:nlsdata.obj
 0002:00010a58       ??_C@_06LBBHFDDG@August@   10032a58     libucrt:nlsdata.obj
 0002:00010a60       ??_C@_09BHHEALKD@September@ 10032a60     libucrt:nlsdata.obj
 0002:00010a6c       ??_C@_07JJNFCEND@October@  10032a6c     libucrt:nlsdata.obj
 0002:00010a74       ??_C@_08HCHEGEOA@November@ 10032a74     libucrt:nlsdata.obj
 0002:00010a80       ??_C@_08EDHMEBNP@December@ 10032a80     libucrt:nlsdata.obj
 0002:00010a8c       ??_C@_02DEDBPAFC@AM@       10032a8c     libucrt:nlsdata.obj
 0002:00010a90       ??_C@_02CJNFDJBF@PM@       10032a90     libucrt:nlsdata.obj
 0002:00010a94       ??_C@_08BPBNCDIB@MM?1dd?1yy@ 10032a94     libucrt:nlsdata.obj
 0002:00010aa0       ??_C@_0BE@CKGJFCPC@dddd?0?5MMMM?5dd?0?5yyyy@ 10032aa0     libucrt:nlsdata.obj
 0002:00010ab4       ??_C@_08JCCMCCIL@HH?3mm?3ss@ 10032ab4     libucrt:nlsdata.obj
 0002:00010ac0       ??_C@_17MBGCMIPB@?$AAS?$AAu?$AAn@ 10032ac0     libucrt:nlsdata.obj
 0002:00010ac8       ??_C@_17KBOMKBF@?$AAM?$AAo?$AAn@ 10032ac8     libucrt:nlsdata.obj
 0002:00010ad0       ??_C@_17BMKGEGOJ@?$AAT?$AAu?$AAe@ 10032ad0     libucrt:nlsdata.obj
 0002:00010ad8       ??_C@_17CJEDCEPE@?$AAW?$AAe?$AAd@ 10032ad8     libucrt:nlsdata.obj
 0002:00010ae0       ??_C@_17PDPHAADD@?$AAT?$AAh?$AAu@ 10032ae0     libucrt:nlsdata.obj
 0002:00010ae8       ??_C@_17HFOLPPLP@?$AAF?$AAr?$AAi@ 10032ae8     libucrt:nlsdata.obj
 0002:00010af0       ??_C@_17GGIBDPIH@?$AAS?$AAa?$AAt@ 10032af0     libucrt:nlsdata.obj
 0002:00010af8       ??_C@_1O@IHNHDHPB@?$AAS?$AAu?$AAn?$AAd?$AAa?$AAy@ 10032af8     libucrt:nlsdata.obj
 0002:00010b08       ??_C@_1O@MMNBFLIA@?$AAM?$AAo?$AAn?$AAd?$AAa?$AAy@ 10032b08     libucrt:nlsdata.obj
 0002:00010b18       ??_C@_1BA@ENFBFFEK@?$AAT?$AAu?$AAe?$AAs?$AAd?$AAa?$AAy@ 10032b18     libucrt:nlsdata.obj
 0002:00010b28       ??_C@_1BE@EBOGMDOH@?$AAW?$AAe?$AAd?$AAn?$AAe?$AAs?$AAd?$AAa?$AAy@ 10032b28     libucrt:nlsdata.obj
 0002:00010b3c       ??_C@_1BC@HHMNLIHE@?$AAT?$AAh?$AAu?$AAr?$AAs?$AAd?$AAa?$AAy@ 10032b3c     libucrt:nlsdata.obj
 0002:00010b50       ??_C@_1O@PDICJHAG@?$AAF?$AAr?$AAi?$AAd?$AAa?$AAy@ 10032b50     libucrt:nlsdata.obj
 0002:00010b60       ??_C@_1BC@ENMNNPAJ@?$AAS?$AAa?$AAt?$AAu?$AAr?$AAd?$AAa?$AAy@ 10032b60     libucrt:nlsdata.obj
 0002:00010b74       ??_C@_17DKNBKCHM@?$AAJ?$AAa?$AAn@ 10032b74     libucrt:nlsdata.obj
 0002:00010b7c       ??_C@_17LMDJEKJN@?$AAF?$AAe?$AAb@ 10032b7c     libucrt:nlsdata.obj
 0002:00010b84       ??_C@_17CKNLEDEC@?$AAM?$AAa?$AAr@ 10032b84     libucrt:nlsdata.obj
 0002:00010b8c       ??_C@_17LFPOIHDD@?$AAA?$AAp?$AAr@ 10032b8c     libucrt:nlsdata.obj
 0002:00010b94       ??_C@_17PNNKMEED@?$AAM?$AAa?$AAy@ 10032b94     libucrt:nlsdata.obj
 0002:00010b9c       ??_C@_17KCJGOCPB@?$AAJ?$AAu?$AAn@ 10032b9c     libucrt:nlsdata.obj
 0002:00010ba4       ??_C@_17IJPCKHK@?$AAJ?$AAu?$AAl@ 10032ba4     libucrt:nlsdata.obj
 0002:00010bac       ??_C@_17ICPELBCN@?$AAA?$AAu?$AAg@ 10032bac     libucrt:nlsdata.obj
 0002:00010bb4       ??_C@_17HCHCOKMG@?$AAS?$AAe?$AAp@ 10032bb4     libucrt:nlsdata.obj
 0002:00010bbc       ??_C@_17FNLKOI@?$AAO?$AAc?$AAt@ 10032bbc     libucrt:nlsdata.obj
 0002:00010bc4       ??_C@_17BBDMLCIG@?$AAN?$AAo?$AAv@ 10032bc4     libucrt:nlsdata.obj
 0002:00010bcc       ??_C@_17EGKACKIF@?$AAD?$AAe?$AAc@ 10032bcc     libucrt:nlsdata.obj
 0002:00010bd4       ??_C@_1BA@EFMEIEBA@?$AAJ?$AAa?$AAn?$AAu?$AAa?$AAr?$AAy@ 10032bd4     libucrt:nlsdata.obj
 0002:00010be4       ??_C@_1BC@JGDDFFAM@?$AAF?$AAe?$AAb?$AAr?$AAu?$AAa?$AAr?$AAy@ 10032be4     libucrt:nlsdata.obj
 0002:00010bf8       ??_C@_1M@IKEENEDF@?$AAM?$AAa?$AAr?$AAc?$AAh@ 10032bf8     libucrt:nlsdata.obj
 0002:00010c04       ??_C@_1M@GJNLMHFD@?$AAA?$AAp?$AAr?$AAi?$AAl@ 10032c04     libucrt:nlsdata.obj
 0002:00010c10       ??_C@_19EPFLPGAP@?$AAJ?$AAu?$AAn?$AAe@ 10032c10     libucrt:nlsdata.obj
 0002:00010c1c       ??_C@_19BIFMLPCD@?$AAJ?$AAu?$AAl?$AAy@ 10032c1c     libucrt:nlsdata.obj
 0002:00010c28       ??_C@_1O@PAHLKOAC@?$AAA?$AAu?$AAg?$AAu?$AAs?$AAt@ 10032c28     libucrt:nlsdata.obj
 0002:00010c38       ??_C@_1BE@DKAAMBJL@?$AAS?$AAe?$AAp?$AAt?$AAe?$AAm?$AAb?$AAe?$AAr@ 10032c38     libucrt:nlsdata.obj
 0002:00010c4c       ??_C@_1BA@EPANDLNG@?$AAO?$AAc?$AAt?$AAo?$AAb?$AAe?$AAr@ 10032c4c     libucrt:nlsdata.obj
 0002:00010c5c       ??_C@_1BC@BGLIFPF@?$AAN?$AAo?$AAv?$AAe?$AAm?$AAb?$AAe?$AAr@ 10032c5c     libucrt:nlsdata.obj
 0002:00010c70       ??_C@_1BC@FEMKIFH@?$AAD?$AAe?$AAc?$AAe?$AAm?$AAb?$AAe?$AAr@ 10032c70     libucrt:nlsdata.obj
 0002:00010c84       ??_C@_15ODEHAHHF@?$AAA?$AAM@ 10032c84     libucrt:nlsdata.obj
 0002:00010c8c       ??_C@_15CLMNNGEL@?$AAP?$AAM@ 10032c8c     libucrt:nlsdata.obj
 0002:00010c94       ??_C@_1BC@IEBCMHCM@?$AAM?$AAM?$AA?1?$AAd?$AAd?$AA?1?$AAy?$AAy@ 10032c94     libucrt:nlsdata.obj
 0002:00010ca8       ??_C@_1CI@KNAKOEBC@?$AAd?$AAd?$AAd?$AAd?$AA?0?$AA?5?$AAM?$AAM?$AAM?$AAM?$AA?5?$AAd?$AAd?$AA?0?$AA?5@ 10032ca8     libucrt:nlsdata.obj
 0002:00010cd0       ??_C@_1BC@GDGBMEMK@?$AAH?$AAH?$AA?3?$AAm?$AAm?$AA?3?$AAs?$AAs@ 10032cd0     libucrt:nlsdata.obj
 0002:00010ce4       ??_C@_1M@BMHNFIME@?$AAe?$AAn?$AA?9?$AAU?$AAS@ 10032ce4     libucrt:nlsdata.obj
 0002:00010cf0       ?ccs@?1???$__acrt_stdio_parse_mode@D@@YA?AU__acrt_stdio_stream_mode@@QBD@Z@4QBDB 10032cf0     libucrt:openfile.obj
 0002:00010cf4       ?utf8_encoding@?1???$__acrt_stdio_parse_mode@D@@YA?AU__acrt_stdio_stream_mode@@QBD@Z@4QBDB 10032cf4     libucrt:openfile.obj
 0002:00010cfc       ?utf16_encoding@?1???$__acrt_stdio_parse_mode@D@@YA?AU__acrt_stdio_stream_mode@@QBD@Z@4QBDB 10032cfc     libucrt:openfile.obj
 0002:00010d04       ?unicode_encoding@?1???$__acrt_stdio_parse_mode@D@@YA?AU__acrt_stdio_stream_mode@@QBD@Z@4QBDB 10032d04     libucrt:openfile.obj
 0002:00010d1c       ??_C@_1M@HPNHIDJI@?$AAj?$AAa?$AA?9?$AAJ?$AAP@ 10032d1c     libucrt:mbctype.obj
 0002:00010d28       ??_C@_1M@BIBDDEMK@?$AAz?$AAh?$AA?9?$AAC?$AAN@ 10032d28     libucrt:mbctype.obj
 0002:00010d34       ??_C@_1M@JLOOOEGK@?$AAk?$AAo?$AA?9?$AAK?$AAR@ 10032d34     libucrt:mbctype.obj
 0002:00010d40       ??_C@_1M@CLNBBOPM@?$AAz?$AAh?$AA?9?$AAT?$AAW@ 10032d40     libucrt:mbctype.obj
 0002:00010d50       ___newctype                10032d50     libucrt:ctype.obj
 0002:00011050       ___newclmap                10033050     libucrt:ctype.obj
 0002:000111d0       ___newcumap                100331d0     libucrt:ctype.obj
 0002:00011350       __wctype                   10033350     libucrt:ctype.obj
 0002:00011c78       ??_C@_15EMKDOKLE@?$AAa?$AAr@ 10033c78     libucrt:lcidtoname_downlevel.obj
 0002:00011c80       ??_C@_15KNPADPLH@?$AAb?$AAg@ 10033c80     libucrt:lcidtoname_downlevel.obj
 0002:00011c88       ??_C@_15EDMHLDMO@?$AAc?$AAa@ 10033c88     libucrt:lcidtoname_downlevel.obj
 0002:00011c90       ??_C@_1O@BPEAJADD@?$AAz?$AAh?$AA?9?$AAC?$AAH?$AAS@ 10033c90     libucrt:lcidtoname_downlevel.obj
 0002:00011ca0       ??_C@_15LJNHCMNK@?$AAc?$AAs@ 10033ca0     libucrt:lcidtoname_downlevel.obj
 0002:00011ca8       ??_C@_15FOMCIDHG@?$AAd?$AAa@ 10033ca8     libucrt:lcidtoname_downlevel.obj
 0002:00011cb0       ??_C@_15NBKABECB@?$AAd?$AAe@ 10033cb0     libucrt:lcidtoname_downlevel.obj
 0002:00011cb8       ??_C@_15GHPEIIAO@?$AAe?$AAl@ 10033cb8     libucrt:lcidtoname_downlevel.obj
 0002:00011cc0       ??_C@_15MNPNEAIF@?$AAe?$AAn@ 10033cc0     libucrt:lcidtoname_downlevel.obj
 0002:00011cc8       ??_C@_15GPIOMPMH@?$AAe?$AAs@ 10033cc8     libucrt:lcidtoname_downlevel.obj
 0002:00011cd0       ??_C@_15NGLOAKJC@?$AAf?$AAi@ 10033cd0     libucrt:lcidtoname_downlevel.obj
 0002:00011cd8       ??_C@_15FBKGNKAM@?$AAf?$AAr@ 10033cd8     libucrt:lcidtoname_downlevel.obj
 0002:00011ce0       ??_C@_15KGGCNEFK@?$AAh?$AAe@ 10033ce0     libucrt:lcidtoname_downlevel.obj
 0002:00011ce8       ??_C@_15PGHLIDMF@?$AAh?$AAu@ 10033ce8     libucrt:lcidtoname_downlevel.obj
 0002:00011cf0       ??_C@_15BIEMAPLM@?$AAi?$AAs@ 10033cf0     libucrt:lcidtoname_downlevel.obj
 0002:00011cf8       ??_C@_15IFJLDHAF@?$AAi?$AAt@ 10033cf8     libucrt:lcidtoname_downlevel.obj
 0002:00011d00       ??_C@_15GEMIOCAG@?$AAj?$AAa@ 10033d00     libucrt:lcidtoname_downlevel.obj
 0002:00011d08       ??_C@_15EPELEGJA@?$AAk?$AAo@ 10033d08     libucrt:lcidtoname_downlevel.obj
 0002:00011d10       ??_C@_15NDDHIMN@?$AAn?$AAl@ 10033d10     libucrt:lcidtoname_downlevel.obj
 0002:00011d18       ??_C@_15BPIGNHCD@?$AAn?$AAo@ 10033d18     libucrt:lcidtoname_downlevel.obj
 0002:00011d20       ??_C@_15DEOPBLCG@?$AAp?$AAl@ 10033d20     libucrt:lcidtoname_downlevel.obj
 0002:00011d28       ??_C@_15KBECGEFG@?$AAp?$AAt@ 10033d28     libucrt:lcidtoname_downlevel.obj
 0002:00011d30       ??_C@_15GLJCBFMD@?$AAr?$AAo@ 10033d30     libucrt:lcidtoname_downlevel.obj
 0002:00011d38       ??_C@_15FEDGKCDI@?$AAr?$AAu@ 10033d38     libucrt:lcidtoname_downlevel.obj
 0002:00011d40       ??_C@_15GLKMLLHM@?$AAh?$AAr@ 10033d40     libucrt:lcidtoname_downlevel.obj
 0002:00011d48       ??_C@_15CPKMFBDB@?$AAs?$AAk@ 10033d48     libucrt:lcidtoname_downlevel.obj
 0002:00011d50       ??_C@_15BAAIOGMK@?$AAs?$AAq@ 10033d50     libucrt:lcidtoname_downlevel.obj
 0002:00011d58       ??_C@_15INNPNOHD@?$AAs?$AAv@ 10033d58     libucrt:lcidtoname_downlevel.obj
 0002:00011d60       ??_C@_15CABMMOGH@?$AAt?$AAh@ 10033d60     libucrt:lcidtoname_downlevel.obj
 0002:00011d68       ??_C@_15BPLIHJJM@?$AAt?$AAr@ 10033d68     libucrt:lcidtoname_downlevel.obj
 0002:00011d70       ??_C@_15NEOEKKDJ@?$AAu?$AAr@ 10033d70     libucrt:lcidtoname_downlevel.obj
 0002:00011d78       ??_C@_15NFICGAJK@?$AAi?$AAd@ 10033d78     libucrt:lcidtoname_downlevel.obj
 0002:00011d80       ??_C@_15PJPFLCCM@?$AAu?$AAk@ 10033d80     libucrt:lcidtoname_downlevel.obj
 0002:00011d88       ??_C@_15HPJPHDM@?$AAb?$AAe@ 10033d88     libucrt:lcidtoname_downlevel.obj
 0002:00011d90       ??_C@_15LCHLGJII@?$AAs?$AAl@ 10033d90     libucrt:lcidtoname_downlevel.obj
 0002:00011d98       ??_C@_15PCFJPHHO@?$AAe?$AAt@ 10033d98     libucrt:lcidtoname_downlevel.obj
 0002:00011da0       ??_C@_15HPFPGODN@?$AAl?$AAv@ 10033da0     libucrt:lcidtoname_downlevel.obj
 0002:00011da8       ??_C@_15NFFGKGLG@?$AAl?$AAt@ 10033da8     libucrt:lcidtoname_downlevel.obj
 0002:00011db0       ??_C@_15BDAKCCHN@?$AAf?$AAa@ 10033db0     libucrt:lcidtoname_downlevel.obj
 0002:00011db8       ??_C@_15NFGIAIAJ@?$AAv?$AAi@ 10033db8     libucrt:lcidtoname_downlevel.obj
 0002:00011dc0       ??_C@_15LMKNDMHN@?$AAh?$AAy@ 10033dc0     libucrt:lcidtoname_downlevel.obj
 0002:00011dc8       ??_C@_15IJBHMCFL@?$AAa?$AAz@ 10033dc8     libucrt:lcidtoname_downlevel.obj
 0002:00011dd0       ??_C@_15EKOFJABL@?$AAe?$AAu@ 10033dd0     libucrt:lcidtoname_downlevel.obj
 0002:00011dd8       ??_C@_15BGHADCNK@?$AAm?$AAk@ 10033dd8     libucrt:lcidtoname_downlevel.obj
 0002:00011de0       ??_C@_15JDNICKHM@?$AAa?$AAf@ 10033de0     libucrt:lcidtoname_downlevel.obj
 0002:00011de8       ??_C@_15KPJEDBKD@?$AAk?$AAa@ 10033de8     libucrt:lcidtoname_downlevel.obj
 0002:00011df0       ??_C@_15PDNFFFEO@?$AAf?$AAo@ 10033df0     libucrt:lcidtoname_downlevel.obj
 0002:00011df8       ??_C@_15OMLEGLOC@?$AAh?$AAi@ 10033df8     libucrt:lcidtoname_downlevel.obj
 0002:00011e00       ??_C@_15IDNNENKK@?$AAm?$AAs@ 10033e00     libucrt:lcidtoname_downlevel.obj
 0002:00011e08       ??_C@_15MACJNBMH@?$AAk?$AAk@ 10033e08     libucrt:lcidtoname_downlevel.obj
 0002:00011e10       ??_C@_15DKDJEOND@?$AAk?$AAy@ 10033e10     libucrt:lcidtoname_downlevel.obj
 0002:00011e18       ??_C@_15DFGDLJBG@?$AAs?$AAw@ 10033e18     libucrt:lcidtoname_downlevel.obj
 0002:00011e20       ??_C@_15BBFAICNG@?$AAu?$AAz@ 10033e20     libucrt:lcidtoname_downlevel.obj
 0002:00011e28       ??_C@_15DKNDCGEA@?$AAt?$AAt@ 10033e28     libucrt:lcidtoname_downlevel.obj
 0002:00011e30       ??_C@_15MGIFMDPL@?$AAp?$AAa@ 10033e30     libucrt:lcidtoname_downlevel.obj
 0002:00011e38       ??_C@_15HCNDBBA@?$AAg?$AAu@ 10033e38     libucrt:lcidtoname_downlevel.obj
 0002:00011e40       ??_C@_15FNBEIBON@?$AAt?$AAa@ 10033e40     libucrt:lcidtoname_downlevel.obj
 0002:00011e48       ??_C@_15NCHGBGLK@?$AAt?$AAe@ 10033e48     libucrt:lcidtoname_downlevel.obj
 0002:00011e50       ??_C@_15PHPHCBPF@?$AAk?$AAn@ 10033e50     libucrt:lcidtoname_downlevel.obj
 0002:00011e58       ??_C@_15DLGBCKMP@?$AAm?$AAr@ 10033e58     libucrt:lcidtoname_downlevel.obj
 0002:00011e60       ??_C@_15EABBLBFF@?$AAs?$AAa@ 10033e60     libucrt:lcidtoname_downlevel.obj
 0002:00011e68       ??_C@_15CBKOMCOI@?$AAm?$AAn@ 10033e68     libucrt:lcidtoname_downlevel.obj
 0002:00011e70       ??_C@_15CKDMCJAF@?$AAg?$AAl@ 10033e70     libucrt:lcidtoname_downlevel.obj
 0002:00011e78       ??_C@_17CNJFBPG@?$AAk?$AAo?$AAk@ 10033e78     libucrt:lcidtoname_downlevel.obj
 0002:00011e80       ??_C@_17FFBJICPL@?$AAs?$AAy?$AAr@ 10033e80     libucrt:lcidtoname_downlevel.obj
 0002:00011e88       ??_C@_17KPNDCPAF@?$AAd?$AAi?$AAv@ 10033e88     libucrt:lcidtoname_downlevel.obj
 0002:00011e90       ??_C@_11LOCGONAA@@         10033e90     libucrt:lcidtoname_downlevel.obj
 0002:00011e94       ??_C@_1M@OKAHONE@?$AAa?$AAr?$AA?9?$AAS?$AAA@ 10033e94     libucrt:lcidtoname_downlevel.obj
 0002:00011ea0       ??_C@_1M@FFFIGIGK@?$AAb?$AAg?$AA?9?$AAB?$AAG@ 10033ea0     libucrt:lcidtoname_downlevel.obj
 0002:00011eac       ??_C@_1M@BJNKEDC@?$AAc?$AAa?$AA?9?$AAE?$AAS@ 10033eac     libucrt:lcidtoname_downlevel.obj
 0002:00011eb8       ??_C@_1M@IJJHFJHA@?$AAc?$AAs?$AA?9?$AAC?$AAZ@ 10033eb8     libucrt:lcidtoname_downlevel.obj
 0002:00011ec4       ??_C@_1M@CLPEOBGI@?$AAd?$AAa?$AA?9?$AAD?$AAK@ 10033ec4     libucrt:lcidtoname_downlevel.obj
 0002:00011ed0       ??_C@_1M@MCMADGCB@?$AAd?$AAe?$AA?9?$AAD?$AAE@ 10033ed0     libucrt:lcidtoname_downlevel.obj
 0002:00011edc       ??_C@_1M@OOCKEMAM@?$AAe?$AAl?$AA?9?$AAG?$AAR@ 10033edc     libucrt:lcidtoname_downlevel.obj
 0002:00011ee8       ??_C@_1M@DDNJFGID@?$AAf?$AAi?$AA?9?$AAF?$AAI@ 10033ee8     libucrt:lcidtoname_downlevel.obj
 0002:00011ef4       ??_C@_1M@GLIPPMAC@?$AAf?$AAr?$AA?9?$AAF?$AAR@ 10033ef4     libucrt:lcidtoname_downlevel.obj
 0002:00011f00       ??_C@_1M@GFMCHPE@?$AAh?$AAe?$AA?9?$AAI?$AAL@ 10033f00     libucrt:lcidtoname_downlevel.obj
 0002:00011f0c       ??_C@_1M@MHLPGNKM@?$AAh?$AAu?$AA?9?$AAH?$AAU@ 10033f0c     libucrt:lcidtoname_downlevel.obj
 0002:00011f18       ??_C@_1M@LPDDNNPN@?$AAi?$AAs?$AA?9?$AAI?$AAS@ 10033f18     libucrt:lcidtoname_downlevel.obj
 0002:00011f24       ??_C@_1M@MADIPODN@?$AAi?$AAt?$AA?9?$AAI?$AAT@ 10033f24     libucrt:lcidtoname_downlevel.obj
 0002:00011f30       ??_C@_1M@IHBJJGG@?$AAn?$AAl?$AA?9?$AAN?$AAL@ 10033f30     libucrt:lcidtoname_downlevel.obj
 0002:00011f3c       ??_C@_1M@EANAGDL@?$AAn?$AAb?$AA?9?$AAN?$AAO@ 10033f3c     libucrt:lcidtoname_downlevel.obj
 0002:00011f48       ??_C@_1M@NEIEMEGP@?$AAp?$AAl?$AA?9?$AAP?$AAL@ 10033f48     libucrt:lcidtoname_downlevel.obj
 0002:00011f54       ??_C@_1M@BOCFIGEP@?$AAp?$AAt?$AA?9?$AAB?$AAR@ 10033f54     libucrt:lcidtoname_downlevel.obj
 0002:00011f60       ??_C@_1M@IMPFOPBG@?$AAr?$AAo?$AA?9?$AAR?$AAO@ 10033f60     libucrt:lcidtoname_downlevel.obj
 0002:00011f6c       ??_C@_1M@IDNNEJMM@?$AAr?$AAu?$AA?9?$AAR?$AAU@ 10033f6c     libucrt:lcidtoname_downlevel.obj
 0002:00011f78       ??_C@_1M@LILEEOGM@?$AAh?$AAr?$AA?9?$AAH?$AAR@ 10033f78     libucrt:lcidtoname_downlevel.obj
 0002:00011f84       ??_C@_1M@FKIFEHPB@?$AAs?$AAk?$AA?9?$AAS?$AAK@ 10033f84     libucrt:lcidtoname_downlevel.obj
 0002:00011f90       ??_C@_1M@LJMAMNPJ@?$AAs?$AAq?$AA?9?$AAA?$AAL@ 10033f90     libucrt:lcidtoname_downlevel.obj
 0002:00011f9c       ??_C@_1M@GIAKDKJK@?$AAs?$AAv?$AA?9?$AAS?$AAE@ 10033f9c     libucrt:lcidtoname_downlevel.obj
 0002:00011fa8       ??_C@_1M@MKJKIKCL@?$AAt?$AAh?$AA?9?$AAT?$AAH@ 10033fa8     libucrt:lcidtoname_downlevel.obj
 0002:00011fb4       ??_C@_1M@MFLCCMPB@?$AAt?$AAr?$AA?9?$AAT?$AAR@ 10033fb4     libucrt:lcidtoname_downlevel.obj
 0002:00011fc0       ??_C@_1M@OIJHDKJN@?$AAu?$AAr?$AA?9?$AAP?$AAK@ 10033fc0     libucrt:lcidtoname_downlevel.obj
 0002:00011fcc       ??_C@_1M@LHIPCIEK@?$AAi?$AAd?$AA?9?$AAI?$AAD@ 10033fcc     libucrt:lcidtoname_downlevel.obj
 0002:00011fd8       ??_C@_1M@MFMOBGI@?$AAu?$AAk?$AA?9?$AAU?$AAA@ 10033fd8     libucrt:lcidtoname_downlevel.obj
 0002:00011fe4       ??_C@_1M@OBGLJIPL@?$AAb?$AAe?$AA?9?$AAB?$AAY@ 10033fe4     libucrt:lcidtoname_downlevel.obj
 0002:00011ff0       ??_C@_1M@BCFAJEAD@?$AAs?$AAl?$AA?9?$AAS?$AAI@ 10033ff0     libucrt:lcidtoname_downlevel.obj
 0002:00011ffc       ??_C@_1M@FKFFEDDN@?$AAe?$AAt?$AA?9?$AAE?$AAE@ 10033ffc     libucrt:lcidtoname_downlevel.obj
 0002:00012008       ??_C@_1M@KGKKAACI@?$AAl?$AAv?$AA?9?$AAL?$AAV@ 10034008     libucrt:lcidtoname_downlevel.obj
 0002:00012014       ??_C@_1M@IFGBIJO@?$AAl?$AAt?$AA?9?$AAL?$AAT@ 10034014     libucrt:lcidtoname_downlevel.obj
 0002:00012020       ??_C@_1M@FGEAHEDM@?$AAf?$AAa?$AA?9?$AAI?$AAR@ 10034020     libucrt:lcidtoname_downlevel.obj
 0002:0001202c       ??_C@_1M@KBMAIBFN@?$AAv?$AAi?$AA?9?$AAV?$AAN@ 1003402c     libucrt:lcidtoname_downlevel.obj
 0002:00012038       ??_C@_1M@GPCBKDJK@?$AAh?$AAy?$AA?9?$AAA?$AAM@ 10034038     libucrt:lcidtoname_downlevel.obj
 0002:00012044       ??_C@_1BG@BECMDDJB@?$AAa?$AAz?$AA?9?$AAA?$AAZ?$AA?9?$AAL?$AAa?$AAt?$AAn@ 10034044     libucrt:lcidtoname_downlevel.obj
 0002:0001205c       ??_C@_1M@MAOFCAEA@?$AAe?$AAu?$AA?9?$AAE?$AAS@ 1003405c     libucrt:lcidtoname_downlevel.obj
 0002:00012068       ??_C@_1M@IGHABKPI@?$AAm?$AAk?$AA?9?$AAM?$AAK@ 10034068     libucrt:lcidtoname_downlevel.obj
 0002:00012074       ??_C@_1M@IAIGNEJG@?$AAt?$AAn?$AA?9?$AAZ?$AAA@ 10034074     libucrt:lcidtoname_downlevel.obj
 0002:00012080       ??_C@_1M@IIJCOJFA@?$AAx?$AAh?$AA?9?$AAZ?$AAA@ 10034080     libucrt:lcidtoname_downlevel.obj
 0002:0001208c       ??_C@_1M@LGPJHNJH@?$AAz?$AAu?$AA?9?$AAZ?$AAA@ 1003408c     libucrt:lcidtoname_downlevel.obj
 0002:00012098       ??_C@_1M@HOKAOIO@?$AAa?$AAf?$AA?9?$AAZ?$AAA@ 10034098     libucrt:lcidtoname_downlevel.obj
 0002:000120a4       ??_C@_1M@DPCLHLIE@?$AAk?$AAa?$AA?9?$AAG?$AAE@ 100340a4     libucrt:lcidtoname_downlevel.obj
 0002:000120b0       ??_C@_1M@BLKMHJBI@?$AAf?$AAo?$AA?9?$AAF?$AAO@ 100340b0     libucrt:lcidtoname_downlevel.obj
 0002:000120bc       ??_C@_1M@LGGJAPPB@?$AAh?$AAi?$AA?9?$AAI?$AAN@ 100340bc     libucrt:lcidtoname_downlevel.obj
 0002:000120c8       ??_C@_1M@FIKPIHFE@?$AAm?$AAt?$AA?9?$AAM?$AAT@ 100340c8     libucrt:lcidtoname_downlevel.obj
 0002:000120d4       ??_C@_1M@HEGGPBFA@?$AAs?$AAe?$AA?9?$AAN?$AAO@ 100340d4     libucrt:lcidtoname_downlevel.obj
 0002:000120e0       ??_C@_1M@EIBJEEPA@?$AAm?$AAs?$AA?9?$AAM?$AAY@ 100340e0     libucrt:lcidtoname_downlevel.obj
 0002:000120ec       ??_C@_1M@FHLBGMPP@?$AAk?$AAk?$AA?9?$AAK?$AAZ@ 100340ec     libucrt:lcidtoname_downlevel.obj
 0002:000120f8       ??_C@_1M@NGJJLCGI@?$AAk?$AAy?$AA?9?$AAK?$AAG@ 100340f8     libucrt:lcidtoname_downlevel.obj
 0002:00012104       ??_C@_1M@GIENNBFC@?$AAs?$AAw?$AA?9?$AAK?$AAE@ 10034104     libucrt:lcidtoname_downlevel.obj
 0002:00012110       ??_C@_1BG@NDGMJIMJ@?$AAu?$AAz?$AA?9?$AAU?$AAZ?$AA?9?$AAL?$AAa?$AAt?$AAn@ 10034110     libucrt:lcidtoname_downlevel.obj
 0002:00012128       ??_C@_1M@IDCCIHBC@?$AAt?$AAt?$AA?9?$AAR?$AAU@ 10034128     libucrt:lcidtoname_downlevel.obj
 0002:00012134       ??_C@_1M@LOICPMOJ@?$AAb?$AAn?$AA?9?$AAI?$AAN@ 10034134     libucrt:lcidtoname_downlevel.obj
 0002:00012140       ??_C@_1M@KPKKNEAH@?$AAp?$AAa?$AA?9?$AAI?$AAN@ 10034140     libucrt:lcidtoname_downlevel.obj
 0002:0001214c       ??_C@_1M@PJGPPBOG@?$AAg?$AAu?$AA?9?$AAI?$AAN@ 1003414c     libucrt:lcidtoname_downlevel.obj
 0002:00012158       ??_C@_1M@KMKMOPHI@?$AAt?$AAa?$AA?9?$AAI?$AAN@ 10034158     libucrt:lcidtoname_downlevel.obj
 0002:00012164       ??_C@_1M@KFEHEPAC@?$AAt?$AAe?$AA?9?$AAI?$AAN@ 10034164     libucrt:lcidtoname_downlevel.obj
 0002:00012170       ??_C@_1M@CDCLMGHI@?$AAk?$AAn?$AA?9?$AAI?$AAN@ 10034170     libucrt:lcidtoname_downlevel.obj
 0002:0001217c       ??_C@_1M@MIODLDKF@?$AAm?$AAl?$AA?9?$AAI?$AAN@ 1003417c     libucrt:lcidtoname_downlevel.obj
 0002:00012188       ??_C@_1M@PBIEACPO@?$AAm?$AAr?$AA?9?$AAI?$AAN@ 10034188     libucrt:lcidtoname_downlevel.obj
 0002:00012194       ??_C@_1M@NIDEAGPH@?$AAs?$AAa?$AA?9?$AAI?$AAN@ 10034194     libucrt:lcidtoname_downlevel.obj
 0002:000121a0       ??_C@_1M@FHIHCBIO@?$AAm?$AAn?$AA?9?$AAM?$AAN@ 100341a0     libucrt:lcidtoname_downlevel.obj
 0002:000121ac       ??_C@_1M@JAIJPENP@?$AAc?$AAy?$AA?9?$AAG?$AAB@ 100341ac     libucrt:lcidtoname_downlevel.obj
 0002:000121b8       ??_C@_1M@PHGFBEPN@?$AAg?$AAl?$AA?9?$AAE?$AAS@ 100341b8     libucrt:lcidtoname_downlevel.obj
 0002:000121c4       ??_C@_1O@KPIPDNCP@?$AAk?$AAo?$AAk?$AA?9?$AAI?$AAN@ 100341c4     libucrt:lcidtoname_downlevel.obj
 0002:000121d4       ??_C@_1O@KNHJLDJA@?$AAs?$AAy?$AAr?$AA?9?$AAS?$AAY@ 100341d4     libucrt:lcidtoname_downlevel.obj
 0002:000121e4       ??_C@_1O@MKEKBLAH@?$AAd?$AAi?$AAv?$AA?9?$AAM?$AAV@ 100341e4     libucrt:lcidtoname_downlevel.obj
 0002:000121f4       ??_C@_1O@OHDCKDDF@?$AAq?$AAu?$AAz?$AA?9?$AAB?$AAO@ 100341f4     libucrt:lcidtoname_downlevel.obj
 0002:00012204       ??_C@_1M@LEPJNLFD@?$AAn?$AAs?$AA?9?$AAZ?$AAA@ 10034204     libucrt:lcidtoname_downlevel.obj
 0002:00012210       ??_C@_1M@OMLEIIJB@?$AAm?$AAi?$AA?9?$AAN?$AAZ@ 10034210     libucrt:lcidtoname_downlevel.obj
 0002:0001221c       ??_C@_1M@PMPEAILG@?$AAa?$AAr?$AA?9?$AAI?$AAQ@ 1003421c     libucrt:lcidtoname_downlevel.obj
 0002:00012228       ??_C@_1M@CNKPNOEE@?$AAd?$AAe?$AA?9?$AAC?$AAH@ 10034228     libucrt:lcidtoname_downlevel.obj
 0002:00012234       ??_C@_1M@LKMGMLKO@?$AAe?$AAn?$AA?9?$AAG?$AAB@ 10034234     libucrt:lcidtoname_downlevel.obj
 0002:00012240       ??_C@_1M@PGKJFFGL@?$AAe?$AAs?$AA?9?$AAM?$AAX@ 10034240     libucrt:lcidtoname_downlevel.obj
 0002:0001224c       ??_C@_1M@DNNANBDC@?$AAf?$AAr?$AA?9?$AAB?$AAE@ 1003424c     libucrt:lcidtoname_downlevel.obj
 0002:00012258       ??_C@_1M@HLGMDFHM@?$AAi?$AAt?$AA?9?$AAC?$AAH@ 10034258     libucrt:lcidtoname_downlevel.obj
 0002:00012264       ??_C@_1M@CLLBGJH@?$AAn?$AAl?$AA?9?$AAB?$AAE@ 10034264     libucrt:lcidtoname_downlevel.obj
 0002:00012270       ??_C@_1M@BODBOGLF@?$AAn?$AAn?$AA?9?$AAN?$AAO@ 10034270     libucrt:lcidtoname_downlevel.obj
 0002:0001227c       ??_C@_1M@HFFAHKAD@?$AAp?$AAt?$AA?9?$AAP?$AAT@ 1003427c     libucrt:lcidtoname_downlevel.obj
 0002:00012288       ??_C@_1BG@LNOAKHIE@?$AAs?$AAr?$AA?9?$AAS?$AAP?$AA?9?$AAL?$AAa?$AAt?$AAn@ 10034288     libucrt:lcidtoname_downlevel.obj
 0002:000122a0       ??_C@_1M@HBMHBGAK@?$AAs?$AAv?$AA?9?$AAF?$AAI@ 100342a0     libucrt:lcidtoname_downlevel.obj
 0002:000122ac       ??_C@_1BG@DGCJGJBE@?$AAa?$AAz?$AA?9?$AAA?$AAZ?$AA?9?$AAC?$AAy?$AAr?$AAl@ 100342ac     libucrt:lcidtoname_downlevel.obj
 0002:000122c4       ??_C@_1M@KEJDAAHB@?$AAs?$AAe?$AA?9?$AAS?$AAE@ 100342c4     libucrt:lcidtoname_downlevel.obj
 0002:000122d0       ??_C@_1M@HEIBJJAD@?$AAm?$AAs?$AA?9?$AAB?$AAN@ 100342d0     libucrt:lcidtoname_downlevel.obj
 0002:000122dc       ??_C@_1BG@PBGJMCEM@?$AAu?$AAz?$AA?9?$AAU?$AAZ?$AA?9?$AAC?$AAy?$AAr?$AAl@ 100342dc     libucrt:lcidtoname_downlevel.obj
 0002:000122f4       ??_C@_1O@LAOBCMDF@?$AAq?$AAu?$AAz?$AA?9?$AAE?$AAC@ 100342f4     libucrt:lcidtoname_downlevel.obj
 0002:00012304       ??_C@_1M@POEEMAIO@?$AAa?$AAr?$AA?9?$AAE?$AAG@ 10034304     libucrt:lcidtoname_downlevel.obj
 0002:00012310       ??_C@_1M@EFAKDEDL@?$AAz?$AAh?$AA?9?$AAH?$AAK@ 10034310     libucrt:lcidtoname_downlevel.obj
 0002:0001231c       ??_C@_1M@HKKIJHGI@?$AAd?$AAe?$AA?9?$AAA?$AAT@ 1003431c     libucrt:lcidtoname_downlevel.obj
 0002:00012328       ??_C@_1M@KBFBEHJF@?$AAe?$AAn?$AA?9?$AAA?$AAU@ 10034328     libucrt:lcidtoname_downlevel.obj
 0002:00012334       ??_C@_1M@MNPLFAAH@?$AAe?$AAs?$AA?9?$AAE?$AAS@ 10034334     libucrt:lcidtoname_downlevel.obj
 0002:00012340       ??_C@_1M@HJOOJFMA@?$AAf?$AAr?$AA?9?$AAC?$AAA@ 10034340     libucrt:lcidtoname_downlevel.obj
 0002:0001234c       ??_C@_1BG@JPOFPNAB@?$AAs?$AAr?$AA?9?$AAS?$AAP?$AA?9?$AAC?$AAy?$AAr?$AAl@ 1003434c     libucrt:lcidtoname_downlevel.obj
 0002:00012364       ??_C@_1M@LNFOCMOB@?$AAs?$AAe?$AA?9?$AAF?$AAI@ 10034364     libucrt:lcidtoname_downlevel.obj
 0002:00012370       ??_C@_1O@MGJBOAMB@?$AAq?$AAu?$AAz?$AA?9?$AAP?$AAE@ 10034370     libucrt:lcidtoname_downlevel.obj
 0002:00012380       ??_C@_1M@GJINLBOK@?$AAa?$AAr?$AA?9?$AAL?$AAY@ 10034380     libucrt:lcidtoname_downlevel.obj
 0002:0001238c       ??_C@_1M@GGMNHJNL@?$AAz?$AAh?$AA?9?$AAS?$AAG@ 1003438c     libucrt:lcidtoname_downlevel.obj
 0002:00012398       ??_C@_1M@HOIKODND@?$AAd?$AAe?$AA?9?$AAL?$AAU@ 10034398     libucrt:lcidtoname_downlevel.obj
 0002:000123a4       ??_C@_1M@DDOCCGFG@?$AAe?$AAn?$AA?9?$AAC?$AAA@ 100343a4     libucrt:lcidtoname_downlevel.obj
 0002:000123b0       ??_C@_1M@BNOEMJLF@?$AAe?$AAs?$AA?9?$AAG?$AAT@ 100343b0     libucrt:lcidtoname_downlevel.obj
 0002:000123bc       ??_C@_1M@EOGNKEK@?$AAf?$AAr?$AA?9?$AAC?$AAH@ 100343bc     libucrt:lcidtoname_downlevel.obj
 0002:000123c8       ??_C@_1M@FLIDJFHL@?$AAh?$AAr?$AA?9?$AAB?$AAA@ 100343c8     libucrt:lcidtoname_downlevel.obj
 0002:000123d4       ??_C@_1O@FMCELNAJ@?$AAs?$AAm?$AAj?$AA?9?$AAN?$AAO@ 100343d4     libucrt:lcidtoname_downlevel.obj
 0002:000123e4       ??_C@_1M@JHGLJMGJ@?$AAa?$AAr?$AA?9?$AAD?$AAZ@ 100343e4     libucrt:lcidtoname_downlevel.obj
 0002:000123f0       ??_C@_1M@JKKFDCNP@?$AAz?$AAh?$AA?9?$AAM?$AAO@ 100343f0     libucrt:lcidtoname_downlevel.obj
 0002:000123fc       ??_C@_1M@GEEFALPE@?$AAd?$AAe?$AA?9?$AAL?$AAI@ 100343fc     libucrt:lcidtoname_downlevel.obj
 0002:00012408       ??_C@_1M@IGEOFBG@?$AAe?$AAn?$AA?9?$AAN?$AAZ@ 10034408     libucrt:lcidtoname_downlevel.obj
 0002:00012414       ??_C@_1M@KDBONEHP@?$AAe?$AAs?$AA?9?$AAC?$AAR@ 10034414     libucrt:lcidtoname_downlevel.obj
 0002:00012420       ??_C@_1M@FHMDOHNN@?$AAf?$AAr?$AA?9?$AAL?$AAU@ 10034420     libucrt:lcidtoname_downlevel.obj
 0002:0001242c       ??_C@_1BG@NFKKMAFG@?$AAb?$AAs?$AA?9?$AAB?$AAA?$AA?9?$AAL?$AAa?$AAt?$AAn@ 1003442c     libucrt:lcidtoname_downlevel.obj
 0002:00012444       ??_C@_1O@IMNBEMCI@?$AAs?$AAm?$AAj?$AA?9?$AAS?$AAE@ 10034444     libucrt:lcidtoname_downlevel.obj
 0002:00012454       ??_C@_1M@DHHMBNDP@?$AAa?$AAr?$AA?9?$AAM?$AAA@ 10034454     libucrt:lcidtoname_downlevel.obj
 0002:00012460       ??_C@_1M@BNBLJCGH@?$AAe?$AAn?$AA?9?$AAI?$AAE@ 10034460     libucrt:lcidtoname_downlevel.obj
 0002:0001246c       ??_C@_1M@GEPAFMDL@?$AAe?$AAs?$AA?9?$AAP?$AAA@ 1003446c     libucrt:lcidtoname_downlevel.obj
 0002:00012478       ??_C@_1M@OJONDMDL@?$AAf?$AAr?$AA?9?$AAM?$AAC@ 10034478     libucrt:lcidtoname_downlevel.obj
 0002:00012484       ??_C@_1BG@OBCNFJB@?$AAs?$AAr?$AA?9?$AAB?$AAA?$AA?9?$AAL?$AAa?$AAt?$AAn@ 10034484     libucrt:lcidtoname_downlevel.obj
 0002:0001249c       ??_C@_1O@KEMEEGPO@?$AAs?$AAm?$AAa?$AA?9?$AAN?$AAO@ 1003449c     libucrt:lcidtoname_downlevel.obj
 0002:000124ac       ??_C@_1M@ELMGFODK@?$AAa?$AAr?$AA?9?$AAT?$AAN@ 100344ac     libucrt:lcidtoname_downlevel.obj
 0002:000124b8       ??_C@_1M@BHDLHFAF@?$AAe?$AAn?$AA?9?$AAZ?$AAA@ 100344b8     libucrt:lcidtoname_downlevel.obj
 0002:000124c4       ??_C@_1M@BMGIGLIF@?$AAe?$AAs?$AA?9?$AAD?$AAO@ 100344c4     libucrt:lcidtoname_downlevel.obj
 0002:000124d0       ??_C@_1BG@CMBHIPBE@?$AAs?$AAr?$AA?9?$AAB?$AAA?$AA?9?$AAC?$AAy?$AAr?$AAl@ 100344d0     libucrt:lcidtoname_downlevel.obj
 0002:000124e8       ??_C@_1O@HEDBLHNP@?$AAs?$AAm?$AAa?$AA?9?$AAS?$AAE@ 100344e8     libucrt:lcidtoname_downlevel.obj
 0002:000124f8       ??_C@_1M@DAGCADIM@?$AAa?$AAr?$AA?9?$AAO?$AAM@ 100344f8     libucrt:lcidtoname_downlevel.obj
 0002:00012504       ??_C@_1M@FODLMICG@?$AAe?$AAn?$AA?9?$AAJ?$AAM@ 10034504     libucrt:lcidtoname_downlevel.obj
 0002:00012510       ??_C@_1M@DNMLCIHB@?$AAe?$AAs?$AA?9?$AAV?$AAE@ 10034510     libucrt:lcidtoname_downlevel.obj
 0002:0001251c       ??_C@_1O@EOKHMKJK@?$AAs?$AAm?$AAs?$AA?9?$AAF?$AAI@ 1003451c     libucrt:lcidtoname_downlevel.obj
 0002:0001252c       ??_C@_1M@CAFJMKOF@?$AAa?$AAr?$AA?9?$AAY?$AAE@ 1003452c     libucrt:lcidtoname_downlevel.obj
 0002:00012538       ??_C@_1M@CBFHIJLI@?$AAe?$AAn?$AA?9?$AAC?$AAB@ 10034538     libucrt:lcidtoname_downlevel.obj
 0002:00012544       ??_C@_1M@BGNFLDN@?$AAe?$AAs?$AA?9?$AAC?$AAO@ 10034544     libucrt:lcidtoname_downlevel.obj
 0002:00012550       ??_C@_1O@JMPHMAMC@?$AAs?$AAm?$AAn?$AA?9?$AAF?$AAI@ 10034550     libucrt:lcidtoname_downlevel.obj
 0002:00012560       ??_C@_1M@JLANABKE@?$AAa?$AAr?$AA?9?$AAS?$AAY@ 10034560     libucrt:lcidtoname_downlevel.obj
 0002:0001256c       ??_C@_1M@HPKGCFGN@?$AAe?$AAn?$AA?9?$AAB?$AAZ@ 1003456c     libucrt:lcidtoname_downlevel.obj
 0002:00012578       ??_C@_1M@OLJCMLGM@?$AAe?$AAs?$AA?9?$AAP?$AAE@ 10034578     libucrt:lcidtoname_downlevel.obj
 0002:00012584       ??_C@_1M@MKKGFKLE@?$AAa?$AAr?$AA?9?$AAJ?$AAO@ 10034584     libucrt:lcidtoname_downlevel.obj
 0002:00012590       ??_C@_1M@EKPGLDNI@?$AAe?$AAn?$AA?9?$AAT?$AAT@ 10034590     libucrt:lcidtoname_downlevel.obj
 0002:0001259c       ??_C@_1M@OONGHFHE@?$AAe?$AAs?$AA?9?$AAA?$AAR@ 1003459c     libucrt:lcidtoname_downlevel.obj
 0002:000125a8       ??_C@_1M@OOJFGBHE@?$AAa?$AAr?$AA?9?$AAL?$AAB@ 100345a8     libucrt:lcidtoname_downlevel.obj
 0002:000125b4       ??_C@_1M@GCEJHNEG@?$AAe?$AAn?$AA?9?$AAZ?$AAW@ 100345b4     libucrt:lcidtoname_downlevel.obj
 0002:000125c0       ??_C@_1M@JNOCAHJI@?$AAe?$AAs?$AA?9?$AAE?$AAC@ 100345c0     libucrt:lcidtoname_downlevel.obj
 0002:000125cc       ??_C@_1M@JEFHPGGB@?$AAa?$AAr?$AA?9?$AAK?$AAW@ 100345cc     libucrt:lcidtoname_downlevel.obj
 0002:000125d8       ??_C@_1M@MLKIBJOJ@?$AAe?$AAn?$AA?9?$AAP?$AAH@ 100345d8     libucrt:lcidtoname_downlevel.obj
 0002:000125e4       ??_C@_1M@BDNIPEND@?$AAe?$AAs?$AA?9?$AAC?$AAL@ 100345e4     libucrt:lcidtoname_downlevel.obj
 0002:000125f0       ??_C@_1M@MPNMEKBD@?$AAa?$AAr?$AA?9?$AAA?$AAE@ 100345f0     libucrt:lcidtoname_downlevel.obj
 0002:000125fc       ??_C@_1M@KBJALCPI@?$AAe?$AAs?$AA?9?$AAU?$AAY@ 100345fc     libucrt:lcidtoname_downlevel.obj
 0002:00012608       ??_C@_1M@LLCCOAGA@?$AAa?$AAr?$AA?9?$AAB?$AAH@ 10034608     libucrt:lcidtoname_downlevel.obj
 0002:00012614       ??_C@_1M@PBFNCDEL@?$AAe?$AAs?$AA?9?$AAP?$AAY@ 10034614     libucrt:lcidtoname_downlevel.obj
 0002:00012620       ??_C@_1M@EDGINPNP@?$AAa?$AAr?$AA?9?$AAQ?$AAA@ 10034620     libucrt:lcidtoname_downlevel.obj
 0002:0001262c       ??_C@_1M@MKDBIIJI@?$AAe?$AAs?$AA?9?$AAB?$AAO@ 1003462c     libucrt:lcidtoname_downlevel.obj
 0002:00012638       ??_C@_1M@CPKKEBLD@?$AAe?$AAs?$AA?9?$AAS?$AAV@ 10034638     libucrt:lcidtoname_downlevel.obj
 0002:00012644       ??_C@_1M@NDBGMMJL@?$AAe?$AAs?$AA?9?$AAH?$AAN@ 10034644     libucrt:lcidtoname_downlevel.obj
 0002:00012650       ??_C@_1M@JIJIBHDP@?$AAe?$AAs?$AA?9?$AAN?$AAI@ 10034650     libucrt:lcidtoname_downlevel.obj
 0002:0001265c       ??_C@_1M@CGFMKEEK@?$AAe?$AAs?$AA?9?$AAP?$AAR@ 1003465c     libucrt:lcidtoname_downlevel.obj
 0002:00012668       ??_C@_1O@ICJHKIIK@?$AAz?$AAh?$AA?9?$AAC?$AAH?$AAT@ 10034668     libucrt:lcidtoname_downlevel.obj
 0002:00012678       ??_C@_15CLNEJCE@?$AAs?$AAr@ 10034678     libucrt:lcidtoname_downlevel.obj
 0002:00012da0       ??_C@_1M@KAHEKEIG@?$AAa?$AAf?$AA?9?$AAz?$AAa@ 10034da0     libucrt:lcidtoname_downlevel.obj
 0002:00012dac       ??_C@_1M@GIECOABL@?$AAa?$AAr?$AA?9?$AAa?$AAe@ 10034dac     libucrt:lcidtoname_downlevel.obj
 0002:00012db8       ??_C@_1M@BMLMEKGI@?$AAa?$AAr?$AA?9?$AAb?$AAh@ 10034db8     libucrt:lcidtoname_downlevel.obj
 0002:00012dc4       ??_C@_1M@DAPFDGGB@?$AAa?$AAr?$AA?9?$AAd?$AAz@ 10034dc4     libucrt:lcidtoname_downlevel.obj
 0002:00012dd0       ??_C@_1M@FJNKGKIG@?$AAa?$AAr?$AA?9?$AAe?$AAg@ 10034dd0     libucrt:lcidtoname_downlevel.obj
 0002:00012ddc       ??_C@_1M@FLGKKCLO@?$AAa?$AAr?$AA?9?$AAi?$AAq@ 10034ddc     libucrt:lcidtoname_downlevel.obj
 0002:00012de8       ??_C@_1M@GNDIPALM@?$AAa?$AAr?$AA?9?$AAj?$AAo@ 10034de8     libucrt:lcidtoname_downlevel.obj
 0002:00012df4       ??_C@_1M@DDMJFMGJ@?$AAa?$AAr?$AA?9?$AAk?$AAw@ 10034df4     libucrt:lcidtoname_downlevel.obj
 0002:00012e00       ??_C@_1M@EJALMLHM@?$AAa?$AAr?$AA?9?$AAl?$AAb@ 10034e00     libucrt:lcidtoname_downlevel.obj
 0002:00012e0c       ??_C@_1M@MOBDBLOC@?$AAa?$AAr?$AA?9?$AAl?$AAy@ 10034e0c     libucrt:lcidtoname_downlevel.obj
 0002:00012e18       ??_C@_1M@JAOCLHDH@?$AAa?$AAr?$AA?9?$AAm?$AAa@ 10034e18     libucrt:lcidtoname_downlevel.obj
 0002:00012e24       ??_C@_1M@JHPMKJIE@?$AAa?$AAr?$AA?9?$AAo?$AAm@ 10034e24     libucrt:lcidtoname_downlevel.obj
 0002:00012e30       ??_C@_1M@OEPGHFNH@?$AAa?$AAr?$AA?9?$AAq?$AAa@ 10034e30     libucrt:lcidtoname_downlevel.obj
 0002:00012e3c       ??_C@_1M@KJDONENM@?$AAa?$AAr?$AA?9?$AAs?$AAa@ 10034e3c     libucrt:lcidtoname_downlevel.obj
 0002:00012e48       ??_C@_1M@DMJDKLKM@?$AAa?$AAr?$AA?9?$AAs?$AAy@ 10034e48     libucrt:lcidtoname_downlevel.obj
 0002:00012e54       ??_C@_1M@OMFIPEDC@?$AAa?$AAr?$AA?9?$AAt?$AAn@ 10034e54     libucrt:lcidtoname_downlevel.obj
 0002:00012e60       ??_C@_1M@IHMHGAON@?$AAa?$AAr?$AA?9?$AAy?$AAe@ 10034e60     libucrt:lcidtoname_downlevel.obj
 0002:00012e6c       ??_C@_1BG@KDCPGJGB@?$AAa?$AAz?$AA?9?$AAa?$AAz?$AA?9?$AAc?$AAy?$AAr?$AAl@ 10034e6c     libucrt:lcidtoname_downlevel.obj
 0002:00012e84       ??_C@_1BG@IBCKDDOE@?$AAa?$AAz?$AA?9?$AAa?$AAz?$AA?9?$AAl?$AAa?$AAt?$AAn@ 10034e84     libucrt:lcidtoname_downlevel.obj
 0002:00012e9c       ??_C@_1M@EGPFDCPD@?$AAb?$AAe?$AA?9?$AAb?$AAy@ 10034e9c     libucrt:lcidtoname_downlevel.obj
 0002:00012ea8       ??_C@_1M@PCMGMCGC@?$AAb?$AAg?$AA?9?$AAb?$AAg@ 10034ea8     libucrt:lcidtoname_downlevel.obj
 0002:00012eb4       ??_C@_1M@BJBMFGOB@?$AAb?$AAn?$AA?9?$AAi?$AAn@ 10034eb4     libucrt:lcidtoname_downlevel.obj
 0002:00012ec0       ??_C@_1BG@EAKMMACD@?$AAb?$AAs?$AA?9?$AAb?$AAa?$AA?9?$AAl?$AAa?$AAt?$AAn@ 10034ec0     libucrt:lcidtoname_downlevel.obj
 0002:00012ed8       ??_C@_1M@KGADAODK@?$AAc?$AAa?$AA?9?$AAe?$AAs@ 10034ed8     libucrt:lcidtoname_downlevel.obj
 0002:00012ee4       ??_C@_1M@COAJPDHI@?$AAc?$AAs?$AA?9?$AAc?$AAz@ 10034ee4     libucrt:lcidtoname_downlevel.obj
 0002:00012ef0       ??_C@_1M@DHBHFONH@?$AAc?$AAy?$AA?9?$AAg?$AAb@ 10034ef0     libucrt:lcidtoname_downlevel.obj
 0002:00012efc       ??_C@_1M@IMGKELGA@?$AAd?$AAa?$AA?9?$AAd?$AAk@ 10034efc     libucrt:lcidtoname_downlevel.obj
 0002:00012f08       ??_C@_1M@NNDGDNGA@?$AAd?$AAe?$AA?9?$AAa?$AAt@ 10034f08     libucrt:lcidtoname_downlevel.obj
 0002:00012f14       ??_C@_1M@IKDBHEEM@?$AAd?$AAe?$AA?9?$AAc?$AAh@ 10034f14     libucrt:lcidtoname_downlevel.obj
 0002:00012f20       ??_C@_1M@GFFOJMCJ@?$AAd?$AAe?$AA?9?$AAd?$AAe@ 10034f20     libucrt:lcidtoname_downlevel.obj
 0002:00012f2c       ??_C@_1M@MDNLKBPM@?$AAd?$AAe?$AA?9?$AAl?$AAi@ 10034f2c     libucrt:lcidtoname_downlevel.obj
 0002:00012f38       ??_C@_1M@NJBEEJNL@?$AAd?$AAe?$AA?9?$AAl?$AAu@ 10034f38     libucrt:lcidtoname_downlevel.obj
 0002:00012f44       ??_C@_1O@GNNELBAP@?$AAd?$AAi?$AAv?$AA?9?$AAm?$AAv@ 10034f44     libucrt:lcidtoname_downlevel.obj
 0002:00012f54       ??_C@_1M@EJLEOGAE@?$AAe?$AAl?$AA?9?$AAg?$AAr@ 10034f54     libucrt:lcidtoname_downlevel.obj
 0002:00012f60       ??_C@_1M@GMPONJN@?$AAe?$AAn?$AA?9?$AAa?$AAu@ 10034f60     libucrt:lcidtoname_downlevel.obj
 0002:00012f6c       ??_C@_1M@NIDIIPGF@?$AAe?$AAn?$AA?9?$AAb?$AAz@ 10034f6c     libucrt:lcidtoname_downlevel.obj
 0002:00012f78       ??_C@_1M@JEHMIMFO@?$AAe?$AAn?$AA?9?$AAc?$AAa@ 10034f78     libucrt:lcidtoname_downlevel.obj
 0002:00012f84       ??_C@_1M@IGMJCDLA@?$AAe?$AAn?$AA?9?$AAc?$AAb@ 10034f84     libucrt:lcidtoname_downlevel.obj
 0002:00012f90       ??_C@_1M@BNFIGBKG@?$AAe?$AAn?$AA?9?$AAg?$AAb@ 10034f90     libucrt:lcidtoname_downlevel.obj
 0002:00012f9c       ??_C@_1M@LKIFDIGP@?$AAe?$AAn?$AA?9?$AAi?$AAe@ 10034f9c     libucrt:lcidtoname_downlevel.obj
 0002:00012fa8       ??_C@_1M@PJKFGCCO@?$AAe?$AAn?$AA?9?$AAj?$AAm@ 10034fa8     libucrt:lcidtoname_downlevel.obj
 0002:00012fb4       ??_C@_1M@KPPKEPBO@?$AAe?$AAn?$AA?9?$AAn?$AAz@ 10034fb4     libucrt:lcidtoname_downlevel.obj
 0002:00012fc0       ??_C@_1M@GMDGLDOB@?$AAe?$AAn?$AA?9?$AAp?$AAh@ 10034fc0     libucrt:lcidtoname_downlevel.obj
 0002:00012fcc       ??_C@_1M@ONGIBJNA@?$AAe?$AAn?$AA?9?$AAt?$AAt@ 10034fcc     libucrt:lcidtoname_downlevel.obj
 0002:00012fd8       ??_C@_1M@LLODPCMM@?$AAe?$AAn?$AA?9?$AAu?$AAs@ 10034fd8     libucrt:lcidtoname_downlevel.obj
 0002:00012fe4       ??_C@_1M@LAKFNPAN@?$AAe?$AAn?$AA?9?$AAz?$AAa@ 10034fe4     libucrt:lcidtoname_downlevel.obj
 0002:00012ff0       ??_C@_1M@MFNHNHEO@?$AAe?$AAn?$AA?9?$AAz?$AAw@ 10034ff0     libucrt:lcidtoname_downlevel.obj
 0002:00012ffc       ??_C@_1M@EJEINPHM@?$AAe?$AAs?$AA?9?$AAa?$AAr@ 10034ffc     libucrt:lcidtoname_downlevel.obj
 0002:00013008       ??_C@_1M@GNKPCCJA@?$AAe?$AAs?$AA?9?$AAb?$AAo@ 10035008     libucrt:lcidtoname_downlevel.obj
 0002:00013014       ??_C@_1M@LEEGFONL@?$AAe?$AAs?$AA?9?$AAc?$AAl@ 10035014     libucrt:lcidtoname_downlevel.obj
 0002:00013020       ??_C@_1M@KGPDPBDF@?$AAe?$AAs?$AA?9?$AAc?$AAo@ 10035020     libucrt:lcidtoname_downlevel.obj
 0002:0001302c       ??_C@_1M@EIAHOHH@?$AAe?$AAs?$AA?9?$AAc?$AAr@ 1003502c     libucrt:lcidtoname_downlevel.obj
 0002:00013038       ??_C@_1M@LLPGMBIN@?$AAe?$AAs?$AA?9?$AAd?$AAo@ 10035038     libucrt:lcidtoname_downlevel.obj
 0002:00013044       ??_C@_1M@DKHMKNJA@?$AAe?$AAs?$AA?9?$AAe?$AAc@ 10035044     libucrt:lcidtoname_downlevel.obj
 0002:00013050       ??_C@_1M@GKGFPKAP@?$AAe?$AAs?$AA?9?$AAe?$AAs@ 10035050     libucrt:lcidtoname_downlevel.obj
 0002:0001305c       ??_C@_1M@LKHKGDLN@?$AAe?$AAs?$AA?9?$AAg?$AAt@ 1003505c     libucrt:lcidtoname_downlevel.obj
 0002:00013068       ??_C@_1M@HEIIGGJD@?$AAe?$AAs?$AA?9?$AAh?$AAn@ 10035068     libucrt:lcidtoname_downlevel.obj
 0002:00013074       ??_C@_1M@FBDHPPGD@?$AAe?$AAs?$AA?9?$AAm?$AAx@ 10035074     libucrt:lcidtoname_downlevel.obj
 0002:00013080       ??_C@_1M@DPAGLNDH@?$AAe?$AAs?$AA?9?$AAn?$AAi@ 10035080     libucrt:lcidtoname_downlevel.obj
 0002:0001308c       ??_C@_1M@MDGOPGDD@?$AAe?$AAs?$AA?9?$AAp?$AAa@ 1003508c     libucrt:lcidtoname_downlevel.obj
 0002:00013098       ??_C@_1M@EMAMGBGE@?$AAe?$AAs?$AA?9?$AAp?$AAe@ 10035098     libucrt:lcidtoname_downlevel.obj
 0002:000130a4       ??_C@_1M@IBMCAOEC@?$AAe?$AAs?$AA?9?$AAp?$AAr@ 100350a4     libucrt:lcidtoname_downlevel.obj
 0002:000130b0       ??_C@_1M@FGMDIJED@?$AAe?$AAs?$AA?9?$AAp?$AAy@ 100350b0     libucrt:lcidtoname_downlevel.obj
 0002:000130bc       ??_C@_1M@IIDEOLLL@?$AAe?$AAs?$AA?9?$AAs?$AAv@ 100350bc     libucrt:lcidtoname_downlevel.obj
 0002:000130c8       ??_C@_1M@GAOBIPA@?$AAe?$AAs?$AA?9?$AAu?$AAy@ 100350c8     libucrt:lcidtoname_downlevel.obj
 0002:000130d4       ??_C@_1M@JKFFICHJ@?$AAe?$AAs?$AA?9?$AAv?$AAe@ 100350d4     libucrt:lcidtoname_downlevel.obj
 0002:000130e0       ??_C@_1M@PNMLOJDF@?$AAe?$AAt?$AA?9?$AAe?$AAe@ 100350e0     libucrt:lcidtoname_downlevel.obj
 0002:000130ec       ??_C@_1M@GHHLIKEI@?$AAe?$AAu?$AA?9?$AAe?$AAs@ 100350ec     libucrt:lcidtoname_downlevel.obj
 0002:000130f8       ??_C@_1M@PBNONODE@?$AAf?$AAa?$AA?9?$AAi?$AAr@ 100350f8     libucrt:lcidtoname_downlevel.obj
 0002:00013104       ??_C@_1M@JEEHPMIL@?$AAf?$AAi?$AA?9?$AAf?$AAi@ 10035104     libucrt:lcidtoname_downlevel.obj
 0002:00013110       ??_C@_1M@LMDCNDBA@?$AAf?$AAo?$AA?9?$AAf?$AAo@ 10035110     libucrt:lcidtoname_downlevel.obj
 0002:0001311c       ??_C@_1M@JKEOHLDK@?$AAf?$AAr?$AA?9?$AAb?$AAe@ 1003511c     libucrt:lcidtoname_downlevel.obj
 0002:00013128       ??_C@_1M@NOHADPMI@?$AAf?$AAr?$AA?9?$AAc?$AAa@ 10035128     libucrt:lcidtoname_downlevel.obj
 0002:00013134       ??_C@_1M@KDHIHAEC@?$AAf?$AAr?$AA?9?$AAc?$AAh@ 10035134     libucrt:lcidtoname_downlevel.obj
 0002:00013140       ??_C@_1M@MMBBFGAK@?$AAf?$AAr?$AA?9?$AAf?$AAr@ 10035140     libucrt:lcidtoname_downlevel.obj
 0002:0001314c       ??_C@_1M@PAFNENNF@?$AAf?$AAr?$AA?9?$AAl?$AAu@ 1003514c     libucrt:lcidtoname_downlevel.obj
 0002:00013158       ??_C@_1M@EOHDJGDD@?$AAf?$AAr?$AA?9?$AAm?$AAc@ 10035158     libucrt:lcidtoname_downlevel.obj
 0002:00013164       ??_C@_1M@FAPLLOPF@?$AAg?$AAl?$AA?9?$AAe?$AAs@ 10035164     libucrt:lcidtoname_downlevel.obj
 0002:00013170       ??_C@_1M@FOPBFLOO@?$AAg?$AAu?$AA?9?$AAi?$AAn@ 10035170     libucrt:lcidtoname_downlevel.obj
 0002:0001317c       ??_C@_1M@KBMCINPM@?$AAh?$AAe?$AA?9?$AAi?$AAl@ 1003517c     libucrt:lcidtoname_downlevel.obj
 0002:00013188       ??_C@_1M@BBPHKFPJ@?$AAh?$AAi?$AA?9?$AAi?$AAn@ 10035188     libucrt:lcidtoname_downlevel.obj
 0002:00013194       ??_C@_1M@PMBNDPHD@?$AAh?$AAr?$AA?9?$AAb?$AAa@ 10035194     libucrt:lcidtoname_downlevel.obj
 0002:000131a0       ??_C@_1M@BPCKOEGE@?$AAh?$AAr?$AA?9?$AAh?$AAr@ 100351a0     libucrt:lcidtoname_downlevel.obj
 0002:000131ac       ??_C@_1M@GACBMHKE@?$AAh?$AAu?$AA?9?$AAh?$AAu@ 100351ac     libucrt:lcidtoname_downlevel.obj
 0002:000131b8       ??_C@_1M@MILPAJJC@?$AAh?$AAy?$AA?9?$AAa?$AAm@ 100351b8     libucrt:lcidtoname_downlevel.obj
 0002:000131c4       ??_C@_1M@BABBICEC@?$AAi?$AAd?$AA?9?$AAi?$AAd@ 100351c4     libucrt:lcidtoname_downlevel.obj
 0002:000131d0       ??_C@_1M@BIKNHHPF@?$AAi?$AAs?$AA?9?$AAi?$AAs@ 100351d0     libucrt:lcidtoname_downlevel.obj
 0002:000131dc       ??_C@_1M@NMPCJPHE@?$AAi?$AAt?$AA?9?$AAc?$AAh@ 100351dc     libucrt:lcidtoname_downlevel.obj
 0002:000131e8       ??_C@_1M@GHKGFEDF@?$AAi?$AAt?$AA?9?$AAi?$AAt@ 100351e8     libucrt:lcidtoname_downlevel.obj
 0002:000131f4       ??_C@_1M@NIEJCJJA@?$AAj?$AAa?$AA?9?$AAj?$AAp@ 100351f4     libucrt:lcidtoname_downlevel.obj
 0002:00013200       ??_C@_1M@JILFNBIM@?$AAk?$AAa?$AA?9?$AAg?$AAe@ 10035200     libucrt:lcidtoname_downlevel.obj
 0002:0001320c       ??_C@_1M@PACPMGPH@?$AAk?$AAk?$AA?9?$AAk?$AAz@ 1003520c     libucrt:lcidtoname_downlevel.obj
 0002:00013218       ??_C@_1M@IELFGMHA@?$AAk?$AAn?$AA?9?$AAi?$AAn@ 10035218     libucrt:lcidtoname_downlevel.obj
 0002:00013224       ??_C@_1O@IBBJHCH@?$AAk?$AAo?$AAk?$AA?9?$AAi?$AAn@ 10035224     libucrt:lcidtoname_downlevel.obj
 0002:00013234       ??_C@_1M@DMHAEOGC@?$AAk?$AAo?$AA?9?$AAk?$AAr@ 10035234     libucrt:lcidtoname_downlevel.obj
 0002:00013240       ??_C@_1M@HBAHBIGA@?$AAk?$AAy?$AA?9?$AAk?$AAg@ 10035240     libucrt:lcidtoname_downlevel.obj
 0002:0001324c       ??_C@_1M@KPMILCJG@?$AAl?$AAt?$AA?9?$AAl?$AAt@ 1003524c     libucrt:lcidtoname_downlevel.obj
 0002:00013258       ??_C@_1M@BDEKKCA@?$AAl?$AAv?$AA?9?$AAl?$AAv@ 10035258     libucrt:lcidtoname_downlevel.obj
 0002:00013264       ??_C@_1M@ELCKCCJJ@?$AAm?$AAi?$AA?9?$AAn?$AAz@ 10035264     libucrt:lcidtoname_downlevel.obj
 0002:00013270       ??_C@_1M@CBOOLAPA@?$AAm?$AAk?$AA?9?$AAm?$AAk@ 10035270     libucrt:lcidtoname_downlevel.obj
 0002:0001327c       ??_C@_1M@GPHNBJKN@?$AAm?$AAl?$AA?9?$AAi?$AAn@ 1003527c     libucrt:lcidtoname_downlevel.obj
 0002:00013288       ??_C@_1M@PABJILIG@?$AAm?$AAn?$AA?9?$AAm?$AAn@ 10035288     libucrt:lcidtoname_downlevel.obj
 0002:00013294       ??_C@_1M@FGBKKIPG@?$AAm?$AAr?$AA?9?$AAi?$AAn@ 10035294     libucrt:lcidtoname_downlevel.obj
 0002:000132a0       ??_C@_1M@NDBPDDAL@?$AAm?$AAs?$AA?9?$AAb?$AAn@ 100352a0     libucrt:lcidtoname_downlevel.obj
 0002:000132ac       ??_C@_1M@OPIHOOPI@?$AAm?$AAs?$AA?9?$AAm?$AAy@ 100352ac     libucrt:lcidtoname_downlevel.obj
 0002:000132b8       ??_C@_1M@PPDBCNFM@?$AAm?$AAt?$AA?9?$AAm?$AAt@ 100352b8     libucrt:lcidtoname_downlevel.obj
 0002:000132c4       ??_C@_1M@KDJDKMDD@?$AAn?$AAb?$AA?9?$AAn?$AAo@ 100352c4     libucrt:lcidtoname_downlevel.obj
 0002:000132d0       ??_C@_1M@KFCFLMJP@?$AAn?$AAl?$AA?9?$AAb?$AAe@ 100352d0     libucrt:lcidtoname_downlevel.obj
 0002:000132dc       ??_C@_1M@KPOPDDGO@?$AAn?$AAl?$AA?9?$AAn?$AAl@ 100352dc     libucrt:lcidtoname_downlevel.obj
 0002:000132e8       ??_C@_1M@LJKPEMLN@?$AAn?$AAn?$AA?9?$AAn?$AAo@ 100352e8     libucrt:lcidtoname_downlevel.obj
 0002:000132f4       ??_C@_1M@BDGHHBFL@?$AAn?$AAs?$AA?9?$AAz?$AAa@ 100352f4     libucrt:lcidtoname_downlevel.obj
 0002:00013300       ??_C@_1M@IDEHOAP@?$AAp?$AAa?$AA?9?$AAi?$AAn@ 10035300     libucrt:lcidtoname_downlevel.obj
 0002:0001330c       ??_C@_1M@HDBKGOGH@?$AAp?$AAl?$AA?9?$AAp?$AAl@ 1003530c     libucrt:lcidtoname_downlevel.obj
 0002:00013318       ??_C@_1M@LJLLCMEH@?$AAp?$AAt?$AA?9?$AAb?$AAr@ 10035318     libucrt:lcidtoname_downlevel.obj
 0002:00013324       ??_C@_1M@NCMONAAL@?$AAp?$AAt?$AA?9?$AAp?$AAt@ 10035324     libucrt:lcidtoname_downlevel.obj
 0002:00013330       ??_C@_1O@EAKMAJDN@?$AAq?$AAu?$AAz?$AA?9?$AAb?$AAo@ 10035330     libucrt:lcidtoname_downlevel.obj
 0002:00013340       ??_C@_1O@BHHPIGDN@?$AAq?$AAu?$AAz?$AA?9?$AAe?$AAc@ 10035340     libucrt:lcidtoname_downlevel.obj
 0002:00013350       ??_C@_1O@GBAPEKMJ@?$AAq?$AAu?$AAz?$AA?9?$AAp?$AAe@ 10035350     libucrt:lcidtoname_downlevel.obj
 0002:00013360       ??_C@_1M@CLGLEFBO@?$AAr?$AAo?$AA?9?$AAr?$AAo@ 10035360     libucrt:lcidtoname_downlevel.obj
 0002:0001336c       ??_C@_1M@CEEDODME@?$AAr?$AAu?$AA?9?$AAr?$AAu@ 1003536c     libucrt:lcidtoname_downlevel.obj
 0002:00013378       ??_C@_1M@HPKKKMPP@?$AAs?$AAa?$AA?9?$AAi?$AAn@ 10035378     libucrt:lcidtoname_downlevel.obj
 0002:00013384       ??_C@_1M@BKMAIGOJ@?$AAs?$AAe?$AA?9?$AAf?$AAi@ 10035384     libucrt:lcidtoname_downlevel.obj
 0002:00013390       ??_C@_1M@NDPIFLFI@?$AAs?$AAe?$AA?9?$AAn?$AAo@ 10035390     libucrt:lcidtoname_downlevel.obj
 0002:0001339c       ??_C@_1M@DANKKHJ@?$AAs?$AAe?$AA?9?$AAs?$AAe@ 1003539c     libucrt:lcidtoname_downlevel.obj
 0002:000133a8       ??_C@_1M@PNBLONPJ@?$AAs?$AAk?$AA?9?$AAs?$AAk@ 100353a8     libucrt:lcidtoname_downlevel.obj
 0002:000133b4       ??_C@_1M@LFMODOAL@?$AAs?$AAl?$AA?9?$AAs?$AAi@ 100353b4     libucrt:lcidtoname_downlevel.obj
 0002:000133c0       ??_C@_1O@DFKOMPG@?$AAs?$AAm?$AAa?$AA?9?$AAn?$AAo@ 100353c0     libucrt:lcidtoname_downlevel.obj
 0002:000133d0       ??_C@_1O@NDKPBNNH@?$AAs?$AAm?$AAa?$AA?9?$AAs?$AAe@ 100353d0     libucrt:lcidtoname_downlevel.obj
 0002:000133e0       ??_C@_1O@PLLKBHAB@?$AAs?$AAm?$AAj?$AA?9?$AAn?$AAo@ 100353e0     libucrt:lcidtoname_downlevel.obj
 0002:000133f0       ??_C@_1O@CLEPOGCA@?$AAs?$AAm?$AAj?$AA?9?$AAs?$AAe@ 100353f0     libucrt:lcidtoname_downlevel.obj
 0002:00013400       ??_C@_1O@DLGJGKMK@?$AAs?$AAm?$AAn?$AA?9?$AAf?$AAi@ 10035400     libucrt:lcidtoname_downlevel.obj
 0002:00013410       ??_C@_1O@OJDJGAJC@?$AAs?$AAm?$AAs?$AA?9?$AAf?$AAi@ 10035410     libucrt:lcidtoname_downlevel.obj
 0002:00013420       ??_C@_1M@BOFOGHPB@?$AAs?$AAq?$AA?9?$AAa?$AAl@ 10035420     libucrt:lcidtoname_downlevel.obj
 0002:0001342c       ??_C@_1BG@LJBBIPGB@?$AAs?$AAr?$AA?9?$AAb?$AAa?$AA?9?$AAc?$AAy?$AAr?$AAl@ 1003542c     libucrt:lcidtoname_downlevel.obj
 0002:00013444       ??_C@_1BG@JLBENFOE@?$AAs?$AAr?$AA?9?$AAb?$AAa?$AA?9?$AAl?$AAa?$AAt?$AAn@ 10035444     libucrt:lcidtoname_downlevel.obj
 0002:0001345c       ??_C@_1BG@KODPNHE@?$AAs?$AAr?$AA?9?$AAs?$AAp?$AA?9?$AAc?$AAy?$AAr?$AAl@ 1003545c     libucrt:lcidtoname_downlevel.obj
 0002:00013474       ??_C@_1BG@CIOGKHPB@?$AAs?$AAr?$AA?9?$AAs?$AAp?$AA?9?$AAl?$AAa?$AAt?$AAn@ 10035474     libucrt:lcidtoname_downlevel.obj
 0002:0001348c       ??_C@_1M@NGFJLMAC@?$AAs?$AAv?$AA?9?$AAf?$AAi@ 1003548c     libucrt:lcidtoname_downlevel.obj
 0002:00013498       ??_C@_1M@MPJEJAJC@?$AAs?$AAv?$AA?9?$AAs?$AAe@ 10035498     libucrt:lcidtoname_downlevel.obj
 0002:000134a4       ??_C@_1M@MPNDHLFK@?$AAs?$AAw?$AA?9?$AAk?$AAe@ 100354a4     libucrt:lcidtoname_downlevel.obj
 0002:000134b0       ??_C@_1O@KOHBJJI@?$AAs?$AAy?$AAr?$AA?9?$AAs?$AAy@ 100354b0     libucrt:lcidtoname_downlevel.obj
 0002:000134c0       ??_C@_1M@LDCEFHA@?$AAt?$AAa?$AA?9?$AAi?$AAn@ 100354c0     libucrt:lcidtoname_downlevel.obj
 0002:000134cc       ??_C@_1M@CNJOFAK@?$AAt?$AAe?$AA?9?$AAi?$AAn@ 100354cc     libucrt:lcidtoname_downlevel.obj
 0002:000134d8       ??_C@_1M@GNAECACD@?$AAt?$AAh?$AA?9?$AAt?$AAh@ 100354d8     libucrt:lcidtoname_downlevel.obj
 0002:000134e4       ??_C@_1M@CHBIHOJO@?$AAt?$AAn?$AA?9?$AAz?$AAa@ 100354e4     libucrt:lcidtoname_downlevel.obj
 0002:000134f0       ??_C@_1M@GCCMIGPJ@?$AAt?$AAr?$AA?9?$AAt?$AAr@ 100354f0     libucrt:lcidtoname_downlevel.obj
 0002:000134fc       ??_C@_1M@CELMCNBK@?$AAt?$AAt?$AA?9?$AAr?$AAu@ 100354fc     libucrt:lcidtoname_downlevel.obj
 0002:00013508       ??_C@_1M@KLMCELGA@?$AAu?$AAk?$AA?9?$AAu?$AAa@ 10035508     libucrt:lcidtoname_downlevel.obj
 0002:00013514       ??_C@_1M@EPAJJAJF@?$AAu?$AAr?$AA?9?$AAp?$AAk@ 10035514     libucrt:lcidtoname_downlevel.obj
 0002:00013520       ??_C@_1BG@GEGPMCDJ@?$AAu?$AAz?$AA?9?$AAu?$AAz?$AA?9?$AAc?$AAy?$AAr?$AAl@ 10035520     libucrt:lcidtoname_downlevel.obj
 0002:00013538       ??_C@_1BG@EGGKJILM@?$AAu?$AAz?$AA?9?$AAu?$AAz?$AA?9?$AAl?$AAa?$AAt?$AAn@ 10035538     libucrt:lcidtoname_downlevel.obj
 0002:00013550       ??_C@_1M@GFOCLFF@?$AAv?$AAi?$AA?9?$AAv?$AAn@ 10035550     libucrt:lcidtoname_downlevel.obj
 0002:0001355c       ??_C@_1M@CPAMEDFI@?$AAx?$AAh?$AA?9?$AAz?$AAa@ 1003555c     libucrt:lcidtoname_downlevel.obj
 0002:00013568       ??_C@_1O@EBKIFIGN@?$AAz?$AAh?$AA?9?$AAc?$AAh?$AAs@ 10035568     libucrt:lcidtoname_downlevel.obj
 0002:00013578       ??_C@_1O@NMHPGANE@?$AAz?$AAh?$AA?9?$AAc?$AAh?$AAt@ 10035578     libucrt:lcidtoname_downlevel.obj
 0002:00013588       ??_C@_1M@LPINJOMC@?$AAz?$AAh?$AA?9?$AAc?$AAn@ 10035588     libucrt:lcidtoname_downlevel.obj
 0002:00013594       ??_C@_1M@OCJEJODD@?$AAz?$AAh?$AA?9?$AAh?$AAk@ 10035594     libucrt:lcidtoname_downlevel.obj
 0002:000135a0       ??_C@_1M@DNDLJINH@?$AAz?$AAh?$AA?9?$AAm?$AAo@ 100355a0     libucrt:lcidtoname_downlevel.obj
 0002:000135ac       ??_C@_1M@MBFDNDND@?$AAz?$AAh?$AA?9?$AAs?$AAg@ 100355ac     libucrt:lcidtoname_downlevel.obj
 0002:000135b8       ??_C@_1M@IMEPLEPE@?$AAz?$AAh?$AA?9?$AAt?$AAw@ 100355b8     libucrt:lcidtoname_downlevel.obj
 0002:000135c4       ??_C@_1M@BBGHNHJP@?$AAz?$AAu?$AA?9?$AAz?$AAa@ 100355c4     libucrt:lcidtoname_downlevel.obj
 0002:000135d0       ?large_power_data@?1??multiply_by_power_of_ten@__crt_strtox@@YA_NAAUbig_integer@2@I@Z@4QBIB 100355d0     libucrt:cfout.obj
 0002:00013f70       ?small_powers_of_ten@?1??multiply_by_power_of_ten@__crt_strtox@@YA_NAAUbig_integer@2@I@Z@4QBIB 10035f70     libucrt:cfout.obj
 0002:00013f94       ??_C@_01GBGANLPD@0@        10035f94     libucrt:cfout.obj
 0002:00013f98       ??_C@_05DNEBIAHO@1?$CDINF@ 10035f98     libucrt:cfout.obj
 0002:00013fa0       ??_C@_06IMKFLFPG@1?$CDQNAN@ 10035fa0     libucrt:cfout.obj
 0002:00013fa8       ??_C@_06PGGFOGJG@1?$CDSNAN@ 10035fa8     libucrt:cfout.obj
 0002:00013fb0       ??_C@_05PHHOCPM@1?$CDIND@  10035fb0     libucrt:cfout.obj
 0002:00014018       ??_C@_1BA@BALFACEM@?$AAC?$AAO?$AAN?$AAO?$AAU?$AAT?$AA$@ 10036018     libucrt:initcon.obj
 0002:00014130       __infinity                 10036130     libucrt:87tran.obj
 0002:0001413a       __minfinity                1003613a     libucrt:87tran.obj
 0002:00014144       __logemax                  10036144     libucrt:87tran.obj
 0002:0001416a       __OP_EXPjmptab             1003616a     libucrt:87tran.obj
 0002:00014190       __indefinite               10036190     libucrt:87disp.obj
 0002:0001419a       __piby2                    1003619a     libucrt:87disp.obj
 0002:000141a4       __piby4                    100361a4     libucrt:87disp.obj
 0002:000141d8       __DEFAULT_CW_in_mem        100361d8     libucrt:common.obj
 0002:000141da       __pi_by_2_to_61            100361da     libucrt:common.obj
 0002:00014214       ??_C@_03MGHMBJCF@log@      10036214     libucrt:libm_error.obj
 0002:00014218       ??_C@_05HGHHAHAP@log10@    10036218     libucrt:libm_error.obj
 0002:00014220       ??_C@_03KHJOGHMM@exp@      10036220     libucrt:libm_error.obj
 0002:00014224       ??_C@_03JGHBODFD@pow@      10036224     libucrt:libm_error.obj
 0002:00014228       ??_C@_04FIHNOPOL@asin@     10036228     libucrt:libm_error.obj
 0002:00014230       ??_C@_04PDIFKINK@acos@     10036230     libucrt:libm_error.obj
 0002:00014238       ??_C@_04EIAKFFMI@sqrt@     10036238     libucrt:libm_error.obj
 0002:00014240       __real@3ff0000000000000    10036240     libucrt:libm_error.obj
 0002:00014260       ___acrt_log10_table_t      10036260     libucrt:log10_tables.obj
 0002:00014670       ___acrt_log10_table_cb     10036670     libucrt:log10_tables.obj
 0002:00014a80       __real@3fe0000000000000    10036a80     libucrt:powhlp.obj
 0002:00014b70       ??_C@_04COOMCNPB@sinh@     10036b70     libucrt:fpexcept.obj
 0002:00014b78       ??_C@_04HPJJNFIM@cosh@     10036b78     libucrt:fpexcept.obj
 0002:00014b80       ??_C@_04FJHINJAO@tanh@     10036b80     libucrt:fpexcept.obj
 0002:00014b88       ??_C@_04MLLJIGOK@atan@     10036b88     libucrt:fpexcept.obj
 0002:00014b90       ??_C@_05KNGEOGJB@atan2@    10036b90     libucrt:fpexcept.obj
 0002:00014b98       ??_C@_03BLEJJJBH@sin@      10036b98     libucrt:fpexcept.obj
 0002:00014b9c       ??_C@_03LALBNOCG@cos@      10036b9c     libucrt:fpexcept.obj
 0002:00014ba0       ??_C@_03IIINPABG@tan@      10036ba0     libucrt:fpexcept.obj
 0002:00014ba4       ??_C@_04GFPJNGEK@ceil@     10036ba4     libucrt:fpexcept.obj
 0002:00014bac       ??_C@_05PBJFFIGL@floor@    10036bac     libucrt:fpexcept.obj
 0002:00014bb4       ??_C@_04ODHECPBC@fabs@     10036bb4     libucrt:fpexcept.obj
 0002:00014bbc       ??_C@_04EHEDPDJG@modf@     10036bbc     libucrt:fpexcept.obj
 0002:00014bc4       ??_C@_05CEJMAHNP@ldexp@    10036bc4     libucrt:fpexcept.obj
 0002:00014bcc       ??_C@_05KBKMEMPO@_cabs@    10036bcc     libucrt:fpexcept.obj
 0002:00014bd4       ??_C@_06MEIMCGCF@_hypot@   10036bd4     libucrt:fpexcept.obj
 0002:00014bdc       ??_C@_04KEPJIHGP@fmod@     10036bdc     libucrt:fpexcept.obj
 0002:00014be4       ??_C@_05GKKHEGJL@frexp@    10036be4     libucrt:fpexcept.obj
 0002:00014bec       ??_C@_03MJLDFKDL@_y0@      10036bec     libucrt:fpexcept.obj
 0002:00014bf0       ??_C@_03NAKIGLHK@_y1@      10036bf0     libucrt:fpexcept.obj
 0002:00014bf4       ??_C@_03ONILCKOB@_yn@      10036bf4     libucrt:fpexcept.obj
 0002:00014bf8       ??_C@_05JGDBENOH@_logb@    10036bf8     libucrt:fpexcept.obj
 0002:00014c00       ??_C@_0L@KDOEJCKC@_nextafter@ 10036c00     libucrt:fpexcept.obj
 0002:00014c10       __d_inf                    10036c10     libucrt:util.obj
 0002:00014c18       __d_max                    10036c18     libucrt:util.obj
 0002:00014c20       __d_mzero                  10036c20     libucrt:util.obj
 0002:00014cb0       __load_config_used         10036cb0     LIBCMT:loadcfg.obj
 0002:00014d68       ??_R4exception@std@@6B@    10036d68     LIBCMT:throw_bad_alloc.obj
 0002:00014d7c       ??_R3exception@std@@8      10036d7c     LIBCMT:throw_bad_alloc.obj
 0002:00014d8c       ??_R2exception@std@@8      10036d8c     LIBCMT:throw_bad_alloc.obj
 0002:00014d94       ??_R1A@?0A@EA@exception@std@@8 10036d94     LIBCMT:throw_bad_alloc.obj
 0002:00014db0       ??_R4bad_alloc@std@@6B@    10036db0     LIBCMT:throw_bad_alloc.obj
 0002:00014dc4       ??_R3bad_alloc@std@@8      10036dc4     LIBCMT:throw_bad_alloc.obj
 0002:00014dd4       ??_R2bad_alloc@std@@8      10036dd4     LIBCMT:throw_bad_alloc.obj
 0002:00014de0       ??_R1A@?0A@EA@bad_alloc@std@@8 10036de0     LIBCMT:throw_bad_alloc.obj
 0002:00014dfc       ??_R4bad_array_new_length@std@@6B@ 10036dfc     LIBCMT:throw_bad_alloc.obj
 0002:00014e10       ??_R3bad_array_new_length@std@@8 10036e10     LIBCMT:throw_bad_alloc.obj
 0002:00014e20       ??_R2bad_array_new_length@std@@8 10036e20     LIBCMT:throw_bad_alloc.obj
 0002:00014e30       ??_R1A@?0A@EA@bad_array_new_length@std@@8 10036e30     LIBCMT:throw_bad_alloc.obj
 0002:00014e4c       ??_R4type_info@@6B@        10036e4c     LIBCMT:std_type_info_static.obj
 0002:00014e60       ??_R3type_info@@8          10036e60     LIBCMT:std_type_info_static.obj
 0002:00014e70       ??_R2type_info@@8          10036e70     LIBCMT:std_type_info_static.obj
 0002:00014e78       ??_R1A@?0A@EA@type_info@@8 10036e78     LIBCMT:std_type_info_static.obj
 0002:00014e94       ___safe_se_handler_table   10036e94     <linker-defined>
 0002:00015190       ___rtc_iaa                 10037190     LIBCMT:initsect.obj
 0002:00015194       ___rtc_izz                 10037194     LIBCMT:initsect.obj
 0002:00015198       ___rtc_taa                 10037198     LIBCMT:initsect.obj
 0002:0001519c       ___rtc_tzz                 1003719c     LIBCMT:initsect.obj
 0002:00015204       __TI2?AVbad_alloc@std@@    10037204     LIBCMT:throw_bad_alloc.obj
 0002:00015214       __CTA2?AVbad_alloc@std@@   10037214     LIBCMT:throw_bad_alloc.obj
 0002:00015220       __CT??_R0?AVbad_alloc@std@@@8??0bad_alloc@std@@QAE@ABV01@@Z12 10037220     LIBCMT:throw_bad_alloc.obj
 0002:0001523c       __CT??_R0?AVexception@std@@@8??0exception@std@@QAE@ABV01@@Z12 1003723c     LIBCMT:throw_bad_alloc.obj
 0002:00015258       __TI3?AVbad_array_new_length@std@@ 10037258     LIBCMT:throw_bad_alloc.obj
 0002:00015268       __CTA3?AVbad_array_new_length@std@@ 10037268     LIBCMT:throw_bad_alloc.obj
 0002:00015278       __CT??_R0?AVbad_array_new_length@std@@@8??0bad_array_new_length@std@@QAE@ABV01@@Z12 10037278     LIBCMT:throw_bad_alloc.obj
 0002:00016198       __IMPORT_DESCRIPTOR_KERNEL32 10038198     kernel32:KERNEL32.dll
 0002:000161ac       __IMPORT_DESCRIPTOR_USER32 100381ac     user32:USER32.dll
 0002:000161c0       __IMPORT_DESCRIPTOR_jawt   100381c0     jawt:jawt.dll
 0002:000161d4       __NULL_IMPORT_DESCRIPTOR   100381d4     kernel32:KERNEL32.dll
 0003:00000000       ___security_cookie_complement 10039000     LIBCMT:gs_cookie.obj
 0003:00000004       ___security_cookie         10039004     LIBCMT:gs_cookie.obj
 0003:00000008       __fltused                  10039008     LIBCMT:fltused.obj
 0003:0000000c       ___scrt_native_dllmain_reason 1003900c     LIBCMT:utility.obj
 0003:00000010       ___isa_enabled             10039010     LIBCMT:cpu_disp.obj
 0003:00000030       __NLG_Destination          10039030     libvcruntime:exsup.obj
 0003:00000040       __iob                      10039040     libucrt:_file.obj
 0003:000000e8       ___abort_behavior          100390e8     libucrt:abort.obj
 0003:00000100       ___badioinfo               10039100     libucrt:ioinit.obj
 0003:00000138       ___acrt_initial_locale_data 10039138     libucrt:nlsdata.obj
 0003:000001f0       ___acrt_initial_locale_pointers 100391f0     libucrt:nlsdata.obj
 0003:000001f8       ___acrt_wide_c_locale_string 100391f8     libucrt:nlsdata.obj
 0003:00000200       ___acrt_initial_multibyte_data 10039200     libucrt:mbctype.obj
 0003:00000720       __pwctype                  10039720     libucrt:ctype.obj
 0003:00000724       ___globallocalestatus      10039724     libucrt:glstatus.obj
 0003:00000728       ___acrt_lconv_c            10039728     libucrt:localeconv.obj
 0003:00000778       ___acrt_lconv_static_decimal 10039778     libucrt:localeconv.obj
 0003:0000077c       ___acrt_lconv_static_W_decimal 1003977c     libucrt:localeconv.obj
 0003:00000780       __lookuptrailbytes         10039780     libucrt:read.obj
 0003:00000890       ??_R0?AVbad_alloc@std@@@8  10039890     LIBCMT:throw_bad_alloc.obj
 0003:000008ac       ??_R0?AVexception@std@@@8  100398ac     LIBCMT:throw_bad_alloc.obj
 0003:000008c8       ??_R0?AVbad_array_new_length@std@@@8 100398c8     LIBCMT:throw_bad_alloc.obj
 0003:000008f0       ??_R0?AVtype_info@@@8      100398f0     LIBCMT:std_type_info_static.obj
 0003:00000908       ?JavaBridgeThreadId@@3KA   10039908     AccessBridgeATInstance.obj
 0003:00000910       ?_OptionsStorage@?1??__local_stdio_printf_options@@9@4_KA 10039910     AccessBridgeDebug.obj
 0003:0000091c       ?theFromJavaHelloMsgID@@3IA 1003991c     AccessBridgeMessages.obj
 0003:00000920       ?theFromWindowsHelloMsgID@@3IA 10039920     AccessBridgeMessages.obj
 0003:00000924       ?theJavaAccessBridge@@3PAVJavaAccessBridge@@A 10039924     JavaAccessBridge.obj
 0003:00000928       ?theDialogWindow@@3PAUHWND__@@A 10039928     JavaAccessBridge.obj
 0003:0000092c       ?receiveMemoryIPCLock@@3U_RTL_CRITICAL_SECTION@@A 1003992c     JavaAccessBridge.obj
 0003:00000c68       ?__type_info_root_node@@3U__type_info_node@@A 10039c68     LIBCMT:tncleanup.obj
 0003:00000c70       ?_OptionsStorage@?1??__local_stdio_scanf_options@@9@4_KA 10039c70     LIBCMT:default_local_stdio_options.obj
 0003:00000c78       ___scrt_current_native_startup_state 10039c78     LIBCMT:utility.obj
 0003:00000c7c       ___scrt_native_startup_lock 10039c7c     LIBCMT:utility.obj
 0003:00000c9c       ___scrt_debugger_hook_flag 10039c9c     LIBCMT:utility_desktop.obj
 0003:00000ca0       ___isa_available           10039ca0     LIBCMT:cpu_disp.obj
 0003:00000ca4       ___favor                   10039ca4     LIBCMT:cpu_disp.obj
 0003:00000ca8       ?__WinRTOutOfMemoryExceptionCallback@@3P6GPAXXZA 10039ca8     libvcruntime:ehhelpers.obj
 0003:00000cac       ?pArgList@UnDecorator@@0PAVReplicator@@A 10039cac     libvcruntime:undname.obj
 0003:00000cb0       ?pZNameList@UnDecorator@@0PAVReplicator@@A 10039cb0     libvcruntime:undname.obj
 0003:00000cb4       ?pTemplateArgList@UnDecorator@@0PAVReplicator@@A 10039cb4     libvcruntime:undname.obj
 0003:00000cb8       ?gName@UnDecorator@@0PBDB  10039cb8     libvcruntime:undname.obj
 0003:00000cbc       ?name@UnDecorator@@0PBDB   10039cbc     libvcruntime:undname.obj
 0003:00000cc0       ?disableFlags@UnDecorator@@0KA 10039cc0     libvcruntime:undname.obj
 0003:00000cc4       ?fExplicitTemplateParams@UnDecorator@@0_NA 10039cc4     libvcruntime:undname.obj
 0003:00000cc5       ?fGetTemplateArgumentList@UnDecorator@@0_NA 10039cc5     libvcruntime:undname.obj
 0003:00000cc8       ?m_pGetParameter@UnDecorator@@0P6APADJ@ZA 10039cc8     libvcruntime:undname.obj
 0003:00000ccc       ?m_CHPENameOffset@UnDecorator@@0KA 10039ccc     libvcruntime:undname.obj
 0003:00000cd0       ?m_recursionLevel@UnDecorator@@0KA 10039cd0     libvcruntime:undname.obj
 0003:00000d4c       ___pPurecall               10039d4c     libvcruntime:purevirt_data.obj
 0003:00000d50       __nstream                  10039d50     libucrt:_file.obj
 0003:00000d54       ___piob                    10039d54     libucrt:_file.obj
 0003:00000d58       __cflush                   10039d58     libucrt:_file.obj
 0003:00000d68       ?c_exit_complete@?1???R<lambda_6e4b09c48022b2350581041d5f6b0c4c>@@QBE@XZ@4_NA 10039d68     libucrt:exit.obj
 0003:00000e78       __environ_table            10039e78     libucrt:environment_initialization.obj
 0003:00000e7c       __wenviron_table           10039e7c     libucrt:environment_initialization.obj
 0003:00000e80       ___dcrt_initial_wide_environment 10039e80     libucrt:environment_initialization.obj
 0003:00000e84       ___dcrt_initial_narrow_environment 10039e84     libucrt:environment_initialization.obj
 0003:00000e88       ___acrt_atexit_table       10039e88     libucrt:onexit.obj
 0003:00000e94       ___acrt_at_quick_exit_table 10039e94     libucrt:onexit.obj
 0003:00000f88       ___pioinfo                 10039f88     libucrt:ioinit.obj
 0003:00001188       __nhandle                  1003a188     libucrt:ioinit.obj
 0003:00001198       ___acrt_stdout_buffer      1003a198     libucrt:_sftbuf.obj
 0003:0000119c       ___acrt_stderr_buffer      1003a19c     libucrt:_sftbuf.obj
 0003:000011a0       ___acrt_locale_changed_data 1003a1a0     libucrt:wsetlocale.obj
 0003:000011a4       ___acrt_current_locale_data 1003a1a4     libucrt:nlsdata.obj
 0003:000012fc       __mbctype                  1003a2fc     libucrt:mbctype.obj
 0003:00001300       __mbcasemap                1003a300     libucrt:mbctype.obj
 0003:00001304       ___acrt_current_multibyte_data 1003a304     libucrt:mbctype.obj
 0003:00001310       __pgmptr                   1003a310     libucrt:argv_data.obj
 0003:00001314       ___argc                    1003a314     libucrt:argv_data.obj
 0003:00001318       ___argv                    1003a318     libucrt:argv_data.obj
 0003:0000131c       ___wargv                   1003a31c     libucrt:argv_data.obj
 0003:00001320       __acmdln                   1003a320     libucrt:argv_data.obj
 0003:00001324       __wcmdln                   1003a324     libucrt:argv_data.obj
 0003:00001328       ___acrt_heap               1003a328     libucrt:heap_handle.obj
 0003:00001344       ___acrt_lconv_static_null  1003a344     libucrt:localeconv.obj
 0003:00001348       ___acrt_lconv_static_W_null 1003a348     libucrt:localeconv.obj
 0003:0000134c       __commode                  1003a34c     libucrt:ncommode.obj
 0003:0000135c       __umaskval                 1003a35c     libucrt:umask.obj
 0003:00001360       ___fastflag                1003a360     libucrt:fp_flags.obj
 0003:00001368       __fmode                    1003a368     libucrt:txtmode.obj
 0003:0000136c       ___scrt_ucrt_dll_is_in_use 1003a36c     <common>
 0003:00001370       ___dyn_tls_init_callback   1003a370     <common>
 0003:00001374       __pmatherr                 1003a374     <common>
 0003:00001378       ___use_sse2_mathfcns       1003a378     <common>

 entry point at        0001:0000c689

 Static symbols

 0000:fffc2000       .debug$S                   10000000     javaaccessbridge.exp
 0000:fffc2000       .debug$S                   10000000     kernel32:KERNEL32.dll
 0000:fffc2000       .debug$S                   10000000     kernel32:KERNEL32.dll
 0000:fffc2000       .debug$S                   10000000     kernel32:KERNEL32.dll
 0000:fffc2000       .debug$S                   10000000     kernel32:KERNEL32.dll
 0000:fffc2000       .debug$S                   10000000     kernel32:KERNEL32.dll
 0000:fffc2000       .debug$S                   10000000     kernel32:KERNEL32.dll
 0000:fffc2000       .debug$S                   10000000     kernel32:KERNEL32.dll
 0000:fffc2000       .debug$S                   10000000     kernel32:KERNEL32.dll
 0000:fffc2000       .debug$S                   10000000     kernel32:KERNEL32.dll
 0000:fffc2000       .debug$S                   10000000     kernel32:KERNEL32.dll
 0000:fffc2000       .debug$S                   10000000     kernel32:KERNEL32.dll
 0000:fffc2000       .debug$S                   10000000     kernel32:KERNEL32.dll
 0000:fffc2000       .debug$S                   10000000     kernel32:KERNEL32.dll
 0000:fffc2000       .debug$S                   10000000     kernel32:KERNEL32.dll
 0000:fffc2000       .debug$S                   10000000     kernel32:KERNEL32.dll
 0000:fffc2000       .debug$S                   10000000     kernel32:KERNEL32.dll
 0000:fffc2000       .debug$S                   10000000     kernel32:KERNEL32.dll
 0000:fffc2000       .debug$S                   10000000     kernel32:KERNEL32.dll
 0000:fffc2000       .debug$S                   10000000     kernel32:KERNEL32.dll
 0000:fffc2000       .debug$S                   10000000     kernel32:KERNEL32.dll
 0000:fffc2000       .debug$S                   10000000     kernel32:KERNEL32.dll
 0000:fffc2000       .debug$S                   10000000     kernel32:KERNEL32.dll
 0000:fffc2000       .debug$S                   10000000     kernel32:KERNEL32.dll
 0000:fffc2000       .debug$S                   10000000     kernel32:KERNEL32.dll
 0000:fffc2000       .debug$S                   10000000     kernel32:KERNEL32.dll
 0000:fffc2000       .debug$S                   10000000     kernel32:KERNEL32.dll
 0000:fffc2000       .debug$S                   10000000     kernel32:KERNEL32.dll
 0000:fffc2000       .debug$S                   10000000     kernel32:KERNEL32.dll
 0000:fffc2000       .debug$S                   10000000     kernel32:KERNEL32.dll
 0000:fffc2000       .debug$S                   10000000     kernel32:KERNEL32.dll
 0000:fffc2000       .debug$S                   10000000     kernel32:KERNEL32.dll
 0000:fffc2000       .debug$S                   10000000     kernel32:KERNEL32.dll
 0000:fffc2000       .debug$S                   10000000     kernel32:KERNEL32.dll
 0000:fffc2000       .debug$S                   10000000     kernel32:KERNEL32.dll
 0000:fffc2000       .debug$S                   10000000     kernel32:KERNEL32.dll
 0000:fffc2000       .debug$S                   10000000     kernel32:KERNEL32.dll
 0000:fffc2000       .debug$S                   10000000     kernel32:KERNEL32.dll
 0000:fffc2000       .debug$S                   10000000     kernel32:KERNEL32.dll
 0000:fffc2000       .debug$S                   10000000     kernel32:KERNEL32.dll
 0000:fffc2000       .debug$S                   10000000     kernel32:KERNEL32.dll
 0000:fffc2000       .debug$S                   10000000     kernel32:KERNEL32.dll
 0000:fffc2000       .debug$S                   10000000     kernel32:KERNEL32.dll
 0000:fffc2000       .debug$S                   10000000     kernel32:KERNEL32.dll
 0000:fffc2000       .debug$S                   10000000     kernel32:KERNEL32.dll
 0000:fffc2000       .debug$S                   10000000     kernel32:KERNEL32.dll
 0000:fffc2000       .debug$S                   10000000     kernel32:KERNEL32.dll
 0000:fffc2000       .debug$S                   10000000     kernel32:KERNEL32.dll
 0000:fffc2000       .debug$S                   10000000     kernel32:KERNEL32.dll
 0000:fffc2000       .debug$S                   10000000     kernel32:KERNEL32.dll
 0000:fffc2000       .debug$S                   10000000     kernel32:KERNEL32.dll
 0000:fffc2000       .debug$S                   10000000     kernel32:KERNEL32.dll
 0000:fffc2000       .debug$S                   10000000     kernel32:KERNEL32.dll
 0000:fffc2000       .debug$S                   10000000     kernel32:KERNEL32.dll
 0000:fffc2000       .debug$S                   10000000     kernel32:KERNEL32.dll
 0000:fffc2000       .debug$S                   10000000     kernel32:KERNEL32.dll
 0000:fffc2000       .debug$S                   10000000     kernel32:KERNEL32.dll
 0000:fffc2000       .debug$S                   10000000     kernel32:KERNEL32.dll
 0000:fffc2000       .debug$S                   10000000     kernel32:KERNEL32.dll
 0000:fffc2000       .debug$S                   10000000     kernel32:KERNEL32.dll
 0000:fffc2000       .debug$S                   10000000     kernel32:KERNEL32.dll
 0000:fffc2000       .debug$S                   10000000     kernel32:KERNEL32.dll
 0000:fffc2000       .debug$S                   10000000     kernel32:KERNEL32.dll
 0000:fffc2000       .debug$S                   10000000     kernel32:KERNEL32.dll
 0000:fffc2000       .debug$S                   10000000     kernel32:KERNEL32.dll
 0000:fffc2000       .debug$S                   10000000     kernel32:KERNEL32.dll
 0000:fffc2000       .debug$S                   10000000     kernel32:KERNEL32.dll
 0000:fffc2000       .debug$S                   10000000     kernel32:KERNEL32.dll
 0000:fffc2000       .debug$S                   10000000     kernel32:KERNEL32.dll
 0000:fffc2000       .debug$S                   10000000     kernel32:KERNEL32.dll
 0000:fffc2000       .debug$S                   10000000     kernel32:KERNEL32.dll
 0000:fffc2000       .debug$S                   10000000     kernel32:KERNEL32.dll
 0000:fffc2000       .debug$S                   10000000     kernel32:KERNEL32.dll
 0000:fffc2000       .debug$S                   10000000     kernel32:KERNEL32.dll
 0000:fffc2000       .debug$S                   10000000     kernel32:KERNEL32.dll
 0000:fffc2000       .debug$S                   10000000     kernel32:KERNEL32.dll
 0000:fffc2000       .debug$S                   10000000     kernel32:KERNEL32.dll
 0000:fffc2000       .debug$S                   10000000     kernel32:KERNEL32.dll
 0000:fffc2000       .debug$S                   10000000     kernel32:KERNEL32.dll
 0000:fffc2000       .debug$S                   10000000     kernel32:KERNEL32.dll
 0000:fffc2000       .debug$S                   10000000     kernel32:KERNEL32.dll
 0000:fffc2000       .debug$S                   10000000     kernel32:KERNEL32.dll
 0000:fffc2000       .debug$S                   10000000     kernel32:KERNEL32.dll
 0000:fffc2000       .debug$S                   10000000     kernel32:KERNEL32.dll
 0000:fffc2000       .debug$S                   10000000     kernel32:KERNEL32.dll
 0000:fffc2000       .debug$S                   10000000     kernel32:KERNEL32.dll
 0000:fffc2000       .debug$S                   10000000     kernel32:KERNEL32.dll
 0000:fffc2000       .debug$S                   10000000     kernel32:KERNEL32.dll
 0000:fffc2000       .debug$S                   10000000     kernel32:KERNEL32.dll
 0000:fffc2000       .debug$S                   10000000     kernel32:KERNEL32.dll
 0000:fffc2000       .debug$S                   10000000     kernel32:KERNEL32.dll
 0000:fffc2000       .debug$S                   10000000     kernel32:KERNEL32.dll
 0000:fffc2000       .debug$S                   10000000     kernel32:KERNEL32.dll
 0000:fffc2000       .debug$S                   10000000     user32:USER32.dll
 0000:fffc2000       .debug$S                   10000000     user32:USER32.dll
 0000:fffc2000       .debug$S                   10000000     user32:USER32.dll
 0000:fffc2000       .debug$S                   10000000     user32:USER32.dll
 0000:fffc2000       .debug$S                   10000000     user32:USER32.dll
 0000:fffc2000       .debug$S                   10000000     user32:USER32.dll
 0000:fffc2000       .debug$S                   10000000     user32:USER32.dll
 0000:fffc2000       .debug$S                   10000000     user32:USER32.dll
 0000:fffc2000       .debug$S                   10000000     user32:USER32.dll
 0000:fffc2000       .debug$S                   10000000     jawt:jawt.dll
 0001:0000008e       ?JavaBridgeThread@@YGIPAX@Z 1000108e f   AccessBridgeATInstance.obj
 0001:0000011a       ?do_event@@YAXPADHPAUHWND__@@1@Z 1000111a f   AccessBridgeATInstance.obj
 0001:0000bccf       $LN244                     1000cccf     JavaAccessBridge.obj
 0001:0000c2d0       $$000000                   1000d2d0     LIBCMT:ulldiv.obj
 0001:0000c349       ?dllmain_crt_dispatch@@YGHQAUHINSTANCE__@@KQAX@Z 1000d349 f   LIBCMT:dll_dllmain.obj
 0001:0000c39c       ?dllmain_crt_process_attach@@YAHQAUHINSTANCE__@@QAX@Z 1000d39c f   LIBCMT:dll_dllmain.obj
 0001:0000c4a3       ?dllmain_crt_process_detach@@YAH_N@Z 1000d4a3 f   LIBCMT:dll_dllmain.obj
 0001:0000c553       ?dllmain_dispatch@@YAHQAUHINSTANCE__@@KQAX@Z 1000d553 f   LIBCMT:dll_dllmain.obj
 0001:0000c65e       ?dllmain_raw@@YGHQAUHINSTANCE__@@KQAX@Z 1000d65e f   LIBCMT:dll_dllmain.obj
 0001:0000c8e9       ___get_entropy             1000d8e9 f   LIBCMT:gs_support.obj
 0001:0000c9bc       ?find_pe_section@@YAPAU_IMAGE_SECTION_HEADER@@QAEI@Z 1000d9bc f   LIBCMT:utility.obj
 0001:0000ce20       $$000000                   1000de20     LIBCMT:sehprolg4.obj
 0001:0000d080       $$000000                   1000e080     libvcruntime:memcpy.obj
 0001:0000d2e4       TrailingUpVec              1000e2e4     libvcruntime:memcpy.obj
 0001:0000d390       TrailingDownVec            1000e390     libvcruntime:memcpy.obj
 0001:0000d600       $$000000                   1000e600     libvcruntime:memset.obj
 0001:0000d760       _ValidateLocalCookies      1000e760 f   libvcruntime:chandler4.obj
 0001:0000db11       ?_FilterSetCurrentException@@YAKPAU_EXCEPTION_POINTERS@@E@Z 1000eb11 f   libvcruntime:ehhelpers.obj
 0001:0000db70       $$000000                   1000eb70     libvcruntime:exsup4.obj
 0001:0000dbfd       __unwind_handler4          1000ebfd f   libvcruntime:exsup4.obj
 0001:0000def0       $$000000                   1000eef0     libvcruntime:exsup.obj
 0001:0000df11       __unwind_handler           1000ef11 f   libvcruntime:exsup.obj
 0001:0000e02e       ?try_get_first_available_module@@YAPAUHINSTANCE__@@QBW4module_id@?A0x15fb64ad@@0@Z 1000f02e f   libvcruntime:winapi_downlevel.obj
 0001:0000e0c8       ?try_get_function@@YAPAXW4function_id@?A0x15fb64ad@@QBDQBW4module_id@2@2@Z 1000f0c8 f   libvcruntime:winapi_downlevel.obj
 0001:0000e250       $$000000                   1000f250     libvcruntime:lowhelpr.obj
 0001:0000e2a0       $$000000                   1000f2a0     libvcruntime:memmove.obj
 0001:0000e504       TrailingUpVec              1000f504     libvcruntime:memmove.obj
 0001:0000e5b0       TrailingDownVec            1000f5b0     libvcruntime:memmove.obj
 0001:0000e820       $$000000                   1000f820     libucrt:strcmp.obj
 0001:0000e8b0       $$000000                   1000f8b0     libucrt:strcat.obj
 0001:0000e9b0       $$000000                   1000f9b0     libucrt:strncpy.obj
 0001:0000ead4       ??$thread_start@P6GIPAX@Z$00@@YGKQAX@Z 1000fad4 f   libucrt:thread.obj
 0001:0000eb52       ??1?$__crt_unique_heap_ptr@U__acrt_thread_parameter@@Uthread_parameter_free_policy@?A0x4e93fcdd@@@@QAE@XZ 1000fb52 f   libucrt:thread.obj
 0001:0000eb89       ?common_end_thread@@YAXI@Z 1000fb89 f   libucrt:thread.obj
 0001:0000ebe0       ?create_thread_parameter@@YAPAU__acrt_thread_parameter@@QAX0@Z 1000fbe0 f   libucrt:thread.obj
 0001:0000ecd0       $$000000                   1000fcd0     libucrt:strlen.obj
 0001:0000ed60       $$000000                   1000fd60     libucrt:strncat.obj
 0001:0000efe1       ??$?RV<lambda_9b2bd5c6bb91c5c032542faa5c3cb611>@@AAV<lambda_be68057ced330f874c40fe9612235e36>@@V<lambda_dbd837d1c0b7fc6e2d81c287c81c071b>@@@?$__crt_seh_guarded_call@H@@QAEH$$QAV<lambda_9b2bd5c6bb91c5c032542faa5c3cb611>@@AAV<lambda_be68057ced330f874c40fe9612235e36>@@$$QAV<lambda_dbd837d1c0b7fc6e2d81c287c81c071b>@@@Z 1000ffe1 f   libucrt:output.obj
 0001:0000f03c       ??$?RV<lambda_c29ee0499b841886b80d843682cc403a>@@AAV<lambda_0be4ab1c2a6918fda4e39227d83ea893>@@V<lambda_5a3ed3da325c8ea037a470278c0f2d16>@@@?$__crt_seh_guarded_call@H@@QAEH$$QAV<lambda_c29ee0499b841886b80d843682cc403a>@@AAV<lambda_0be4ab1c2a6918fda4e39227d83ea893>@@$$QAV<lambda_5a3ed3da325c8ea037a470278c0f2d16>@@@Z 1001003c f   libucrt:output.obj
 0001:0000f6cd       ??R<lambda_0be4ab1c2a6918fda4e39227d83ea893>@@QBEHXZ 100106cd f   libucrt:output.obj
 0001:0000f78c       ??R<lambda_be68057ced330f874c40fe9612235e36>@@QBEHXZ 1001078c f   libucrt:output.obj
 0001:0000fb61       $LN53                      10010b61     libucrt:output.obj
 0001:0000fc7d       $LN53                      10010c7d     libucrt:output.obj
 0001:0001065b       $LN20                      1001165b     libucrt:output.obj
 0001:0001066f       $LN17                      1001166f     libucrt:output.obj
 0001:000115e2       ??$common_fsopen@D@@YAPAU_iobuf@@QBD0H@Z 100125e2 f   libucrt:fopen.obj
 0001:000116b0       ??$common_getenv@D@@YAPADQBD@Z 100126b0 f   libucrt:getenv.obj
 0001:0001172f       ??$common_getenv_nolock@D@@YAPADQBD@Z 1001272f f   libucrt:getenv.obj
 0001:00011ecd       ??$?RV<lambda_03b1d95aef87969028cfba75ccab2455>@@AAV<lambda_6e4b09c48022b2350581041d5f6b0c4c>@@V<lambda_22bdf7517842c4b3e53723af5aa32b9e>@@@?$__crt_seh_guarded_call@X@@QAEX$$QAV<lambda_03b1d95aef87969028cfba75ccab2455>@@AAV<lambda_6e4b09c48022b2350581041d5f6b0c4c>@@$$QAV<lambda_22bdf7517842c4b3e53723af5aa32b9e>@@@Z 10012ecd f   libucrt:exit.obj
 0001:00011f1a       ??R<lambda_6e4b09c48022b2350581041d5f6b0c4c>@@QBE@XZ 10012f1a f   libucrt:exit.obj
 0001:00011ff4       ?atexit_exception_filter@@YAHK@Z 10012ff4 f   libucrt:exit.obj
 0001:00012007       ?common_exit@@YAXHW4_crt_exit_cleanup_mode@@W4_crt_exit_return_mode@@@Z 10013007 f   libucrt:exit.obj
 0001:0001206b       ?exit_or_terminate_process@@YAXI@Z 1001306b f   libucrt:exit.obj
 0001:000120ad       ?is_managed_app@@YA_NXZ    100130ad f   libucrt:exit.obj
 0001:000120f0       ?try_cor_exit_process@@YAXI@Z 100130f0 f   libucrt:exit.obj
 0001:0001217e       ??$common_configure_argv@D@@YAHW4_crt_argv_mode@@@Z 1001317e f   libucrt:argv_parsing.obj
 0001:000122b4       ??$parse_command_line@D@@YAXPADPAPAD0PAI2@Z 100132b4 f   libucrt:argv_parsing.obj
 0001:00012485       ??$common_get_or_create_environment_nolock@D@@YAPAPADXZ 10013485 f   libucrt:environment_initialization.obj
 0001:000124b1       ??$common_initialize_environment_nolock@D@@YAHXZ 100134b1 f   libucrt:environment_initialization.obj
 0001:00012504       ??$create_environment@D@@YAQAPADQAD@Z 10013504 f   libucrt:environment_initialization.obj
 0001:000125d4       ??$free_environment@D@@YAXQAPAD@Z 100135d4 f   libucrt:environment_initialization.obj
 0001:000125d4       ??$free_environment@_W@@YAXQAPA_W@Z 100135d4 f   libucrt:environment_initialization.obj
 0001:00012603       ??$initialize_environment_by_cloning_nolock@D@@YAHXZ 10013603 f   libucrt:environment_initialization.obj
 0001:000126af       ??$uninitialize_environment_internal@D@@YAXAAPAPAD@Z 100136af f   libucrt:environment_initialization.obj
 0001:000126ca       ??$uninitialize_environment_internal@_W@@YAXAAPAPA_W@Z 100136ca f   libucrt:environment_initialization.obj
 0001:00012726       ??$?RV<lambda_69a2805e680e0e292e8ba93315fe43a8>@@AAV<lambda_f03950bc5685219e0bcd2087efbe011e>@@V<lambda_03fcd07e894ec930e3f35da366ca99d6>@@@?$__crt_seh_guarded_call@H@@QAEH$$QAV<lambda_69a2805e680e0e292e8ba93315fe43a8>@@AAV<lambda_f03950bc5685219e0bcd2087efbe011e>@@$$QAV<lambda_03fcd07e894ec930e3f35da366ca99d6>@@@Z 10013726 f   libucrt:onexit.obj
 0001:00012781       ??R<lambda_f03950bc5685219e0bcd2087efbe011e>@@QBEHXZ 10013781 f   libucrt:onexit.obj
 0001:000128b1       _initialize_environment    100138b1 f   libucrt:initialization.obj
 0001:000128b1       _initialize_global_state_isolation 100138b1 f   libucrt:initialization.obj
 0001:000128b1       _report_memory_leaks       100138b1 f   libucrt:initialization.obj
 0001:000128b1       _uninitialize_c            100138b1 f   libucrt:initialization.obj
 0001:000128b1       _uninitialize_global_state_isolation 100138b1 f   libucrt:initialization.obj
 0001:000128b4       _initialize_global_variables 100138b4 f   libucrt:initialization.obj
 0001:000128c1       _initialize_c              100138c1 f   libucrt:initialization.obj
 0001:000128db       _uninitialize_environment  100138db f   libucrt:initialization.obj
 0001:000128e3       _initialize_pointers       100138e3 f   libucrt:initialization.obj
 0001:00012911       _uninitialize_vcruntime    10013911 f   libucrt:initialization.obj
 0001:0001291a       _uninitialize_allocated_memory 1001391a f   libucrt:initialization.obj
 0001:00012931       _uninitialize_allocated_io_buffers 10013931 f   libucrt:initialization.obj
 0001:000129a0       ??R<lambda_af42a3ee9806e9a7305d451646e05244>@@QBEXAAPAU__crt_multibyte_data@@@Z 100139a0 f   libucrt:initialization.obj
 0001:00013420       $$000000                   10014420     libucrt:strncmp.obj
 0001:000137f0       ??$?RV<lambda_15ade71b0218206bbe3333a0c9b79046>@@AAV<lambda_da44e0f8b0f19ba52fefafb335991732>@@V<lambda_207f2d024fc103971653565357d6cd41>@@@?$__crt_seh_guarded_call@X@@QAEX$$QAV<lambda_15ade71b0218206bbe3333a0c9b79046>@@AAV<lambda_da44e0f8b0f19ba52fefafb335991732>@@$$QAV<lambda_207f2d024fc103971653565357d6cd41>@@@Z 100147f0 f   libucrt:per_thread_data.obj
 0001:00013842       ??$?RV<lambda_38edbb1296d33220d7e4dd0ed76b244a>@@AAV<lambda_5ce1d447e08cb34b2473517608e21441>@@V<lambda_fb385d3da700c9147fc39e65dd577a8c>@@@?$__crt_seh_guarded_call@X@@QAEX$$QAV<lambda_38edbb1296d33220d7e4dd0ed76b244a>@@AAV<lambda_5ce1d447e08cb34b2473517608e21441>@@$$QAV<lambda_fb385d3da700c9147fc39e65dd577a8c>@@@Z 10014842 f   libucrt:per_thread_data.obj
 0001:000138ad       ??$?RV<lambda_6affb1475c98b40b75cdec977db92e3c>@@AAV<lambda_b8d4b9c228a6ecc3f80208dbb4b4a104>@@V<lambda_608742c3c92a14382c1684fc64f96c88>@@@?$__crt_seh_guarded_call@X@@QAEX$$QAV<lambda_6affb1475c98b40b75cdec977db92e3c>@@AAV<lambda_b8d4b9c228a6ecc3f80208dbb4b4a104>@@$$QAV<lambda_608742c3c92a14382c1684fc64f96c88>@@@Z 100148ad f   libucrt:per_thread_data.obj
 0001:00013902       ??$?RV<lambda_a7e850c220f1c8d1e6efeecdedd162c6>@@AAV<lambda_46720907175c18b6c9d2717bc0d2d362>@@V<lambda_9048902d66e8d99359bc9897bbb930a8>@@@?$__crt_seh_guarded_call@X@@QAEX$$QAV<lambda_a7e850c220f1c8d1e6efeecdedd162c6>@@AAV<lambda_46720907175c18b6c9d2717bc0d2d362>@@$$QAV<lambda_9048902d66e8d99359bc9897bbb930a8>@@@Z 10014902 f   libucrt:per_thread_data.obj
 0001:0001395c       ?construct_ptd@@YAXQAU__acrt_ptd@@QAPAU__crt_locale_data@@@Z 1001495c f   libucrt:per_thread_data.obj
 0001:000139f5       ?destroy_fls@@YGXPAX@Z     100149f5 f   libucrt:per_thread_data.obj
 0001:00013a16       ?destroy_ptd@@YAXQAU__acrt_ptd@@@Z 10014a16 f   libucrt:per_thread_data.obj
 0001:00013ae3       ?replace_current_thread_locale_nolock@@YAXQAU__acrt_ptd@@QAU__crt_locale_data@@@Z 10014ae3 f   libucrt:per_thread_data.obj
 0001:00013dac       ?try_get_AreFileApisANSI@@YAP6GHXZXZ 10014dac f   libucrt:winapi_thunks.obj
 0001:00013dc6       ?try_get_CompareStringEx@@YAP6GHPB_WK0H0HPAU_nlsversioninfo@@PAXJ@ZXZ 10014dc6 f   libucrt:winapi_thunks.obj
 0001:00013de0       ?try_get_LCMapStringEx@@YAP6GHPB_WK0HPA_WHPAU_nlsversioninfo@@PAXJ@ZXZ 10014de0 f   libucrt:winapi_thunks.obj
 0001:00013dfa       ?try_get_LocaleNameToLCID@@YAP6GKPB_WK@ZXZ 10014dfa f   libucrt:winapi_thunks.obj
 0001:00013e14       ?try_get_first_available_module@@YAPAUHINSTANCE__@@QBW4module_id@?A0x391cf84c@@0@Z 10014e14 f   libucrt:winapi_thunks.obj
 0001:00013edb       ?try_get_function@@YAPAXW4function_id@?A0x391cf84c@@QBDQBW4module_id@2@2@Z 10014edb f   libucrt:winapi_thunks.obj
 0001:0001441c       ??$?RV<lambda_2866be3712abc81a800a822484c830d8>@@AAV<lambda_39ca0ed439415581b5b15c265174cece>@@V<lambda_2b24c74d71094a6cd0cb82e44167d71b>@@@?$__crt_seh_guarded_call@X@@QAEX$$QAV<lambda_2866be3712abc81a800a822484c830d8>@@AAV<lambda_39ca0ed439415581b5b15c265174cece>@@$$QAV<lambda_2b24c74d71094a6cd0cb82e44167d71b>@@@Z 1001541c f   libucrt:fflush.obj
 0001:000144a8       ??$?RV<lambda_2cc53f568c5a2bb6f192f930a45d44ea>@@AAV<lambda_ab61a845afdef5b7c387490eaf3616ee>@@V<lambda_c2ffc0b7726aa6be21d5f0026187e748>@@@?$__crt_seh_guarded_call@X@@QAEX$$QAV<lambda_2cc53f568c5a2bb6f192f930a45d44ea>@@AAV<lambda_ab61a845afdef5b7c387490eaf3616ee>@@$$QAV<lambda_c2ffc0b7726aa6be21d5f0026187e748>@@@Z 100154a8 f   libucrt:fflush.obj
 0001:00014554       ?common_flush_all@@YAH_N@Z 10015554 f   libucrt:fflush.obj
 0001:000145a1       ?common_flush_all_should_try_to_flush_stream@@YA_NV__crt_stdio_stream@@QAH@Z 100155a1 f   libucrt:fflush.obj
 0001:000145d4       ?is_stream_flushable_or_commitable@@YA_NJ@Z 100155d4 f   libucrt:fflush.obj
 0001:000146ef       ?initialize_inherited_file_handles_nolock@@YAXXZ 100156ef f   libucrt:ioinit.obj
 0001:000147a5       ?initialize_stdio_handles_nolock@@YAXXZ 100157a5 f   libucrt:ioinit.obj
 0001:00014d32       ?fp_format_a@@YAHQBNPADIQADIH_NIQAU__crt_locale_pointers@@@Z 10015d32 f   libucrt:cvt.obj
 0001:0001504b       ?fp_format_e@@YAHQBNQADI1IH_NIQAU__crt_locale_pointers@@@Z 1001604b f   libucrt:cvt.obj
 0001:000150ed       ?fp_format_e_internal@@YAHQADIH_NIQAU_strflt@@1QAU__crt_locale_pointers@@@Z 100160ed f   libucrt:cvt.obj
 0001:00015235       ?fp_format_f@@YAHQBNQADI1IHQAU__crt_locale_pointers@@@Z 10016235 f   libucrt:cvt.obj
 0001:000152c0       ?fp_format_f_internal@@YAHQADIHQAU_strflt@@_NQAU__crt_locale_pointers@@@Z 100162c0 f   libucrt:cvt.obj
 0001:00015391       ?fp_format_g@@YAHQBNQADI1IH_NIQAU__crt_locale_pointers@@@Z 10016391 f   libucrt:cvt.obj
 0001:00015452       ?fp_format_nan_or_infinity@@YAHW4__acrt_fp_class@@_NPADI1@Z 10016452 f   libucrt:cvt.obj
 0001:000154e7       ?shift_bytes@@YAXQADI0H@Z  100164e7 f   libucrt:cvt.obj
 0001:00015656       ?fputwc_binary_nolock@@YAG_WV__crt_stdio_stream@@@Z 10016656 f   libucrt:fputwc.obj
 0001:00015901       ??$?RV<lambda_e5124f882df8998aaf41531e079ba474>@@AAV<lambda_3e16ef9562a7dcce91392c22ab16ea36>@@V<lambda_e25ca0880e6ef98be67edffd8c599615>@@@?$__crt_seh_guarded_call@X@@QAEX$$QAV<lambda_e5124f882df8998aaf41531e079ba474>@@AAV<lambda_3e16ef9562a7dcce91392c22ab16ea36>@@$$QAV<lambda_e25ca0880e6ef98be67edffd8c599615>@@@Z 10016901 f   libucrt:wsetlocale.obj
 0001:000159a1       ??$?RV<lambda_218ce3db14220d0be481dae8ef3383b6>@@AAV<lambda_628dfdc04ba53c8bfc02c9951375f3f5>@@V<lambda_57dc472bd5c9d5f3b2cbca59b8a843ae>@@@?$__crt_seh_guarded_call@H@@QAEH$$QAV<lambda_218ce3db14220d0be481dae8ef3383b6>@@AAV<lambda_628dfdc04ba53c8bfc02c9951375f3f5>@@$$QAV<lambda_57dc472bd5c9d5f3b2cbca59b8a843ae>@@@Z 100169a1 f   libucrt:close.obj
 0001:00015bfa       ?find_or_allocate_unused_stream_nolock@@YA?AV__crt_stdio_stream@@XZ 10016bfa f   libucrt:stream.obj
 0001:00015ee6       ??$common_openfile@D@@YAPAU_iobuf@@QBD0HV__crt_stdio_stream@@@Z 10016ee6 f   libucrt:openfile.obj
 0001:00016219       ?<lambda_invoker_cdecl>@<lambda_838c7f62c73c983481e27c09e84b0b5d>@@CAHPBX0@Z 10017219 f   libucrt:argv_wildcards.obj
 0001:00016231       ??$__acrt_convert_wcs_mbs_cp@D_WV<lambda_62f6974d9771e494a5ea317cc32e971c>@@U__crt_win32_buffer_internal_dynamic_resizing@@@@YAHQBDAAV?$__crt_win32_buffer@_WU__crt_win32_buffer_internal_dynamic_resizing@@@@ABV<lambda_62f6974d9771e494a5ea317cc32e971c>@@I@Z 10017231 f   libucrt:argv_wildcards.obj
 0001:000162e3       ??$__acrt_convert_wcs_mbs_cp@_WDV<lambda_28bda7af82a03b66c1cb3803a755f95d>@@U__crt_win32_buffer_internal_dynamic_resizing@@@@YAHQB_WAAV?$__crt_win32_buffer@DU__crt_win32_buffer_internal_dynamic_resizing@@@@ABV<lambda_28bda7af82a03b66c1cb3803a755f95d>@@I@Z 100172e3 f   libucrt:argv_wildcards.obj
 0001:000163cf       ??$common_expand_argv_wildcards@D@@YAHQAPADQAPAPAD@Z 100173cf f   libucrt:argv_wildcards.obj
 0001:000165be       ??$copy_and_add_argument_to_buffer@D@@YAHQBD0IAAV?$argument_list@D@?A0x5f5c8891@@@Z 100175be f   libucrt:argv_wildcards.obj
 0001:0001666f       ??$expand_argument_wildcards@D@@YAHQAD0AAV?$argument_list@D@?A0x5f5c8891@@@Z 1001766f f   libucrt:argv_wildcards.obj
 0001:000169b9       ?expand_if_necessary@?$argument_list@D@?A0x5f5c8891@@AAEHXZ 100179b9 f   libucrt:argv_wildcards.obj
 0001:00016a4b       ??$__acrt_convert_wcs_mbs_cp@_WDV<lambda_0fec1a7b3f42a53036604e18c2d5e07e>@@U__crt_win32_buffer_no_resizing@@@@YAHQB_WAAV?$__crt_win32_buffer@DU__crt_win32_buffer_no_resizing@@@@ABV<lambda_0fec1a7b3f42a53036604e18c2d5e07e>@@I@Z 10017a4b f   libucrt:getmodulefilenamea.obj
 0001:00016bee       ??$?RV<lambda_ceb1ee4838e85a9d631eb091e2fbe199>@@AAV<lambda_ae742caa10f662c28703da3d2ea5e57e>@@V<lambda_cd08b5d6af4937fe54fc07d0c9bf6b37>@@@?$__crt_seh_guarded_call@X@@QAEX$$QAV<lambda_ceb1ee4838e85a9d631eb091e2fbe199>@@AAV<lambda_ae742caa10f662c28703da3d2ea5e57e>@@$$QAV<lambda_cd08b5d6af4937fe54fc07d0c9bf6b37>@@@Z 10017bee f   libucrt:mbctype.obj
 0001:00016c3b       ??R<lambda_ae742caa10f662c28703da3d2ea5e57e>@@QBEXXZ 10017c3b f   libucrt:mbctype.obj
 0001:00016cbe       ?CPtoLocaleName@@YAPB_WH@Z 10017cbe f   libucrt:mbctype.obj
 0001:00016cfc       ?getSystemCP@@YAHH@Z       10017cfc f   libucrt:mbctype.obj
 0001:00016d6d       ?setSBCS@@YAXPAU__crt_multibyte_data@@@Z 10017d6d f   libucrt:mbctype.obj
 0001:00016dd2       ?setSBUpLow@@YAXPAU__crt_multibyte_data@@@Z 10017dd2 f   libucrt:mbctype.obj
 0001:00016f53       ?setmbcp_internal@@YAHH_NQAU__acrt_ptd@@QAPAU__crt_multibyte_data@@@Z 10017f53 f   libucrt:mbctype.obj
 0001:0001706c       ?update_thread_multibyte_data_internal@@YAPAU__crt_multibyte_data@@QAU__acrt_ptd@@QAPAU1@@Z 1001806c f   libucrt:mbctype.obj
 0001:0001735a       _memcpy_s                  1001835a f   libucrt:cfout.obj
 0001:0001735a       _memcpy_s                  1001835a f   libucrt:mbctype.obj
 0001:000173db       ?x_ismbbtype_l@@YAHPAU__crt_locale_pointers@@IHH@Z 100183db f   libucrt:ismbbyte.obj
 0001:0001758c       ?find_end_of_double_null_terminated_sequence@@YAPB_WQB_W@Z 1001858c f   libucrt:get_environment_from_os.obj
 0001:00017647       ??$common_set_variable_in_environment_nolock@D@@YAHQADH@Z 10018647 f   libucrt:setenv.obj
 0001:00017885       ??$copy_environment@D@@YAPAPADQAPAD@Z 10018885 f   libucrt:setenv.obj
 0001:00017935       ??$ensure_current_environment_is_not_initial_environment_nolock@D@@YAXXZ 10018935 f   libucrt:setenv.obj
 0001:0001794f       ??$find_in_environment_nolock@D@@YAHQBDI@Z 1001894f f   libucrt:setenv.obj
 0001:00017ad0       ??$?RV<lambda_cbab9ec6f41b0180b23cc171c22676b0>@@AAV<lambda_44731a7d0e6d81c3e6aa82d741081786>@@V<lambda_4b292cb8dd18144e164572427af410ab>@@@?$__crt_seh_guarded_call@P6AXH@Z@@QAEP6AXH@Z$$QAV<lambda_cbab9ec6f41b0180b23cc171c22676b0>@@AAV<lambda_44731a7d0e6d81c3e6aa82d741081786>@@$$QAV<lambda_4b292cb8dd18144e164572427af410ab>@@@Z 10018ad0 f   libucrt:signal.obj
 0001:00017b34       ?get_global_action_nolock@@YAPAP6AXH@ZH@Z 10018b34 f   libucrt:signal.obj
 0001:00017b76       ?siglookup@@YAPAU__crt_signal_action_t@@HQAU1@@Z 10018b76 f   libucrt:signal.obj
 0001:00018339       ?GetTableIndexFromLocaleName@@YAHPB_W@Z 10019339 f   libucrt:lcidtoname_downlevel.obj
 0001:000183b5       ??$?RV<lambda_9e9de3de5fa147e2223d7db92bc10aa6>@@AAV<lambda_38ce7e780aa69e748d6df282ebc68efe>@@V<lambda_8ca6da459f0f6780f1cff60fdc3d00e5>@@@?$__crt_seh_guarded_call@H@@QAEH$$QAV<lambda_9e9de3de5fa147e2223d7db92bc10aa6>@@AAV<lambda_38ce7e780aa69e748d6df282ebc68efe>@@$$QAV<lambda_8ca6da459f0f6780f1cff60fdc3d00e5>@@@Z 100193b5 f   libucrt:commit.obj
 0001:000184d4       ?write_double_translated_ansi_nolock@@YA?AUwrite_result@?A0x17268360@@HQBDI@Z 100194d4 f   libucrt:write.obj
 0001:0001887e       ?write_double_translated_unicode_nolock@@YA?AUwrite_result@?A0x17268360@@QBDI@Z 1001987e f   libucrt:write.obj
 0001:000188e6       ?write_requires_double_translation_nolock@@YA_NH@Z 100198e6 f   libucrt:write.obj
 0001:00018957       ?write_text_ansi_nolock@@YA?AUwrite_result@?A0x17268360@@HQBDI@Z 10019957 f   libucrt:write.obj
 0001:00018a32       ?write_text_utf16le_nolock@@YA?AUwrite_result@?A0x17268360@@HQBDI@Z 10019a32 f   libucrt:write.obj
 0001:00018b1b       ?write_text_utf8_nolock@@YA?AUwrite_result@?A0x17268360@@HQBDI@Z 10019b1b f   libucrt:write.obj
 0001:0001938f       ??R<lambda_3d301b9e52f5099be73030e1f0bf487e>@@QBEIPBD@Z 1001a38f f   libucrt:mbrtowc.obj
 0001:0001ae62       ??$common_flush_and_write_nolock@D@@YAHHV__crt_stdio_stream@@@Z 1001be62 f   libucrt:_flsbuf.obj
 0001:0001af77       ??$common_flush_and_write_nolock@_W@@YAHHV__crt_stdio_stream@@@Z 1001bf77 f   libucrt:_flsbuf.obj
 0001:0001b090       ??$write_buffer_nolock@D@@YA_NDV__crt_stdio_stream@@@Z 1001c090 f   libucrt:_flsbuf.obj
 0001:0001b15c       ??$write_buffer_nolock@_W@@YA_N_WV__crt_stdio_stream@@@Z 1001c15c f   libucrt:_flsbuf.obj
 0001:0001b22a       ?stream_is_at_end_of_file_nolock@@YA_NV__crt_stdio_stream@@@Z 1001c22a f   libucrt:_flsbuf.obj
 0001:0001b482       ?free_crt_array_internal@@YAXQAPBXI@Z 1001c482 f   libucrt:inittime.obj
 0001:0001b846       ??$common_sopen_dispatch@D@@YAHQBDHHHQAHH@Z 1001c846 f   libucrt:open.obj
 0001:0001b907       ?configure_text_mode@@YAHHUfile_options@?A0xa9d50aae@@HAAW4__crt_lowio_text_mode@@@Z 1001c907 f   libucrt:open.obj
 0001:0001bb5a       ?create_file@@YAPAXQB_WQAU_SECURITY_ATTRIBUTES@@Ufile_options@?A0xa9d50aae@@@Z 1001cb5a f   libucrt:open.obj
 0001:0001bb7f       ?decode_open_create_flags@@YAKH@Z 1001cb7f f   libucrt:open.obj
 0001:0001bbef       ?decode_options@@YA?AUfile_options@?A0xa9d50aae@@HHH@Z 1001cbef f   libucrt:open.obj
 0001:0001bd69       ?truncate_ctrl_z_if_present@@YAHH@Z 1001cd69 f   libucrt:open.obj
 0001:0001c1ce       ?InternalCompareStringA@@YAHPAU__crt_locale_pointers@@PB_WKPBDH2HH@Z 1001d1ce f   libucrt:comparestringa.obj
 0001:0001c4a0       ?swap@@YAXPAD0I@Z          1001d4a0 f   libucrt:qsort.obj
 0001:0001c924       ??$common_tcsncpy_s@D@@YAHQADIQBDI@Z 1001d924 f   libucrt:strncpy_s.obj
 0001:0001c9f0       $$000000                   1001d9f0     libucrt:strpbrk.obj
 0001:0001cad4       ?__acrt_LCMapStringA_stat@@YAHPAU__crt_locale_pointers@@PB_WKPBDHPADHHH@Z 1001dad4 f   libucrt:lcmapstringa.obj
 0001:0001cd07       ?initialize_multibyte@@YAHXZ 1001dd07 f   libucrt:multibyte_initializer.obj
 0001:0001ce60       ??$common_lseek@_J@@YA_JH_JH@Z 1001de60 f   libucrt:lseek.obj
 0001:0001cf6c       ??$common_lseek_nolock@_J@@YA_JH_JH@Z 1001df6c f   libucrt:lseek.obj
 0001:0001d050       ??$translate_text_mode_nolock@D@@YAHHQADI@Z 1001e050 f   libucrt:read.obj
 0001:0001d1b1       ??$translate_text_mode_nolock@_W@@YAHHQA_WI@Z 1001e1b1 f   libucrt:read.obj
 0001:0001d382       ?translate_ansi_or_utf8_nolock@@YAHHQADIQA_WI@Z 1001e382 f   libucrt:read.obj
 0001:0001d4d9       ?translate_utf16_from_console_nolock@@YAHHQA_WI@Z 1001e4d9 f   libucrt:read.obj
 0001:0001db70       $$000000                   1001eb70     libucrt:log10_impl.obj
 0001:0001dc80       $$000000                   1001ec80     libucrt:ceil_pentium4.obj
 0001:0001de00       $$000000                   1001ee00     libucrt:_strnicm.obj
 0001:0001e136       ?__dcrt_lowio_initialize_console_output@@YAXXZ 1001f136 f   libucrt:initcon.obj
 0001:0001e1e0       ?to_abstract_control@@YA?AW4__acrt_fenv_abstract_control@@W4__acrt_fenv_machine_sse_control@@@Z 1001f1e0 f   libucrt:_fenvutils.obj
 0001:0001e29c       ?to_abstract_control@@YA?AW4__acrt_fenv_abstract_control@@W4__acrt_fenv_machine_x87_control@@@Z 1001f29c f   libucrt:_fenvutils.obj
 0001:0001e355       ?to_machine_sse_control@@YA?AW4__acrt_fenv_machine_sse_control@@W4__acrt_fenv_abstract_control@@@Z 1001f355 f   libucrt:_fenvutils.obj
 0001:0001e422       ?to_machine_x87_control@@YA?AW4__acrt_fenv_machine_x87_control@@W4__acrt_fenv_abstract_control@@@Z 1001f422 f   libucrt:_fenvutils.obj
 0001:0001e880       $$000000                   1001f880     libucrt:log10_pentium4.obj
 0001:0001eb10       $$000000                   1001fb10     libucrt:87tran.obj
 0001:0001ed20       $$000000                   1001fd20     libucrt:87disp.obj
 0001:0001ef80       $$000000                   1001ff80     libucrt:common.obj
 0001:0001f110       $$000000                   10020110     libucrt:genexcep.obj
 0001:00020190       $$000000                   10021190     LIBCMT:ulldvrm.obj
 0001:00020230       $$000000                   10021230     LIBCMT:llmul.obj
 0001:00020270       $$000000                   10021270     LIBCMT:lldvrm.obj
 0001:00020350       $$000000                   10021350     LIBCMT:ullshr.obj
 0001:00020370       $$000000                   10021370     LIBCMT:chkstk.obj
 0001:000203a0       $$000000                   100213a0     LIBCMT:llshl.obj
 0001:000203c0       $$000000                   100213c0     LIBCMT:ftol2.obj
 0001:00020660       $$000000                   10021660     LIBCMT:alloca16.obj
 0001:00020690       $$000000                   10021690     libvcruntime:strrchr.obj
 0001:000207d0       $$000000                   100217d0     libvcruntime:strchr.obj
 0002:0000f444       _GS_ExceptionPointers      10031444     LIBCMT:gs_report.obj
 0002:0000f458       ?tokenTable@@3QBUStringLiteral@@B 10031458     libvcruntime:undname.obj
 0002:0000f4d8       ?nameTable@@3QBUStringLiteral@@B 100314d8     libvcruntime:undname.obj
 0002:0000f770       ?rttiTable@@3QBUStringLiteral@@B 10031770     libvcruntime:undname.obj
 0002:0000f798       ?IndirectionName@@3QBUStringLiteral@@B 10031798     libvcruntime:undname.obj
 0002:0000f7c8       ?PrefixName@@3QBUStringLiteral@@B 100317c8     libvcruntime:undname.obj
 0002:0000fdf8       ?module_names@?A0x15fb64ad@@3QBQB_WB 10031df8     libvcruntime:winapi_downlevel.obj
 0002:0000fea0       ?candidate_modules@?1??try_get_FlsAlloc@@YAP6GKP6GXPAX@Z@ZXZ@4QBW4module_id@?A0x15fb64ad@@B 10031ea0     libvcruntime:winapi_downlevel.obj
 0002:0000feb4       ?candidate_modules@?1??try_get_FlsFree@@YAP6GHK@ZXZ@4QBW4module_id@?A0x15fb64ad@@B 10031eb4     libvcruntime:winapi_downlevel.obj
 0002:0000fec4       ?candidate_modules@?1??try_get_FlsGetValue@@YAP6GPAXK@ZXZ@4QBW4module_id@?A0x15fb64ad@@B 10031ec4     libvcruntime:winapi_downlevel.obj
 0002:0000fed8       ?candidate_modules@?1??try_get_FlsSetValue@@YAP6GHKPAX@ZXZ@4QBW4module_id@?A0x15fb64ad@@B 10031ed8     libvcruntime:winapi_downlevel.obj
 0002:0000feec       ?candidate_modules@?1??try_get_InitializeCriticalSectionEx@@YAP6GHPAU_RTL_CRITICAL_SECTION@@KK@ZXZ@4QBW4module_id@?A0x15fb64ad@@B 10031eec     libvcruntime:winapi_downlevel.obj
 0002:00010040       ___acrt_initializers       10032040     libucrt:initialization.obj
 0002:000100c0       ?errtable@@3QBUerrentry@?A0x31fdb9ec@@B 100320c0     libucrt:errno.obj
 0002:00010228       ?module_names@?A0x391cf84c@@3QBQB_WB 10032228     libucrt:winapi_thunks.obj
 0002:000106a0       ?candidate_modules@?1??try_get_AreFileApisANSI@@YAP6GHXZXZ@4QBW4module_id@?A0x391cf84c@@B 100326a0     libucrt:winapi_thunks.obj
 0002:000106b4       ?candidate_modules@?1??try_get_CompareStringEx@@YAP6GHPB_WK0H0HPAU_nlsversioninfo@@PAXJ@ZXZ@4QBW4module_id@?A0x391cf84c@@B 100326b4     libucrt:winapi_thunks.obj
 0002:000106cc       ?candidate_modules@?1??try_get_FlsAlloc@@YAP6GKP6GXPAX@Z@ZXZ@4QBW4module_id@?A0x391cf84c@@B 100326cc     libucrt:winapi_thunks.obj
 0002:000106d4       ?candidate_modules@?1??try_get_FlsFree@@YAP6GHK@ZXZ@4QBW4module_id@?A0x391cf84c@@B 100326d4     libucrt:winapi_thunks.obj
 0002:000106dc       ?candidate_modules@?1??try_get_FlsGetValue@@YAP6GPAXK@ZXZ@4QBW4module_id@?A0x391cf84c@@B 100326dc     libucrt:winapi_thunks.obj
 0002:000106e4       ?candidate_modules@?1??try_get_FlsSetValue@@YAP6GHKPAX@ZXZ@4QBW4module_id@?A0x391cf84c@@B 100326e4     libucrt:winapi_thunks.obj
 0002:000106ec       ?candidate_modules@?1??try_get_InitializeCriticalSectionEx@@YAP6GHPAU_RTL_CRITICAL_SECTION@@KK@ZXZ@4QBW4module_id@?A0x391cf84c@@B 100326ec     libucrt:winapi_thunks.obj
 0002:000106f4       ?candidate_modules@?1??try_get_LCMapStringEx@@YAP6GHPB_WK0HPA_WHPAU_nlsversioninfo@@PAXJ@ZXZ@4QBW4module_id@?A0x391cf84c@@B 100326f4     libucrt:winapi_thunks.obj
 0002:0001070c       ?candidate_modules@?1??try_get_LocaleNameToLCID@@YAP6GKPB_WK@ZXZ@4QBW4module_id@?A0x391cf84c@@B 1003270c     libucrt:winapi_thunks.obj
 0002:00010728       ?candidate_modules@?1??try_get_RoInitialize@@YAP6GJW4RO_INIT_TYPE@@@ZXZ@4QBW4module_id@?A0x391cf84c@@B 10032728     libucrt:winapi_thunks.obj
 0002:0001073c       ?candidate_modules@?1??try_get_RoUninitialize@@YAP6GXXZXZ@4QBW4module_id@?A0x391cf84c@@B 1003273c     libucrt:winapi_thunks.obj
 0002:00010750       ?candidate_modules@?1??try_get_AppPolicyGetProcessTerminationMethod@@YAP6GJPAXPAW4AppPolicyProcessTerminationMethod@@@ZXZ@4QBW4module_id@?A0x391cf84c@@B 10032750     libucrt:winapi_thunks.obj
 0002:0001077c       ?candidate_modules@?1??try_get_AppPolicyGetThreadInitializationType@@YAP6GJPAXPAW4AppPolicyThreadInitializationType@@@ZXZ@4QBW4module_id@?A0x391cf84c@@B 1003277c     libucrt:winapi_thunks.obj
 0002:000107a8       ?strings@?1??fp_format_nan_or_infinity@@YAHW4__acrt_fp_class@@_NPADI1@Z@4QAY03QBDA 100327a8     libucrt:cvt.obj
 0002:00010d0c       ?_mb_locale_names@@3QBQB_WB 10032d0c     libucrt:mbctype.obj
 0002:00011558       ?LcidToLocaleNameTable@?A0x881e4c05@@3QBULcidToLocaleName@1@B 10033558     libucrt:lcidtoname_downlevel.obj
 0002:00012680       ?LocaleNameToIndexTable@?A0x881e4c05@@3QBULocaleNameIndex@1@B 10034680     libucrt:lcidtoname_downlevel.obj
 0002:00013ed8       ?large_power_indices@?1??multiply_by_power_of_ten@__crt_strtox@@YA_NAAUbig_integer@2@I@Z@4QBUunpack_index@?1??12@YA_N0I@Z@B 10035ed8     libucrt:cfout.obj
 0002:00013fc0       LOG_name                   10035fc0     libucrt:log10_impl.obj
 0002:00013fd0       _One                       10035fd0     libucrt:ceil_pentium4.obj
 0002:00013fe0       _Bns                       10035fe0     libucrt:ceil_pentium4.obj
 0002:00013ff0       _Zero                      10035ff0     libucrt:ceil_pentium4.obj
 0002:00014000       _S                         10036000     libucrt:ceil_pentium4.obj
 0002:00014010       _NegZero                   10036010     libucrt:ceil_pentium4.obj
 0002:00014030       emask                      10036030     libucrt:log10_pentium4.obj
 0002:00014040       CC                         10036040     libucrt:log10_pentium4.obj
 0002:00014050       Magic                      10036050     libucrt:log10_pentium4.obj
 0002:00014060       hi_mask                    10036060     libucrt:log10_pentium4.obj
 0002:00014070       LOG10_2                    10036070     libucrt:log10_pentium4.obj
 0002:00014080       place_L                    10036080     libucrt:log10_pentium4.obj
 0002:000140a0       One                        100360a0     libucrt:log10_pentium4.obj
 0002:000140b0       Zero                       100360b0     libucrt:log10_pentium4.obj
 0002:000140c0       Two52                      100360c0     libucrt:log10_pentium4.obj
 0002:000140d0       Infs                       100360d0     libucrt:log10_pentium4.obj
 0002:000140e0       NaN                        100360e0     libucrt:log10_pentium4.obj
 0002:000140f0       coeff                      100360f0     libucrt:log10_pentium4.obj
 0002:0001414e       _log2max                   1003614e     libucrt:87tran.obj
 0002:00014158       _smallarg                  10036158     libucrt:87tran.obj
 0002:00014162       _half                      10036162     libucrt:87tran.obj
 0002:000141ae       One                        100361ae     libucrt:87disp.obj
 0002:000141b6       Three                      100361b6     libucrt:87disp.obj
 0002:000141be       XAMtoTagTab                100361be     libucrt:87disp.obj
 0002:000141d0       One                        100361d0     libucrt:common.obj
 0002:000141e4       DblMax                     100361e4     libucrt:common.obj
 0002:000141ec       DblMin                     100361ec     libucrt:common.obj
 0002:000141f4       IeeeAdjO                   100361f4     libucrt:common.obj
 0002:000141fc       IeeeAdjU                   100361fc     libucrt:common.obj
 0002:00014204       _infinity                  10036204     libucrt:common.obj
 0002:0001420c       _zero                      1003620c     libucrt:common.obj
 0002:00014248       _over                      10036248     libucrt:fpctrl.obj
 0002:00014254       _under                     10036254     libucrt:fpctrl.obj
 0002:00014a88       ?_names@?1??_get_fname@@9@9 10036a88     libucrt:fpexcept.obj
 0002:00014c30       two32                      10036c30     LIBCMT:ftol2.obj
 0002:00014c34       two63                      10036c34     LIBCMT:ftol2.obj
 0002:00014c38       _NaN                       10036c38     LIBCMT:ftol2.obj
 0002:000151a0       __sehtable$?dllmain_crt_process_attach@@YAHQAUHINSTANCE__@@QAX@Z 100371a0     LIBCMT:dll_dllmain.obj
 0002:000151c0       __sehtable$?dllmain_crt_process_detach@@YAH_N@Z 100371c0     LIBCMT:dll_dllmain.obj
 0002:000151e8       __sehtable$?dllmain_dispatch@@YAHQAUHINSTANCE__@@KQAX@Z 100371e8     LIBCMT:dll_dllmain.obj
 0002:00015298       __sehtable$___scrt_is_nonwritable_in_current_image 10037298     LIBCMT:utility.obj
 0002:000152b8       __sehtable$___DestructExceptionObject 100372b8     libvcruntime:ehhelpers.obj
 0002:000152d8       __sehtable$??$thread_start@P6GIPAX@Z$00@@YGKQAX@Z 100372d8     libucrt:thread.obj
 0002:000152f8       __sehtable$??$?RV<lambda_c29ee0499b841886b80d843682cc403a>@@AAV<lambda_0be4ab1c2a6918fda4e39227d83ea893>@@V<lambda_5a3ed3da325c8ea037a470278c0f2d16>@@@?$__crt_seh_guarded_call@H@@QAEH$$QAV<lambda_c29ee0499b841886b80d843682cc403a>@@AAV<lambda_0be4ab1c2a6918fda4e39227d83ea893>@@$$QAV<lambda_5a3ed3da325c8ea037a470278c0f2d16>@@@Z 100372f8     libucrt:output.obj
 0002:00015318       __sehtable$??$?RV<lambda_9b2bd5c6bb91c5c032542faa5c3cb611>@@AAV<lambda_be68057ced330f874c40fe9612235e36>@@V<lambda_dbd837d1c0b7fc6e2d81c287c81c071b>@@@?$__crt_seh_guarded_call@H@@QAEH$$QAV<lambda_9b2bd5c6bb91c5c032542faa5c3cb611>@@AAV<lambda_be68057ced330f874c40fe9612235e36>@@$$QAV<lambda_dbd837d1c0b7fc6e2d81c287c81c071b>@@@Z 10037318     libucrt:output.obj
 0002:00015338       __sehtable$_fclose         10037338     libucrt:fclose.obj
 0002:00015358       __sehtable$??$common_fsopen@D@@YAPAU_iobuf@@QBD0H@Z 10037358     libucrt:fopen.obj
 0002:00015378       __sehtable$??$common_getenv@D@@YAPADQBD@Z 10037378     libucrt:getenv.obj
 0002:00015398       __sehtable$__query_new_handler 10037398     libucrt:new_handler.obj
 0002:000153b8       __sehtable$??R<lambda_6e4b09c48022b2350581041d5f6b0c4c>@@QBE@XZ 100373b8     libucrt:exit.obj
 0002:000153d8       __sehtable$??$?RV<lambda_03b1d95aef87969028cfba75ccab2455>@@AAV<lambda_6e4b09c48022b2350581041d5f6b0c4c>@@V<lambda_22bdf7517842c4b3e53723af5aa32b9e>@@@?$__crt_seh_guarded_call@X@@QAEX$$QAV<lambda_03b1d95aef87969028cfba75ccab2455>@@AAV<lambda_6e4b09c48022b2350581041d5f6b0c4c>@@$$QAV<lambda_22bdf7517842c4b3e53723af5aa32b9e>@@@Z 100373d8     libucrt:exit.obj
 0002:000153f8       __sehtable$??$?RV<lambda_69a2805e680e0e292e8ba93315fe43a8>@@AAV<lambda_f03950bc5685219e0bcd2087efbe011e>@@V<lambda_03fcd07e894ec930e3f35da366ca99d6>@@@?$__crt_seh_guarded_call@H@@QAEH$$QAV<lambda_69a2805e680e0e292e8ba93315fe43a8>@@AAV<lambda_f03950bc5685219e0bcd2087efbe011e>@@$$QAV<lambda_03fcd07e894ec930e3f35da366ca99d6>@@@Z 100373f8     libucrt:onexit.obj
 0002:00015418       __sehtable$_terminate      10037418     libucrt:terminate.obj
 0002:00015438       __sehtable$??$?RV<lambda_15ade71b0218206bbe3333a0c9b79046>@@AAV<lambda_da44e0f8b0f19ba52fefafb335991732>@@V<lambda_207f2d024fc103971653565357d6cd41>@@@?$__crt_seh_guarded_call@X@@QAEX$$QAV<lambda_15ade71b0218206bbe3333a0c9b79046>@@AAV<lambda_da44e0f8b0f19ba52fefafb335991732>@@$$QAV<lambda_207f2d024fc103971653565357d6cd41>@@@Z 10037438     libucrt:per_thread_data.obj
 0002:00015458       __sehtable$??$?RV<lambda_a7e850c220f1c8d1e6efeecdedd162c6>@@AAV<lambda_46720907175c18b6c9d2717bc0d2d362>@@V<lambda_9048902d66e8d99359bc9897bbb930a8>@@@?$__crt_seh_guarded_call@X@@QAEX$$QAV<lambda_a7e850c220f1c8d1e6efeecdedd162c6>@@AAV<lambda_46720907175c18b6c9d2717bc0d2d362>@@$$QAV<lambda_9048902d66e8d99359bc9897bbb930a8>@@@Z 10037458     libucrt:per_thread_data.obj
 0002:00015478       __sehtable$??$?RV<lambda_38edbb1296d33220d7e4dd0ed76b244a>@@AAV<lambda_5ce1d447e08cb34b2473517608e21441>@@V<lambda_fb385d3da700c9147fc39e65dd577a8c>@@@?$__crt_seh_guarded_call@X@@QAEX$$QAV<lambda_38edbb1296d33220d7e4dd0ed76b244a>@@AAV<lambda_5ce1d447e08cb34b2473517608e21441>@@$$QAV<lambda_fb385d3da700c9147fc39e65dd577a8c>@@@Z 10037478     libucrt:per_thread_data.obj
 0002:00015498       __sehtable$??$?RV<lambda_6affb1475c98b40b75cdec977db92e3c>@@AAV<lambda_b8d4b9c228a6ecc3f80208dbb4b4a104>@@V<lambda_608742c3c92a14382c1684fc64f96c88>@@@?$__crt_seh_guarded_call@X@@QAEX$$QAV<lambda_6affb1475c98b40b75cdec977db92e3c>@@AAV<lambda_b8d4b9c228a6ecc3f80208dbb4b4a104>@@$$QAV<lambda_608742c3c92a14382c1684fc64f96c88>@@@Z 10037498     libucrt:per_thread_data.obj
 0002:000154b8       __sehtable$__fcloseall     100374b8     libucrt:closeall.obj
 0002:000154d8       __sehtable$??$?RV<lambda_2866be3712abc81a800a822484c830d8>@@AAV<lambda_39ca0ed439415581b5b15c265174cece>@@V<lambda_2b24c74d71094a6cd0cb82e44167d71b>@@@?$__crt_seh_guarded_call@X@@QAEX$$QAV<lambda_2866be3712abc81a800a822484c830d8>@@AAV<lambda_39ca0ed439415581b5b15c265174cece>@@$$QAV<lambda_2b24c74d71094a6cd0cb82e44167d71b>@@@Z 100374d8     libucrt:fflush.obj
 0002:000154f8       __sehtable$??$?RV<lambda_2cc53f568c5a2bb6f192f930a45d44ea>@@AAV<lambda_ab61a845afdef5b7c387490eaf3616ee>@@V<lambda_c2ffc0b7726aa6be21d5f0026187e748>@@@?$__crt_seh_guarded_call@X@@QAEX$$QAV<lambda_2cc53f568c5a2bb6f192f930a45d44ea>@@AAV<lambda_ab61a845afdef5b7c387490eaf3616ee>@@$$QAV<lambda_c2ffc0b7726aa6be21d5f0026187e748>@@@Z 100374f8     libucrt:fflush.obj
 0002:00015518       __sehtable$___acrt_initialize_lowio 10037518     libucrt:ioinit.obj
 0002:00015538       __sehtable$??$?RV<lambda_e5124f882df8998aaf41531e079ba474>@@AAV<lambda_3e16ef9562a7dcce91392c22ab16ea36>@@V<lambda_e25ca0880e6ef98be67edffd8c599615>@@@?$__crt_seh_guarded_call@X@@QAEX$$QAV<lambda_e5124f882df8998aaf41531e079ba474>@@AAV<lambda_3e16ef9562a7dcce91392c22ab16ea36>@@$$QAV<lambda_e25ca0880e6ef98be67edffd8c599615>@@@Z 10037538     libucrt:wsetlocale.obj
 0002:00015558       __sehtable$??$?RV<lambda_218ce3db14220d0be481dae8ef3383b6>@@AAV<lambda_628dfdc04ba53c8bfc02c9951375f3f5>@@V<lambda_57dc472bd5c9d5f3b2cbca59b8a843ae>@@@?$__crt_seh_guarded_call@H@@QAEH$$QAV<lambda_218ce3db14220d0be481dae8ef3383b6>@@AAV<lambda_628dfdc04ba53c8bfc02c9951375f3f5>@@$$QAV<lambda_57dc472bd5c9d5f3b2cbca59b8a843ae>@@@Z 10037558     libucrt:close.obj
 0002:00015578       __sehtable$?__acrt_stdio_allocate_stream@@YA?AV__crt_stdio_stream@@XZ 10037578     libucrt:stream.obj
 0002:00015598       __sehtable$?update_thread_multibyte_data_internal@@YAPAU__crt_multibyte_data@@QAU__acrt_ptd@@QAPAU1@@Z 10037598     libucrt:mbctype.obj
 0002:000155b8       __sehtable$??$?RV<lambda_ceb1ee4838e85a9d631eb091e2fbe199>@@AAV<lambda_ae742caa10f662c28703da3d2ea5e57e>@@V<lambda_cd08b5d6af4937fe54fc07d0c9bf6b37>@@@?$__crt_seh_guarded_call@X@@QAEX$$QAV<lambda_ceb1ee4838e85a9d631eb091e2fbe199>@@AAV<lambda_ae742caa10f662c28703da3d2ea5e57e>@@$$QAV<lambda_cd08b5d6af4937fe54fc07d0c9bf6b37>@@@Z 100375b8     libucrt:mbctype.obj
 0002:000155d8       __sehtable$_raise          100375d8     libucrt:signal.obj
 0002:000155f8       __sehtable$??$?RV<lambda_cbab9ec6f41b0180b23cc171c22676b0>@@AAV<lambda_44731a7d0e6d81c3e6aa82d741081786>@@V<lambda_4b292cb8dd18144e164572427af410ab>@@@?$__crt_seh_guarded_call@P6AXH@Z@@QAEP6AXH@Z$$QAV<lambda_cbab9ec6f41b0180b23cc171c22676b0>@@AAV<lambda_44731a7d0e6d81c3e6aa82d741081786>@@$$QAV<lambda_4b292cb8dd18144e164572427af410ab>@@@Z 100375f8     libucrt:signal.obj
 0002:00015618       __sehtable$___acrt_update_thread_locale_data 10037618     libucrt:locale_refcounting.obj
 0002:00015638       __sehtable$??$?RV<lambda_9e9de3de5fa147e2223d7db92bc10aa6>@@AAV<lambda_38ce7e780aa69e748d6df282ebc68efe>@@V<lambda_8ca6da459f0f6780f1cff60fdc3d00e5>@@@?$__crt_seh_guarded_call@H@@QAEH$$QAV<lambda_9e9de3de5fa147e2223d7db92bc10aa6>@@AAV<lambda_38ce7e780aa69e748d6df282ebc68efe>@@$$QAV<lambda_8ca6da459f0f6780f1cff60fdc3d00e5>@@@Z 10037638     libucrt:commit.obj
 0002:00015658       __sehtable$__write         10037658     libucrt:write.obj
 0002:00015678       __sehtable$__alloc_osfhnd  10037678     libucrt:osfinfo.obj
 0002:00015698       __sehtable$___acrt_lowio_ensure_fh_exists 10037698     libucrt:osfinfo.obj
 0002:000156b8       __sehtable$??$common_sopen_dispatch@D@@YAHQBDHHHQAHH@Z 100376b8     libucrt:open.obj
 0002:000156d8       __sehtable$??$common_lseek@_J@@YA_JH_JH@Z 100376d8     libucrt:lseek.obj
 0002:000156f8       __sehtable$__IsNonwritableInCurrentImage 100376f8     LIBCMT:pesect.obj
 0002:00015720       .edata                     10037720     javaaccessbridge.exp
 0002:00015748       rgpv                       10037748     javaaccessbridge.exp
 0002:000157c0       rgszName                   100377c0     javaaccessbridge.exp
 0002:00015838       rgwOrd                     10037838     javaaccessbridge.exp
 0002:00015874       szName                     10037874     javaaccessbridge.exp
 0002:00015889       $N00001                    10037889     javaaccessbridge.exp
 0002:000158cf       $N00002                    100378cf     javaaccessbridge.exp
 0002:00015915       $N00003                    10037915     javaaccessbridge.exp
 0002:00015959       $N00004                    10037959     javaaccessbridge.exp
 0002:0001599f       $N00005                    1003799f     javaaccessbridge.exp
 0002:00015a00       $N00006                    10037a00     javaaccessbridge.exp
 0002:00015a61       $N00007                    10037a61     javaaccessbridge.exp
 0002:00015aa8       $N00008                    10037aa8     javaaccessbridge.exp
 0002:00015af1       $N00009                    10037af1     javaaccessbridge.exp
 0002:00015b38       $N00010                    10037b38     javaaccessbridge.exp
 0002:00015b7f       $N00011                    10037b7f     javaaccessbridge.exp
 0002:00015bc6       $N00012                    10037bc6     javaaccessbridge.exp
 0002:00015c0c       $N00013                    10037c0c     javaaccessbridge.exp
 0002:00015c53       $N00014                    10037c53     javaaccessbridge.exp
 0002:00015c9b       $N00015                    10037c9b     javaaccessbridge.exp
 0002:00015ce7       $N00016                    10037ce7     javaaccessbridge.exp
 0002:00015d3e       $N00017                    10037d3e     javaaccessbridge.exp
 0002:00015d93       $N00018                    10037d93     javaaccessbridge.exp
 0002:00015dec       $N00019                    10037dec     javaaccessbridge.exp
 0002:00015e3a       $N00020                    10037e3a     javaaccessbridge.exp
 0002:00015e88       $N00021                    10037e88     javaaccessbridge.exp
 0002:00015edc       $N00022                    10037edc     javaaccessbridge.exp
 0002:00015f29       $N00023                    10037f29     javaaccessbridge.exp
 0002:00015f7b       $N00024                    10037f7b     javaaccessbridge.exp
 0002:00015fc9       $N00025                    10037fc9     javaaccessbridge.exp
 0002:0001601c       $N00026                    1003801c     javaaccessbridge.exp
 0002:00016069       $N00027                    10038069     javaaccessbridge.exp
 0002:000160b7       $N00028                    100380b7     javaaccessbridge.exp
 0002:0001610b       $N00029                    1003810b     javaaccessbridge.exp
 0002:0001614b       $N00030                    1003814b     javaaccessbridge.exp
 0002:0001642e       .idata$6                   1003842e     kernel32:KERNEL32.dll
 0002:000164ea       .idata$6                   100384ea     user32:USER32.dll
 0002:00016508       .idata$6                   10038508     jawt:jawt.dll
 0003:00000020       ?__vcrt_flsindex@@3KA      10039020     libvcruntime:per_thread_data.obj
 0003:000000f0       ?errno_no_memory@@3HA      100390f0     libucrt:errno.obj
 0003:000000f4       ?doserrno_no_memory@@3KA   100390f4     libucrt:errno.obj
 0003:000000f8       ?__acrt_flsindex@@3KA      100390f8     libucrt:per_thread_data.obj
 0003:00000420       __mbctypes                 10039420     libucrt:mbctype.obj
 0003:00000528       __mbcasemaps               10039528     libucrt:mbctype.obj
 0003:00000628       ?__rgctypeflag@@3PADA      10039628     libucrt:mbctype.obj
 0003:00000630       ?__rgcode_page_info@@3PAUcode_page_info@@A 10039630     libucrt:mbctype.obj
 0003:00000880       ?__dcrt_lowio_console_output_handle@@3PAXA 10039880     libucrt:initcon.obj
 0003:00000918       _logFP                     10039918     AccessBridgeDebug.obj
 0003:00000944       ?__proc_attached@@3HA      10039944     LIBCMT:dll_dllmain.obj
 0003:00000948       _GS_ExceptionRecord        10039948     LIBCMT:gs_report.obj
 0003:00000998       _GS_ContextRecord          10039998     LIBCMT:gs_report.obj
 0003:00000c80       ?is_initialized_as_dll@@3_NA 10039c80     LIBCMT:utility.obj
 0003:00000c81       ?module_local_atexit_table_initialized@@3_NA 10039c81     LIBCMT:utility.obj
 0003:00000c84       ?module_local_atexit_table@@3U_onexit_table_t@@A 10039c84     LIBCMT:utility.obj
 0003:00000c90       ?module_local_at_quick_exit_table@@3U_onexit_table_t@@A 10039c90     LIBCMT:utility.obj
 0003:00000cd4       ?heap@@3V_HeapManager@@A   10039cd4     libvcruntime:undname.obj
 0003:00000ce8       ?__vcrt_startup_thread_ptd@@3U__vcrt_ptd@@A 10039ce8     libvcruntime:per_thread_data.obj
 0003:00000d10       ___vcrt_lock_table         10039d10     libvcruntime:locks.obj
 0003:00000d28       ___vcrt_locks_initialized  10039d28     libvcruntime:locks.obj
 0003:00000d2c       ?module_handles@@3PAPAUHINSTANCE__@@A 10039d2c     libvcruntime:winapi_downlevel.obj
 0003:00000d38       ?function_pointers@@3PAPAXA 10039d38     libvcruntime:winapi_downlevel.obj
 0003:00000d5c       ?__acrt_new_handler@@3V?$dual_state_global@P6AHI@Z@__crt_state_management@@A 10039d5c     libucrt:new_handler.obj
 0003:00000d60       ?c_termination_complete@@3JA 10039d60     libucrt:exit.obj
 0003:00000d64       ?thread_local_exit_callback_func@@3P6GXPAXK0@ZA 10039d64     libucrt:exit.obj
 0003:00000d70       ?program_name@?1???$common_configure_argv@D@@YAHW4_crt_argv_mode@@@Z@4PADA 10039d70     libucrt:argv_parsing.obj
 0003:00000ea0       ?__acrt_invalid_parameter_handler@@3V?$dual_state_global@P6AXPB_W00II@Z@__crt_state_management@@A 10039ea0     libucrt:invalid_parameter.obj
 0003:00000ea8       ?module_handles@@3PAPAUHINSTANCE__@@A 10039ea8     libucrt:winapi_thunks.obj
 0003:00000ef8       ?encoded_function_pointers@@3PAPAXA 10039ef8     libucrt:winapi_thunks.obj
 0003:00000f80       ?state_cache@?1???$get_cached_win_policy@Ubegin_thread_init_policy_properties@?1??__acrt_get_begin_thread_init_policy@@YA?AW4begin_thread_init_policy@@XZ@@@YA?AW4begin_thread_init_policy@@W4AppPolicyThreadInitializationType@@@Z@4JA 10039f80     libucrt:win_policies.obj
 0003:0000118c       ?internal_state@?1??_mbtowc_l@@9@4U_Mbstatet@@A 1003a18c     libucrt:mbtowc.obj
 0003:00001194       ?enable_percent_n@@3IA     1003a194     libucrt:printf_count_output.obj
 0003:000011a8       ?__acrt_lock_table@@3PAU_RTL_CRITICAL_SECTION@@A 1003a1a8     libucrt:locks.obj
 0003:000012f8       ?__acrt_locks_initialized@@3IA 1003a2f8     libucrt:locks.obj
 0003:00001308       ?fSystemSet@@3HA           1003a308     libucrt:mbctype.obj
 0003:0000130c       ?initialized@?1??__acrt_initialize_multibyte@@9@4_NA 1003a30c     libucrt:mbctype.obj
 0003:0000132c       ?ctrlc_action@@3V?$dual_state_global@P6AXH@Z@__crt_state_management@@A 1003a32c     libucrt:signal.obj
 0003:00001330       ?ctrlbreak_action@@3V?$dual_state_global@P6AXH@Z@__crt_state_management@@A 1003a330     libucrt:signal.obj
 0003:00001334       ?abort_action@@3V?$dual_state_global@P6AXH@Z@__crt_state_management@@A 1003a334     libucrt:signal.obj
 0003:00001338       ?term_action@@3V?$dual_state_global@P6AXH@Z@__crt_state_management@@A 1003a338     libucrt:signal.obj
 0003:0000133c       ?user_matherr@@3V?$dual_state_global@P6AHPAU_exception@@@Z@__crt_state_management@@A 1003a33c     libucrt:matherr.obj
 0003:00001340       ?__acrt_global_new_mode@@3V?$dual_state_global@J@__crt_state_management@@A 1003a340     libucrt:new_mode.obj
 0003:00001350       ?__acrt_app_type@@3W4_crt_app_type@@A 1003a350     libucrt:report_runtime_error.obj
 0003:00001354       ?internal_pst@?1??__mbrtoc32_utf8@__crt_mbstring@@YAIPA_UPBDIPAU_Mbstatet@@@Z@4U3@A 1003a354     libucrt:mbrtoc32.obj
 0003:00001364       __pmatherr_set             1003a364     libucrt:libm_error.obj
 0004:00000120       $R000000                   1003b120     javaaccessbridge.dll.res
 0004:000004a8       $R000388                   1003b4a8     javaaccessbridge.dll.res
 0004:000006c0       $R0005A0                   1003b6c0     javaaccessbridge.dll.res
